 LuaPlugin

 Timestamp is 4aa85097 (Thu Sep 10 02:04:23 2009)

 Preferred load address is 11000000

 Start         Length     Name                   Class
 0001:00000000 000a76ebH .text                   CODE
 0001:000a76f0 000000c2H .text$x                 CODE
 0001:000a77b2 00000044H .text$yc                CODE
 0001:000a77f6 0000003cH .text$yd                CODE
 0002:00000000 0000023cH .idata$5                DATA
 0002:0000023c 00000004H .CRT$XCA                DATA
 0002:00000240 0000000cH .CRT$XCC                DATA
 0002:0000024c 00000004H .CRT$XCU                DATA
 0002:00000250 00000004H .CRT$XCZ                DATA
 0002:00000254 00000004H .CRT$XIA                DATA
 0002:00000258 00000018H .CRT$XIC                DATA
 0002:00000270 00000004H .CRT$XID                DATA
 0002:00000274 00000004H .CRT$XIZ                DATA
 0002:00000278 00000004H .CRT$XPA                DATA
 0002:0000027c 00000008H .CRT$XPX                DATA
 0002:00000284 00000004H .CRT$XPXA               DATA
 0002:00000288 00000004H .CRT$XPZ                DATA
 0002:0000028c 00000004H .CRT$XTA                DATA
 0002:00000290 00000004H .CRT$XTZ                DATA
 0002:000002a0 000154e8H .rdata                  DATA
 0002:00015788 00000049H .rdata$debug            DATA
 0002:000157d4 000004f0H .rdata$r                DATA
 0002:00015cd0 00000030H .rdata$sxdata           DATA
 0002:00015d00 00000004H .rtc$IAA                DATA
 0002:00015d04 00000004H .rtc$IZZ                DATA
 0002:00015d08 00000004H .rtc$TAA                DATA
 0002:00015d0c 00000004H .rtc$TZZ                DATA
 0002:00015d10 00000c3cH .xdata$x                DATA
 0002:0001694c 00000050H .idata$2                DATA
 0002:0001699c 00000014H .idata$3                DATA
 0002:000169b0 0000023cH .idata$4                DATA
 0002:00016bec 000008d4H .idata$6                DATA
 0002:000174c0 000001e6H .edata                  DATA
 0003:00000000 000020baH .data                   DATA
 0003:000020c0 00002d64H .bss                    DATA

  Address         Publics by Value              Rva+Base       Lib:Object

 0000:00000000       __except_list              00000000     <absolute>
 0000:0000000c       ___safe_se_handler_count   0000000c     <absolute>
 0000:00000000       ___ImageBase               11000000     <linker-defined>
 0001:00000000       ??1bad_alloc@std@@UAE@XZ   11001000 f i engine_gm.obj
 0001:00000010       ??_Ebad_alloc@std@@UAEPAXI@Z 11001010 f i  CIL library: CIL module
 0001:00000010       ??_Gbad_alloc@std@@UAEPAXI@Z 11001010 f i engine_gm.obj
 0001:00000040       ?InitEngineSSGM@@YAXXZ     11001040 f   engine_gm.obj
 0001:000000c0       ?Translate_Preset_ID_To_PT_String_Name@@YAPB_WHI@Z 110010c0 f   engine_gm.obj
 0001:00000160       ??0?$basic_string@DU?$char_traits@D@std@@V?$allocator@D@2@@std@@QAE@PBD@Z 11001160 f i engine_gm.obj
 0001:000001a0       ??1?$basic_string@DU?$char_traits@D@std@@V?$allocator@D@2@@std@@QAE@XZ 110011a0 f i engine_gm.obj
 0001:000001d0       ?assign@?$basic_string@DU?$char_traits@D@std@@V?$allocator@D@2@@std@@QAEAAV12@ABV12@II@Z 110011d0 f i engine_gm.obj
 0001:000002b0       ?assign@?$basic_string@DU?$char_traits@D@std@@V?$allocator@D@2@@std@@QAEAAV12@PBDI@Z 110012b0 f i engine_gm.obj
 0001:00000390       ?erase@?$basic_string@DU?$char_traits@D@std@@V?$allocator@D@2@@std@@QAEAAV12@II@Z 11001390 f i engine_gm.obj
 0001:00000420       ?_Copy@?$basic_string@DU?$char_traits@D@std@@V?$allocator@D@2@@std@@IAEXII@Z 11001420 f i engine_gm.obj
 0001:00000550       ?allocate@?$allocator@D@std@@QAEPADI@Z 11001550 f i engine_gm.obj
 0001:000005b0       ??0bad_alloc@std@@QAE@ABV01@@Z 110015b0 f i engine_gm.obj
 0001:000005d0       ??0logic_error@std@@QAE@ABV?$basic_string@DU?$char_traits@D@std@@V?$allocator@D@2@@1@@Z 110015d0 f i gmcommandclass.obj
 0001:00000630       ?what@logic_error@std@@UBEPBDXZ 11001630 f i gmcommandclass.obj
 0001:00000640       ??0length_error@std@@QAE@ABV?$basic_string@DU?$char_traits@D@std@@V?$allocator@D@2@@1@@Z 11001640 f i gmcommandclass.obj
 0001:00000660       ??1logic_error@std@@UAE@XZ 11001660 f i gmcommandclass.obj
 0001:00000660       ??1length_error@std@@UAE@XZ 11001660 f i gmcommandclass.obj
 0001:000006a0       ??_Glength_error@std@@UAEPAXI@Z 110016a0 f i gmcommandclass.obj
 0001:000006a0       ??_Elogic_error@std@@UAEPAXI@Z 110016a0 f i  CIL library: CIL module
 0001:000006a0       ??_Elength_error@std@@UAEPAXI@Z 110016a0 f i  CIL library: CIL module
 0001:000006a0       ??_Glogic_error@std@@UAEPAXI@Z 110016a0 f i gmcommandclass.obj
 0001:000006f0       ??0logic_error@std@@QAE@ABV01@@Z 110016f0 f i gmcommandclass.obj
 0001:00000760       ??0length_error@std@@QAE@ABV01@@Z 11001760 f i gmcommandclass.obj
 0001:00000780       ??1locale@std@@QAE@XZ      11001780 f i gmfunc.obj
 0001:000007d0       ?Load_Hooks@@YAXXZ         110017d0 f   Hooks.obj
 0001:00000a00       ?Plugin_Load@@YAXXZ        11001a00 f   plugin.obj
 0001:00000c70       _SSGM_Host_Hook            11001c70 f   plugin.obj
 0001:00000c80       _SSGM_Player_Join_Hook     11001c80 f   plugin.obj
 0001:00000c90       _SSGM_Player_Leave_Hook    11001c90 f   plugin.obj
 0001:00000ca0       _SSGM_Level_Loaded_Hook    11001ca0 f   plugin.obj
 0001:00000cb0       _SSGM_GameOver_Hook        11001cb0 f   plugin.obj
 0001:00000cc0       _SSGM_Console_Output_Hook  11001cc0 f   plugin.obj
 0001:00000cd0       _SSGM_DDE_Hook             11001cd0 f   plugin.obj
 0001:00000ce0       _DllMain@12                11001ce0 f   dllmain.obj
 0001:00000d10       _Create_Script             11001d10 f   dllmain.obj
 0001:00000d30       _Set_Script_Commands       11001d30 f   dllmain.obj
 0001:00002070       _Set_Request_Destroy_Func  11003070 f   dllmain.obj
 0001:00002080       _SSGM_Check_Version        11003080 f   dllmain.obj
 0001:000020a0       _SSGM_Plugin_Load          110030a0 f   dllmain.obj
 0001:00002100       _SSGM_Plugin_Unload        11003100 f   dllmain.obj
 0001:000022e0       ?erase@?$vector@PAUChatCommandInfo@@V?$allocator@PAUChatCommandInfo@@@std@@@std@@QAE?AV?$_Vector_iterator@PAUChatCommandInfo@@V?$allocator@PAUChatCommandInfo@@@std@@@2@V?$_Vector_const_iterator@PAUChatCommandInfo@@V?$allocator@PAUChatCommandInfo@@@std@@@2@0@Z 110032e0 f i dllmain.obj
 0001:00002370       ??_E?$VectorClass@PAE@@UAEPAXI@Z 11003370 f i  CIL library: CIL module
 0001:00002370       ??_G?$VectorClass@PAE@@UAEPAXI@Z 11003370 f i engine_bhs.obj
 0001:00002390       ??1?$VectorClass@PAE@@UAE@XZ 11003390 f i engine_bhs.obj
 0001:000023a0       ??8?$VectorClass@PAE@@UAE_NAAV0@@Z 110033a0 f i engine_bhs.obj
 0001:000023b0       ?Resize@?$VectorClass@PAE@@UAE_NHPAPAE@Z 110033b0 f i engine_bhs.obj
 0001:000023c0       ?ID@?$VectorClass@PAE@@UAEHAAPAE@Z 110033c0 f i engine_bhs.obj
 0001:000023c0       ?ID@?$VectorClass@PAE@@UAEHPAPAE@Z 110033c0 f i engine_bhs.obj
 0001:000023d0       ?InitEngineCommon@@YAXI@Z  110033d0 f   engine_common.obj
 0001:00002590       ?Console_Output@@YAXPBDZZ  11003590 f   engine_common.obj
 0001:000025a0       ?InitEngine@@YAXXZ         110035a0 f   engine_common.obj
 0001:000026e0       ?Get@IntDataSafeClass@@QAEHXZ 110036e0 f   engine_def.obj
 0001:000026f0       ?Get@FloatDataSafeClass@@QAEMXZ 110036f0 f   engine_def.obj
 0001:00002700       ?Get@UIntDataSafeClass@@QAEIXZ 11003700 f   engine_def.obj
 0001:00002710       ?InitEngineDef@@YAXI@Z     11003710 f   engine_def.obj
 0001:00002830       ?Get_Phys_Definition@@YAPAVDefinitionClass@@PAE@Z 11003830 f   engine_def.obj
 0001:00002880       ?InitEngineDmg@@YAXI@Z     11003880 f   engine_dmg.obj
 0001:00002910       ?Set_Skin@@YAXPAEPBD@Z     11003910 f   engine_dmg.obj
 0001:00002970       ?The_Game@@YAPAVcGameData@@XZ 11003970 f   engine_game.obj
 0001:00002980       ?Find_Base@BaseControllerClass@@SAPAV1@H@Z 11003980 f   engine_game.obj
 0001:00002990       ?Get_Harvester_Vehicle@BaseControllerClass@@QAEPAEXZ 11003990 f   engine_game.obj
 0001:000029a0       ?Power_Base@BaseControllerClass@@QAEX_N@Z 110039a0 f   engine_game.obj
 0001:000029b0       ?Set_Can_Generate_Soldiers@BaseControllerClass@@QAEX_N@Z 110039b0 f   engine_game.obj
 0001:000029c0       ?Set_Can_Generate_Vehicles@BaseControllerClass@@QAEX_N@Z 110039c0 f   engine_game.obj
 0001:000029d0       ?Destroy_Base@BaseControllerClass@@QAEXXZ 110039d0 f   engine_game.obj
 0001:000029e0       ?Enable_Radar@BaseControllerClass@@QAEX_N@Z 110039e0 f   engine_game.obj
 0001:000029f0       ?Set_Beacon_Destroyed_Base@BaseControllerClass@@QAEX_N@Z 110039f0 f   engine_game.obj
 0001:00002a00       ?Find_Building@BaseControllerClass@@QAEPAEI@Z 11003a00 f   engine_game.obj
 0001:00002a10       ?InitEngineGame@@YAXI@Z    11003a10 f   engine_game.obj
 0001:00002e50       ?Is_Harvester@@YA_NPAE@Z   11003e50 f   engine_game.obj
 0001:00002ee0       ?Building_Type@@YAHPAE@Z   11003ee0 f   engine_game.obj
 0001:00002f50       ?Get_Building_Count_Team@@YAHH@Z 11003f50 f   engine_game.obj
 0001:00003000       ?Find_Building_By_Class_ID@@YAPAEHK@Z 11004000 f   engine_game.obj
 0001:000030c0       ?Find_Building_By_Team@@YAPAEH@Z 110040c0 f   engine_game.obj
 0001:00003140       ?Get_Current_Game_Mode@@YAIXZ 11004140 f   engine_game.obj
 0001:000031c0       ?Is_Harvester_Preset@@YA_NPAE@Z 110041c0 f   engine_game.obj
 0001:00003240       ?InitEngineIO@@YAXI@Z      11004240 f   engine_io.obj
 0001:000033b0       ?InitEngineMath@@YAXXZ     110043b0 f   engine_math.obj
 0001:00003430       ?Add@_Vector3MathFunctions@@UAEXPAUVector3@@00@Z 11004430 f   engine_math.obj
 0001:00003480       ?Subtract@_Vector3MathFunctions@@UAEXPAUVector3@@00@Z 11004480 f   engine_math.obj
 0001:000034d0       ?Multiply@_Vector3MathFunctions@@UAEXPAUVector3@@00@Z 110044d0 f   engine_math.obj
 0001:00003520       ?Divide@_Vector3MathFunctions@@UAEXPAUVector3@@00@Z 11004520 f   engine_math.obj
 0001:00003570       ?Multiply@_Vector3MathFunctions@@UAEXPAUVector3@@PAM0@Z 11004570 f   engine_math.obj
 0001:000035c0       ?Divide@_Vector3MathFunctions@@UAEXPAUVector3@@PAM0@Z 110045c0 f   engine_math.obj
 0001:00003610       ?Cross@_Vector3MathFunctions@@UAEXPAUVector3@@00@Z 11004610 f   engine_math.obj
 0001:00003670       ?Normalize@_Vector3MathFunctions@@UAEXPAUVector3@@0@Z 11004670 f   engine_math.obj
 0001:00003700       ?Dot@_Vector3MathFunctions@@UAEXPAUVector3@@0PAM@Z 11004700 f   engine_math.obj
 0001:00003730       ?Add@_Vector3MathFunctions@@UAE?AUVector3@@PAU2@0@Z 11004730 f   engine_math.obj
 0001:00003760       ?Subtract@_Vector3MathFunctions@@UAE?AUVector3@@PAU2@0@Z 11004760 f   engine_math.obj
 0001:00003790       ?Multiply@_Vector3MathFunctions@@UAE?AUVector3@@PAU2@0@Z 11004790 f   engine_math.obj
 0001:000037c0       ?Divide@_Vector3MathFunctions@@UAE?AUVector3@@PAU2@0@Z 110047c0 f   engine_math.obj
 0001:000037f0       ?Multiply@_Vector3MathFunctions@@UAE?AUVector3@@PAU2@PAM@Z 110047f0 f   engine_math.obj
 0001:00003820       ?Divide@_Vector3MathFunctions@@UAE?AUVector3@@PAU2@PAM@Z 11004820 f   engine_math.obj
 0001:00003850       ?Cross@_Vector3MathFunctions@@UAE?AUVector3@@PAU2@0@Z 11004850 f   engine_math.obj
 0001:00003880       ?Normalize@_Vector3MathFunctions@@UAE?AUVector3@@PAU2@@Z 11004880 f   engine_math.obj
 0001:000038b0       ?Dot@_Vector3MathFunctions@@UAEMPAUVector3@@0@Z 110048b0 f   engine_math.obj
 0001:000038d0       ?Subtract@_Vector4MathFunctions@@UAEXPAUVector4@@00@Z 110048d0 f   engine_math.obj
 0001:000038d0       ?Add@_Vector4MathFunctions@@UAEXPAUVector4@@00@Z 110048d0 f   engine_math.obj
 0001:00003930       ?Multiply@_Vector4MathFunctions@@UAEXPAUVector4@@00@Z 11004930 f   engine_math.obj
 0001:00003990       ?Divide@_Vector4MathFunctions@@UAEXPAUVector4@@00@Z 11004990 f   engine_math.obj
 0001:000039f0       ?Multiply@_Vector4MathFunctions@@UAEXPAUVector4@@PAM0@Z 110049f0 f   engine_math.obj
 0001:00003a50       ?Divide@_Vector4MathFunctions@@UAEXPAUVector4@@PAM0@Z 11004a50 f   engine_math.obj
 0001:00003ab0       ?Add@_Vector4MathFunctions@@UAE?AUVector4@@PAU2@0@Z 11004ab0 f   engine_math.obj
 0001:00003ae0       ?Subtract@_Vector4MathFunctions@@UAE?AUVector4@@PAU2@0@Z 11004ae0 f   engine_math.obj
 0001:00003b10       ?Multiply@_Vector4MathFunctions@@UAE?AUVector4@@PAU2@0@Z 11004b10 f   engine_math.obj
 0001:00003b40       ?Divide@_Vector4MathFunctions@@UAE?AUVector4@@PAU2@0@Z 11004b40 f   engine_math.obj
 0001:00003b70       ?Multiply@_Vector4MathFunctions@@UAE?AUVector4@@PAU2@PAM@Z 11004b70 f   engine_math.obj
 0001:00003ba0       ?Divide@_Vector4MathFunctions@@UAE?AUVector4@@PAU2@PAM@Z 11004ba0 f   engine_math.obj
 0001:00003bd0       ?Add@_Vector4MathFunctionsSSE@@UAEXPAUVector4@@00@Z 11004bd0 f   engine_math.obj
 0001:00003c00       ?Subtract@_Vector4MathFunctionsSSE@@UAEXPAUVector4@@00@Z 11004c00 f   engine_math.obj
 0001:00003c30       ?Multiply@_Vector4MathFunctionsSSE@@UAEXPAUVector4@@00@Z 11004c30 f   engine_math.obj
 0001:00003c60       ?Divide@_Vector4MathFunctionsSSE@@UAEXPAUVector4@@00@Z 11004c60 f   engine_math.obj
 0001:00003c90       ?Multiply@_Vector4MathFunctionsSSE@@UAEXPAUVector4@@PAM0@Z 11004c90 f   engine_math.obj
 0001:00003c90       ?Divide@_Vector4MathFunctionsSSE@@UAEXPAUVector4@@PAM0@Z 11004c90 f   engine_math.obj
 0001:00003cc0       ?Destroy_Connection@@YAXH@Z 11004cc0 f   engine_net.obj
 0001:00003cd0       ?InitEngineNet@@YAXI@Z     11004cd0 f   engine_net.obj
 0001:00003e10       ?Get_IP_Address@@YAPBDH@Z  11004e10 f   engine_net.obj
 0001:00003ea0       ?Get_IP_Port@@YAPBDH@Z     11004ea0 f   engine_net.obj
 0001:00003f50       ?Grant@PowerupGameObjDef@@QAEXPAEH_N@Z 11004f50 f   engine_obj.obj
 0001:00003f60       ?Set_Max_Health@DefenseObjectClass@@QAEXM@Z 11004f60 f   engine_obj.obj
 0001:00003f70       ?Set_Max_Shield_Strength@DefenseObjectClass@@QAEXM@Z 11004f70 f   engine_obj.obj
 0001:00003f80       ?Mark_Owner_Dirty@DefenseObjectClass@@QAEXXZ 11004f80 f   engine_obj.obj
 0001:00003f90       ?Start_Observers@ScriptableGameObj@@QAEXXZ 11004f90 f   engine_obj.obj
 0001:00003fa0       ?InitEngineObj@@YAXI@Z     11004fa0 f   engine_obj.obj
 0001:00004170       ?Get_Object_Type@@YAHPAE@Z 11005170 f   engine_obj.obj
 0001:000041a0       ?As_BeaconGameObj@@YAPAEPAE@Z 110051a0 f   engine_obj.obj
 0001:000041e0       ?As_PowerPlantGameObj@@YAPAEPAE@Z 110051e0 f   engine_obj.obj
 0001:00004240       ?As_SoldierFactoryGameObj@@YAPAEPAE@Z 11005240 f   engine_obj.obj
 0001:000042a0       ?As_VehicleFactoryGameObj@@YAPAEPAE@Z 110052a0 f   engine_obj.obj
 0001:00004300       ?As_AirstripGameObj@@YAPAEPAE@Z 11005300 f   engine_obj.obj
 0001:00004360       ?As_WarFactoryGameObj@@YAPAEPAE@Z 11005360 f   engine_obj.obj
 0001:000043c0       ?As_RefineryGameObj@@YAPAEPAE@Z 110053c0 f   engine_obj.obj
 0001:00004420       ?As_ComCenterGameObj@@YAPAEPAE@Z 11005420 f   engine_obj.obj
 0001:00004480       ?As_RepairBayGameObj@@YAPAEPAE@Z 11005480 f   engine_obj.obj
 0001:000044e0       ?As_VehicleGameObj@@YAPAEPAE@Z 110054e0 f   engine_obj.obj
 0001:00004510       ?As_SmartGameObj@@YAPAEPAE@Z 11005510 f   engine_obj.obj
 0001:00004540       ?As_SoldierGameObj@@YAPAEPAE@Z 11005540 f   engine_obj.obj
 0001:00004570       ?As_ScriptZoneGameObj@@YAPAEPAE@Z 11005570 f   engine_obj.obj
 0001:000045a0       ?Get_Building_Type@@YAPBDPAE@Z 110055a0 f   engine_obj.obj
 0001:00004630       ?Get_Object_Count@@YAHHPBD@Z 11005630 f   engine_obj.obj
 0001:000046b0       ?Find_Random_Preset@@YAPAEPBDHH@Z 110056b0 f   engine_obj.obj
 0001:00004730       ?Send_Custom_To_Team_Buildings@@YAXHPAEHHM@Z 11005730 f   engine_obj.obj
 0001:00004830       ?Send_Custom_To_Team_Preset@@YAXHPBDPAEHHM@Z 11005830 f   engine_obj.obj
 0001:00004920       ?Send_Custom_All_Objects@@YAXHPAEH@Z 11005920 f   engine_obj.obj
 0001:000049f0       ?Send_Custom_Event_To_Object@@YAXPAEPBDHHM@Z 110059f0 f   engine_obj.obj
 0001:00004ac0       ?Grant_Powerup@@YAXPAEPBD@Z 11005ac0 f   engine_obj.obj
 0001:00004b20       ?Overlap_Test@@YAIABVOBBoxClass@@ABUVector3@@@Z 11005b20 f   engine_obj2.obj
 0001:00004b30       ?GrantSupplies@@YAXPAE@Z   11005b30 f   engine_obj2.obj
 0001:00004b40       ?Check_Transitions@@YA_NPAE_N@Z 11005b40 f   engine_obj2.obj
 0001:00004b50       ?InitEngineObj2@@YAXI@Z    11005b50 f   engine_obj2.obj
 0001:00004dd0       ?Get_Vehicle@@YAPAEPAE@Z   11005dd0 f   engine_obj2.obj
 0001:00004e20       ?Soldier_Re_Init@@YAXPAEPAVDefinitionClass@@@Z 11005e20 f   engine_obj2.obj
 0001:00004e60       ?Change_Character@@YA_NPAEPBD@Z 11005e60 f   engine_obj2.obj
 0001:00004ee0       ?Create_Vehicle@@YAXPBDMPAEH@Z 11005ee0 f   engine_obj2.obj
 0001:00004fa0       ?Toggle_Fly_Mode@@YAXPAE@Z 11005fa0 f   engine_obj2.obj
 0001:00005010       ?Get_Vehicle_Occupant_Count@@YAHPAE@Z 11006010 f   engine_obj2.obj
 0001:00005080       ?Get_Vehicle_Driver@@YAPAEPAE@Z 11006080 f   engine_obj2.obj
 0001:000050d0       ?Get_Vehicle_Gunner_Pos@@YAPAEPAE@Z 110060d0 f   engine_obj2.obj
 0001:00005120       ?Get_Vehicle_Gunner@@YAPAEPAE@Z 11006120 f   engine_obj2.obj
 0001:00005180       ?Force_Occupant_Exit@@YAXPAEH@Z 11006180 f   engine_obj2.obj
 0001:000051e0       ?Force_Occupants_Exit@@YAXPAE@Z 110061e0 f   engine_obj2.obj
 0001:00005250       ?Change_Spawn_Char@@YAXHPBD@Z 11006250 f   engine_obj2.obj
 0001:000052a0       ?Get_Vehicle_Mode@@YAIPAE@Z 110062a0 f   engine_obj2.obj
 0001:00005320       ?Force_Occupants_Exit_Team@@YAXPAEH@Z 11006320 f   engine_obj2.obj
 0001:00005400       ?IsInsideZone@@YA_NPAE0@Z  11006400 f   engine_obj2.obj
 0001:000054a0       ?Get_Zone_Type@@YAIPAE@Z   110064a0 f   engine_obj2.obj
 0001:00005510       ?Create_Zone@@YAPAEPBDABVOBBoxClass@@@Z 11006510 f   engine_obj2.obj
 0001:00005560       ?PointInZone@@YA_NPAEABUVector3@@@Z 11006560 f   engine_obj2.obj
 0001:000055e0       ?Set_Vehicle_Gunner@@YAXPAEH@Z 110065e0 f   engine_obj2.obj
 0001:00005650       ?Set_Transform@PhysicalGameObj@@QAEXPAUMatrix3D@@@Z 11006650 f   engine_phys.obj
 0001:00005660       ?Get_Transform@PhysicalGameObj@@QAEPAUMatrix3D@@XZ 11006660 f   engine_phys.obj
 0001:00005670       ?InitEnginePhys@@YAXI@Z    11006670 f   engine_phys.obj
 0001:00005700       ?Get_Model@@YAPBDPAE@Z     11006700 f   engine_phys.obj
 0001:00005760       ?Is_TrackedVehicle@@YA_NPAE@Z 11006760 f   engine_phys.obj
 0001:000057c0       ?Is_VTOLVehicle@@YA_NPAE@Z 110067c0 f   engine_phys.obj
 0001:00005820       ?Is_WheeledVehicle@@YA_NPAE@Z 11006820 f   engine_phys.obj
 0001:00005880       ?Is_Motorcycle@@YA_NPAE@Z  11006880 f   engine_phys.obj
 0001:000058e0       ?Is_Door@@YA_NPAE@Z        110068e0 f   engine_phys.obj
 0001:00005940       ?Is_Elevator@@YA_NPAE@Z    11006940 f   engine_phys.obj
 0001:000059a0       ?Is_DamageableStaticPhys@@YA_NPAE@Z 110069a0 f   engine_phys.obj
 0001:00005a00       ?Is_AccessablePhys@@YA_NPAE@Z 11006a00 f   engine_phys.obj
 0001:00005a60       ?Is_DecorationPhys@@YA_NPAE@Z 11006a60 f   engine_phys.obj
 0001:00005ac0       ?Is_HumanPhys@@YA_NPAE@Z   11006ac0 f   engine_phys.obj
 0001:00005b20       ?Is_MotorVehicle@@YA_NPAE@Z 11006b20 f   engine_phys.obj
 0001:00005b80       ?Is_Phys3@@YA_NPAE@Z       11006b80 f   engine_phys.obj
 0001:00005be0       ?Is_RigidBody@@YA_NPAE@Z   11006be0 f   engine_phys.obj
 0001:00005c40       ?Is_ShakeableStatricPhys@@YA_NPAE@Z 11006c40 f   engine_phys.obj
 0001:00005ca0       ?Is_StaticAnimPhys@@YA_NPAE@Z 11006ca0 f   engine_phys.obj
 0001:00005d00       ?Is_StaticPhys@@YA_NPAE@Z  11006d00 f   engine_phys.obj
 0001:00005d60       ?Is_TimedDecorationPhys@@YA_NPAE@Z 11006d60 f   engine_phys.obj
 0001:00005dc0       ?Is_VehiclePhys@@YA_NPAE@Z 11006dc0 f   engine_phys.obj
 0001:00005e20       ?Is_DynamicAnimPhys@@YA_NPAE@Z 11006e20 f   engine_phys.obj
 0001:00005e80       ?Is_BuildingAggregate@@YA_NPAE@Z 11006e80 f   engine_phys.obj
 0001:00005ee0       ?Is_Projectile@@YA_NPAE@Z  11006ee0 f   engine_phys.obj
 0001:00005f40       ?Get_Physics@@YAPBDPAE@Z   11006f40 f   engine_phys.obj
 0001:00006070       ?Copy_Transform@@YAXPAE0@Z 11007070 f   engine_phys.obj
 0001:000060e0       ?Get_Htree_Name@@YAPBDPAE@Z 110070e0 f   engine_phys.obj
 0001:00006150       ?Create_Effect_All_Of_Preset@@YAXPBD0M_N@Z 11007150 f   engine_phys.obj
 0001:00006220       ?Get_Player_Count@@YAHXZ   11007220 f   engine_player.obj
 0001:00006230       ?Set_Player_Type@cPlayer@@QAEXH@Z 11007230 f   engine_player.obj
 0001:00006240       ?Set_Ladder_Points@cPlayer@@QAEXH@Z 11007240 f   engine_player.obj
 0001:00006250       ?Set_Rung@cPlayer@@QAEXH@Z 11007250 f   engine_player.obj
 0001:00006260       ?InitEnginePlayer@@YAXI@Z  11007260 f   engine_player.obj
 0001:00006450       ?Get_Player_Name@@YAPBDPAE@Z 11007450 f   engine_player.obj
 0001:000064d0       ?Change_Team@@YAXPAEH@Z    110074d0 f   engine_player.obj
 0001:00006530       ?Get_Player_ID@@YAJPAE@Z   11007530 f   engine_player.obj
 0001:00006580       ?Get_Kill_To_Death_Ratio@@YAMH@Z 11007580 f   engine_player.obj
 0001:000065e0       ?Get_GameObj_By_Player_Name@@YAPAEPBD@Z 110075e0 f   engine_player.obj
 0001:000066a0       ?Find_First_Player@@YAPAEH@Z 110076a0 f   engine_player.obj
 0001:00006740       ?Change_Player_Team@@YA_NPAE_N11@Z 11007740 f   engine_player.obj
 0001:00006930       ?stristr@@YAPADPBD0@Z      11007930 f   engine_player.obj
 0001:000069b0       ?Get_Part_Name@@YAPAEPBD@Z 110079b0 f   engine_player.obj
 0001:00006a60       ?Get_Part_Names@@YAHPBD@Z  11007a60 f   engine_player.obj
 0001:00006ae0       ?Get_Team_Player_Count@@YAHH@Z 11007ae0 f   engine_player.obj
 0001:00006b70       ?Send_Custom_All_Players@@YAXHPAEH@Z 11007b70 f   engine_player.obj
 0001:00006bf0       ?Steal_Team_Credits@@YAMMH@Z 11007bf0 f   engine_player.obj
 0001:00006c70       ?Get_Team_Credits@@YAMH@Z  11007c70 f   engine_player.obj
 0001:00006ce0       ?Get_Definition@TeamPurchaseSettingsDefClass@@SAPAV1@K@Z 11007ce0 f   engine_pt.obj
 0001:00006cf0       ?Find_Definition@PurchaseSettingsDefClass@@SAPAV1@KK@Z 11007cf0 f   engine_pt.obj
 0001:00006d00       ?InitEnginePT@@YAXI@Z      11007d00 f   engine_pt.obj
 0001:00006dc0       ?Get_Team_Cost@@YAIPBDI@Z  11007dc0 f   engine_pt.obj
 0001:00006e70       ?Disable_Preset_By_Name@@YAXIPBD@Z 11007e70 f   engine_pt.obj
 0001:00006ef0       ?Disable_Enlisted_By_Name@@YAXIPBD@Z 11007ef0 f   engine_pt.obj
 0001:00006f50       ?Disable_Preset@@YAXIII@Z  11007f50 f   engine_pt.obj
 0001:00006fc0       ?Disable_All_Ground_Vehicles@@YAXI@Z 11007fc0 f   engine_pt.obj
 0001:00007050       ?Disable_All_Flying_Vehicles@@YAXI@Z 11008050 f   engine_pt.obj
 0001:000070e0       ?Get_Team_Icon@@YAPADPBDI@Z 110080e0 f   engine_pt.obj
 0001:000071c0       ?Remove_Script@@YAXPAEPBD@Z 110081c0 f   engine_script.obj
 0001:00007230       ?Remove_Duplicate_Script@@YAXPAEPBD@Z 11008230 f   engine_script.obj
 0001:000072b0       ?Remove_Script_Preset@@YAXPBD0H@Z 110082b0 f   engine_script.obj
 0001:00007380       ?Remove_Script_Type@@YAXPBDKH@Z 11008380 f   engine_script.obj
 0001:00007450       ?Remove_All_Scripts@@YAXPAE@Z 11008450 f   engine_script.obj
 0001:000074b0       ?Attach_Script_Preset@@YAXPBD00H@Z 110084b0 f   engine_script.obj
 0001:00007590       ?Attach_Script_Type@@YAXPBD0KH@Z 11008590 f   engine_script.obj
 0001:00007660       ?Is_Script_Attached@@YA_NPAEPBD@Z 11008660 f   engine_script.obj
 0001:000076d0       ?Attach_Script_Preset_Once@@YAXPBD00H@Z 110086d0 f   engine_script.obj
 0001:000077c0       ?Attach_Script_Type_Once@@YAXPBD0KH@Z 110087c0 f   engine_script.obj
 0001:000078a0       ?Attach_Script_Player_Once@@YAXPBD0H@Z 110088a0 f   engine_script.obj
 0001:00007960       ?Attach_Script_Building@@YAXPBD0H@Z 11008960 f   engine_script.obj
 0001:00007a00       ?Attach_Script_Is_Preset@@YAXPAEPBD11H@Z 11008a00 f   engine_script.obj
 0001:00007a80       ?Attach_Script_Is_Type@@YAXPAEKPBD1H@Z 11008a80 f   engine_script.obj
 0001:00007af0       ?Attach_Script_All_Buildings_Team@@YAXHPBD0_N@Z 11008af0 f   engine_script.obj
 0001:00007bd0       ?Attach_Script_All_Turrets_Team@@YAXHPBD0_N@Z 11008bd0 f   engine_script.obj
 0001:00007d40       ?Find_Building_With_Script@@YAPAEHHPBDPAE@Z 11008d40 f   engine_script.obj
 0001:00007e20       ?Find_Object_With_Script@@YAPAEPBD@Z 11008e20 f   engine_script.obj
 0001:00007e80       ?InitEngineString@@YAXI@Z  11008e80 f   engine_string.obj
 0001:000080a0       ??1StringClass@@QAE@XZ     110090a0 f   engine_string.obj
 0001:000080b0       ??4StringClass@@QAEAAV0@PBD@Z 110090b0 f   engine_string.obj
 0001:00008100       ?Format@StringClass@@QAAHPADZZ 11009100 f   engine_string.obj
 0001:00008120       ?Format_Args@StringClass@@QAAHPADAAPAD@Z 11009120 f   engine_string.obj
 0001:000081a0       ?Uninitialised_Grow@StringClass@@QAEXH@Z 110091a0 f   engine_string.obj
 0001:00008210       ?Free_String@StringClass@@QAEXXZ 11009210 f   engine_string.obj
 0001:00008280       ?Uninitialised_Grow@WideStringClass@@QAEXH@Z 11009280 f   engine_string.obj
 0001:00008300       ?Free_String@WideStringClass@@QAEXXZ 11009300 f   engine_string.obj
 0001:00008380       ?Convert_From@WideStringClass@@QAE_NPBD@Z 11009380 f   engine_string.obj
 0001:000083f0       ?WideCharToChar@@YAPBDPB_W@Z 110093f0 f   engine_string.obj
 0001:00008440       ?newstr@@YAPADPBD@Z        11009440 f   engine_string.obj
 0001:00008480       ?InitEngineTDB@@YAXI@Z     11009480 f   engine_tdb.obj
 0001:00008510       ?Get_Translated_String@@YAPBDK@Z 11009510 f   engine_tdb.obj
 0001:00008570       ?Get_Wide_Translated_String@@YAPB_WK@Z 11009570 f   engine_tdb.obj
 0001:000085a0       ?Get_Translated_Preset_Name@@YAPBDPAE@Z 110095a0 f   engine_tdb.obj
 0001:00008610       ?Get_Current_Wide_Translated_Weapon@@YAPB_WPAE@Z 11009610 f   engine_tdb.obj
 0001:00008680       ?Get_Translated_Weapon@@YAPBDPAEH@Z 11009680 f   engine_tdb.obj
 0001:000086f0       ?Get_Team_Name@@YAPBDH@Z   110096f0 f   engine_tdb.obj
 0001:00008760       ?Get_Wide_Vehicle_Name@@YAPB_WPAE@Z 11009760 f   engine_tdb.obj
 0001:000087c0       ?Lock@CriticalSectionClass@@QAEXXZ 110097c0 f   engine_threading.obj
 0001:000087d0       ?Get_Beacon_Owner@BeaconGameObj@@QAEPAEXZ 110097d0 f   engine_weap.obj
 0001:000087e0       ?Defuse@C4GameObj@@QAEXXZ  110097e0 f   engine_weap.obj
 0001:000087f0       ?InitEngineWeap@@YAXI@Z    110097f0 f   engine_weap.obj
 0001:000088b0       ?Get_Current_Bullets@@YAHPAE@Z 110098b0 f   engine_weap.obj
 0001:00008910       ?Get_Current_Clip_Bullets@@YAHPAE@Z 11009910 f   engine_weap.obj
 0001:00008970       ?Get_Current_Total_Bullets@@YAHPAE@Z 11009970 f   engine_weap.obj
 0001:000089f0       ?Get_Position_Total_Bullets@@YAHPAEH@Z 110099f0 f   engine_weap.obj
 0001:00008a70       ?Get_Bullets@@YAHPAEPBD@Z  11009a70 f   engine_weap.obj
 0001:00008b10       ?Get_Clip_Bullets@@YAHPAEPBD@Z 11009b10 f   engine_weap.obj
 0001:00008bb0       ?Get_Total_Bullets@@YAHPAEPBD@Z 11009bb0 f   engine_weap.obj
 0001:00008c60       ?Get_Current_Max_Bullets@@YAHPAE@Z 11009c60 f   engine_weap.obj
 0001:00008cc0       ?Get_Current_Clip_Max_Bullets@@YAHPAE@Z 11009cc0 f   engine_weap.obj
 0001:00008d20       ?Get_Current_Total_Max_Bullets@@YAHPAE@Z 11009d20 f   engine_weap.obj
 0001:00008da0       ?Get_Position_Max_Bullets@@YAHPAEH@Z 11009da0 f   engine_weap.obj
 0001:00008e00       ?Get_Position_Clip_Max_Bullets@@YAHPAEH@Z 11009e00 f   engine_weap.obj
 0001:00008e60       ?Get_Position_Total_Max_Bullets@@YAHPAEH@Z 11009e60 f   engine_weap.obj
 0001:00008ee0       ?Get_Max_Bullets@@YAHPAEPBD@Z 11009ee0 f   engine_weap.obj
 0001:00008f80       ?Get_Max_Total_Bullets@@YAHPAEPBD@Z 11009f80 f   engine_weap.obj
 0001:00009040       ?Set_Current_Bullets@@YAXPAEH@Z 1100a040 f   engine_weap.obj
 0001:000090a0       ?Set_Current_Clip_Bullets@@YAXPAEH@Z 1100a0a0 f   engine_weap.obj
 0001:00009100       ?Set_Position_Bullets@@YAXPAEHH@Z 1100a100 f   engine_weap.obj
 0001:00009160       ?Set_Position_Clip_Bullets@@YAXPAEHH@Z 1100a160 f   engine_weap.obj
 0001:000091c0       ?Set_Bullets@@YAXPAEPBDH@Z 1100a1c0 f   engine_weap.obj
 0001:00009260       ?Set_Clip_Bullets@@YAXPAEPBDH@Z 1100a260 f   engine_weap.obj
 0001:00009300       ?Get_Current_Weapon_Style@@YAHPAE@Z 1100a300 f   engine_weap.obj
 0001:00009360       ?Disarm_Beacon@@YAXPAE@Z   1100a360 f   engine_weap.obj
 0001:000093a0       ?Disarm_Beacons@@YAXH@Z    1100a3a0 f   engine_weap.obj
 0001:00009510       ?Disarm_Nearest_Beacon@@YAXPAEH_N@Z 1100a510 f   engine_weap.obj
 0001:00009730       ?Disarm_All_Proxy_C4@@YAXH@Z 1100a730 f   engine_weap.obj
 0001:000098f0       ?Disarm_All_C4@@YAXH@Z     1100a8f0 f   engine_weap.obj
 0001:00009a60       ?Get_Current_Weapon@@YAPBDPAE@Z 1100aa60 f   engine_weap.obj
 0001:00009ac0       ?Get_Weapon@@YAPBDPAEH@Z   1100aac0 f   engine_weap.obj
 0001:00009b20       ?Has_Weapon@@YA_NPAEPBD@Z  1100ab20 f   engine_weap.obj
 0001:00009bb0       ?Find_Beacon@@YAPAEHH@Z    1100abb0 f   engine_weap.obj
 0001:00009c60       ?Get_C4_Count@@YAHH@Z      1100ac60 f   engine_weap.obj
 0001:00009cf0       ?Get_Beacon_Count@@YAHH@Z  1100acf0 f   engine_weap.obj
 0001:00009d80       ?Get_C4_Count_Proximity@@YAHH@Z 1100ad80 f   engine_weap.obj
 0001:00009ea0       ?Get_C4_Count_Remote@@YAHH@Z 1100aea0 f   engine_weap.obj
 0001:00009fc0       ?UnregisterScript@ScriptRegistrar@@SAXPAVScriptFactory@@@Z 1100afc0 f   scriptregistrar.obj
 0001:00009ff0       ?CreateScript@ScriptRegistrar@@SAPAVScriptImpClass@@PBD@Z 1100aff0 f   scriptregistrar.obj
 0001:0000a030       ??_GLuaScript@LuaScriptManager@@UAEPAXI@Z 1100b030 f i LuaManager.obj
 0001:0000a030       ??_ELuaScript@LuaScriptManager@@UAEPAXI@Z 1100b030 f i  CIL library: CIL module
 0001:0000a030       ??_GScriptImpClass@@UAEPAXI@Z 1100b030 f i scripts.obj
 0001:0000a030       ??_EScriptImpClass@@UAEPAXI@Z 1100b030 f i  CIL library: CIL module
 0001:0000a050       ??_GGameObjObserverClass@@UAEPAXI@Z 1100b050 f i scripts.obj
 0001:0000a050       ??_EGameObjObserverClass@@UAEPAXI@Z 1100b050 f i  CIL library: CIL module
 0001:0000a070       ?Get_Name@ScriptImpClass@@UAEPADXZ 1100b070 f   scripts.obj
 0001:0000a080       ?Attach@ScriptImpClass@@UAEXPAE@Z 1100b080 f   scripts.obj
 0001:0000a090       ?Detach@ScriptImpClass@@UAEXPAE@Z 1100b090 f   scripts.obj
 0001:0000a0b0       ?Damaged@ScriptImpClass@@UAEXPAE0M@Z 1100b0b0 f   scripts.obj
 0001:0000a0b0       ?Action_Complete@ScriptImpClass@@UAEXPAEHW4ActionCompleteReason@@@Z 1100b0b0 f   scripts.obj
 0001:0000a0c0       ?Custom@ScriptImpClass@@UAEXPAEHH0@Z 1100b0c0 f   scripts.obj
 0001:0000a0d0       ?Killed@ScriptImpClass@@UAEXPAE0@Z 1100b0d0 f   scripts.obj
 0001:0000a0d0       ?Timer_Expired@ScriptImpClass@@UAEXPAEH@Z 1100b0d0 f   scripts.obj
 0001:0000a0d0       ?Sound_Heard@ScriptImpClass@@UAEXPAEABUCombatSound@@@Z 1100b0d0 f   scripts.obj
 0001:0000a0d0       ?Animation_Complete@ScriptImpClass@@UAEXPAEPBD@Z 1100b0d0 f   scripts.obj
 0001:0000a0d0       ?Exited@ScriptImpClass@@UAEXPAE0@Z 1100b0d0 f   scripts.obj
 0001:0000a0d0       ?Entered@ScriptImpClass@@UAEXPAE0@Z 1100b0d0 f   scripts.obj
 0001:0000a0d0       ?Enemy_Seen@ScriptImpClass@@UAEXPAE0@Z 1100b0d0 f   scripts.obj
 0001:0000a0d0       ?Poked@ScriptImpClass@@UAEXPAE0@Z 1100b0d0 f   scripts.obj
 0001:0000a0e0       ?Owner@ScriptImpClass@@UAEPAEXZ 1100b0e0 f   scripts.obj
 0001:0000a0f0       ?Get_Owner_Ptr@ScriptImpClass@@UAEPAPAEXZ 1100b0f0 f   scripts.obj
 0001:0000a100       ?Set_Parameters_String@ScriptImpClass@@UAEXPBD@Z 1100b100 f   scripts.obj
 0001:0000a240       ?Get_Parameters_String@ScriptImpClass@@UAEXPADI@Z 1100b240 f   scripts.obj
 0001:0000a2f0       ?Save@ScriptImpClass@@UAEXAAE@Z 1100b2f0 f   scripts.obj
 0001:0000a350       ?Load@ScriptImpClass@@UAEXAAE@Z 1100b350 f   scripts.obj
 0001:0000a440       ?Destroyed@ScriptImpClass@@UAEXPAE@Z 1100b440 f   scripts.obj
 0001:0000a440       ?Load_Data@ScriptImpClass@@UAEXAAE@Z 1100b440 f   scripts.obj
 0001:0000a440       ?Created@ScriptImpClass@@UAEXPAE@Z 1100b440 f   scripts.obj
 0001:0000a440       ?Save_Data@ScriptImpClass@@UAEXAAE@Z 1100b440 f   scripts.obj
 0001:0000a450       ??1ScriptImpClass@@UAE@XZ  1100b450 f   scripts.obj
 0001:0000a4b0       ?Clear_Parameters@ScriptImpClass@@QAEXXZ 1100b4b0 f   scripts.obj
 0001:0000a500       ?Get_Parameter_Index@ScriptImpClass@@QAEHPBD@Z 1100b500 f   scripts.obj
 0001:0000a640       ?Set_Parameter@ScriptImpClass@@QAEXHPBD@Z 1100b640 f   scripts.obj
 0001:0000a6a0       ?cCallback@sqlite_wrapper@@CAHPAXHPAPAD1@Z 1100b6a0 f i Lua_Class.obj
 0001:0000a840       ?Query@sqlite_wrapper@@QAEXPAUlua_State@@PBD11@Z 1100b840 f i Lua_Class.obj
 0001:0000a8f0       ?Query@Lua_sqlite_wrapper@@CAHPAUlua_State@@@Z 1100b8f0 f i Lua_Class.obj
 0001:0000aa30       ?GetInstance@Lua_sqlite_wrapper@@SAPAVsqlite_wrapper@@PAUlua_State@@H@Z 1100ba30 f i Lua_Class.obj
 0001:0000ab00       ??0ActionParamsStruct@@QAE@XZ 1100bb00 f i LuaFunctions.obj
 0001:0000ac50       ?RegisterTable@Lua_sqlite_wrapper@@CAHPAUlua_State@@@Z 1100bc50 f i LuaFunctions.obj
 0001:0000ae10       ?DeleteInstance@Lua_sqlite_wrapper@@CAHPAUlua_State@@@Z 1100be10 f i LuaFunctions.obj
 0001:0000ae60       ?Register@Lua_sqlite_wrapper@@SAXPAUlua_State@@@Z 1100be60 f i LuaFunctions.obj
 0001:0000b080       ?Get_Vector3@@YAPAUVector3@@PAUlua_State@@HPAU1@@Z 1100c080 f   LuaFunctions.obj
 0001:0000b130       ?Lua_Get_ID@@YAHPAUlua_State@@@Z 1100c130 f   LuaFunctions.obj
 0001:0000b1a0       ?Lua_Console_Input@@YAHPAUlua_State@@@Z 1100c1a0 f   LuaFunctions.obj
 0001:0000b1e0       ?Lua_Console_Output@@YAHPAUlua_State@@@Z 1100c1e0 f   LuaFunctions.obj
 0001:0000b200       ?Lua_Get_Definition_Name@@YAHPAUlua_State@@@Z 1100c200 f   LuaFunctions.obj
 0001:0000b280       ?Lua_Get_Definition_ID@@YAHPAUlua_State@@@Z 1100c280 f   LuaFunctions.obj
 0001:0000b2f0       ?Lua_Get_Definition_Class_ID@@YAHPAUlua_State@@@Z 1100c2f0 f   LuaFunctions.obj
 0001:0000b360       ?Lua_Is_Valid_Preset_ID@@YAHPAUlua_State@@@Z 1100c360 f   LuaFunctions.obj
 0001:0000b3d0       ?Lua_Is_Valid_Preset@@YAHPAUlua_State@@@Z 1100c3d0 f   LuaFunctions.obj
 0001:0000b420       ?Lua_Set_Max_Health@@YAHPAUlua_State@@@Z 1100c420 f   LuaFunctions.obj
 0001:0000b4b0       ?Lua_Set_Max_Shield_Strength@@YAHPAUlua_State@@@Z 1100c4b0 f   LuaFunctions.obj
 0001:0000b540       ?Lua_Get_Shield_Type@@YAHPAUlua_State@@@Z 1100c540 f   LuaFunctions.obj
 0001:0000b5d0       ?Lua_Get_Skin@@YAHPAUlua_State@@@Z 1100c5d0 f   LuaFunctions.obj
 0001:0000b650       ?Lua_Set_Skin@@YAHPAUlua_State@@@Z 1100c650 f   LuaFunctions.obj
 0001:0000b6a0       ?Lua_Power_Base@@YAHPAUlua_State@@@Z 1100c6a0 f   LuaFunctions.obj
 0001:0000b700       ?Lua_Set_Can_Generate_Soldiers@@YAHPAUlua_State@@@Z 1100c700 f   LuaFunctions.obj
 0001:0000b760       ?Lua_Set_Can_Generate_Vehicles@@YAHPAUlua_State@@@Z 1100c760 f   LuaFunctions.obj
 0001:0000b7c0       ?Lua_Destroy_Base@@YAHPAUlua_State@@@Z 1100c7c0 f   LuaFunctions.obj
 0001:0000b7f0       ?Lua_Beacon_Destroyed_Base@@YAHPAUlua_State@@@Z 1100c7f0 f   LuaFunctions.obj
 0001:0000b850       ?Lua_Enable_Base_Radar@@YAHPAUlua_State@@@Z 1100c850 f   LuaFunctions.obj
 0001:0000b8b0       ?Lua_Is_Harvester@@YAHPAUlua_State@@@Z 1100c8b0 f   LuaFunctions.obj
 0001:0000b900       ?Lua_Is_Radar_Enabled@@YAHPAUlua_State@@@Z 1100c900 f   LuaFunctions.obj
 0001:0000b950       ?Lua_Building_Type@@YAHPAUlua_State@@@Z 1100c950 f   LuaFunctions.obj
 0001:0000b9b0       ?Lua_Is_Building_Dead@@YAHPAUlua_State@@@Z 1100c9b0 f   LuaFunctions.obj
 0001:0000ba40       ?Lua_Find_Building@@YAHPAUlua_State@@@Z 1100ca40 f   LuaFunctions.obj
 0001:0000bac0       ?Lua_Find_Base_Defense@@YAHPAUlua_State@@@Z 1100cac0 f   LuaFunctions.obj
 0001:0000bb30       ?Lua_Is_Map_Flying@@YAHPAUlua_State@@@Z 1100cb30 f   LuaFunctions.obj
 0001:0000bb60       ?Lua_Find_Harvester@@YAHPAUlua_State@@@Z 1100cb60 f   LuaFunctions.obj
 0001:0000bbd0       ?Lua_Is_Base_Powered@@YAHPAUlua_State@@@Z 1100cbd0 f   LuaFunctions.obj
 0001:0000bc20       ?Lua_Can_Generate_Vehicles@@YAHPAUlua_State@@@Z 1100cc20 f   LuaFunctions.obj
 0001:0000bc70       ?Lua_Can_Generate_Soliders@@YAHPAUlua_State@@@Z 1100cc70 f   LuaFunctions.obj
 0001:0000bcc0       ?Lua_Is_A_Building@@YAHPAUlua_State@@@Z 1100ccc0 f   LuaFunctions.obj
 0001:0000bd30       ?Lua_Get_Building_Count_Team@@YAHPAUlua_State@@@Z 1100cd30 f   LuaFunctions.obj
 0001:0000bd70       ?Lua_Find_Building_By_Team@@YAHPAUlua_State@@@Z 1100cd70 f   LuaFunctions.obj
 0001:0000bd70       ?Lua_Find_Building_By_Name@@YAHPAUlua_State@@@Z 1100cd70 f   LuaFunctions.obj
 0001:0000bdd0       ?Lua_Find_Power_Plant@@YAHPAUlua_State@@@Z 1100cdd0 f   LuaFunctions.obj
 0001:0000be40       ?Lua_Find_Refinery@@YAHPAUlua_State@@@Z 1100ce40 f   LuaFunctions.obj
 0001:0000beb0       ?Lua_Find_Repair_Bay@@YAHPAUlua_State@@@Z 1100ceb0 f   LuaFunctions.obj
 0001:0000bf20       ?Lua_Find_Soldier_Factory@@YAHPAUlua_State@@@Z 1100cf20 f   LuaFunctions.obj
 0001:0000bf90       ?Lua_Find_Airstrip@@YAHPAUlua_State@@@Z 1100cf90 f   LuaFunctions.obj
 0001:0000c000       ?Lua_Find_War_Factory@@YAHPAUlua_State@@@Z 1100d000 f   LuaFunctions.obj
 0001:0000c070       ?Lua_Find_Vehicle_Factory@@YAHPAUlua_State@@@Z 1100d070 f   LuaFunctions.obj
 0001:0000c0e0       ?Lua_Find_Com_Center@@YAHPAUlua_State@@@Z 1100d0e0 f   LuaFunctions.obj
 0001:0000c150       ?Lua_Is_Gameplay_Permitted@@YAHPAUlua_State@@@Z 1100d150 f   LuaFunctions.obj
 0001:0000c190       ?Lua_Is_Dedicated@@YAHPAUlua_State@@@Z 1100d190 f   LuaFunctions.obj
 0001:0000c1c0       ?Lua_Is_Linux@@YAHPAUlua_State@@@Z 1100d1c0 f   LuaFunctions.obj
 0001:0000c200       ?Lua_Get_Current_Game_Mode@@YAHPAUlua_State@@@Z 1100d200 f   LuaFunctions.obj
 0001:0000c240       ?Lua_Get_Harvester_Preset_ID@@YAHPAUlua_State@@@Z 1100d240 f   LuaFunctions.obj
 0001:0000c2b0       ?Lua_Is_Harvester_Preset@@YAHPAUlua_State@@@Z 1100d2b0 f   LuaFunctions.obj
 0001:0000c300       ?Lua_Destroy_Connection@@YAHPAUlua_State@@@Z 1100d300 f   LuaFunctions.obj
 0001:0000c320       ?Lua_Get_IP_Address@@YAHPAUlua_State@@@Z 1100d320 f   LuaFunctions.obj
 0001:0000c360       ?Lua_Get_IP_Port@@YAHPAUlua_State@@@Z 1100d360 f   LuaFunctions.obj
 0001:0000c3a0       ?Lua_Get_Bandwidth@@YAHPAUlua_State@@@Z 1100d3a0 f   LuaFunctions.obj
 0001:0000c400       ?Lua_Get_Ping@@YAHPAUlua_State@@@Z 1100d400 f   LuaFunctions.obj
 0001:0000c470       ?Lua_Get_Kbits@@YAHPAUlua_State@@@Z 1100d470 f   LuaFunctions.obj
 0001:0000c4f0       ?Lua_Get_Object_Type@@YAHPAUlua_State@@@Z 1100d4f0 f   LuaFunctions.obj
 0001:0000c580       ?Lua_Set_Object_Type@@YAHPAUlua_State@@@Z 1100d580 f   LuaFunctions.obj
 0001:0000c5f0       ?Lua_Is_Building@@YAHPAUlua_State@@@Z 1100d5f0 f   LuaFunctions.obj
 0001:0000c660       ?Lua_Is_Soldier@@YAHPAUlua_State@@@Z 1100d660 f   LuaFunctions.obj
 0001:0000c6d0       ?Lua_Is_Vehicle@@YAHPAUlua_State@@@Z 1100d6d0 f   LuaFunctions.obj
 0001:0000c740       ?Lua_Is_Cinematic@@YAHPAUlua_State@@@Z 1100d740 f   LuaFunctions.obj
 0001:0000c7c0       ?Lua_Is_ScriptZone@@YAHPAUlua_State@@@Z 1100d7c0 f   LuaFunctions.obj
 0001:0000c830       ?Lua_Is_Powerup@@YAHPAUlua_State@@@Z 1100d830 f   LuaFunctions.obj
 0001:0000c8b0       ?Lua_Is_C4@@YAHPAUlua_State@@@Z 1100d8b0 f   LuaFunctions.obj
 0001:0000c930       ?Lua_Is_Beacon@@YAHPAUlua_State@@@Z 1100d930 f   LuaFunctions.obj
 0001:0000c9b0       ?Lua_Is_Armed@@YAHPAUlua_State@@@Z 1100d9b0 f   LuaFunctions.obj
 0001:0000ca30       ?Lua_Is_Simple@@YAHPAUlua_State@@@Z 1100da30 f   LuaFunctions.obj
 0001:0000cab0       ?Lua_Is_PowerPlant@@YAHPAUlua_State@@@Z 1100dab0 f   LuaFunctions.obj
 0001:0000cb00       ?Lua_Is_SoldierFactory@@YAHPAUlua_State@@@Z 1100db00 f   LuaFunctions.obj
 0001:0000cb50       ?Lua_Is_VehicleFactory@@YAHPAUlua_State@@@Z 1100db50 f   LuaFunctions.obj
 0001:0000cba0       ?Lua_Is_Airstrip@@YAHPAUlua_State@@@Z 1100dba0 f   LuaFunctions.obj
 0001:0000cbf0       ?Lua_Is_WarFactory@@YAHPAUlua_State@@@Z 1100dbf0 f   LuaFunctions.obj
 0001:0000cc40       ?Lua_Is_Refinery@@YAHPAUlua_State@@@Z 1100dc40 f   LuaFunctions.obj
 0001:0000cc90       ?Lua_Is_ComCenter@@YAHPAUlua_State@@@Z 1100dc90 f   LuaFunctions.obj
 0001:0000cce0       ?Lua_Is_RepairBay@@YAHPAUlua_State@@@Z 1100dce0 f   LuaFunctions.obj
 0001:0000cd30       ?Lua_Is_Scriptable@@YAHPAUlua_State@@@Z 1100dd30 f   LuaFunctions.obj
 0001:0000cda0       ?Lua_Get_Building_Type@@YAHPAUlua_State@@@Z 1100dda0 f   LuaFunctions.obj
 0001:0000cde0       ?Lua_Get_Object_Count@@YAHPAUlua_State@@@Z 1100dde0 f   LuaFunctions.obj
 0001:0000ce40       ?Lua_Find_Random_Preset@@YAHPAUlua_State@@@Z 1100de40 f   LuaFunctions.obj
 0001:0000cee0       ?Lua_Send_Custom_To_Team_Buildings@@YAHPAUlua_State@@@Z 1100dee0 f   LuaFunctions.obj
 0001:0000cf60       ?Lua_Send_Custom_To_Team_Preset@@YAHPAUlua_State@@@Z 1100df60 f   LuaFunctions.obj
 0001:0000d000       ?Lua_Send_Custom_All_Objects@@YAHPAUlua_State@@@Z 1100e000 f   LuaFunctions.obj
 0001:0000d060       ?Lua_Send_Custom_Event_To_Object@@YAHPAUlua_State@@@Z 1100e060 f   LuaFunctions.obj
 0001:0000d0f0       ?Lua_Get_Is_Powerup_Persistant@@YAHPAUlua_State@@@Z 1100e0f0 f   LuaFunctions.obj
 0001:0000d180       ?Lua_Set_Is_Powerup_Persistant@@YAHPAUlua_State@@@Z 1100e180 f   LuaFunctions.obj
 0001:0000d220       ?Lua_Get_Powerup_Always_Allow_Grant@@YAHPAUlua_State@@@Z 1100e220 f   LuaFunctions.obj
 0001:0000d2b0       ?Lua_Set_Powerup_Always_Allow_Grant@@YAHPAUlua_State@@@Z 1100e2b0 f   LuaFunctions.obj
 0001:0000d350       ?Lua_Get_Powerup_Grant_Sound@@YAHPAUlua_State@@@Z 1100e350 f   LuaFunctions.obj
 0001:0000d3f0       ?Lua_Set_Powerup_Grant_Sound@@YAHPAUlua_State@@@Z 1100e3f0 f   LuaFunctions.obj
 0001:0000d480       ?Lua_Grant_Powerup@@YAHPAUlua_State@@@Z 1100e480 f   LuaFunctions.obj
 0001:0000d4d0       ?Lua_Get_Vehicle@@YAHPAUlua_State@@@Z 1100e4d0 f   LuaFunctions.obj
 0001:0000d580       ?Lua_Grant_Refill@@YAHPAUlua_State@@@Z 1100e580 f   LuaFunctions.obj
 0001:0000d5f0       ?Lua_Change_Character@@YAHPAUlua_State@@@Z 1100e5f0 f   LuaFunctions.obj
 0001:0000d670       ?Lua_Create_Vehicle@@YAHPAUlua_State@@@Z 1100e670 f   LuaFunctions.obj
 0001:0000d6f0       ?Lua_Toggle_Fly_Mode@@YAHPAUlua_State@@@Z 1100e6f0 f   LuaFunctions.obj
 0001:0000d720       ?Lua_Get_Vehicle_Occupant_Count@@YAHPAUlua_State@@@Z 1100e720 f   LuaFunctions.obj
 0001:0000d780       ?Lua_Get_Vehicle_Occupant@@YAHPAUlua_State@@@Z 1100e780 f   LuaFunctions.obj
 0001:0000d850       ?Lua_Get_Vehicle_Driver@@YAHPAUlua_State@@@Z 1100e850 f   LuaFunctions.obj
 0001:0000d910       ?Lua_Get_Vehicle_Gunner@@YAHPAUlua_State@@@Z 1100e910 f   LuaFunctions.obj
 0001:0000d990       ?Lua_Force_Occupant_Exit@@YAHPAUlua_State@@@Z 1100e990 f   LuaFunctions.obj
 0001:0000d9e0       ?Lua_Force_Occupants_Exit@@YAHPAUlua_State@@@Z 1100e9e0 f   LuaFunctions.obj
 0001:0000da20       ?Lua_Get_Vehicle_Return@@YAHPAUlua_State@@@Z 1100ea20 f   LuaFunctions.obj
 0001:0000dae0       ?Lua_Is_Stealth@@YAHPAUlua_State@@@Z 1100eae0 f   LuaFunctions.obj
 0001:0000db70       ?Lua_Get_Fly_Mode@@YAHPAUlua_State@@@Z 1100eb70 f   LuaFunctions.obj
 0001:0000dc10       ?Lua_Get_Vehicle_Seat_Count@@YAHPAUlua_State@@@Z 1100ec10 f   LuaFunctions.obj
 0001:0000dcb0       ?Lua_Get_Spawn_Char@@YAHPAUlua_State@@@Z 1100ecb0 f   LuaFunctions.obj
 0001:0000dd00       ?Lua_Change_Spawn_Char@@YAHPAUlua_State@@@Z 1100ed00 f   LuaFunctions.obj
 0001:0000dd40       ?Lua_Soldier_Transition_Vehicle@@YAHPAUlua_State@@@Z 1100ed40 f   LuaFunctions.obj
 0001:0000ddb0       ?Lua_Get_Vehicle_Mode@@YAHPAUlua_State@@@Z 1100edb0 f   LuaFunctions.obj
 0001:0000de10       ?Lua_Get_Team_Vehicle_Count@@YAHPAUlua_State@@@Z 1100ee10 f   LuaFunctions.obj
 0001:0000de80       ?Lua_Get_Vehicle_Owner@@YAHPAUlua_State@@@Z 1100ee80 f   LuaFunctions.obj
 0001:0000df30       ?Lua_Force_Occupants_Exit_Team@@YAHPAUlua_State@@@Z 1100ef30 f   LuaFunctions.obj
 0001:0000df80       ?Lua_Get_Vehicle_Definition_Mode@@YAHPAUlua_State@@@Z 1100ef80 f   LuaFunctions.obj
 0001:0000dff0       ?Lua_IsInsideZone@@YAHPAUlua_State@@@Z 1100eff0 f   LuaFunctions.obj
 0001:0000e060       ?Lua_Get_Vehicle_Definition_Mode_By_ID@@YAHPAUlua_State@@@Z 1100f060 f   LuaFunctions.obj
 0001:0000e0e0       ?Lua_Get_Zone_Type@@YAHPAUlua_State@@@Z 1100f0e0 f   LuaFunctions.obj
 0001:0000e140       ?Lua_IsAvailableForPurchase@@YAHPAUlua_State@@@Z 1100f140 f   LuaFunctions.obj
 0001:0000e1a0       ?Lua_Check_Transitions@@YAHPAUlua_State@@@Z 1100f1a0 f   LuaFunctions.obj
 0001:0000e220       ?Lua_Get_Vehicle_Gunner_Pos@@YAHPAUlua_State@@@Z 1100f220 f   LuaFunctions.obj
 0001:0000e2e0       ?Lua_Set_Vehicle_Is_Visible@@YAHPAUlua_State@@@Z 1100f2e0 f   LuaFunctions.obj
 0001:0000e340       ?Lua_Set_Vehicle_Gunner@@YAHPAUlua_State@@@Z 1100f340 f   LuaFunctions.obj
 0001:0000e390       ?Lua_Get_Model@@YAHPAUlua_State@@@Z 1100f390 f   LuaFunctions.obj
 0001:0000e3d0       ?Lua_Get_Animation_Frame@@YAHPAUlua_State@@@Z 1100f3d0 f   LuaFunctions.obj
 0001:0000e450       ?Lua_Is_TrackedVehicle@@YAHPAUlua_State@@@Z 1100f450 f   LuaFunctions.obj
 0001:0000e4a0       ?Lua_Is_VTOLVehicle@@YAHPAUlua_State@@@Z 1100f4a0 f   LuaFunctions.obj
 0001:0000e4f0       ?Lua_Is_WheeledVehicle@@YAHPAUlua_State@@@Z 1100f4f0 f   LuaFunctions.obj
 0001:0000e540       ?Lua_Is_Motorcycle@@YAHPAUlua_State@@@Z 1100f540 f   LuaFunctions.obj
 0001:0000e590       ?Lua_Is_Door@@YAHPAUlua_State@@@Z 1100f590 f   LuaFunctions.obj
 0001:0000e5e0       ?Lua_Is_Elevator@@YAHPAUlua_State@@@Z 1100f5e0 f   LuaFunctions.obj
 0001:0000e630       ?Lua_Is_DamageableStaticPhys@@YAHPAUlua_State@@@Z 1100f630 f   LuaFunctions.obj
 0001:0000e680       ?Lua_Is_AccessablePhys@@YAHPAUlua_State@@@Z 1100f680 f   LuaFunctions.obj
 0001:0000e6d0       ?Lua_Is_DecorationPhys@@YAHPAUlua_State@@@Z 1100f6d0 f   LuaFunctions.obj
 0001:0000e720       ?Lua_Is_HumanPhys@@YAHPAUlua_State@@@Z 1100f720 f   LuaFunctions.obj
 0001:0000e770       ?Lua_Is_MotorVehicle@@YAHPAUlua_State@@@Z 1100f770 f   LuaFunctions.obj
 0001:0000e7c0       ?Lua_Is_Phys3@@YAHPAUlua_State@@@Z 1100f7c0 f   LuaFunctions.obj
 0001:0000e810       ?Lua_Is_RigidBody@@YAHPAUlua_State@@@Z 1100f810 f   LuaFunctions.obj
 0001:0000e860       ?Lua_Is_ShakeableStatricPhys@@YAHPAUlua_State@@@Z 1100f860 f   LuaFunctions.obj
 0001:0000e8b0       ?Lua_Is_StaticAnimPhys@@YAHPAUlua_State@@@Z 1100f8b0 f   LuaFunctions.obj
 0001:0000e900       ?Lua_Is_StaticPhys@@YAHPAUlua_State@@@Z 1100f900 f   LuaFunctions.obj
 0001:0000e950       ?Lua_Is_TimedDecorationPhys@@YAHPAUlua_State@@@Z 1100f950 f   LuaFunctions.obj
 0001:0000e9a0       ?Lua_Is_VehiclePhys@@YAHPAUlua_State@@@Z 1100f9a0 f   LuaFunctions.obj
 0001:0000ea00       ?Lua_Is_DynamicAnimPhys@@YAHPAUlua_State@@@Z 1100fa00 f   LuaFunctions.obj
 0001:0000ea50       ?Lua_Is_BuildingAggregate@@YAHPAUlua_State@@@Z 1100fa50 f   LuaFunctions.obj
 0001:0000eaa0       ?Lua_Is_Projectile@@YAHPAUlua_State@@@Z 1100faa0 f   LuaFunctions.obj
 0001:0000eaf0       ?Lua_Get_Physics@@YAHPAUlua_State@@@Z 1100faf0 f   LuaFunctions.obj
 0001:0000eb30       ?Lua_Copy_Transform@@YAHPAUlua_State@@@Z 1100fb30 f   LuaFunctions.obj
 0001:0000eb90       ?Lua_Get_Mass@@YAHPAUlua_State@@@Z 1100fb90 f   LuaFunctions.obj
 0001:0000ec10       ?Lua_Get_Htree_Name@@YAHPAUlua_State@@@Z 1100fc10 f   LuaFunctions.obj
 0001:0000ec50       ?Lua_Get_Sex@@YAHPAUlua_State@@@Z 1100fc50 f   LuaFunctions.obj
 0001:0000ecb0       ?Lua_Create_Effect_All_Of_Preset@@YAHPAUlua_State@@@Z 1100fcb0 f   LuaFunctions.obj
 0001:0000ed30       ?Lua_Get_GameObj@@YAHPAUlua_State@@@Z 1100fd30 f   LuaFunctions.obj
 0001:0000eda0       ?Lua_Get_Player_ID@@YAHPAUlua_State@@@Z 1100fda0 f   LuaFunctions.obj
 0001:0000ee40       ?Lua_Get_Player_Name@@YAHPAUlua_State@@@Z 1100fe40 f   LuaFunctions.obj
 0001:0000eea0       ?Lua_Get_Player_Name_By_ID@@YAHPAUlua_State@@@Z 1100fea0 f   LuaFunctions.obj
 0001:0000ef00       ?Lua_Change_Team@@YAHPAUlua_State@@@Z 1100ff00 f   LuaFunctions.obj
 0001:0000ef50       ?Lua_Change_Team_By_ID@@YAHPAUlua_State@@@Z 1100ff50 f   LuaFunctions.obj
 0001:0000efd0       ?Lua_Get_Player_Count@@YAHPAUlua_State@@@Z 1100ffd0 f   LuaFunctions.obj
 0001:0000f010       ?Lua_Get_Team_Player_Count@@YAHPAUlua_State@@@Z 11010010 f   LuaFunctions.obj
 0001:0000f060       ?Lua_Get_Team@@YAHPAUlua_State@@@Z 11010060 f   LuaFunctions.obj
 0001:0000f0c0       ?Lua_Get_Rank@@YAHPAUlua_State@@@Z 110100c0 f   LuaFunctions.obj
 0001:0000f120       ?Lua_Get_Kills@@YAHPAUlua_State@@@Z 11010120 f   LuaFunctions.obj
 0001:0000f180       ?Lua_Get_Deaths@@YAHPAUlua_State@@@Z 11010180 f   LuaFunctions.obj
 0001:0000f1e0       ?Lua_Get_Score@@YAHPAUlua_State@@@Z 110101e0 f   LuaFunctions.obj
 0001:0000f230       ?Lua_Get_Money@@YAHPAUlua_State@@@Z 11010230 f   LuaFunctions.obj
 0001:0000f280       ?Lua_Get_Kill_To_Death_Ratio@@YAHPAUlua_State@@@Z 11010280 f   LuaFunctions.obj
 0001:0000f2c0       ?Lua_Get_Part_Name@@YAHPAUlua_State@@@Z 110102c0 f   LuaFunctions.obj
 0001:0000f320       ?Lua_Get_Part_Names@@YAHPAUlua_State@@@Z 11010320 f   LuaFunctions.obj
 0001:0000f370       ?Lua_Get_GameObj_By_Player_Name@@YAHPAUlua_State@@@Z 11010370 f   LuaFunctions.obj
 0001:0000f3e0       ?Lua_Purchase_Item@@YAHPAUlua_State@@@Z 110103e0 f   LuaFunctions.obj
 0001:0000f490       ?Lua_Set_Ladder_Points@@YAHPAUlua_State@@@Z 11010490 f   LuaFunctions.obj
 0001:0000f4e0       ?Lua_Set_Rung@@YAHPAUlua_State@@@Z 110104e0 f   LuaFunctions.obj
 0001:0000f530       ?Lua_Set_Money@@YAHPAUlua_State@@@Z 11010530 f   LuaFunctions.obj
 0001:0000f580       ?Lua_Set_Score@@YAHPAUlua_State@@@Z 11010580 f   LuaFunctions.obj
 0001:0000f5d0       ?Lua_Find_First_Player@@YAHPAUlua_State@@@Z 110105d0 f   LuaFunctions.obj
 0001:0000f630       ?Lua_Change_Player_Team@@YAHPAUlua_State@@@Z 11010630 f   LuaFunctions.obj
 0001:0000f6f0       ?Lua_Tally_Team_Size@@YAHPAUlua_State@@@Z 110106f0 f   LuaFunctions.obj
 0001:0000f740       ?Lua_Get_Team_Score@@YAHPAUlua_State@@@Z 11010740 f   LuaFunctions.obj
 0001:0000f790       ?Lua_Send_Custom_All_Players@@YAHPAUlua_State@@@Z 11010790 f   LuaFunctions.obj
 0001:0000f7f0       ?Lua_Steal_Team_Credits@@YAHPAUlua_State@@@Z 110107f0 f   LuaFunctions.obj
 0001:0000f840       ?Lua_Get_Team_Credits@@YAHPAUlua_State@@@Z 11010840 f   LuaFunctions.obj
 0001:0000f880       ?Lua_Change_Team_2@@YAHPAUlua_State@@@Z 11010880 f   LuaFunctions.obj
 0001:0000f910       ?Lua_Get_Player_Type@@YAHPAUlua_State@@@Z 11010910 f   LuaFunctions.obj
 0001:0000f9c0       ?Lua_Get_Team_Cost@@YAHPAUlua_State@@@Z 110109c0 f   LuaFunctions.obj
 0001:0000fa50       ?Lua_Get_Cost@@YAHPAUlua_State@@@Z 11010a50 f   LuaFunctions.obj
 0001:0000fac0       ?Lua_Set_Enlisted@@YAHPAUlua_State@@@Z 11010ac0 f   LuaFunctions.obj
 0001:0000fbd0       ?Lua_Set_Beacon@@YAHPAUlua_State@@@Z 11010bd0 f   LuaFunctions.obj
 0001:0000fce0       ?Lua_Set_Refill@@YAHPAUlua_State@@@Z 11010ce0 f   LuaFunctions.obj
 0001:0000fd80       ?Lua_Set_Preset@@YAHPAUlua_State@@@Z 11010d80 f   LuaFunctions.obj
 0001:0000ff10       ?Lua_Set_Alternate@@YAHPAUlua_State@@@Z 11010f10 f   LuaFunctions.obj
 0001:00010070       ?Lua_Disable_Enlisted@@YAHPAUlua_State@@@Z 11011070 f   LuaFunctions.obj
 0001:00010110       ?Lua_Disable_Preset@@YAHPAUlua_State@@@Z 11011110 f   LuaFunctions.obj
 0001:000101c0       ?Lua_Disable_Enlisted_By_Name@@YAHPAUlua_State@@@Z 110111c0 f   LuaFunctions.obj
 0001:00010220       ?Lua_Disable_Preset_By_Name@@YAHPAUlua_State@@@Z 11011220 f   LuaFunctions.obj
 0001:00010280       ?Lua_Disable_All_Ground_Vehicles@@YAHPAUlua_State@@@Z 11011280 f   LuaFunctions.obj
 0001:000102c0       ?Lua_Disable_All_Flying_Vehicles@@YAHPAUlua_State@@@Z 110112c0 f   LuaFunctions.obj
 0001:00010300       ?Lua_Get_Team_Icon@@YAHPAUlua_State@@@Z 11011300 f   LuaFunctions.obj
 0001:00010370       ?Lua_Get_Icon@@YAHPAUlua_State@@@Z 11011370 f   LuaFunctions.obj
 0001:000103c0       ?Lua_Remove_Script@@YAHPAUlua_State@@@Z 110113c0 f   LuaFunctions.obj
 0001:00010410       ?Lua_Remove_All_Scripts@@YAHPAUlua_State@@@Z 11011410 f   LuaFunctions.obj
 0001:00010440       ?Lua_Attach_Script_Preset@@YAHPAUlua_State@@@Z 11011440 f   LuaFunctions.obj
 0001:000104b0       ?Lua_Attach_Script_Type@@YAHPAUlua_State@@@Z 110114b0 f   LuaFunctions.obj
 0001:00010540       ?Lua_Remove_Script_Preset@@YAHPAUlua_State@@@Z 11011540 f   LuaFunctions.obj
 0001:00010590       ?Lua_Remove_Script_Type@@YAHPAUlua_State@@@Z 11011590 f   LuaFunctions.obj
 0001:00010610       ?Lua_Is_Script_Attached@@YAHPAUlua_State@@@Z 11011610 f   LuaFunctions.obj
 0001:00010680       ?Lua_Attach_Script_Once@@YAHPAUlua_State@@@Z 11011680 f   LuaFunctions.obj
 0001:00010710       ?Lua_Attach_Script_Preset_Once@@YAHPAUlua_State@@@Z 11011710 f   LuaFunctions.obj
 0001:00010780       ?Lua_Attach_Script_Type_Once@@YAHPAUlua_State@@@Z 11011780 f   LuaFunctions.obj
 0001:00010810       ?Lua_Attach_Script_Building@@YAHPAUlua_State@@@Z 11011810 f   LuaFunctions.obj
 0001:00010860       ?Lua_Attach_Script_Is_Preset@@YAHPAUlua_State@@@Z 11011860 f   LuaFunctions.obj
 0001:00010900       ?Lua_Attach_Script_Is_Type@@YAHPAUlua_State@@@Z 11011900 f   LuaFunctions.obj
 0001:000109c0       ?Lua_Attach_Script_Player_Once@@YAHPAUlua_State@@@Z 110119c0 f   LuaFunctions.obj
 0001:00010a10       ?Lua_Remove_Duplicate_Script@@YAHPAUlua_State@@@Z 11011a10 f   LuaFunctions.obj
 0001:00010a60       ?Lua_Attach_Script_All_Buildings_Team@@YAHPAUlua_State@@@Z 11011a60 f   LuaFunctions.obj
 0001:00010ae0       ?Lua_Attach_Script_All_Turrets_Team@@YAHPAUlua_State@@@Z 11011ae0 f   LuaFunctions.obj
 0001:00010b60       ?Lua_Find_Building_With_Script@@YAHPAUlua_State@@@Z 11011b60 f   LuaFunctions.obj
 0001:00010c20       ?Lua_Find_Object_With_Script@@YAHPAUlua_State@@@Z 11011c20 f   LuaFunctions.obj
 0001:00010c90       ?Lua_Get_Translated_String@@YAHPAUlua_State@@@Z 11011c90 f   LuaFunctions.obj
 0001:00010d20       ?Lua_Get_Translated_Preset_Name@@YAHPAUlua_State@@@Z 11011d20 f   LuaFunctions.obj
 0001:00010d70       ?Lua_Get_Translated_Weapon@@YAHPAUlua_State@@@Z 11011d70 f   LuaFunctions.obj
 0001:00010df0       ?Lua_Get_Current_Translated_Weapon@@YAHPAUlua_State@@@Z 11011df0 f   LuaFunctions.obj
 0001:00010ea0       ?Lua_Get_Team_Name@@YAHPAUlua_State@@@Z 11011ea0 f   LuaFunctions.obj
 0001:00010ee0       ?Lua_Get_Vehicle_Name@@YAHPAUlua_State@@@Z 11011ee0 f   LuaFunctions.obj
 0001:00010f90       ?Lua_Get_Translated_Definition_Name@@YAHPAUlua_State@@@Z 11011f90 f   LuaFunctions.obj
 0001:00010ff0       ?Lua_Get_Current_Bullets@@YAHPAUlua_State@@@Z 11011ff0 f   LuaFunctions.obj
 0001:00011050       ?Lua_Get_Current_Clip_Bullets@@YAHPAUlua_State@@@Z 11012050 f   LuaFunctions.obj
 0001:000110b0       ?Lua_Get_Current_Total_Bullets@@YAHPAUlua_State@@@Z 110120b0 f   LuaFunctions.obj
 0001:00011110       ?Lua_Get_Total_Bullets@@YAHPAUlua_State@@@Z 11012110 f   LuaFunctions.obj
 0001:00011180       ?Lua_Get_Clip_Bullets@@YAHPAUlua_State@@@Z 11012180 f   LuaFunctions.obj
 0001:000111f0       ?Lua_Get_Bullets@@YAHPAUlua_State@@@Z 110121f0 f   LuaFunctions.obj
 0001:00011260       ?Lua_Get_Current_Max_Bullets@@YAHPAUlua_State@@@Z 11012260 f   LuaFunctions.obj
 0001:000112c0       ?Lua_Get_Current_Clip_Max_Bullets@@YAHPAUlua_State@@@Z 110122c0 f   LuaFunctions.obj
 0001:00011320       ?Lua_Get_Current_Total_Max_Bullets@@YAHPAUlua_State@@@Z 11012320 f   LuaFunctions.obj
 0001:00011380       ?Lua_Get_Max_Total_Bullets@@YAHPAUlua_State@@@Z 11012380 f   LuaFunctions.obj
 0001:00011380       ?Lua_Get_Max_Clip_Bullets@@YAHPAUlua_State@@@Z 11012380 f   LuaFunctions.obj
 0001:000113f0       ?Lua_Get_Max_Bullets@@YAHPAUlua_State@@@Z 110123f0 f   LuaFunctions.obj
 0001:00011460       ?Lua_Get_Position_Total_Bullets@@YAHPAUlua_State@@@Z 11012460 f   LuaFunctions.obj
 0001:000114d0       ?Lua_Get_Position_Bullets@@YAHPAUlua_State@@@Z 110124d0 f   LuaFunctions.obj
 0001:00011590       ?Lua_Get_Position_Clip_Bullets@@YAHPAUlua_State@@@Z 11012590 f   LuaFunctions.obj
 0001:00011650       ?Lua_Get_Position_Total_Max_Bullets@@YAHPAUlua_State@@@Z 11012650 f   LuaFunctions.obj
 0001:000116c0       ?Lua_Get_Position_Max_Bullets@@YAHPAUlua_State@@@Z 110126c0 f   LuaFunctions.obj
 0001:00011730       ?Lua_Get_Position_Clip_Max_Bullets@@YAHPAUlua_State@@@Z 11012730 f   LuaFunctions.obj
 0001:000117a0       ?Lua_Set_Current_Bullets@@YAHPAUlua_State@@@Z 110127a0 f   LuaFunctions.obj
 0001:000117f0       ?Lua_Set_Current_Clip_Bullets@@YAHPAUlua_State@@@Z 110127f0 f   LuaFunctions.obj
 0001:00011840       ?Lua_Set_Position_Bullets@@YAHPAUlua_State@@@Z 11012840 f   LuaFunctions.obj
 0001:000118a0       ?Lua_Set_Position_Clip_Bullets@@YAHPAUlua_State@@@Z 110128a0 f   LuaFunctions.obj
 0001:00011900       ?Lua_Set_Bullets@@YAHPAUlua_State@@@Z 11012900 f   LuaFunctions.obj
 0001:00011970       ?Lua_Set_Clip_Bullets@@YAHPAUlua_State@@@Z 11012970 f   LuaFunctions.obj
 0001:000119e0       ?Lua_Get_Powerup_Weapon@@YAHPAUlua_State@@@Z 110129e0 f   LuaFunctions.obj
 0001:00011a60       ?Lua_Get_Powerup_Weapon_By_Obj@@YAHPAUlua_State@@@Z 11012a60 f   LuaFunctions.obj
 0001:00011af0       ?Lua_Get_Current_Weapon_Style@@YAHPAUlua_State@@@Z 11012af0 f   LuaFunctions.obj
 0001:00011b50       ?Lua_Disarm_Beacon@@YAHPAUlua_State@@@Z 11012b50 f   LuaFunctions.obj
 0001:00011bc0       ?Lua_Disarm_Beacons@@YAHPAUlua_State@@@Z 11012bc0 f   LuaFunctions.obj
 0001:00011be0       ?Lua_Disarm_Nearest_Beacon@@YAHPAUlua_State@@@Z 11012be0 f   LuaFunctions.obj
 0001:00011c50       ?Lua_Disarm_C4@@YAHPAUlua_State@@@Z 11012c50 f   LuaFunctions.obj
 0001:00011cc0       ?Lua_Disarm_All_Proxy_C4@@YAHPAUlua_State@@@Z 11012cc0 f   LuaFunctions.obj
 0001:00011ce0       ?Lua_Disarm_All_C4@@YAHPAUlua_State@@@Z 11012ce0 f   LuaFunctions.obj
 0001:00011d00       ?Lua_Get_Current_Weapon@@YAHPAUlua_State@@@Z 11012d00 f   LuaFunctions.obj
 0001:00011d40       ?Lua_Get_Weapon_Count@@YAHPAUlua_State@@@Z 11012d40 f   LuaFunctions.obj
 0001:00011de0       ?Lua_Get_Weapon@@YAHPAUlua_State@@@Z 11012de0 f   LuaFunctions.obj
 0001:00011e40       ?Lua_Has_Weapon@@YAHPAUlua_State@@@Z 11012e40 f   LuaFunctions.obj
 0001:00011ec0       ?Lua_Find_Beacon@@YAHPAUlua_State@@@Z 11012ec0 f   LuaFunctions.obj
 0001:00011f40       ?Lua_Get_C4_Count@@YAHPAUlua_State@@@Z 11012f40 f   LuaFunctions.obj
 0001:00011f90       ?Lua_Get_Beacon_Count@@YAHPAUlua_State@@@Z 11012f90 f   LuaFunctions.obj
 0001:00011fe0       ?Lua_Get_Mine_Limit@@YAHPAUlua_State@@@Z 11012fe0 f   LuaFunctions.obj
 0001:00012020       ?Lua_Get_C4_Mode@@YAHPAUlua_State@@@Z 11013020 f   LuaFunctions.obj
 0001:000120c0       ?Lua_Get_C4_Count_Proximity@@YAHPAUlua_State@@@Z 110130c0 f   LuaFunctions.obj
 0001:00012110       ?Lua_Get_C4_Count_Remote@@YAHPAUlua_State@@@Z 11013110 f   LuaFunctions.obj
 0001:00012160       ?Lua_Get_C4_Planter@@YAHPAUlua_State@@@Z 11013160 f   LuaFunctions.obj
 0001:00012210       ?Lua_Get_C4_Attached@@YAHPAUlua_State@@@Z 11013210 f   LuaFunctions.obj
 0001:000122c0       ?Lua_Get_Beacon_Planter@@YAHPAUlua_State@@@Z 110132c0 f   LuaFunctions.obj
 0001:00012370       ?Lua_Create_Object@@YAHPAUlua_State@@@Z 11013370 f   LuaFunctions.obj
 0001:00012410       ?Lua_Destroy_Object@@YAHPAUlua_State@@@Z 11013410 f   LuaFunctions.obj
 0001:00012440       ?Lua_Get_Preset_Name@@YAHPAUlua_State@@@Z 11013440 f   LuaFunctions.obj
 0001:00012490       ?Lua_Get_Position@@YAHPAUlua_State@@@Z 11013490 f   LuaFunctions.obj
 0001:000125f0       ?Lua_Enable_Vehicle_Transitions@@YAHPAUlua_State@@@Z 110135f0 f   LuaFunctions.obj
 0001:00012650       ?Lua_Set_Model@@YAHPAUlua_State@@@Z 11013650 f   LuaFunctions.obj
 0001:000126a0       ?Lua_Goto_Location@@YAHPAUlua_State@@@Z 110136a0 f   LuaFunctions.obj
 0001:00012790       ?Lua_Goto_Object@@YAHPAUlua_State@@@Z 11013790 f   LuaFunctions.obj
 0001:00012830       ?Lua_Disable_Physical_Collisions@@YAHPAUlua_State@@@Z 11013830 f   LuaFunctions.obj
 0001:00012860       ?Lua_Enable_Collisions@@YAHPAUlua_State@@@Z 11013860 f   LuaFunctions.obj
 0001:00012890       ?Lua_Random_Building@@YAHPAUlua_State@@@Z 11013890 f   LuaFunctions.obj
 0001:00012960       ?Lua_Get_Current_Map@@YAHPAUlua_State@@@Z 11013960 f   LuaFunctions.obj
 0001:00012980       ?Lua_Get_Next_Map@@YAHPAUlua_State@@@Z 11013980 f   LuaFunctions.obj
 0001:000129f0       ?Lua_Set_Position@@YAHPAUlua_State@@@Z 110139f0 f   LuaFunctions.obj
 0001:00012a70       ?Lua_Apply_Damage@@YAHPAUlua_State@@@Z 11013a70 f   LuaFunctions.obj
 0001:00012b20       ?Lua_Get_Facing@@YAHPAUlua_State@@@Z 11013b20 f   LuaFunctions.obj
 0001:00012b70       ?Lua_Set_Facing@@YAHPAUlua_State@@@Z 11013b70 f   LuaFunctions.obj
 0001:00012bc0       ?Lua_Set_Clouds@@YAHPAUlua_State@@@Z 11013bc0 f   LuaFunctions.obj
 0001:00012c20       ?Lua_Set_Ash@@YAHPAUlua_State@@@Z 11013c20 f   LuaFunctions.obj
 0001:00012c90       ?Lua_Set_Rain@@YAHPAUlua_State@@@Z 11013c90 f   LuaFunctions.obj
 0001:00012c90       ?Lua_Set_Snow@@YAHPAUlua_State@@@Z 11013c90 f   LuaFunctions.obj
 0001:00012d00       ?Lua_Set_Wind@@YAHPAUlua_State@@@Z 11013d00 f   LuaFunctions.obj
 0001:00012d70       ?Lua_Attach_Script@@YAHPAUlua_State@@@Z 11013d70 f   LuaFunctions.obj
 0001:00012de0       ?Lua_Create_Object_At_Bone@@YAHPAUlua_State@@@Z 11013de0 f   LuaFunctions.obj
 0001:00012e90       ?Lua_Attach_To_Object_Bone@@YAHPAUlua_State@@@Z 11013e90 f   LuaFunctions.obj
 0001:00012f10       ?Lua_Display_Health_Bar@@YAHPAUlua_State@@@Z 11013f10 f   LuaFunctions.obj
 0001:00012f80       ?Lua_Create_Script_Zone@@YAHPAUlua_State@@@Z 11013f80 f   LuaFunctions.obj
 0001:000130c0       ?Lua_tClock@@YAHPAUlua_State@@@Z 110140c0 f   LuaFunctions.obj
 0001:00013100       ?Lua_Invoke@@YAHPAUlua_State@@@Z 11014100 f   LuaFunctions.obj
 0001:00013140       ?Lua_RequestSerial@@YAHPAUlua_State@@@Z 11014140 f   LuaFunctions.obj
 0001:000131d0       ?Lua_GetTimeRemaining@@YAHPAUlua_State@@@Z 110141d0 f   LuaFunctions.obj
 0001:00013220       ?Lua_Get_Health@@YAHPAUlua_State@@@Z 11014220 f   LuaFunctions.obj
 0001:00013280       ?Lua_Get_Max_Health@@YAHPAUlua_State@@@Z 11014280 f   LuaFunctions.obj
 0001:000132e0       ?Lua_Get_Shield_Strength@@YAHPAUlua_State@@@Z 110142e0 f   LuaFunctions.obj
 0001:00013340       ?Lua_Get_Max_Shield_Strength@@YAHPAUlua_State@@@Z 11014340 f   LuaFunctions.obj
 0001:000133a0       ?Lua_LongToIP@@YAHPAUlua_State@@@Z 110143a0 f   LuaFunctions.obj
 0001:00013450       ?Lua_IPToLong@@YAHPAUlua_State@@@Z 11014450 f   LuaFunctions.obj
 0001:00013550       ?Lua_Is_A_Star@@YAHPAUlua_State@@@Z 11014550 f   LuaFunctions.obj
 0001:000135e0       ?Lua_Enable_Stealth@@YAHPAUlua_State@@@Z 110145e0 f   LuaFunctions.obj
 0001:00013680       ?Lua_Get_Rotation@@YAHPAUlua_State@@@Z 11014680 f   LuaFunctions.obj
 0001:00013760       ?Lua_Get_All_Players@@YAHPAUlua_State@@@Z 11014760 f   LuaFunctions.obj
 0001:00013810       ?Lua_Get_All_Vehicles@@YAHPAUlua_State@@@Z 11014810 f   LuaFunctions.obj
 0001:00013900       ?Lua_Get_All_Buildings@@YAHPAUlua_State@@@Z 11014900 f   LuaFunctions.obj
 0001:000139b0       ?Lua_Get_All_Objects@@YAHPAUlua_State@@@Z 110149b0 f   LuaFunctions.obj
 0001:00013a60       ?Lua_Display_GDI_Player_Terminal_Player@@YAHPAUlua_State@@@Z 11014a60 f   LuaFunctions.obj
 0001:00013aa0       ?Lua_Display_Nod_Player_Terminal_Player@@YAHPAUlua_State@@@Z 11014aa0 f   LuaFunctions.obj
 0001:00013ae0       ?Lua_Reload_All_Plugins@@YAHPAUlua_State@@@Z 11014ae0 f   LuaFunctions.obj
 0001:00013af0       ?Lua_Set_Health@@YAHPAUlua_State@@@Z 11014af0 f   LuaFunctions.obj
 0001:00013b50       ?Lua_Set_Shield_Strength@@YAHPAUlua_State@@@Z 11014b50 f   LuaFunctions.obj
 0001:00013bb0       ?Lua_cPlayer@@YAHPAUlua_State@@@Z 11014bb0 f   LuaFunctions.obj
 0001:00014c60       ?Lua_The_Game@@YAHPAUlua_State@@@Z 11015c60 f   LuaFunctions.obj
 0001:00015db0       ?Lua_Set_cPlayer@@YAHPAUlua_State@@@Z 11016db0 f   LuaFunctions.obj
 0001:00016b80       ?Lua_Set_The_Game@@YAHPAUlua_State@@@Z 11017b80 f   LuaFunctions.obj
 0001:00017920       ?Lua_Memory_Write@@YAHPAUlua_State@@@Z 11018920 f   LuaFunctions.obj
 0001:00017ab0       ?Lua_Memory_Read@@YAHPAUlua_State@@@Z 11018ab0 f   LuaFunctions.obj
 0001:00017bd0       ?Lua_Set_Shield_Type@@YAHPAUlua_State@@@Z 11018bd0 f   LuaFunctions.obj
 0001:00017c30       ?AddFunctions@@YAXPAUlua_State@@@Z 11018c30 f   LuaFunctions.obj
 0001:0001a7d0       ?Lua_DestroyScript@LuaScriptManager@@SAXPAEH@Z 1101b7d0 f   LuaManager.obj
 0001:0001a820       ?Lua_Get_Float_Parameter@LuaScriptManager@@SAMPAEHPBD@Z 1101b820 f   LuaManager.obj
 0001:0001a8a0       ?Lua_Get_Int_Parameter@LuaScriptManager@@SAHPAEHPBD@Z 1101b8a0 f   LuaManager.obj
 0001:0001a920       ?Lua_Get_String_Parameter@LuaScriptManager@@SAPBDPAEHPBD@Z 1101b920 f   LuaManager.obj
 0001:0001a990       ?Register_Script@LuaScriptManager@@SAHPAUlua_State@@@Z 1101b990 f   LuaManager.obj
 0001:0001ab00       ?Lua_Start_Timer@LuaScriptManager@@SAXPAEHMH@Z 1101bb00 f   LuaManager.obj
 0001:0001ab60       ?Cleanup@LuaScriptManager@@SAXXZ 1101bb60 f   LuaManager.obj
 0001:0001abb0       ?RegisterScriptFunctions@LuaScriptManager@@SAXPAUlua_State@@@Z 1101bbb0 f   LuaManager.obj
 0001:0001ad60       ?Lua_DestroyScript_Wrap@LuaScriptManager@@SAHPAUlua_State@@@Z 1101bd60 f   LuaManager.obj
 0001:0001ae50       ?Lua_Get_Float_Parameter_Wrap@LuaScriptManager@@SAHPAUlua_State@@@Z 1101be50 f   LuaManager.obj
 0001:0001afb0       ?Lua_Get_Int_Parameter_Wrap@LuaScriptManager@@SAHPAUlua_State@@@Z 1101bfb0 f   LuaManager.obj
 0001:0001b110       ?Lua_Get_String_Parameter_Wrap@LuaScriptManager@@SAHPAUlua_State@@@Z 1101c110 f   LuaManager.obj
 0001:0001b190       ?Lua_Start_Timer_Wrap@LuaScriptManager@@SAHPAUlua_State@@@Z 1101c190 f   LuaManager.obj
 0001:0001b350       ?Created@LuaScript@LuaScriptManager@@EAEXPAE@Z 1101c350 f   LuaManager.obj
 0001:0001b4e0       ?Destroyed@LuaScript@LuaScriptManager@@EAEXPAE@Z 1101c4e0 f   LuaManager.obj
 0001:0001b670       ?Killed@LuaScript@LuaScriptManager@@EAEXPAE0@Z 1101c670 f   LuaManager.obj
 0001:0001b830       ?Damaged@LuaScript@LuaScriptManager@@EAEXPAE0M@Z 1101c830 f   LuaManager.obj
 0001:0001b9f0       ?Custom@LuaScript@LuaScriptManager@@EAEXPAEHH0@Z 1101c9f0 f   LuaManager.obj
 0001:0001bbc0       ?Enemy_Seen@LuaScript@LuaScriptManager@@EAEXPAE0@Z 1101cbc0 f   LuaManager.obj
 0001:0001bd80       ?Action_Complete@LuaScript@LuaScriptManager@@EAEXPAEHW4ActionCompleteReason@@@Z 1101cd80 f   LuaManager.obj
 0001:0001bf20       ?Timer_Expired@LuaScript@LuaScriptManager@@EAEXPAEH@Z 1101cf20 f   LuaManager.obj
 0001:0001c0c0       ?Animation_Complete@LuaScript@LuaScriptManager@@EAEXPAEPBD@Z 1101d0c0 f   LuaManager.obj
 0001:0001c260       ?Poked@LuaScript@LuaScriptManager@@EAEXPAE0@Z 1101d260 f   LuaManager.obj
 0001:0001c420       ?Entered@LuaScript@LuaScriptManager@@EAEXPAE0@Z 1101d420 f   LuaManager.obj
 0001:0001c5e0       ?Exited@LuaScript@LuaScriptManager@@EAEXPAE0@Z 1101d5e0 f   LuaManager.obj
 0001:0001c7a0       ?LoadLua@LuaManager@@SAXPBD@Z 1101d7a0 f   LuaManager.obj
 0001:0001c910       ?Cleanup@LuaManager@@SAXXZ 1101d910 f   LuaManager.obj
 0001:0001c950       ?Report_Errors@LuaManager@@SA_NPAUlua_State@@H@Z 1101d950 f   LuaManager.obj
 0001:0001caa0       ?Call_Unload@LuaManager@@SAXXZ 1101daa0 f   LuaManager.obj
 0001:0001cb90       ?Call_Chat_Hook@LuaManager@@SA_NHHAAVWideStringClass@@H@Z 1101db90 f   LuaManager.obj
 0001:0001cd90       ?Call_Host_Hook@LuaManager@@SAXHHPBD@Z 1101dd90 f   LuaManager.obj
 0001:0001cec0       ?Call_Player_Join_Hook@LuaManager@@SAXHPBD@Z 1101dec0 f   LuaManager.obj
 0001:0001cfe0       ?Call_Player_Leave_Hook@LuaManager@@SAXH@Z 1101dfe0 f   LuaManager.obj
 0001:0001d0f0       ?Call_Level_Loaded_Hook@LuaManager@@SAXXZ 1101e0f0 f   LuaManager.obj
 0001:0001d1e0       ?Call_GameOver_Hook@LuaManager@@SAXXZ 1101e1e0 f   LuaManager.obj
 0001:0001d2d0       ?Call_Console_Output_Hook@LuaManager@@SAXPBD@Z 1101e2d0 f   LuaManager.obj
 0001:0001d3e0       ?Call_Version_Hook@LuaManager@@SAXHM@Z 1101e3e0 f   LuaManager.obj
 0001:0001d500       ?Purchase_Hook@LuaManager@@SAXPAVBaseControllerClass@@PAEIIIPBD@Z 1101e500 f   LuaManager.obj
 0001:0001d6a0       ?Call_Object_Hook@LuaManager@@SAXPAXPAE@Z 1101e6a0 f   LuaManager.obj
 0001:0001d7d0       ?Call_DDE_Hook@LuaManager@@SAXPBD@Z 1101e7d0 f   LuaManager.obj
 0001:0001d8e0       ?Call_Think_Hook@LuaManager@@SAXXZ 1101e8e0 f   LuaManager.obj
 0001:0001d9e0       ?Call_Serial_Hook@LuaManager@@SAXHPBD@Z 1101e9e0 f   LuaManager.obj
 0001:0001db00       ?Call_LoadingE_Hook@LuaManager@@SAXH_N@Z 1101eb00 f   LuaManager.obj
 0001:0001dc30       ?Call_Damage_Hook@LuaManager@@SA_NHHHMI@Z 1101ec30 f   LuaManager.obj
 0001:0001ddf0       ?Call_Ping_Hook@LuaManager@@SAXHH@Z 1101edf0 f   LuaManager.obj
 0001:0001df10       ?Call_Suicide_Hook@LuaManager@@SA_NH@Z 1101ef10 f   LuaManager.obj
 0001:0001e090       ?Call_Radio_Hook@LuaManager@@SA_NHHHHH@Z 1101f090 f   LuaManager.obj
 0001:0001e240       ?CallInvoke@LuaManager@@SAXPBD0@Z 1101f240 f   LuaManager.obj
 0001:0001e320       ?Reload_All@LuaManager@@SAXXZ 1101f320 f   LuaManager.obj
 0001:0001e410       ?Connect@LuaSocketManager@@SAHPBDH@Z 1101f410 f   LuaManager.obj
 0001:0001e4c0       ??_GTCPSocket@@QAEPAXI@Z   1101f4c0 f i LuaManager.obj
 0001:0001e4f0       ?Server@LuaSocketManager@@SAHPBDH@Z 1101f4f0 f   LuaManager.obj
 0001:0001e5a0       ?Accept@LuaSocketManager@@SAHH@Z 1101f5a0 f   LuaManager.obj
 0001:0001e660       ?Lua_Connect_Wrap@LuaSocketManager@@SAHPAUlua_State@@@Z 1101f660 f   LuaManager.obj
 0001:0001e760       ?Lua_Server_Wrap@LuaSocketManager@@SAHPAUlua_State@@@Z 1101f760 f   LuaManager.obj
 0001:0001e860       ?Lua_Accept_Wrap@LuaSocketManager@@SAHPAUlua_State@@@Z 1101f860 f   LuaManager.obj
 0001:0001e900       ?Lua_Recv_Wrap@LuaSocketManager@@SAHPAUlua_State@@@Z 1101f900 f   LuaManager.obj
 0001:0001e9d0       ?Lua_Send_Wrap@LuaSocketManager@@SAHPAUlua_State@@@Z 1101f9d0 f   LuaManager.obj
 0001:0001eb00       ?Lua_DataAvaliable_Wrap@LuaSocketManager@@SAHPAUlua_State@@@Z 1101fb00 f   LuaManager.obj
 0001:0001ebc0       ?Lua_ClientWaiting_Wrap@LuaSocketManager@@SAHPAUlua_State@@@Z 1101fbc0 f   LuaManager.obj
 0001:0001ec80       ?Lua_Disconnect_Wrap@LuaSocketManager@@SAHPAUlua_State@@@Z 1101fc80 f   LuaManager.obj
 0001:0001ed40       ?Register@LuaSocketManager@@SAXPAUlua_State@@@Z 1101fd40 f   LuaManager.obj
 0001:0001f030       ?Cleanup@LuaSocketManager@@SAXXZ 11020030 f   LuaManager.obj
 0001:0001f0a0       ?Upload@LuaSocketManager@@SGKPAX@Z 110200a0 f   LuaManager.obj
 0001:0001f180       ?Lua_Upload@LuaSocketManager@@SAHPAUlua_State@@@Z 11020180 f   LuaManager.obj
 0001:0001f510       ?Lua_Check_Upload@LuaSocketManager@@SAHPAUlua_State@@@Z 11020510 f   LuaManager.obj
 0001:0001f550       ?Lua_Check_Upload_Error@LuaSocketManager@@SAHPAUlua_State@@@Z 11020550 f   LuaManager.obj
 0001:0001f590       ??_G?$ScriptRegistrant@VLuaScript@LuaScriptManager@@@@UAEPAXI@Z 11020590 f i LuaManager.obj
 0001:0001f590       ??_GScriptFactory@@UAEPAXI@Z 11020590 f i scriptfactory.obj
 0001:0001f590       ??_EScriptFactory@@UAEPAXI@Z 11020590 f i  CIL library: CIL module
 0001:0001f590       ??_E?$ScriptRegistrant@VLuaScript@LuaScriptManager@@@@UAEPAXI@Z 11020590 f i  CIL library: CIL module
 0001:0001f5c0       ?Create@?$ScriptRegistrant@VLuaScript@LuaScriptManager@@@@UAEPAVScriptImpClass@@XZ 110205c0 f i LuaManager.obj
 0001:0001f600       ?GetFiles@@YAXPBDPAPADH@Z  11020600 f   Misc.obj
 0001:0001f6f0       ?Client@TCPSocket@@QAE_NPBDH@Z 110206f0 f   Misc.obj
 0001:0001f7b0       ?Server@TCPSocket@@QAE_NPBDHH@Z 110207b0 f   Misc.obj
 0001:0001f850       ?Is_Connected@TCPSocket@@QAE_NXZ 11020850 f   Misc.obj
 0001:0001f940       ?Is_DataAvaliable@TCPSocket@@QAE_NXZ 11020940 f   Misc.obj
 0001:0001fa40       ?Is_ConnectionWaiting@TCPSocket@@QAE_NXZ 11020a40 f   Misc.obj
 0001:0001fb30       ?RecviveData@TCPSocket@@QAE_NPADPAH@Z 11020b30 f   Misc.obj
 0001:0001fb90       ?SendData@TCPSocket@@QAE_NPBDH@Z 11020b90 f   Misc.obj
 0001:0001fbe0       ?Accept@TCPSocket@@QAE_NPAV1@@Z 11020be0 f   Misc.obj
 0001:0001fcd0       _lua_checkstack            11020cd0 f   lapi.obj
 0001:0001fd40       _lua_xmove                 11020d40 f   lapi.obj
 0001:0001fd90       _lua_settop                11020d90 f   lapi.obj
 0001:0001fde0       _lua_remove                11020de0 f   lapi.obj
 0001:0001fe20       _lua_insert                11020e20 f   lapi.obj
 0001:0001fe70       _lua_pushvalue             11020e70 f   lapi.obj
 0001:0001fe90       _lua_isnumber              11020e90 f   lapi.obj
 0001:0001fed0       _lua_isstring              11020ed0 f   lapi.obj
 0001:0001ff00       _lua_tonumber              11020f00 f   lapi.obj
 0001:0001ff50       _lua_tointeger             11020f50 f   lapi.obj
 0001:0001ffb0       _lua_toboolean             11020fb0 f   lapi.obj
 0001:0001ffd0       _lua_tolstring             11020fd0 f   lapi.obj
 0001:00020040       _lua_objlen                11021040 f   lapi.obj
 0001:000200a0       _lua_topointer             110210a0 f   lapi.obj
 0001:00020100       _lua_pushlstring           11021100 f   lapi.obj
 0001:00020140       _lua_pushstring            11021140 f   lapi.obj
 0001:000201a0       _lua_pushfstring           110211a0 f   lapi.obj
 0001:000201d0       _lua_pushcclosure          110211d0 f   lapi.obj
 0001:00020260       _lua_getfield              11021260 f   lapi.obj
 0001:000202c0       _lua_getmetatable          110212c0 f   lapi.obj
 0001:00020310       _lua_getfenv               11021310 f   lapi.obj
 0001:00020370       _lua_setfield              11021370 f   lapi.obj
 0001:000203d0       _lua_rawset                110213d0 f   lapi.obj
 0001:00020490       _lua_rawseti               11021490 f   lapi.obj
 0001:00020530       _lua_setmetatable          11021530 f   lapi.obj
 0001:000205d0       _lua_setfenv               110215d0 f   lapi.obj
 0001:00020690       _lua_gc                    11021690 f   lapi.obj
 0001:00020770       _lua_concat                11021770 f   lapi.obj
 0001:000207e0       _lua_newuserdata           110217e0 f   lapi.obj
 0001:00020840       _lua_getupvalue            11021840 f   lapi.obj
 0001:000208c0       _lua_setupvalue            110218c0 f   lapi.obj
 0001:00020970       _luaL_argerror             11021970 f   lauxlib.obj
 0001:00020a50       _luaL_typerror             11021a50 f   lauxlib.obj
 0001:00020aa0       _luaL_where                11021aa0 f   lauxlib.obj
 0001:00020b30       _luaL_error                11021b30 f   lauxlib.obj
 0001:00020ba0       _luaL_checkoption          11021ba0 f   lauxlib.obj
 0001:00020c70       _luaL_newmetatable         11021c70 f   lauxlib.obj
 0001:00020d50       _luaL_checkudata           11021d50 f   lauxlib.obj
 0001:00020e20       _luaL_checklstring         11021e20 f   lauxlib.obj
 0001:00020e90       _luaL_checknumber          11021e90 f   lauxlib.obj
 0001:00020f80       _luaL_checkinteger         11021f80 f   lauxlib.obj
 0001:00021030       _luaL_getmetafield         11022030 f   lauxlib.obj
 0001:000210c0       _luaL_callmeta             110220c0 f   lauxlib.obj
 0001:00021160       _luaL_openlib              11022160 f   lauxlib.obj
 0001:000212d0       _luaL_gsub                 110222d0 f   lauxlib.obj
 0001:000213f0       _luaL_findtable            110223f0 f   lauxlib.obj
 0001:00021780       _luaL_addlstring           11022780 f   lauxlib.obj
 0001:00021820       _luaL_addvalue             11022820 f   lauxlib.obj
 0001:00021890       _luaL_ref                  11022890 f   lauxlib.obj
 0001:00021a80       _luaL_loadfile             11022a80 f   lauxlib.obj
 0001:00024270       _luaopen_base              11025270 f   lbaselib.obj
 0001:000242a0       _luaK_nil                  110252a0 f   lcode.obj
 0001:00024330       _luaK_jump                 11025330 f   lcode.obj
 0001:00024670       _luaK_concat               11025670 f   lcode.obj
 0001:000246c0       _luaK_reserveregs          110256c0 f   lcode.obj
 0001:00024850       _luaK_numberK              11025850 f   lcode.obj
 0001:000248b0       _luaK_setreturns           110258b0 f   lcode.obj
 0001:00024950       _luaK_setoneret            11025950 f   lcode.obj
 0001:000249a0       _luaK_dischargevars        110259a0 f   lcode.obj
 0001:00024d30       _luaK_exp2nextreg          11025d30 f   lcode.obj
 0001:00024da0       _luaK_exp2anyreg           11025da0 f   lcode.obj
 0001:00024df0       _luaK_exp2val              11025df0 f   lcode.obj
 0001:00024e40       _luaK_exp2RK               11025e40 f   lcode.obj
 0001:00024f80       _luaK_storevar             11025f80 f   lcode.obj
 0001:00025060       _luaK_self                 11026060 f   lcode.obj
 0001:00025290       _luaK_goiftrue             11026290 f   lcode.obj
 0001:00025720       _luaK_prefix               11026720 f   lcode.obj
 0001:000257c0       _luaK_infix                110267c0 f   lcode.obj
 0001:00025840       _luaK_posfix               11026840 f   lcode.obj
 0001:00025b00       _luaK_codeABC              11026b00 f   lcode.obj
 0001:00025b30       _luaK_setlist              11026b30 f   lcode.obj
 0001:000271f0       _luaopen_debug             110281f0 f   ldblib.obj
 0001:00027260       _lua_getstack              11028260 f   ldebug.obj
 0001:00027600       _lua_getinfo               11028600 f   ldebug.obj
 0001:00027720       _luaG_checkopenop          11028720 f   ldebug.obj
 0001:00027ea0       _luaG_typeerror            11028ea0 f   ldebug.obj
 0001:00027f20       _luaG_aritherror           11028f20 f   ldebug.obj
 0001:00027f70       _luaG_ordererror           11028f70 f   ldebug.obj
 0001:00028040       _luaG_errormsg             11029040 f   ldebug.obj
 0001:000280d0       _luaG_runerror             110290d0 f   ldebug.obj
 0001:00028110       _luaD_seterrorobj          11029110 f   ldo.obj
 0001:000281f0       _luaD_throw                110291f0 f   ldo.obj
 0001:00028250       _luaD_rawrunprotected      11029250 f   ldo.obj
 0001:00028340       _luaD_reallocstack         11029340 f   ldo.obj
 0001:000283b0       _luaD_reallocCI            110293b0 f   ldo.obj
 0001:00028490       _luaD_callhook             11029490 f   ldo.obj
 0001:00028860       _luaD_precall              11029860 f   ldo.obj
 0001:00028a90       _luaD_poscall              11029a90 f   ldo.obj
 0001:00028b10       _luaD_call                 11029b10 f   ldo.obj
 0001:00028c90       _lua_resume                11029c90 f   ldo.obj
 0001:00028d30       _luaD_pcall                11029d30 f   ldo.obj
 0001:00028fa0       _luaD_protectedparser      11029fa0 f   ldo.obj
 0001:000294a0       _luaU_dump                 1102a4a0 f   ldump.obj
 0001:00029520       _luaF_newCclosure          1102a520 f   lfunc.obj
 0001:00029590       _luaF_newLclosure          1102a590 f   lfunc.obj
 0001:00029600       _luaF_findupval            1102a600 f   lfunc.obj
 0001:00029690       _luaF_freeupval            1102a690 f   lfunc.obj
 0001:000296c0       _luaF_close                1102a6c0 f   lfunc.obj
 0001:000297a0       _luaF_newproto             1102a7a0 f   lfunc.obj
 0001:00029830       _luaF_freeproto            1102a830 f   lfunc.obj
 0001:000298c0       _luaF_freeclosure          1102a8c0 f   lfunc.obj
 0001:00029900       _luaF_getlocalname         1102a900 f   lfunc.obj
 0001:00029a20       _luaC_separateudata        1102aa20 f   lgc.obj
 0001:0002a3c0       _luaC_freeall              1102b3c0 f   lgc.obj
 0001:0002a6f0       _luaC_step                 1102b6f0 f   lgc.obj
 0001:0002a770       _luaC_fullgc               1102b770 f   lgc.obj
 0001:0002a7e0       _luaC_barrierf             1102b7e0 f   lgc.obj
 0001:0002a810       _luaL_openlibs             1102b810 f   linit.obj
 0001:0002c340       _luaopen_io                1102d340 f   liolib.obj
 0001:0002c520       _luaX_init                 1102d520 f   llex.obj
 0001:0002c560       _luaX_token2str            1102d560 f   llex.obj
 0001:0002c620       _luaX_lexerror             1102d620 f   llex.obj
 0001:0002c690       _luaX_newstring            1102d690 f   llex.obj
 0001:0002c790       _luaX_setinput             1102d790 f   llex.obj
 0001:0002dc40       _luaX_next                 1102ec40 f   llex.obj
 0001:0002e590       _luaopen_math              1102f590 f   lmathlib.obj
 0001:0002e6c0       _luaM_growaux_             1102f6c0 f   lmem.obj
 0001:0002e790       _luaM_realloc_             1102f790 f   lmem.obj
 0001:0002fda0       _luaopen_package           11030da0 f   loadlib.obj
 0001:000301c0       _luaO_rawequalObj          110311c0 f   lobject.obj
 0001:00030210       _luaO_str2d                11031210 f   lobject.obj
 0001:00030310       _luaO_pushvfstring         11031310 f   lobject.obj
 0001:000305e0       _luaO_pushfstring          110315e0 f   lobject.obj
 0001:00030600       _luaO_chunkid              11031600 f   lobject.obj
 0001:00030ff0       _luaopen_os                11031ff0 f   loslib.obj
 0001:00031cb0       _luaY_parser               11032cb0 f   lparser.obj
 0001:000350b0       _luaE_newthread            110360b0 f   lstate.obj
 0001:00035180       _luaE_freethread           11036180 f   lstate.obj
 0001:000351d0       _lua_newstate              110361d0 f   lstate.obj
 0001:00035320       _lua_close                 11036320 f   lstate.obj
 0001:00035380       _luaS_resize               11036380 f   lstring.obj
 0001:00035500       _luaS_newlstr              11036500 f   lstring.obj
 0001:000355f0       _luaS_newudata             110365f0 f   lstring.obj
 0001:00037c70       _luaopen_string            11038c70 f   lstrlib.obj
 0001:00037ed0       _luaH_next                 11038ed0 f   ltable.obj
 0001:00038490       _luaH_resizearray          11039490 f   ltable.obj
 0001:000385c0       _luaH_new                  110395c0 f   ltable.obj
 0001:00038630       _luaH_free                 11039630 f   ltable.obj
 0001:00038790       _luaH_getnum               11039790 f   ltable.obj
 0001:00038820       _luaH_getstr               11039820 f   ltable.obj
 0001:00038860       _luaH_get                  11039860 f   ltable.obj
 0001:00038930       _luaH_set                  11039930 f   ltable.obj
 0001:00038990       _luaH_setstr               11039990 f   ltable.obj
 0001:00038ab0       _luaH_getn                 11039ab0 f   ltable.obj
 0001:00039d30       _luaopen_table             1103ad30 f   ltablib.obj
 0001:00039d50       _luaT_init                 1103ad50 f   ltm.obj
 0001:00039da0       _luaT_gettm                1103ada0 f   ltm.obj
 0001:0003a7f0       _luaU_undump               1103b7f0 f   lundump.obj
 0001:0003a860       _luaV_tonumber             1103b860 f   lvm.obj
 0001:0003a8b0       _luaV_tostring             1103b8b0 f   lvm.obj
 0001:0003ab10       _luaV_gettable             1103bb10 f   lvm.obj
 0001:0003ac60       _luaV_settable             1103bc60 f   lvm.obj
 0001:0003b0e0       _luaV_lessthan             1103c0e0 f   lvm.obj
 0001:0003b260       _luaV_equalval             1103c260 f   lvm.obj
 0001:0003b330       _luaV_concat               1103c330 f   lvm.obj
 0001:0003b730       _luaV_execute              1103c730 f   lvm.obj
 0001:0003c990       _luaZ_fill                 1103d990 f   lzio.obj
 0001:0003c9d0       _luaZ_read                 1103d9d0 f   lzio.obj
 0001:0003ca60       _luaZ_openspace            1103da60 f   lzio.obj
 0001:0003e5a0       _sqlite3_vfs_find          1103f5a0 f   sqlite3.obj
 0001:0003e6a0       _sqlite3_vfs_register      1103f6a0 f   sqlite3.obj
 0001:0003e720       _sqlite3_vfs_unregister    1103f720 f   sqlite3.obj
 0001:0003e760       _sqlite3_memory_used       1103f760 f   sqlite3.obj
 0001:0003e7c0       _sqlite3_memory_highwater  1103f7c0 f   sqlite3.obj
 0001:0003e830       _sqlite3_memory_alarm      1103f830 f   sqlite3.obj
 0001:0003e920       _sqlite3_malloc            1103f920 f   sqlite3.obj
 0001:0003ea20       _sqlite3_free              1103fa20 f   sqlite3.obj
 0001:0003ea80       _sqlite3_realloc           1103fa80 f   sqlite3.obj
 0001:0003ebc0       _sqlite3_mutex_alloc       1103fbc0 f   sqlite3.obj
 0001:0003eca0       _sqlite3_mutex_free        1103fca0 f   sqlite3.obj
 0001:0003ecc0       _sqlite3_mutex_enter       1103fcc0 f   sqlite3.obj
 0001:0003ece0       _sqlite3_mutex_try         1103fce0 f   sqlite3.obj
 0001:0003ecf0       _sqlite3_mutex_leave       1103fcf0 f   sqlite3.obj
 0001:0003ed00       _sqlite3_soft_heap_limit   1103fd00 f   sqlite3.obj
 0001:0003ff90       _sqlite3_vmprintf          11040f90 f   sqlite3.obj
 0001:00040030       _sqlite3_mprintf           11041030 f   sqlite3.obj
 0001:00040050       _sqlite3_snprintf          11041050 f   sqlite3.obj
 0001:00042170       _sqlite3_release_memory    11043170 f   sqlite3.obj
 0001:000429b0       _winDlSym                  110439b0 f   sqlite3.obj
 0001:000429d0       _winDlClose                110439d0 f   sqlite3.obj
 0001:00042ab0       _winCurrentTime            11043ab0 f   sqlite3.obj
 0001:00046a80       _sqlite3_enable_shared_cache 11047a80 f   sqlite3.obj
 0001:00052950       _sqlite3_expired           11053950 f   sqlite3.obj
 0001:00052970       _sqlite3_finalize          11053970 f   sqlite3.obj
 0001:000529f0       _sqlite3_reset             110539f0 f   sqlite3.obj
 0001:00052a50       _sqlite3_clear_bindings    11053a50 f   sqlite3.obj
 0001:00052ad0       _sqlite3_value_blob        11053ad0 f   sqlite3.obj
 0001:00052b10       _sqlite3_value_bytes       11053b10 f   sqlite3.obj
 0001:00052b50       _sqlite3_value_bytes16     11053b50 f   sqlite3.obj
 0001:00052b80       _sqlite3_value_double      11053b80 f   sqlite3.obj
 0001:00052b90       _sqlite3_value_int         11053b90 f   sqlite3.obj
 0001:00052b90       _sqlite3_value_int64       11053b90 f   sqlite3.obj
 0001:00052ba0       _sqlite3_value_text        11053ba0 f   sqlite3.obj
 0001:00052bb0       _sqlite3_value_text16be    11053bb0 f   sqlite3.obj
 0001:00052bc0       _sqlite3_value_text16le    11053bc0 f   sqlite3.obj
 0001:00052bc0       _sqlite3_value_text16      11053bc0 f   sqlite3.obj
 0001:00052bd0       _sqlite3_value_type        11053bd0 f   sqlite3.obj
 0001:00052be0       _sqlite3_result_blob       11053be0 f   sqlite3.obj
 0001:00052c10       _sqlite3_result_double     11053c10 f   sqlite3.obj
 0001:00052c40       _sqlite3_result_error      11053c40 f   sqlite3.obj
 0001:00052c70       _sqlite3_result_error16    11053c70 f   sqlite3.obj
 0001:00052ca0       _sqlite3_result_int        11053ca0 f   sqlite3.obj
 0001:00052ce0       _sqlite3_result_int64      11053ce0 f   sqlite3.obj
 0001:00052d20       _sqlite3_result_null       11053d20 f   sqlite3.obj
 0001:00052d50       _sqlite3_result_text       11053d50 f   sqlite3.obj
 0001:00052d80       _sqlite3_result_text16le   11053d80 f   sqlite3.obj
 0001:00052d80       _sqlite3_result_text16     11053d80 f   sqlite3.obj
 0001:00052db0       _sqlite3_result_text16be   11053db0 f   sqlite3.obj
 0001:00052de0       _sqlite3_result_value      11053de0 f   sqlite3.obj
 0001:00052e00       _sqlite3_result_error_toobig 11053e00 f   sqlite3.obj
 0001:00052e40       _sqlite3_result_error_nomem 11053e40 f   sqlite3.obj
 0001:00053020       _sqlite3_step              11054020 f   sqlite3.obj
 0001:00053180       _sqlite3_user_data         11054180 f   sqlite3.obj
 0001:00053230       _sqlite3_aggregate_context 11054230 f   sqlite3.obj
 0001:000532b0       _sqlite3_get_auxdata       110542b0 f   sqlite3.obj
 0001:000532d0       _sqlite3_set_auxdata       110542d0 f   sqlite3.obj
 0001:000533b0       _sqlite3_aggregate_count   110543b0 f   sqlite3.obj
 0001:000533c0       _sqlite3_column_count      110543c0 f   sqlite3.obj
 0001:000533e0       _sqlite3_data_count        110543e0 f   sqlite3.obj
 0001:00053480       _sqlite3_column_blob       11054480 f   sqlite3.obj
 0001:00053520       _sqlite3_column_bytes      11054520 f   sqlite3.obj
 0001:000535b0       _sqlite3_column_bytes16    110545b0 f   sqlite3.obj
 0001:00053640       _sqlite3_column_double     11054640 f   sqlite3.obj
 0001:000536c0       _sqlite3_column_int        110546c0 f   sqlite3.obj
 0001:00053730       _sqlite3_column_int64      11054730 f   sqlite3.obj
 0001:000537b0       _sqlite3_column_text       110547b0 f   sqlite3.obj
 0001:00053820       _sqlite3_column_value      11054820 f   sqlite3.obj
 0001:00053890       _sqlite3_column_text16     11054890 f   sqlite3.obj
 0001:00053900       _sqlite3_column_type       11054900 f   sqlite3.obj
 0001:000539f0       _sqlite3_column_name       110549f0 f   sqlite3.obj
 0001:00053a10       _sqlite3_column_name16     11054a10 f   sqlite3.obj
 0001:00053a30       _sqlite3_column_decltype   11054a30 f   sqlite3.obj
 0001:00053a50       _sqlite3_column_decltype16 11054a50 f   sqlite3.obj
 0001:00053bb0       _sqlite3_bind_blob         11054bb0 f   sqlite3.obj
 0001:00053be0       _sqlite3_bind_double       11054be0 f   sqlite3.obj
 0001:00053c50       _sqlite3_bind_int          11054c50 f   sqlite3.obj
 0001:00053c70       _sqlite3_bind_int64        11054c70 f   sqlite3.obj
 0001:00053cf0       _sqlite3_bind_null         11054cf0 f   sqlite3.obj
 0001:00053d30       _sqlite3_bind_text         11054d30 f   sqlite3.obj
 0001:00053d60       _sqlite3_bind_text16       11054d60 f   sqlite3.obj
 0001:00053d90       _sqlite3_bind_value        11054d90 f   sqlite3.obj
 0001:00053df0       _sqlite3_bind_zeroblob     11054df0 f   sqlite3.obj
 0001:00053e80       _sqlite3_bind_parameter_count 11054e80 f   sqlite3.obj
 0001:00053f00       _sqlite3_bind_parameter_name 11054f00 f   sqlite3.obj
 0001:00053f30       _sqlite3_bind_parameter_index 11054f30 f   sqlite3.obj
 0001:00053fb0       _sqlite3_transfer_bindings 11054fb0 f   sqlite3.obj
 0001:00054060       _sqlite3_db_handle         11055060 f   sqlite3.obj
 0001:00054230       _sqlite3_value_numeric_type 11055230 f   sqlite3.obj
 0001:00057e00       _sqlite3_blob_open         11058e00 f   sqlite3.obj
 0001:00058600       _sqlite3_blob_close        11059600 f   sqlite3.obj
 0001:00058710       _sqlite3_blob_read         11059710 f   sqlite3.obj
 0001:00058740       _sqlite3_blob_write        11059740 f   sqlite3.obj
 0001:00058770       _sqlite3_blob_bytes        11059770 f   sqlite3.obj
 0001:0005fff0       _sqlite3_set_authorizer    11060ff0 f   sqlite3.obj
 0001:0006cb30       _sqlite3_exec              1106db30 f   sqlite3.obj
 0001:000704f0       _sqlite3_prepare           110714f0 f   sqlite3.obj
 0001:00070520       _sqlite3_prepare_v2        11071520 f   sqlite3.obj
 0001:00070640       _sqlite3_prepare16         11071640 f   sqlite3.obj
 0001:00070670       _sqlite3_prepare16_v2      11071670 f   sqlite3.obj
 0001:00076880       _sqlite3_get_table         11077880 f   sqlite3.obj
 0001:00076a10       _sqlite3_free_table        11077a10 f   sqlite3.obj
 0001:0007ba70       _sqlite3_create_module     1107ca70 f   sqlite3.obj
 0001:0007ba90       _sqlite3_create_module_v2  1107ca90 f   sqlite3.obj
 0001:0007c5d0       _sqlite3_declare_vtab      1107d5d0 f   sqlite3.obj
 0001:00084f70       _sqlite3_complete          11085f70 f   sqlite3.obj
 0001:00085260       _sqlite3_complete16        11086260 f   sqlite3.obj
 0001:00085360       _sqlite3_libversion        11086360 f   sqlite3.obj
 0001:00085370       _sqlite3_libversion_number 11086370 f   sqlite3.obj
 0001:00085490       _sqlite3_last_insert_rowid 11086490 f   sqlite3.obj
 0001:000854a0       _sqlite3_changes           110864a0 f   sqlite3.obj
 0001:000854b0       _sqlite3_total_changes     110864b0 f   sqlite3.obj
 0001:000854c0       _sqlite3_close             110864c0 f   sqlite3.obj
 0001:00085c40       _sqlite3_busy_handler      11086c40 f   sqlite3.obj
 0001:00085c90       _sqlite3_progress_handler  11086c90 f   sqlite3.obj
 0001:00085d30       _sqlite3_busy_timeout      11086d30 f   sqlite3.obj
 0001:00085db0       _sqlite3_interrupt         11086db0 f   sqlite3.obj
 0001:00085f50       _sqlite3_create_function   11086f50 f   sqlite3.obj
 0001:00085fd0       _sqlite3_create_function16 11086fd0 f   sqlite3.obj
 0001:00086070       _sqlite3_overload_function 11087070 f   sqlite3.obj
 0001:00086110       _sqlite3_trace             11087110 f   sqlite3.obj
 0001:00086150       _sqlite3_profile           11087150 f   sqlite3.obj
 0001:00086190       _sqlite3_commit_hook       11087190 f   sqlite3.obj
 0001:000861d0       _sqlite3_update_hook       110871d0 f   sqlite3.obj
 0001:00086220       _sqlite3_rollback_hook     11087220 f   sqlite3.obj
 0001:00086330       _sqlite3_errmsg            11087330 f   sqlite3.obj
 0001:000863e0       _sqlite3_errmsg16          110873e0 f   sqlite3.obj
 0001:00086500       _sqlite3_errcode           11087500 f   sqlite3.obj
 0001:00086a80       _sqlite3_open              11087a80 f   sqlite3.obj
 0001:00086aa0       _sqlite3_open_v2           11087aa0 f   sqlite3.obj
 0001:00086ab0       _sqlite3_open16            11087ab0 f   sqlite3.obj
 0001:00086bf0       _sqlite3_create_collation  11087bf0 f   sqlite3.obj
 0001:00086c70       _sqlite3_create_collation_v2 11087c70 f   sqlite3.obj
 0001:00086cf0       _sqlite3_create_collation16 11087cf0 f   sqlite3.obj
 0001:00086d80       _sqlite3_collation_needed  11087d80 f   sqlite3.obj
 0001:00086dd0       _sqlite3_collation_needed16 11087dd0 f   sqlite3.obj
 0001:00086e20       _sqlite3_get_autocommit    11087e20 f   sqlite3.obj
 0001:00086e30       _sqlite3_thread_cleanup    11087e30 f   sqlite3.obj
 0001:00086e30       _SSGM_Chat_Hook            11087e30 f   plugin.obj
 0001:00086e30       ?Clear@?$VectorClass@PAE@@UAEXXZ 11087e30 f   engine_bhs.obj
 0001:00086e30       ?Register_Auto_Save_Variables@ScriptImpClass@@UAEXXZ 11087e30 f   scripts.obj
 0001:00086e40       _sqlite3_sleep             11087e40 f   sqlite3.obj
 0001:00086e70       _sqlite3_file_control      11087e70 f   sqlite3.obj
 0001:00086f5c       ___WSAFDIsSet@8            11087f5c f   ws2_32:WS2_32.dll
 0001:00086f62       _sprintf                   11087f62 f   LIBCMT:sprintf.obj
 0001:00086fdf       __localtime64_s            11087fdf f   LIBCMT:loctim64.obj
 0001:00087297       __localtime64              11088297 f   LIBCMT:loctim64.obj
 0001:000872be       __time64                   110882be f   LIBCMT:time64.obj
 0001:0008730f       _memmove_s                 1108830f f   LIBCMT:memmove_s.obj
 0001:0008736c       ??0exception@std@@QAE@XZ   1108836c f   LIBCMT:stdexcpt.obj
 0001:0008737d       ??0exception@std@@QAE@ABQBD@Z 1108837d f   LIBCMT:stdexcpt.obj
 0001:000873d0       ??0exception@std@@QAE@ABQBDH@Z 110883d0 f   LIBCMT:stdexcpt.obj
 0001:000873ed       ??0exception@std@@QAE@ABV01@@Z 110883ed f   LIBCMT:stdexcpt.obj
 0001:0008744a       ??1exception@std@@UAE@XZ   1108844a f   LIBCMT:stdexcpt.obj
 0001:00087460       ?what@exception@std@@UBEPBDXZ 11088460 f   LIBCMT:stdexcpt.obj
 0001:0008746d       ??_Eexception@std@@UAEPAXI@Z 1108846d f i LIBCMT:stdexcpt.obj
 0001:0008746d       ??_Gexception@std@@UAEPAXI@Z 1108846d f i LIBCMT:stdexcpt.obj
 0001:0008748e       ??_U@YAPAXI@Z              1108848e f   LIBCMT:new2.obj
 0001:00087499       ??_V@YAXPAX@Z              11088499 f   LIBCMT:delete2.obj
 0001:000874a4       ??3@YAXPAX@Z               110884a4 f   LIBCMT:delete.obj
 0001:000874af       _memcpy_s                  110884af f   LIBCMT:memcpy_s.obj
 0001:0008752c       ??0_LocaleUpdate@@QAE@PAUlocaleinfo_struct@@@Z 1108852c f i LIBCMT:wcstombs.obj
 0001:000875b3       __wcstombs_l_helper        110885b3 f   LIBCMT:wcstombs.obj
 0001:000877f5       _wcstombs                  110887f5 f   LIBCMT:wcstombs.obj
 0001:0008780f       ??1type_info@@UAE@XZ       1108880f f   LIBCMT:typinfo.obj
 0001:0008781f       ??_Etype_info@@UAEPAXI@Z   1108881f f i LIBCMT:typinfo.obj
 0001:0008781f       ??_Gtype_info@@UAEPAXI@Z   1108881f f i LIBCMT:typinfo.obj
 0001:00087840       ??8type_info@@QBE_NABV0@@Z 11088840 f   LIBCMT:typinfo.obj
 0001:00087860       ??0bad_alloc@std@@QAE@XZ   11088860 f i LIBCMT:new.obj
 0001:0008787b       ??2@YAPAXI@Z               1108887b f   LIBCMT:new.obj
 0001:000878e0       __initp_misc_invarg        110888e0 f   LIBCMT:invarg.obj
 0001:000878ef       __invoke_watson            110888ef f   LIBCMT:invarg.obj
 0001:00087a17       __invalid_parameter        11088a17 f   LIBCMT:invarg.obj
 0001:00087a3d       __invalid_parameter_noinfo 11088a3d f   LIBCMT:invarg.obj
 0001:00087a4d       _free                      11088a4d f   LIBCMT:free.obj
 0001:00087adb       __ungetc_nolock            11088adb f   LIBCMT:ungetc.obj
 0001:00087bcc       _ungetc                    11088bcc f   LIBCMT:ungetc.obj
 0001:00087c40       _strstr                    11088c40 f   LIBCMT:strstr.obj
 0001:00087cd0       _memchr                    11088cd0 f   LIBCMT:memchr.obj
 0001:00087d7d       __flush                    11088d7d f   LIBCMT:fflush.obj
 0001:00087de5       __fflush_nolock            11088de5 f   LIBCMT:fflush.obj
 0001:00087f07       _fflush                    11088f07 f   LIBCMT:fflush.obj
 0001:00087f5a       __flushall                 11088f5a f   LIBCMT:fflush.obj
 0001:00087f63       _getc                      11088f63 f   LIBCMT:fgetc.obj
 0001:00088067       _localeconv                11089067 f   LIBCMT:lconv.obj
 0001:0008808d       _remove                    1108908d f   LIBCMT:unlink.obj
 0001:000880bd       __tolower_l                110890bd f   LIBCMT:tolower.obj
 0001:000881d2       _tolower                   110891d2 f   LIBCMT:tolower.obj
 0001:000881fe       _printf                    110891fe f   LIBCMT:printf.obj
 0001:000882ad       __get_printf_count_output  110892ad f   LIBCMT:printf.obj
 0001:000882c3       _setvbuf                   110892c3 f   LIBCMT:setvbuf.obj
 0001:000883c1       __fwrite_nolock            110893c1 f   LIBCMT:fwrite.obj
 0001:00088523       _fwrite                    11089523 f   LIBCMT:fwrite.obj
 0001:000885b0       _strcspn                   110895b0 f   LIBCMT:strcspn.obj
 0001:000885f6       __fseek_nolock             110895f6 f   LIBCMT:fseek.obj
 0001:00088680       _fseek                     11089680 f   LIBCMT:fseek.obj
 0001:00088705       __fclose_nolock            11089705 f   LIBCMT:fclose.obj
 0001:0008877c       _fclose                    1108977c f   LIBCMT:fclose.obj
 0001:000887f8       __fsopen                   110897f8 f   LIBCMT:fopen.obj
 0001:000888bc       _fopen                     110898bc f   LIBCMT:fopen.obj
 0001:000888d3       ___ascii_stricmp           110898d3 f   LIBCMT:stricmp.obj
 0001:0008890c       __stricmp_l                1108990c f   LIBCMT:stricmp.obj
 0001:000889e1       __stricmp                  110899e1 f   LIBCMT:stricmp.obj
 0001:000889e1       _stricmp                   110899e1 f   LIBCMT:stricmp.obj
 0001:00088bd8       __mbsrtowcs_helper         11089bd8 f   LIBCMT:mbrtowc.obj
 0001:00088cc2       _mbsrtowcs                 11089cc2 f   LIBCMT:mbrtowc.obj
 0001:00088ccd       __purecall                 11089ccd f   LIBCMT:purevirt.obj
 0001:00088cf7       _atol                      11089cf7 f   LIBCMT:atox.obj
 0001:00088d0d       _atoi                      11089d0d f   LIBCMT:atox.obj
 0001:00088d20       _strncpy                   11089d20 f   LIBCMT:strncpy.obj
 0001:00088e44       _fprintf                   11089e44 f   LIBCMT:fprintf.obj
 0001:00088f60       __atof_l                   11089f60 f   LIBCMT:atof.obj
 0001:0008900b       _atof                      1108a00b f   LIBCMT:atof.obj
 0001:00089020       _strpbrk                   1108a020 f   LIBCMT:strpbrk.obj
 0001:00089060       _clock                     1108a060 f   LIBCMT:clock.obj
 0001:000890a5       ___inittime                1108a0a5 f   LIBCMT:clock.obj
 0001:000890de       _strcpy_s                  1108a0de f   LIBCMT:strcpy_s.obj
 0001:00089146       _feof                      1108a146 f   LIBCMT:feoferr.obj
 0001:0008917a       _ferror                    1108a17a f   LIBCMT:feoferr.obj
 0001:000891ae       __get_sys_err_msg          1108a1ae f i LIBCMT:strerror.obj
 0001:000891d6       _strerror                  1108a1d6 f   LIBCMT:strerror.obj
 0001:00089242       ___iob_func                1108a242 f   LIBCMT:_file.obj
 0001:00089248       ___initstdio               1108a248 f   LIBCMT:_file.obj
 0001:000892f9       ___endstdio                1108a2f9 f   LIBCMT:_file.obj
 0001:00089319       __lock_file                1108a319 f   LIBCMT:_file.obj
 0001:0008935a       __lock_file2               1108a35a f   LIBCMT:_file.obj
 0001:0008938c       __unlock_file              1108a38c f   LIBCMT:_file.obj
 0001:000893c8       __unlock_file2             1108a3c8 f   LIBCMT:_file.obj
 0001:00089410       _strchr                    1108a410 f   LIBCMT:strchr.obj
 0001:00089416       ___from_strstr_to_strchr   1108a416     LIBCMT:strchr.obj
 0001:000894ce       __get_errno_from_oserr     1108a4ce f   LIBCMT:dosmap.obj
 0001:00089510       __errno                    1108a510 f   LIBCMT:dosmap.obj
 0001:00089523       ___doserrno                1108a523 f   LIBCMT:dosmap.obj
 0001:00089536       __dosmaperr                1108a536 f   LIBCMT:dosmap.obj
 0001:00089559       __fread_nolock_s           1108a559 f   LIBCMT:fread.obj
 0001:00089763       _fread_s                   1108a763 f   LIBCMT:fread.obj
 0001:000897f9       _fread                     1108a7f9 f   LIBCMT:fread.obj
 0001:00089816       __freopen_helper           1108a816 f   LIBCMT:freopen.obj
 0001:000898ef       _freopen                   1108a8ef f   LIBCMT:freopen.obj
 0001:00089915       _realloc                   1108a915 f   LIBCMT:realloc.obj
 0001:00089b30       __isalpha_l                1108ab30 f i LIBCMT:_ctype.obj
 0001:00089b86       _isalpha                   1108ab86 f i LIBCMT:_ctype.obj
 0001:00089bb6       __isupper_l                1108abb6 f i LIBCMT:_ctype.obj
 0001:00089c07       _isupper                   1108ac07 f i LIBCMT:_ctype.obj
 0001:00089c35       __islower_l                1108ac35 f i LIBCMT:_ctype.obj
 0001:00089c86       _islower                   1108ac86 f i LIBCMT:_ctype.obj
 0001:00089cb4       __isdigit_l                1108acb4 f i LIBCMT:_ctype.obj
 0001:00089d05       _isdigit                   1108ad05 f i LIBCMT:_ctype.obj
 0001:00089d33       __isxdigit_l               1108ad33 f i LIBCMT:_ctype.obj
 0001:00089d89       _isxdigit                  1108ad89 f i LIBCMT:_ctype.obj
 0001:00089db9       __isspace_l                1108adb9 f i LIBCMT:_ctype.obj
 0001:00089e0a       _isspace                   1108ae0a f i LIBCMT:_ctype.obj
 0001:00089e38       __ispunct_l                1108ae38 f i LIBCMT:_ctype.obj
 0001:00089e89       _ispunct                   1108ae89 f i LIBCMT:_ctype.obj
 0001:00089eb7       __isalnum_l                1108aeb7 f i LIBCMT:_ctype.obj
 0001:00089f0d       _isalnum                   1108af0d f i LIBCMT:_ctype.obj
 0001:00089f3d       __iscntrl_l                1108af3d f i LIBCMT:_ctype.obj
 0001:00089f8e       _iscntrl                   1108af8e f i LIBCMT:_ctype.obj
 0001:00089fbc       _fputs                     1108afbc f   LIBCMT:fputs.obj
 0001:0008a2fa       _strtol                    1108b2fa f   LIBCMT:strtol.obj
 0001:0008a325       _strtoul                   1108b325 f   LIBCMT:strtol.obj
 0001:0008a351       _fgets                     1108b351 f   LIBCMT:fgets.obj
 0001:0008a49c       _longjmp                   1108b49c f   LIBCMT:longjmp.obj
 0001:0008a54d       __crt_waiting_on_module_handle 1108b54d f   LIBCMT:crt0dat.obj
 0001:0008a57d       __amsg_exit                1108b57d f   LIBCMT:crt0dat.obj
 0001:0008a5a6       ___crtCorExitProcess       1108b5a6 f   LIBCMT:crt0dat.obj
 0001:0008a5d1       ___crtExitProcess          1108b5d1 f   LIBCMT:crt0dat.obj
 0001:0008a5e9       __lockexit                 1108b5e9 f   LIBCMT:crt0dat.obj
 0001:0008a5f2       __unlockexit               1108b5f2 f   LIBCMT:crt0dat.obj
 0001:0008a618       __initterm_e               1108b618 f   LIBCMT:crt0dat.obj
 0001:0008a63c       __cinit                    1108b63c f   LIBCMT:crt0dat.obj
 0001:0008a7ed       _exit                      1108b7ed f   LIBCMT:crt0dat.obj
 0001:0008a803       __exit                     1108b803 f   LIBCMT:crt0dat.obj
 0001:0008a819       __cexit                    1108b819 f   LIBCMT:crt0dat.obj
 0001:0008a828       __init_pointers            1108b828 f   LIBCMT:crt0dat.obj
 0001:0008a876       _vfscanf                   1108b876 f   LIBCMT:fscanf.obj
 0001:0008a980       _fscanf                    1108b980 f   LIBCMT:fscanf.obj
 0001:0008ab17       __tmpnam_helper            1108bb17 f   LIBCMT:tmpfile.obj
 0001:0008ac56       _tmpnam                    1108bc56 f   LIBCMT:tmpfile.obj
 0001:0008ac7d       __tmpfile_helper           1108bc7d f   LIBCMT:tmpfile.obj
 0001:0008ae9d       _tmpfile                   1108be9d f   LIBCMT:tmpfile.obj
 0001:0008af17       __popen                    1108bf17 f   LIBCMT:popen.obj
 0001:0008b428       __pclose                   1108c428 f   LIBCMT:popen.obj
 0001:0008b4fb       __ftell_nolock             1108c4fb f   LIBCMT:ftell.obj
 0001:0008b698       _ftell                     1108c698 f   LIBCMT:ftell.obj
 0001:0008b706       _clearerr_s                1108c706 f   LIBCMT:clearerr.obj
 0001:0008b7b3       _clearerr                  1108c7b3 f   LIBCMT:clearerr.obj
 0001:0008b7c0       _ceil                      1108c7c0 f   LIBCMT:_ceil_pentium4_.obj
 0001:0008b800       __ceil_pentium4            1108c800 f   LIBCMT:_ceil_pentium4_.obj
 0001:0008b8e0       _modf                      1108c8e0 f   LIBCMT:_modf_pentium4_.obj
 0001:0008b920       __modf_pentium4            1108c920 f   LIBCMT:_modf_pentium4_.obj
 0001:0008ba28       _ldexp                     1108ca28 f   LIBCMT:_ldexp_.obj
 0001:0008bbda       _srand                     1108cbda f   LIBCMT:rand.obj
 0001:0008bbec       _rand                      1108cbec f   LIBCMT:rand.obj
 0001:0008bc0e       _frexp                     1108cc0e f   LIBCMT:_frexp_.obj
 0001:0008bcf0       _strrchr                   1108ccf0 f   LIBCMT:strrchr.obj
 0001:0008bd1d       __getenv_helper_nolock     1108cd1d f   LIBCMT:getenv.obj
 0001:0008bda4       _getenv                    1108cda4 f   LIBCMT:getenv.obj
 0001:0008be27       __dupenv_s                 1108ce27 f   LIBCMT:getenv.obj
 0001:0008bf0d       __strtod_l                 1108cf0d f   LIBCMT:strtod.obj
 0001:0008c02c       _strtod                    1108d02c f   LIBCMT:strtod.obj
 0001:0008c050       _strncat                   1108d050 f   LIBCMT:strncat.obj
 0001:0008c185       _rename                    1108d185 f   LIBCMT:rename.obj
 0001:0008c46d       __mktime64                 1108d46d f   LIBCMT:mktime64.obj
 0001:0008c47f       __gmtime64_s               1108d47f f   LIBCMT:gmtime64.obj
 0001:0008c6c2       __gmtime64                 1108d6c2 f   LIBCMT:gmtime64.obj
 0001:0008c6e9       _system                    1108d6e9 f   LIBCMT:system.obj
 0001:0008c7c9       __freea                    1108d7c9 f i LIBCMT:strftime.obj
 0001:0008d0cd       __Strftime_l               1108e0cd f   LIBCMT:strftime.obj
 0001:0008d271       _strftime                  1108e271 f   LIBCMT:strftime.obj
 0001:0008d290       ___freetlocinfo            1108e290 f   LIBCMT:setlocal.obj
 0001:0008d3d9       ___addlocaleref            1108e3d9 f   LIBCMT:setlocal.obj
 0001:0008d468       ___removelocaleref         1108e468 f   LIBCMT:setlocal.obj
 0001:0008d565       ___updatetlocinfo          1108e565 f   LIBCMT:setlocal.obj
 0001:0008d62e       __free_locale              1108e62e f   LIBCMT:setlocal.obj
 0001:0008d6f0       __strcats                  1108e6f0 f   LIBCMT:setlocal.obj
 0001:0008d730       ___lc_strtolc              1108e730 f   LIBCMT:setlocal.obj
 0001:0008d859       ___lc_lctostr              1108e859 f   LIBCMT:setlocal.obj
 0001:0008da43       __expandlocale             1108ea43 f   LIBCMT:setlocal.obj
 0001:0008e191       _setlocale                 1108f191 f   LIBCMT:setlocal.obj
 0001:0008e301       __difftime64               1108f301 f   LIBCMT:difftm64.obj
 0001:0008e344       __toupper_l                1108f344 f   LIBCMT:toupper.obj
 0001:0008e45a       _toupper                   1108f45a f   LIBCMT:toupper.obj
 0001:0008e486       __strcoll_l                1108f486 f   LIBCMT:strcoll.obj
 0001:0008e52c       _strcoll                   1108f52c f   LIBCMT:strcoll.obj
 0001:0008e550       _memmove                   1108f550 f   LIBCMT:memmove.obj
 0001:0008e8b5       _strncmp                   1108f8b5 f   LIBCMT:strncmp.obj
 0001:0008e975       _V6_HeapAlloc              1108f975 f   LIBCMT:malloc.obj
 0001:0008e9c4       _malloc                    1108f9c4 f   LIBCMT:malloc.obj
 0001:0008ea8e       __CRT_INIT@12              1108fa8e f   LIBCMT:dllcrt0.obj
 0001:0008ecb9       __DllMainCRTStartup@12     1108fcb9 f   LIBCMT:dllcrt0.obj
 0001:0008ecdc       __flsbuf                   1108fcdc f   LIBCMT:_flsbuf.obj
 0001:0008eee6       __output_l                 1108fee6 f   LIBCMT:output.obj
 0001:0008fa7e       __set_daylight             11090a7e f i LIBCMT:tzset.obj
 0001:0008fa8f       __set_dstbias              11090a8f f i LIBCMT:tzset.obj
 0001:0008faa0       __set_timezone             11090aa0 f i LIBCMT:tzset.obj
 0001:000901c6       ___tzset                   110911c6 f   LIBCMT:tzset.obj
 0001:00090215       __isindst                  11091215 f   LIBCMT:tzset.obj
 0001:00090256       __get_daylight             11091256 f   LIBCMT:timeset.obj
 0001:0009028f       __get_dstbias              1109128f f   LIBCMT:timeset.obj
 0001:000902c8       __get_timezone             110912c8 f   LIBCMT:timeset.obj
 0001:00090301       ___daylight                11091301 f   LIBCMT:timeset.obj
 0001:00090307       ___dstbias                 11091307 f   LIBCMT:timeset.obj
 0001:0009030d       ___timezone                1109130d f   LIBCMT:timeset.obj
 0001:00090313       ___tzname                  11091313 f   LIBCMT:timeset.obj
 0001:00090320       _memset                    11091320 f   LIBCMT:memset.obj
 0001:000903a0       __alldiv                   110913a0 f   LIBCMT:lldiv.obj
 0001:00090450       __allrem                   11091450 f   LIBCMT:llrem.obj
 0001:00090502       ___getgmtimebuf            11091502 f   LIBCMT:gmtime.obj
 0001:00090540       __aulldiv                  11091540 f   LIBCMT:ulldiv.obj
 0001:000905b0       _strlen                    110915b0 f   LIBCMT:strlen.obj
 0001:00090640       _memcpy                    11091640 f   LIBCMT:memcpy.obj
 0001:00090bcb       ___updatetmbcinfo          11091bcb f   LIBCMT:mbctype.obj
 0001:00090ceb       __setmbcp_nolock           11091ceb f   LIBCMT:mbctype.obj
 0001:00090ed0       __setmbcp                  11091ed0 f   LIBCMT:mbctype.obj
 0001:0009106a       ___initmbctable            1109206a f   LIBCMT:mbctype.obj
 0001:00091088       __encode_pointer           11092088 f   LIBCMT:tidtable.obj
 0001:000910fa       __encoded_null             110920fa f   LIBCMT:tidtable.obj
 0001:00091103       __decode_pointer           11092103 f   LIBCMT:tidtable.obj
 0001:00091175       ___crtTlsAlloc@4           11092175 f   LIBCMT:tidtable.obj
 0001:0009117e       ___set_flsgetvalue         1109217e f   LIBCMT:tidtable.obj
 0001:000911b2       __mtterm                   110921b2 f   LIBCMT:tidtable.obj
 0001:000911ef       __initptd                  110921ef f   LIBCMT:tidtable.obj
 0001:000912d6       __getptd_noexit            110922d6 f   LIBCMT:tidtable.obj
 0001:0009134f       __getptd                   1109234f f   LIBCMT:tidtable.obj
 0001:00091369       __freefls@4                11092369 f   LIBCMT:tidtable.obj
 0001:00091498       __freeptd                  11092498 f   LIBCMT:tidtable.obj
 0001:00091506       __mtinit                   11092506 f   LIBCMT:tidtable.obj
 0001:00091693       _wcslen                    11092693 f   LIBCMT:wcslen.obj
 0001:000916ad       @__security_check_cookie@4 110926ad f   LIBCMT:secchk.obj
 0001:000916bc       ?_Type_info_dtor@type_info@@CAXPAV1@@Z 110926bc f   LIBCMT:typname.obj
 0001:00091730       _strcmp                    11092730 f   LIBCMT:strcmp.obj
 0001:00091872       ___onexitinit              11092872 f   LIBCMT:onexit.obj
 0001:000918a3       __onexit                   110928a3 f   LIBCMT:onexit.obj
 0001:000918df       _atexit                    110928df f   LIBCMT:onexit.obj
 0001:000918f6       __initp_heap_handler       110928f6 f   LIBCMT:handler.obj
 0001:00091905       __callnewh                 11092905 f   LIBCMT:handler.obj
 0001:0009192d       __CxxThrowException@8      1109292d f   LIBCMT:throw.obj
 0001:00091979       __crt_debugger_hook        11092979 f   LIBCMT:dbghook.obj
 0001:00091981       __ioinit                   11092981 f   LIBCMT:ioinit.obj
 0001:00091bd5       __ioterm                   11092bd5 f   LIBCMT:ioinit.obj
 0001:00091c23       __fileno                   11092c23 f   LIBCMT:fileno.obj
 0001:00091c58       __SEH_prolog4              11092c58 f   LIBCMT:sehprolg4.obj
 0001:00091c9d       __SEH_epilog4              11092c9d f   LIBCMT:sehprolg4.obj
 0001:00091cc0       __except_handler4          11092cc0 f   LIBCMT:chandler4.obj
 0001:00091e4c       __heap_init                11092e4c f   LIBCMT:heapinit.obj
 0001:00091e7c       __heap_term                11092e7c f   LIBCMT:heapinit.obj
 0001:00091ef0       __mtinitlocks              11092ef0 f   LIBCMT:mlock.obj
 0001:00091f3b       __mtdeletelocks            11092f3b f   LIBCMT:mlock.obj
 0001:00091f92       __unlock                   11092f92 f   LIBCMT:mlock.obj
 0001:00091fa9       __mtinitlocknum            11092fa9 f   LIBCMT:mlock.obj
 0001:0009206c       __lock                     1109306c f   LIBCMT:mlock.obj
 0001:0009209f       ___sbh_find_block          1109309f f   LIBCMT:sbheap.obj
 0001:000920cf       ___sbh_free_block          110930cf f   LIBCMT:sbheap.obj
 0001:000923e5       ___sbh_alloc_new_region    110933e5 f   LIBCMT:sbheap.obj
 0001:00092495       ___sbh_alloc_new_group     11093495 f   LIBCMT:sbheap.obj
 0001:0009259d       ___sbh_resize_block        1109359d f   LIBCMT:sbheap.obj
 0001:0009287e       ___sbh_alloc_block         1109387e f   LIBCMT:sbheap.obj
 0001:00092b63       __getbuf                   11093b63 f   LIBCMT:_getbuf.obj
 0001:00092bac       __write_nolock             11093bac f   LIBCMT:write.obj
 0001:000932df       __write                    110942df f   LIBCMT:write.obj
 0001:000933bb       __commit                   110943bb f   LIBCMT:commit.obj
 0001:0009349c       __filbuf                   1109449c f   LIBCMT:_filbuf.obj
 0001:000935c7       __vsnprintf_l              110945c7 f   LIBCMT:vsnprint.obj
 0001:0009367a       __vsnprintf                1109467a f   LIBCMT:vsnprint.obj
 0001:0009367a       _vsnprintf                 1109467a f   LIBCMT:vsnprint.obj
 0001:00093a3c       ___crtLCMapStringA         11094a3c f   LIBCMT:a_map.obj
 0001:00093a81       __isleadbyte_l             11094a81 f i LIBCMT:_wctype.obj
 0001:00093ab9       _isleadbyte                11094ab9 f i LIBCMT:_wctype.obj
 0001:00093acc       __isctype_l                11094acc f   LIBCMT:isctype.obj
 0001:00093b84       __stbuf                    11094b84 f   LIBCMT:_sftbuf.obj
 0001:00093c20       __ftbuf                    11094c20 f   LIBCMT:_sftbuf.obj
 0001:00093c54       __malloc_crt               11094c54 f   LIBCMT:crtheap.obj
 0001:00093c99       __calloc_crt               11094c99 f   LIBCMT:crtheap.obj
 0001:00093ce5       __realloc_crt              11094ce5 f   LIBCMT:crtheap.obj
 0001:00093d33       __recalloc_crt             11094d33 f   LIBCMT:crtheap.obj
 0001:00093d85       __freebuf                  11094d85 f   LIBCMT:_freebuf.obj
 0001:00093db6       __lseek_nolock             11094db6 f   LIBCMT:lseek.obj
 0001:00093e2b       __lseek                    11094e2b f   LIBCMT:lseek.obj
 0001:00093f07       __close_nolock             11094f07 f   LIBCMT:close.obj
 0001:00093fa3       __close                    11094fa3 f   LIBCMT:close.obj
 0001:00094070       __openfile                 11095070 f   LIBCMT:_open.obj
 0001:00094339       __getstream                11095339 f   LIBCMT:stream.obj
 0001:00094474       __local_unwind4            11095474 f   LIBCMT:exsup4.obj
 0001:0009454a       __seh_longjmp_unwind4@4    1109554a f   LIBCMT:exsup4.obj
 0001:00094566       @_EH4_CallFilterFunc@8     11095566 f   LIBCMT:exsup4.obj
 0001:0009457d       @_EH4_TransferToHandler@8  1109557d f   LIBCMT:exsup4.obj
 0001:00094596       @_EH4_GlobalUnwind@4       11095596 f   LIBCMT:exsup4.obj
 0001:000945b0       @_EH4_LocalUnwind@16       110955b0 f   LIBCMT:exsup4.obj
 0001:000945c7       _abort                     110955c7 f   LIBCMT:abort.obj
 0001:000946de       __set_abort_behavior       110956de f   LIBCMT:abort.obj
 0001:000946ff       __NMSG_WRITE               110956ff f   LIBCMT:crt0msg.obj
 0001:000948aa       __FF_MSGBANNER             110958aa f   LIBCMT:crt0msg.obj
 0001:000948e3       ___getlocaleinfo           110958e3 f   LIBCMT:inithelp.obj
 0001:00094a62       __initp_misc_purevirt      11095a62 f   LIBCMT:inithelp.obj
 0001:00094b3b       __input_l                  11095b3b f   LIBCMT:input.obj
 0001:00095af8       __fltin2                   11096af8 f   LIBCMT:_cfin_.obj
 0001:00095b9f       __cfltcvt_init             11096b9f f   LIBCMT:_fpinit_.obj
 0001:00095bff       __fpmath                   11096bff f   LIBCMT:_fpinit_.obj
 0001:00095c22       ___strgtold12_l            11096c22 f   LIBCMT:_strgtold_.obj
 0001:00096320       __allmul                   11097320 f   LIBCMT:llmul.obj
 0001:00096354       ___sys_nerr                11097354 f   LIBCMT:syserr.obj
 0001:0009635a       ___sys_errlist             1109735a f   LIBCMT:syserr.obj
 0001:00096360       _strncpy_s                 11097360 f   LIBCMT:strncpy_s.obj
 0001:00096415       __fcloseall                11097415 f   LIBCMT:closeall.obj
 0001:000964b4       __read_nolock              110974b4 f   LIBCMT:read.obj
 0001:00096a76       __read                     11097a76 f   LIBCMT:read.obj
 0001:00096b74       __global_unwind2           11097b74 f   LIBCMT:exsup.obj
 0001:00096bd9       __local_unwind2            11097bd9 f   LIBCMT:exsup.obj
 0001:00096c5d       __abnormal_termination     11097c5d f   LIBCMT:exsup.obj
 0001:00096c80       __NLG_Notify1              11097c80 f   LIBCMT:exsup.obj
 0001:00096c89       __NLG_Notify               11097c89 f   LIBCMT:exsup.obj
 0001:00096ca0       __NLG_Dispatch2            11097ca0     LIBCMT:exsup.obj
 0001:00096ca0       __NLG_Dispatch             11097ca0     LIBCMT:exsup.obj
 0001:00096ca8       __NLG_Call                 11097ca8 f   LIBCMT:exsup.obj
 0001:00096caa       __NLG_Return2              11097caa     LIBCMT:exsup.obj
 0001:00096cab       __rt_probe_read4@4         11097cab f   LIBCMT:sehsupp.obj
 0001:00096cf6       __RTC_Initialize           11097cf6 f   LIBCMT:_initsect_.obj
 0001:00096d1c       __RTC_Terminate            11097d1c f   LIBCMT:_initsect_.obj
 0001:00096d42       __initp_misc_cfltcvt_tab   11097d42 f   LIBCMT:cmiscdat.obj
 0001:00096d70       __ValidateImageBase        11097d70 f   LIBCMT:pesect.obj
 0001:00096db0       __FindPESection            11097db0 f   LIBCMT:pesect.obj
 0001:00096e00       __IsNonwritableInCurrentImage 11097e00 f   LIBCMT:pesect.obj
 0001:00096ebd       ?terminate@@YAXXZ          11097ebd f   LIBCMT:hooks.obj
 0001:00096ef6       ?unexpected@@YAXXZ         11097ef6 f   LIBCMT:hooks.obj
 0001:00096f09       ?_inconsistency@@YAXXZ     11097f09 f   LIBCMT:hooks.obj
 0001:00096f41       __initp_eh_hooks           11097f41 f   LIBCMT:hooks.obj
 0001:00096f52       __fpclear                  11097f52 f   LIBCMT:_fpinit_.obj
 0001:00096f52       __initp_misc_winxfltr      11097f52 f   LIBCMT:winxfltr.obj
 0001:00096f53       __XcptFilter               11097f53 f   LIBCMT:winxfltr.obj
 0001:000970b3       ___CppXcptFilter           110980b3 f   LIBCMT:winxfltr.obj
 0001:000970d3       __initp_misc_winsig        110980d3 f   LIBCMT:winsig.obj
 0001:00097128       ___get_sigabrt             11098128 f   LIBCMT:winsig.obj
 0001:00097135       _raise                     11098135 f   LIBCMT:winsig.obj
 0001:000972e5       __initp_misc_rand_s        110982e5 f   LIBCMT:rand_s.obj
 0001:000972f4       __initp_misc_initcrit      110982f4 f   LIBCMT:initcrit.obj
 0001:00097303       ___crtInitCritSecAndSpinCount 11098303 f   LIBCMT:initcrit.obj
 0001:00097363       _strcat_s                  11098363 f   LIBCMT:strcat_s.obj
 0001:000974b4       __itoa_s                   110984b4 f   LIBCMT:xtoas.obj
 0001:000974de       __ultoa_s                  110984de f   LIBCMT:xtoas.obj
 0001:000974f8       __getpid                   110984f8 f   LIBCMT:getpid.obj
 0001:000974fe       __mbsrchr_l                110984fe f   LIBCMT:mbsrchr.obj
 0001:000975ba       __mbsrchr                  110985ba f   LIBCMT:mbsrchr.obj
 0001:000975d1       __rmtmp                    110985d1 f   LIBCMT:rmtmp.obj
 0001:0009767a       __access_s                 1109867a f   LIBCMT:access.obj
 0001:00097703       __strdup                   11098703 f   LIBCMT:strdup.obj
 0001:00097e77       __sopen_helper             11098e77 f   LIBCMT:open.obj
 0001:00097f43       __sopen_s                  11098f43 f   LIBCMT:open.obj
 0001:00097f63       __getpath                  11098f63 f   LIBCMT:getpath.obj
 0001:00097ff8       __fdopen                   11098ff8 f   LIBCMT:fdopen.obj
 0001:0009817e       __pipe                     1109917e f   LIBCMT:pipe.obj
 0001:00098435       __cwait                    11099435 f   LIBCMT:wait.obj
 0001:000984c6       ___libm_error_support      110994c6 f   LIBCMT:_libm_error_.obj
 0001:00098776       __sse2_mathfcns_init       11099776 f   LIBCMT:_mathfcns_.obj
 0001:0009878a       __ceil_default             1109978a f   LIBCMT:_ceil_.obj
 0001:0009885f       __modf_default             1109985f f   LIBCMT:_modf_.obj
 0001:0009896e       __set_exp                  1109996e f   LIBCMT:_util_.obj
 0001:0009899a       __sptype                   1109999a f   LIBCMT:_util_.obj
 0001:000989fa       __decomp                   110999fa f   LIBCMT:_util_.obj
 0001:00098ab3       __copysign                 11099ab3 f   LIBCMT:_ieeemisc_.obj
 0001:00098adb       __fpclass                  11099adb f   LIBCMT:_ieeemisc_.obj
 0001:00098b6f       __raise_exc_ex             11099b6f f   LIBCMT:_fpexcept_.obj
 0001:00098e4b       __raise_exc                11099e4b f   LIBCMT:_fpexcept_.obj
 0001:00098e6e       __handle_exc               11099e6e f   LIBCMT:_fpexcept_.obj
 0001:00099050       __set_errno_from_matherr   1109a050 f   LIBCMT:_fpexcept_.obj
 0001:0009907d       __errcode                  1109a07d f   LIBCMT:_fpexcept_.obj
 0001:000990b1       __umatherr                 1109a0b1 f   LIBCMT:_fpexcept_.obj
 0001:00099151       __handle_qnan1             1109a151 f   LIBCMT:_fpexcept_.obj
 0001:000991a6       __handle_qnan2             1109a1a6 f   LIBCMT:_fpexcept_.obj
 0001:00099207       __except1                  1109a207 f   LIBCMT:_fpexcept_.obj
 0001:000992d0       __except2                  1109a2d0 f   LIBCMT:_fpexcept_.obj
 0001:000993a8       __statfp                   1109a3a8 f   LIBCMT:_fpctrl_.obj
 0001:000993b8       __clrfp                    1109a3b8 f   LIBCMT:_fpctrl_.obj
 0001:000993c9       __ctrlfp                   1109a3c9 f   LIBCMT:_fpctrl_.obj
 0001:000993f2       __set_statfp               1109a3f2 f   LIBCMT:_fpctrl_.obj
 0001:0009944a       ___set_fpsr_sse2           1109a44a f   LIBCMT:_fpctrl_.obj
 0001:000994bc       __mbsnbicoll_l             1109a4bc f   LIBCMT:mbsnbico.obj
 0001:000995aa       __mbsnbicoll               1109a5aa f   LIBCMT:mbsnbico.obj
 0001:000995c4       ___wtomb_environ           1109a5c4 f   LIBCMT:wtombenv.obj
 0001:0009965b       _calloc                    1109a65b f   LIBCMT:calloc.obj
 0001:0009969b       _strnlen                   1109a69b f   LIBCMT:strlen_s.obj
 0001:000996b8       __spawnvpe                 1109a6b8 f   LIBCMT:spawnvpe.obj
 0001:000999aa       __spawnve                  1109a9aa f   LIBCMT:spawnve.obj
 0001:00099bd0       __alloca_probe_16          1109abd0 f   LIBCMT:alloca16.obj
 0001:00099be6       __alloca_probe_8           1109abe6     LIBCMT:alloca16.obj
 0001:0009a017       ___free_lc_time            1109b017 f   LIBCMT:inittime.obj
 0001:0009a1ac       ___init_time               1109b1ac f   LIBCMT:inittime.obj
 0001:0009a225       ___free_lconv_num          1109b225 f   LIBCMT:initnum.obj
 0001:0009a26a       ___init_numeric            1109b26a f   LIBCMT:initnum.obj
 0001:0009a434       ___free_lconv_mon          1109b434 f   LIBCMT:initmon.obj
 0001:0009a4c2       ___init_monetary           1109b4c2 f   LIBCMT:initmon.obj
 0001:0009a788       ___init_ctype              1109b788 f   LIBCMT:initctyp.obj
 0001:0009ab2a       ____lc_codepage_func       1109bb2a f   LIBCMT:initctyp.obj
 0001:0009b10b       ___get_qualified_locale    1109c10b f   LIBCMT:getqloc.obj
 0001:0009b2fc       _memcmp                    1109c2fc f   LIBCMT:memcmp.obj
 0001:0009cb36       ___crtGetStringTypeA       1109db36 f   LIBCMT:a_str.obj
 0001:0009cf06       ___crtCompareStringA       1109df06 f   LIBCMT:a_cmp.obj
 0001:0009cfcf       __VEC_memcpy               1109dfcf f   LIBCMT:p4_memcpy.obj
 0001:0009d0b2       __setenvp                  1109e0b2 f   LIBCMT:stdenvp.obj
 0001:0009d32a       __setargv                  1109e32a f   LIBCMT:stdargv.obj
 0001:0009d3e5       ___crtGetEnvironmentStringsA 1109e3e5 f   LIBCMT:a_env.obj
 0001:0009d51c       ___security_init_cookie    1109e51c f   LIBCMT:gs_support.obj
 0001:0009d5b2       __lseeki64_nolock          1109e5b2 f   LIBCMT:lseeki64.obj
 0001:0009d637       __lseeki64                 1109e637 f   LIBCMT:lseeki64.obj
 0001:0009d750       __isatty                   1109e750 f   LIBCMT:isatty.obj
 0001:0009d7b4       __wctomb_s_l               1109e7b4 f   LIBCMT:wctomb.obj
 0001:0009d920       _wctomb_s                  1109e920 f   LIBCMT:wctomb.obj
 0001:0009d940       __aulldvrm                 1109e940 f   LIBCMT:ulldvrm.obj
 0001:0009da2c       __VEC_memzero              1109ea2c f   LIBCMT:p4_memset.obj
 0001:0009dabb       ___report_gsfailure        1109eabb f   LIBCMT:gs_report.obj
 0001:0009dbc1       __msize                    1109ebc1 f   LIBCMT:msize.obj
 0001:0009dc70       __chkstk                   1109ec70 f   LIBCMT:chkstk.obj
 0001:0009dc70       __alloca_probe             1109ec70     LIBCMT:chkstk.obj
 0001:0009dc9b       __putwch_nolock            1109ec9b f   LIBCMT:putwch.obj
 0001:0009dd60       __mbtowc_l                 1109ed60 f   LIBCMT:mbtowc.obj
 0001:0009de77       _mbtowc                    1109ee77 f   LIBCMT:mbtowc.obj
 0001:0009de91       __set_osfhnd               1109ee91 f   LIBCMT:osfinfo.obj
 0001:0009df12       __free_osfhnd              1109ef12 f   LIBCMT:osfinfo.obj
 0001:0009df98       __get_osfhandle            1109ef98 f   LIBCMT:osfinfo.obj
 0001:0009e00f       ___lock_fhandle            1109f00f f   LIBCMT:osfinfo.obj
 0001:0009e0af       __unlock_fhandle           1109f0af f   LIBCMT:osfinfo.obj
 0001:0009e0d6       __alloc_osfhnd             1109f0d6 f   LIBCMT:osfinfo.obj
 0001:0009e270       ___ansicp                  1109f270 f   LIBCMT:convrtcp.obj
 0001:0009e2b9       ___convertcp               1109f2b9 f   LIBCMT:convrtcp.obj
 0001:0009e46d       __calloc_impl              1109f46d f   LIBCMT:calloc_impl.obj
 0001:0009e58b       __recalloc                 1109f58b f   LIBCMT:recalloc.obj
 0001:0009e606       __mbsnbicmp_l              1109f606 f   LIBCMT:mbsnbicm.obj
 0001:0009e831       __mbsnbicmp                1109f831 f   LIBCMT:mbsnbicm.obj
 0001:0009e84b       __mbsnbcmp_l               1109f84b f   LIBCMT:mbsnbcmp.obj
 0001:0009e9b5       __mbsnbcmp                 1109f9b5 f   LIBCMT:mbsnbcmp.obj
 0001:0009e9cf       ___crtMessageBoxA          1109f9cf f   LIBCMT:crtmbox.obj
 0001:0009eb38       __set_error_mode           1109fb38 f   LIBCMT:errmode.obj
 0001:0009eb83       ___crtGetLocaleInfoW       1109fb83 f   LIBCMT:w_loc.obj
 0001:0009ecf6       ___crtGetLocaleInfoA       1109fcf6 f   LIBCMT:a_loc.obj
 0001:0009ed33       __ld12tod                  1109fd33 f   LIBCMT:_intrncvt_.obj
 0001:0009f277       __ld12tof                  110a0277 f   LIBCMT:_intrncvt_.obj
 0001:0009f7bb       __forcdecpt_l              110a07bb f   LIBCMT:cvt.obj
 0001:0009f82e       __cropzeros_l              110a082e f   LIBCMT:cvt.obj
 0001:0009f8b0       __positive                 110a08b0 f   LIBCMT:cvt.obj
 0001:0009f8cc       __fassign_l                110a08cc f   LIBCMT:cvt.obj
 0001:0009f90e       __fassign                  110a090e f   LIBCMT:cvt.obj
 0001:0009f947       __forcdecpt                110a0947 f   LIBCMT:cvt.obj
 0001:0009f95a       __cropzeros                110a095a f   LIBCMT:cvt.obj
 0001:0009fadc       __cftoe_l                  110a0adc f   LIBCMT:cvt.obj
 0001:0009fbac       __cftoe                    110a0bac f   LIBCMT:cvt.obj
 0001:0009fbcc       __cftoa_l                  110a0bcc f   LIBCMT:cvt.obj
 0001:000a0036       __cftof_l                  110a1036 f   LIBCMT:cvt.obj
 0001:000a00f1       __cftog_l                  110a10f1 f   LIBCMT:cvt.obj
 0001:000a01eb       __cfltcvt_l                110a11eb f   LIBCMT:cvt.obj
 0001:000a0273       __cfltcvt                  110a1273 f   LIBCMT:cvt.obj
 0001:000a0296       __setdefaultprecision      110a1296 f   LIBCMT:fp8.obj
 0001:000a02c1       __ms_p5_test_fdiv          110a12c1 f   LIBCMT:_testfdiv_.obj
 0001:000a02ff       __ms_p5_mp_test_fdiv       110a12ff f   LIBCMT:_testfdiv_.obj
 0001:000a0328       ___mtold12                 110a1328 f   LIBCMT:_mantold_.obj
 0001:000a04f6       __fptrap                   110a14f6 f   LIBCMT:crt0fp.obj
 0001:000a04ff       __chsize_nolock            110a14ff f   LIBCMT:chsize.obj
 0001:000a06b5       __setmode_nolock           110a16b5 f   LIBCMT:setmode.obj
 0001:000a0771       __get_fmode                110a1771 f   LIBCMT:setmode.obj
 0001:000a07aa       __matherr                  110a17aa f   LIBCMT:_matherr_.obj
 0001:000a07aa       ___init_collate            110a17aa f   LIBCMT:initcoll.obj
 0001:000a07aa       ___init_dummy              110a17aa f   LIBCMT:setlocal.obj
 0001:000a07fd       __get_sse2_info            110a17fd f   LIBCMT:cpu_disp.obj
 0001:000a085f       ___sse2_available_init     110a185f f   LIBCMT:cpu_disp.obj
 0001:000a086c       __frnd                     110a186c f   LIBCMT:_frnd_.obj
 0001:000a0880       __strnicoll_l              110a1880 f   LIBCMT:strnicol.obj
 0001:000a0a26       ___crtsetenv               110a1a26 f   LIBCMT:setenv.obj
 0001:000a0c71       __mbschr_l                 110a1c71 f   LIBCMT:mbschr.obj
 0001:000a0d2d       __mbschr                   110a1d2d f   LIBCMT:mbschr.obj
 0001:000a0d44       __dospawn                  110a1d44 f   LIBCMT:dospawn.obj
 0001:000a0f53       __cenvarg                  110a1f53 f   LIBCMT:cenvarg.obj
 0001:000a132c       __strnicmp_l               110a232c f   LIBCMT:strnicmp.obj
 0001:000a141e       __strnicmp                 110a241e f   LIBCMT:strnicmp.obj
 0001:000a14cf       __ismbblead                110a24cf f   LIBCMT:ismbbyte.obj
 0001:000a14e7       ___initconout              110a24e7 f   LIBCMT:initcon.obj
 0001:000a1506       ___termcon                 110a2506 f   LIBCMT:initcon.obj
 0001:000a1533       __atodbl_l                 110a2533 f   LIBCMT:atodbl.obj
 0001:000a15db       __atoflt_l                 110a25db f   LIBCMT:atodbl.obj
 0001:000a1683       __fptostr                  110a2683 f   LIBCMT:_fptostr.obj
 0001:000a1742       ___dtold                   110a2742 f   LIBCMT:_cfout_.obj
 0001:000a17ff       __fltout2                  110a27ff f   LIBCMT:_cfout_.obj
 0001:000a1890       __alldvrm                  110a2890 f   LIBCMT:lldvrm.obj
 0001:000a1970       __aullshr                  110a2970 f   LIBCMT:ullshr.obj
 0001:000a198f       __controlfp_s              110a298f f   LIBCMT:_contrlfp_.obj
 0001:000a19fb       __mbsnicmp_l               110a29fb f   LIBCMT:mbsnicmp.obj
 0001:000a1bc3       __mbsnicmp                 110a2bc3 f   LIBCMT:mbsnicmp.obj
 0001:000a1be0       ___ascii_strnicmp          110a2be0 f   LIBCMT:_strnicm.obj
 0001:000a1c41       _$I10_OUTPUT               110a2c41 f   LIBCMT:_x10fout_.obj
 0001:000a2693       __control87                110a3693 f i LIBCMT:_ieee87_.obj
 0001:000a29a2       ??0out_of_range@std@@QAE@ABV?$basic_string@DU?$char_traits@D@std@@V?$allocator@D@2@@1@@Z 110a39a2 f i libcpmt:string.obj
 0001:000a29bf       ??1out_of_range@std@@UAE@XZ 110a39bf f i libcpmt:string.obj
 0001:000a29ca       ??_Eout_of_range@std@@UAEPAXI@Z 110a39ca f i libcpmt:string.obj
 0001:000a29ca       ??_Gout_of_range@std@@UAEPAXI@Z 110a39ca f i libcpmt:string.obj
 0001:000a29f1       ?_Xlen@_String_base@std@@SAXXZ 110a39f1 f   libcpmt:string.obj
 0001:000a2a29       ?_Xran@_String_base@std@@SAXXZ 110a3a29 f   libcpmt:string.obj
 0001:000a2a61       ??0out_of_range@std@@QAE@ABV01@@Z 110a3a61 f i libcpmt:string.obj
 0001:000a2a7e       ??0_Init_locks@std@@QAE@XZ 110a3a7e f   libcpmt:xlock.obj
 0001:000a2aaf       ??1_Init_locks@std@@QAE@XZ 110a3aaf f   libcpmt:xlock.obj
 0001:000a2ad8       ??0_Lockit@std@@QAE@H@Z    110a3ad8 f   libcpmt:xlock.obj
 0001:000a2b00       ??1_Lockit@std@@QAE@XZ     110a3b00 f   libcpmt:xlock.obj
 0001:000a2b6a       ??1_Init_atexit@@QAE@XZ    110a3b6a f i libcpmt:iosptrs.obj
 0001:000a2b8f       __Mtxinit                  110a3b8f f   libcpmt:xmtx.obj
 0001:000a2b9f       __Mtxdst                   110a3b9f f   libcpmt:xmtx.obj
 0001:000a2baf       __Mtxlock                  110a3baf f   libcpmt:xmtx.obj
 0001:000a2bbf       __Mtxunlock                110a3bbf f   libcpmt:xmtx.obj
 0001:000a2bd0       _RtlUnwind@16              110a3bd0 f   kernel32:KERNEL32.dll
 0001:000a2bd6       ?_JumpToContinuation@@YGXPAXPAUEHRegistrationNode@@@Z 110a3bd6 f   LIBCMT:_trnsctrl_.obj
 0001:000a2c08       ?_CallMemberFunction2@@YGXPAX00H@Z 110a3c08 f   LIBCMT:_trnsctrl_.obj
 0001:000a2c08       ?_CallMemberFunction0@@YGXPAX0@Z 110a3c08 f   LIBCMT:_trnsctrl_.obj
 0001:000a2c08       ?_CallMemberFunction1@@YGXPAX00@Z 110a3c08 f   LIBCMT:_trnsctrl_.obj
 0001:000a2c0f       ?_UnwindNestedFrames@@YGXPAUEHRegistrationNode@@PAUEHExceptionRecord@@@Z 110a3c0f f   LIBCMT:_trnsctrl_.obj
 0001:000a2c63       ___CxxFrameHandler3        110a3c63 f   LIBCMT:_trnsctrl_.obj
 0001:000a2ccc       ?_CallSETranslator@@YAHPAUEHExceptionRecord@@PAUEHRegistrationNode@@PAX2PBU_s_FuncInfo@@H1@Z 110a3ccc f   LIBCMT:_trnsctrl_.obj
 0001:000a2e42       ?_GetRangeOfTrysToCheck@@YAPBU_s_TryBlockMapEntry@@PBU_s_FuncInfo@@HHPAI1@Z 110a3e42 f   LIBCMT:_trnsctrl_.obj
 0001:000a2eb7       __CreateFrameInfo          110a3eb7 f   LIBCMT:_trnsctrl_.obj
 0001:000a2ee3       __IsExceptionObjectToBeDestroyed 110a3ee3 f   LIBCMT:_trnsctrl_.obj
 0001:000a2f0a       __FindAndUnlinkFrame       110a3f0a f   LIBCMT:_trnsctrl_.obj
 0001:000a2f5c       ?_CallCatchBlock2@@YAPAXPAUEHRegistrationNode@@PBU_s_FuncInfo@@PAXHK@Z 110a3f5c f   LIBCMT:_trnsctrl_.obj
 0001:000a2fbc       __EH_prolog3               110a3fbc f   LIBCMT:ehprolg3.obj
 0001:000a2fef       __EH_prolog3_catch         110a3fef f   LIBCMT:ehprolg3.obj
 0001:000a3025       ??0bad_exception@std@@QAE@PBD@Z 110a4025 f i LIBCMT:frame.obj
 0001:000a3043       ??1bad_exception@std@@UAE@XZ 110a4043 f i LIBCMT:frame.obj
 0001:000a304e       ??_Ebad_exception@std@@UAEPAXI@Z 110a404e f i LIBCMT:frame.obj
 0001:000a304e       ??_Gbad_exception@std@@UAEPAXI@Z 110a404e f i LIBCMT:frame.obj
 0001:000a3075       ___TypeMatch               110a4075 f   LIBCMT:frame.obj
 0001:000a30d4       ___FrameUnwindFilter       110a40d4 f   LIBCMT:frame.obj
 0001:000a311d       ___FrameUnwindToState      110a411d f   LIBCMT:frame.obj
 0001:000a3243       ___DestructExceptionObject 110a4243 f   LIBCMT:frame.obj
 0001:000a3298       ___AdjustPointer           110a4298 f   LIBCMT:frame.obj
 0001:000a3521       ___BuildCatchObjectHelper  110a4521 f   LIBCMT:frame.obj
 0001:000a36a0       ___BuildCatchObject        110a46a0 f   LIBCMT:frame.obj
 0001:000a3bdb       ??0bad_exception@std@@QAE@ABV01@@Z 110a4bdb f i LIBCMT:frame.obj
 0001:000a3bf8       ___InternalCxxFrameHandler 110a4bf8 f   LIBCMT:frame.obj
 0001:000a3ce0       __CallSettingFrame@12      110a4ce0 f   LIBCMT:lowhelpr.obj
 0001:000a3d07       __NLG_Return               110a4d07     LIBCMT:lowhelpr.obj
 0001:000a3d2c       ?_ValidateWrite@@YAHPAXI@Z 110a4d2c f   LIBCMT:validate.obj
 0001:000a3d2c       ?_ValidateRead@@YAHPBXI@Z  110a4d2c f   LIBCMT:validate.obj
 0001:000a3d2c       ?_ValidateExecute@@YAHP6GHXZ@Z 110a4d2c f   LIBCMT:validate.obj
 0001:000a3d40       __allshl                   110a4d40 f   LIBCMT:llshl.obj
 0001:000a3d60       __ftol2_sse                110a4d60 f   LIBCMT:ftol2.obj
 0001:000a3d69       __ftol2_pentium4           110a4d69 f   LIBCMT:ftol2.obj
 0001:000a3d7c       __ftol2_sse_excpt          110a4d7c f   LIBCMT:ftol2.obj
 0001:000a3d96       __ftol2                    110a4d96 f   LIBCMT:ftol2.obj
 0001:000a3e0c       __setjmp3                  110a4e0c f   LIBCMT:setjmp3.obj
 0001:000a3e90       _pow                       110a4e90 f   LIBCMT:_pow_.obj
 0001:000a3ed0       __CIpow                    110a4ed0 f   LIBCMT:_pow_.obj
 0001:000a3f0b       __CIpow_default            110a4f0b f   LIBCMT:_pow_.obj
 0001:000a3f24       __pow_default              110a4f24     LIBCMT:_pow_.obj
 0001:000a4120       _floor                     110a5120 f   LIBCMT:_floor_pentium4_.obj
 0001:000a4160       __floor_pentium4           110a5160 f   LIBCMT:_floor_pentium4_.obj
 0001:000a4250       __aullrem                  110a5250 f   LIBCMT:ullrem.obj
 0001:000a42d0       _fmod                      110a52d0 f   LIBCMT:_87fmod_.obj
 0001:000a42da       __CIfmod                   110a52da f   LIBCMT:_87fmod_.obj
 0001:000a4310       _acos                      110a5310 f   LIBCMT:_acos_.obj
 0001:000a4350       __CIacos                   110a5350 f   LIBCMT:_acos_.obj
 0001:000a438b       __CIacos_default           110a538b f   LIBCMT:_acos_.obj
 0001:000a439f       __acos_default             110a539f     LIBCMT:_acos_.obj
 0001:000a4460       _asin                      110a5460 f   LIBCMT:_asin_.obj
 0001:000a44a0       __CIasin                   110a54a0 f   LIBCMT:_asin_.obj
 0001:000a44db       __CIasin_default           110a54db f   LIBCMT:_asin_.obj
 0001:000a44ef       __asin_default             110a54ef     LIBCMT:_asin_.obj
 0001:000a45b0       _sinh                      110a55b0 f   LIBCMT:_87ctrigh_.obj
 0001:000a45ba       _cosh                      110a55ba f   LIBCMT:_87ctrigh_.obj
 0001:000a45c1       _tanh                      110a55c1 f   LIBCMT:_87ctrigh_.obj
 0001:000a45c8       __CIsinh                   110a55c8 f   LIBCMT:_87ctrigh_.obj
 0001:000a45d2       __CIcosh                   110a55d2 f   LIBCMT:_87ctrigh_.obj
 0001:000a45d9       __CItanh                   110a55d9 f   LIBCMT:_87ctrigh_.obj
 0001:000a45e0       __allshr                   110a55e0 f   LIBCMT:llshr.obj
 0001:000a4610       __CIpow_pentium4           110a5610 f   LIBCMT:_pow_pentium4_.obj
 0001:000a4629       __pow_pentium4             110a5629     LIBCMT:_pow_pentium4_.obj
 0001:000a5181       __fFEXP                    110a6181     LIBCMT:_87tran_.obj
 0001:000a51e8       __rtinfpopse               110a61e8     LIBCMT:_87tran_.obj
 0001:000a51ea       __rtinfnpopse              110a61ea     LIBCMT:_87tran_.obj
 0001:000a51fa       __fFLN                     110a61fa     LIBCMT:_87tran_.obj
 0001:000a52af       __rtinfpop                 110a62af     LIBCMT:_87tran_.obj
 0001:000a52b1       __rtinfnpop                110a62b1     LIBCMT:_87tran_.obj
 0001:000a52ce       __ffexpm1                  110a62ce     LIBCMT:_87tran_.obj
 0001:000a5380       __trandisp1                110a6380 f   LIBCMT:_87disp_.obj
 0001:000a53e7       __trandisp2                110a63e7 f   LIBCMT:_87disp_.obj
 0001:000a5473       __rttospopde               110a6473     LIBCMT:_87disp_.obj
 0001:000a5478       __rttospop                 110a6478     LIBCMT:_87disp_.obj
 0001:000a547a       __rtnospop                 110a647a     LIBCMT:_87disp_.obj
 0001:000a547c       __rttosnpop                110a647c     LIBCMT:_87disp_.obj
 0001:000a547d       __rtnospopde               110a647d     LIBCMT:_87disp_.obj
 0001:000a5484       __rtzeropop                110a6484     LIBCMT:_87disp_.obj
 0001:000a5486       __rtzeronpop               110a6486     LIBCMT:_87disp_.obj
 0001:000a548b       __rtonepop                 110a648b     LIBCMT:_87disp_.obj
 0001:000a548d       __rtonenpop                110a648d     LIBCMT:_87disp_.obj
 0001:000a5492       __tosnan1                  110a6492     LIBCMT:_87disp_.obj
 0001:000a54bd       __nosnan2                  110a64bd     LIBCMT:_87disp_.obj
 0001:000a54bf       __tosnan2                  110a64bf     LIBCMT:_87disp_.obj
 0001:000a54e7       __nan2                     110a64e7     LIBCMT:_87disp_.obj
 0001:000a5526       __rtindfpop                110a6526     LIBCMT:_87disp_.obj
 0001:000a5528       __rtindfnpop               110a6528     LIBCMT:_87disp_.obj
 0001:000a5539       __rttosnpopde              110a6539     LIBCMT:_87disp_.obj
 0001:000a5543       __rtchsifneg               110a6543     LIBCMT:_87disp_.obj
 0001:000a5550       __startTwoArgErrorHandling 110a6550 f   LIBCMT:_genexcep_.obj
 0001:000a5567       __startOneArgErrorHandling 110a6567 f   LIBCMT:_genexcep_.obj
 0001:000a55b0       __twoToTOS                 110a65b0 f   LIBCMT:_common_.obj
 0001:000a55c5       __load_CW                  110a65c5 f   LIBCMT:_common_.obj
 0001:000a55dc       __convertTOStoQNaN         110a65dc f   LIBCMT:_common_.obj
 0001:000a55f5       __fload_withFB             110a65f5 f   LIBCMT:_common_.obj
 0001:000a5638       __checkTOS_withFB          110a6638 f   LIBCMT:_common_.obj
 0001:000a564e       __fast_exit                110a664e f   LIBCMT:_common_.obj
 0001:000a565b       __math_exit                110a665b f   LIBCMT:_common_.obj
 0001:000a5685       __check_overflow_exit      110a6685 f   LIBCMT:_common_.obj
 0001:000a5699       __check_range_exit         110a6699 f   LIBCMT:_common_.obj
 0001:000a573c       __d_inttype                110a673c f   LIBCMT:_powhlp_.obj
 0001:000a57a2       __powhlp                   110a67a2 f   LIBCMT:_powhlp_.obj
 0001:000a58e2       __floor_default            110a68e2 f   LIBCMT:_floor_.obj
 0001:000a59c0       __cintrindisp2             110a69c0 f   LIBCMT:_87cdisp_.obj
 0001:000a59fe       __cintrindisp1             110a69fe f   LIBCMT:_87cdisp_.obj
 0001:000a5a3b       __ctrandisp2               110a6a3b f   LIBCMT:_87cdisp_.obj
 0001:000a5bd1       __ctrandisp1               110a6bd1 f   LIBCMT:_87cdisp_.obj
 0001:000a5c04       __fload                    110a6c04 f   LIBCMT:_87cdisp_.obj
 0001:000a5c40       _fdiv_main_routine         110a6c40 f   LIBCMT:_adj_fdiv_.obj
 0001:000a5d57       __adj_fdiv_r               110a6d57 f   LIBCMT:_adj_fdiv_.obj
 0001:000a61f6       __fdivp_sti_st             110a71f6 f   LIBCMT:_adj_fdiv_.obj
 0001:000a6209       __fdivrp_sti_st            110a7209 f   LIBCMT:_adj_fdiv_.obj
 0001:000a621c       __adj_fdiv_m32             110a721c f   LIBCMT:_adj_fdiv_.obj
 0001:000a6268       __adj_fdiv_m64             110a7268 f   LIBCMT:_adj_fdiv_.obj
 0001:000a62b4       __adj_fdiv_m16i            110a72b4 f   LIBCMT:_adj_fdiv_.obj
 0001:000a62e8       __adj_fdiv_m32i            110a72e8 f   LIBCMT:_adj_fdiv_.obj
 0001:000a631c       __adj_fdivr_m32            110a731c f   LIBCMT:_adj_fdiv_.obj
 0001:000a6368       __adj_fdivr_m64            110a7368 f   LIBCMT:_adj_fdiv_.obj
 0001:000a63b4       __adj_fdivr_m16i           110a73b4 f   LIBCMT:_adj_fdiv_.obj
 0001:000a63e8       __adj_fdivr_m32i           110a73e8 f   LIBCMT:_adj_fdiv_.obj
 0001:000a641c       __safe_fdiv                110a741c f   LIBCMT:_adj_fdiv_.obj
 0001:000a6431       __safe_fdivr               110a7431 f   LIBCMT:_adj_fdiv_.obj
 0001:000a6446       __fprem_common             110a7446 f   LIBCMT:_adj_fdiv_.obj
 0001:000a664c       __adj_fprem                110a764c f   LIBCMT:_adj_fdiv_.obj
 0001:000a66fe       __fprem1_common            110a76fe f   LIBCMT:_adj_fdiv_.obj
 0001:000a6904       __adj_fprem1               110a7904 f   LIBCMT:_adj_fdiv_.obj
 0001:000a69b9       __safe_fprem               110a79b9 f   LIBCMT:_adj_fdiv_.obj
 0001:000a69bf       __safe_fprem1              110a79bf f   LIBCMT:_adj_fdiv_.obj
 0001:000a69c5       __adj_fpatan               110a79c5 f   LIBCMT:_adj_fdiv_.obj
 0001:000a69c8       __adj_fptan                110a79c8 f   LIBCMT:_adj_fdiv_.obj
 0001:000a69d0       __CIacos_pentium4          110a79d0 f   LIBCMT:_acos_pentium4_.obj
 0001:000a69e8       __acos_pentium4            110a79e8     LIBCMT:_acos_pentium4_.obj
 0001:000a6f30       __CIasin_pentium4          110a7f30 f   LIBCMT:_asin_pentium4_.obj
 0001:000a6f48       __asin_pentium4            110a7f48     LIBCMT:_asin_pentium4_.obj
 0001:000a74b0       __fFSINH                   110a84b0     LIBCMT:_87trigh_.obj
 0001:000a7502       __fFCOSH                   110a8502     LIBCMT:_87trigh_.obj
 0001:000a75ac       __87except                 110a85ac f   LIBCMT:_87except_.obj
 0002:00000000       __imp__GetModuleHandleA@4  110a9000     kernel32:KERNEL32.dll
 0002:00000004       __imp__GetLocaleInfoW@16   110a9004     kernel32:KERNEL32.dll
 0002:00000008       __imp__SetStdHandle@8      110a9008     kernel32:KERNEL32.dll
 0002:0000000c       __imp__WriteConsoleW@20    110a900c     kernel32:KERNEL32.dll
 0002:00000010       __imp__GetConsoleOutputCP@0 110a9010     kernel32:KERNEL32.dll
 0002:00000014       __imp__WriteConsoleA@20    110a9014     kernel32:KERNEL32.dll
 0002:00000018       __imp__HeapSize@12         110a9018     kernel32:KERNEL32.dll
 0002:0000001c       __imp__GetEnvironmentStringsW@0 110a901c     kernel32:KERNEL32.dll
 0002:00000020       __imp__FreeEnvironmentStringsW@4 110a9020     kernel32:KERNEL32.dll
 0002:00000024       __imp__GetEnvironmentStrings@0 110a9024     kernel32:KERNEL32.dll
 0002:00000028       __imp__FreeEnvironmentStringsA@4 110a9028     kernel32:KERNEL32.dll
 0002:0000002c       __imp__CompareStringW@24   110a902c     kernel32:KERNEL32.dll
 0002:00000030       __imp__CompareStringA@24   110a9030     kernel32:KERNEL32.dll
 0002:00000034       __imp__GetStringTypeW@16   110a9034     kernel32:KERNEL32.dll
 0002:00000038       __imp__GetStringTypeA@20   110a9038     kernel32:KERNEL32.dll
 0002:0000003c       __imp__IsValidLocale@8     110a903c     kernel32:KERNEL32.dll
 0002:00000040       __imp__EnumSystemLocalesA@8 110a9040     kernel32:KERNEL32.dll
 0002:00000044       __imp__GetLocaleInfoA@16   110a9044     kernel32:KERNEL32.dll
 0002:00000048       __imp__GetUserDefaultLCID@0 110a9048     kernel32:KERNEL32.dll
 0002:0000004c       __imp__WaitForSingleObject@8 110a904c     kernel32:KERNEL32.dll
 0002:00000050       __imp__GetExitCodeProcess@8 110a9050     kernel32:KERNEL32.dll
 0002:00000054       __imp__CreatePipe@16       110a9054     kernel32:KERNEL32.dll
 0002:00000058       __imp__GetProcAddress@8    110a9058     kernel32:KERNEL32.dll
 0002:0000005c       __imp__LoadLibraryA@4      110a905c     kernel32:KERNEL32.dll
 0002:00000060       __imp__GetCurrentDirectoryA@8 110a9060     kernel32:KERNEL32.dll
 0002:00000064       __imp__DisableThreadLibraryCalls@4 110a9064     kernel32:KERNEL32.dll
 0002:00000068       __imp__VirtualProtect@16   110a9068     kernel32:KERNEL32.dll
 0002:0000006c       __imp__GetLastError@0      110a906c     kernel32:KERNEL32.dll
 0002:00000070       __imp__CreateThread@24     110a9070     kernel32:KERNEL32.dll
 0002:00000074       __imp__FindFirstFileA@8    110a9074     kernel32:KERNEL32.dll
 0002:00000078       __imp__FindClose@4         110a9078     kernel32:KERNEL32.dll
 0002:0000007c       __imp__FindNextFileA@8     110a907c     kernel32:KERNEL32.dll
 0002:00000080       __imp__FreeLibrary@4       110a9080     kernel32:KERNEL32.dll
 0002:00000084       __imp__FormatMessageA@28   110a9084     kernel32:KERNEL32.dll
 0002:00000088       __imp__GetModuleFileNameA@12 110a9088     kernel32:KERNEL32.dll
 0002:0000008c       __imp__GetProcessHeap@0    110a908c     kernel32:KERNEL32.dll
 0002:00000090       __imp__GetFullPathNameA@16 110a9090     kernel32:KERNEL32.dll
 0002:00000094       __imp__CreateFileA@28      110a9094     kernel32:KERNEL32.dll
 0002:00000098       __imp__GetFileSize@8       110a9098     kernel32:KERNEL32.dll
 0002:0000009c       __imp__SetFilePointer@16   110a909c     kernel32:KERNEL32.dll
 0002:000000a0       __imp__SetEndOfFile@4      110a90a0     kernel32:KERNEL32.dll
 0002:000000a4       __imp__InterlockedIncrement@4 110a90a4     kernel32:KERNEL32.dll
 0002:000000a8       __imp__QueryPerformanceCounter@4 110a90a8     kernel32:KERNEL32.dll
 0002:000000ac       __imp__UnlockFile@20       110a90ac     kernel32:KERNEL32.dll
 0002:000000b0       __imp__LockFile@20         110a90b0     kernel32:KERNEL32.dll
 0002:000000b4       __imp__GetTickCount@0      110a90b4     kernel32:KERNEL32.dll
 0002:000000b8       __imp__GetSystemTimeAsFileTime@4 110a90b8     kernel32:KERNEL32.dll
 0002:000000bc       __imp__WriteFile@20        110a90bc     kernel32:KERNEL32.dll
 0002:000000c0       __imp__InitializeCriticalSection@4 110a90c0     kernel32:KERNEL32.dll
 0002:000000c4       __imp__WideCharToMultiByte@32 110a90c4     kernel32:KERNEL32.dll
 0002:000000c8       __imp__LoadLibraryW@4      110a90c8     kernel32:KERNEL32.dll
 0002:000000cc       __imp__Sleep@4             110a90cc     kernel32:KERNEL32.dll
 0002:000000d0       __imp__LeaveCriticalSection@4 110a90d0     kernel32:KERNEL32.dll
 0002:000000d4       __imp__GetFileAttributesA@4 110a90d4     kernel32:KERNEL32.dll
 0002:000000d8       __imp__GetFileAttributesW@4 110a90d8     kernel32:KERNEL32.dll
 0002:000000dc       __imp__ReadFile@20         110a90dc     kernel32:KERNEL32.dll
 0002:000000e0       __imp__CreateFileW@28      110a90e0     kernel32:KERNEL32.dll
 0002:000000e4       __imp__MultiByteToWideChar@24 110a90e4     kernel32:KERNEL32.dll
 0002:000000e8       __imp__FlushFileBuffers@4  110a90e8     kernel32:KERNEL32.dll
 0002:000000ec       __imp__GetTempPathW@8      110a90ec     kernel32:KERNEL32.dll
 0002:000000f0       __imp__LockFileEx@24       110a90f0     kernel32:KERNEL32.dll
 0002:000000f4       __imp__EnterCriticalSection@4 110a90f4     kernel32:KERNEL32.dll
 0002:000000f8       __imp__DeleteCriticalSection@4 110a90f8     kernel32:KERNEL32.dll
 0002:000000fc       __imp__GetCurrentThreadId@0 110a90fc     kernel32:KERNEL32.dll
 0002:00000100       __imp__GetVersionExA@4     110a9100     kernel32:KERNEL32.dll
 0002:00000104       __imp__CloseHandle@4       110a9104     kernel32:KERNEL32.dll
 0002:00000108       __imp__DeleteFileW@4       110a9108     kernel32:KERNEL32.dll
 0002:0000010c       __imp__GetCurrentProcessId@0 110a910c     kernel32:KERNEL32.dll
 0002:00000110       __imp__GetTempPathA@8      110a9110     kernel32:KERNEL32.dll
 0002:00000114       __imp__GetSystemTime@4     110a9114     kernel32:KERNEL32.dll
 0002:00000118       __imp__AreFileApisANSI@0   110a9118     kernel32:KERNEL32.dll
 0002:0000011c       __imp__SetEnvironmentVariableA@8 110a911c     kernel32:KERNEL32.dll
 0002:00000120       __imp__GetFullPathNameW@16 110a9120     kernel32:KERNEL32.dll
 0002:00000124       __imp__DeleteFileA@4       110a9124     kernel32:KERNEL32.dll
 0002:00000128       __imp__TerminateProcess@8  110a9128     kernel32:KERNEL32.dll
 0002:0000012c       __imp__GetCurrentProcess@0 110a912c     kernel32:KERNEL32.dll
 0002:00000130       __imp__UnhandledExceptionFilter@4 110a9130     kernel32:KERNEL32.dll
 0002:00000134       __imp__SetUnhandledExceptionFilter@4 110a9134     kernel32:KERNEL32.dll
 0002:00000138       __imp__IsDebuggerPresent@0 110a9138     kernel32:KERNEL32.dll
 0002:0000013c       __imp__HeapFree@12         110a913c     kernel32:KERNEL32.dll
 0002:00000140       __imp__HeapReAlloc@16      110a9140     kernel32:KERNEL32.dll
 0002:00000144       __imp__HeapAlloc@12        110a9144     kernel32:KERNEL32.dll
 0002:00000148       __imp__RtlUnwind@16        110a9148     kernel32:KERNEL32.dll
 0002:0000014c       __imp__GetModuleHandleW@4  110a914c     kernel32:KERNEL32.dll
 0002:00000150       __imp__ExitProcess@4       110a9150     kernel32:KERNEL32.dll
 0002:00000154       __imp__CreateProcessA@40   110a9154     kernel32:KERNEL32.dll
 0002:00000158       __imp__DuplicateHandle@28  110a9158     kernel32:KERNEL32.dll
 0002:0000015c       __imp__MoveFileA@8         110a915c     kernel32:KERNEL32.dll
 0002:00000160       __imp__GetTimeFormatA@24   110a9160     kernel32:KERNEL32.dll
 0002:00000164       __imp__GetDateFormatA@24   110a9164     kernel32:KERNEL32.dll
 0002:00000168       __imp__InterlockedDecrement@4 110a9168     kernel32:KERNEL32.dll
 0002:0000016c       __imp__GetCommandLineA@0   110a916c     kernel32:KERNEL32.dll
 0002:00000170       __imp__GetTimeZoneInformation@4 110a9170     kernel32:KERNEL32.dll
 0002:00000174       __imp__GetCPInfo@8         110a9174     kernel32:KERNEL32.dll
 0002:00000178       __imp__GetACP@0            110a9178     kernel32:KERNEL32.dll
 0002:0000017c       __imp__GetOEMCP@0          110a917c     kernel32:KERNEL32.dll
 0002:00000180       __imp__IsValidCodePage@4   110a9180     kernel32:KERNEL32.dll
 0002:00000184       __imp__TlsGetValue@4       110a9184     kernel32:KERNEL32.dll
 0002:00000188       __imp__TlsAlloc@0          110a9188     kernel32:KERNEL32.dll
 0002:0000018c       __imp__TlsSetValue@8       110a918c     kernel32:KERNEL32.dll
 0002:00000190       __imp__TlsFree@4           110a9190     kernel32:KERNEL32.dll
 0002:00000194       __imp__SetLastError@4      110a9194     kernel32:KERNEL32.dll
 0002:00000198       __imp__RaiseException@16   110a9198     kernel32:KERNEL32.dll
 0002:0000019c       __imp__SetHandleCount@4    110a919c     kernel32:KERNEL32.dll
 0002:000001a0       __imp__GetStdHandle@4      110a91a0     kernel32:KERNEL32.dll
 0002:000001a4       __imp__GetFileType@4       110a91a4     kernel32:KERNEL32.dll
 0002:000001a8       __imp__GetStartupInfoA@4   110a91a8     kernel32:KERNEL32.dll
 0002:000001ac       __imp__HeapCreate@12       110a91ac     kernel32:KERNEL32.dll
 0002:000001b0       __imp__HeapDestroy@4       110a91b0     kernel32:KERNEL32.dll
 0002:000001b4       __imp__VirtualFree@12      110a91b4     kernel32:KERNEL32.dll
 0002:000001b8       __imp__VirtualAlloc@16     110a91b8     kernel32:KERNEL32.dll
 0002:000001bc       __imp__GetConsoleCP@0      110a91bc     kernel32:KERNEL32.dll
 0002:000001c0       __imp__GetConsoleMode@8    110a91c0     kernel32:KERNEL32.dll
 0002:000001c4       __imp__LCMapStringA@24     110a91c4     kernel32:KERNEL32.dll
 0002:000001c8       __imp__LCMapStringW@24     110a91c8     kernel32:KERNEL32.dll
 0002:000001cc       __imp__InterlockedExchange@8 110a91cc     kernel32:KERNEL32.dll
 0002:000001d0       __imp__InitializeCriticalSectionAndSpinCount@8 110a91d0     kernel32:KERNEL32.dll
 0002:000001d4       \177KERNEL32_NULL_THUNK_DATA 110a91d4     kernel32:KERNEL32.dll
 0002:000001d8       __imp__MessageBoxA@16      110a91d8     user32:USER32.dll
 0002:000001dc       \177USER32_NULL_THUNK_DATA 110a91dc     user32:USER32.dll
 0002:000001e0       __imp__FtpPutFileA@20      110a91e0     Wininet:WININET.dll
 0002:000001e4       __imp__InternetConnectA@32 110a91e4     Wininet:WININET.dll
 0002:000001e8       __imp__InternetOpenA@20    110a91e8     Wininet:WININET.dll
 0002:000001ec       __imp__InternetCloseHandle@4 110a91ec     Wininet:WININET.dll
 0002:000001f0       \177WININET_NULL_THUNK_DATA 110a91f0     Wininet:WININET.dll
 0002:000001f4       __imp__connect@12          110a91f4     ws2_32:WS2_32.dll
 0002:000001f8       __imp__inet_addr@4         110a91f8     ws2_32:WS2_32.dll
 0002:000001fc       __imp__select@20           110a91fc     ws2_32:WS2_32.dll
 0002:00000200       __imp__htons@4             110a9200     ws2_32:WS2_32.dll
 0002:00000204       __imp__shutdown@8          110a9204     ws2_32:WS2_32.dll
 0002:00000208       __imp__recv@16             110a9208     ws2_32:WS2_32.dll
 0002:0000020c       __imp__bind@12             110a920c     ws2_32:WS2_32.dll
 0002:00000210       __imp__socket@12           110a9210     ws2_32:WS2_32.dll
 0002:00000214       __imp____WSAFDIsSet@8      110a9214     ws2_32:WS2_32.dll
 0002:00000218       __imp__closesocket@4       110a9218     ws2_32:WS2_32.dll
 0002:0000021c       __imp__gethostbyname@4     110a921c     ws2_32:WS2_32.dll
 0002:00000220       __imp__send@16             110a9220     ws2_32:WS2_32.dll
 0002:00000224       __imp__listen@8            110a9224     ws2_32:WS2_32.dll
 0002:00000228       __imp__accept@12           110a9228     ws2_32:WS2_32.dll
 0002:0000022c       __imp__WSAStartup@8        110a922c     ws2_32:WS2_32.dll
 0002:00000230       __imp__WSACleanup@0        110a9230     ws2_32:WS2_32.dll
 0002:00000234       __imp__ntohs@4             110a9234     ws2_32:WS2_32.dll
 0002:00000238       \177WS2_32_NULL_THUNK_DATA 110a9238     ws2_32:WS2_32.dll
 0002:0000023c       ___xc_a                    110a923c     LIBCMT:crt0init.obj
 0002:00000250       ___xc_z                    110a9250     LIBCMT:crt0init.obj
 0002:00000254       ___xi_a                    110a9254     LIBCMT:crt0init.obj
 0002:00000274       ___xi_z                    110a9274     LIBCMT:crt0init.obj
 0002:00000278       ___xp_a                    110a9278     LIBCMT:crt0init.obj
 0002:00000288       ___xp_z                    110a9288     LIBCMT:crt0init.obj
 0002:0000028c       ___xt_a                    110a928c     LIBCMT:crt0init.obj
 0002:00000290       ___xt_z                    110a9290     LIBCMT:crt0init.obj
 0002:000002c0       ??_7exception@std@@6B@     110a92c0     LIBCMT:stdexcpt.obj
 0002:000002c8       ??_C@_0BC@EOODALEL@Unknown?5exception?$AA@ 110a92c8     LIBCMT:stdexcpt.obj
 0002:000002e0       ??_7type_info@@6B@         110a92e0     LIBCMT:typinfo.obj
 0002:000002e8       ??_7bad_alloc@std@@6B@     110a92e8     LIBCMT:new.obj
 0002:000002f0       ??_C@_0EA@FCLIIPNN@Visual?5C?$CL?$CL?5CRT?3?5Not?5enough?5memor@ 110a92f0     LIBCMT:strerror.obj
 0002:00000330       ??_C@_0P@MIGLKIOC@CorExitProcess?$AA@ 110a9330     LIBCMT:crt0dat.obj
 0002:00000340       ??_C@_1BI@BGOHAHKC@?$AAm?$AAs?$AAc?$AAo?$AAr?$AAe?$AAe?$AA?4?$AAd?$AAl?$AAl?$AA?$AA@ 110a9340     LIBCMT:crt0dat.obj
 0002:00000358       ??_C@_04HBHDLLBA@PATH?$AA@ 110a9358     LIBCMT:popen.obj
 0002:00000360       ??_C@_04NPFIMJFF@?5?1c?5?$AA@ 110a9360     LIBCMT:popen.obj
 0002:00000368       ??_C@_07INNMNHPJ@cmd?4exe?$AA@ 110a9368     LIBCMT:popen.obj
 0002:00000370       ??_C@_07CFPBBAOO@COMSPEC?$AA@ 110a9370     LIBCMT:popen.obj
 0002:00000410       ??_C@_02HNHPBPFE@?1c?$AA@  110a9410     LIBCMT:system.obj
 0002:00000414       ??_C@_08JCCMCCIL@HH?3mm?3ss?$AA@ 110a9414     LIBCMT:strftime.obj
 0002:00000420       ??_C@_0BE@CKGJFCPC@dddd?0?5MMMM?5dd?0?5yyyy?$AA@ 110a9420     LIBCMT:strftime.obj
 0002:00000434       ??_C@_08BPBNCDIB@MM?1dd?1yy?$AA@ 110a9434     LIBCMT:strftime.obj
 0002:00000440       ??_C@_02CJNFDJBF@PM?$AA@   110a9440     LIBCMT:strftime.obj
 0002:00000444       ??_C@_02DEDBPAFC@AM?$AA@   110a9444     LIBCMT:strftime.obj
 0002:00000448       ??_C@_08EDHMEBNP@December?$AA@ 110a9448     LIBCMT:strftime.obj
 0002:00000454       ??_C@_08HCHEGEOA@November?$AA@ 110a9454     LIBCMT:strftime.obj
 0002:00000460       ??_C@_07JJNFCEND@October?$AA@ 110a9460     LIBCMT:strftime.obj
 0002:00000468       ??_C@_09BHHEALKD@September?$AA@ 110a9468     LIBCMT:strftime.obj
 0002:00000474       ??_C@_06LBBHFDDG@August?$AA@ 110a9474     LIBCMT:strftime.obj
 0002:0000047c       ??_C@_04MIEPOIFP@July?$AA@ 110a947c     LIBCMT:strftime.obj
 0002:00000484       ??_C@_04CNLMGBGM@June?$AA@ 110a9484     LIBCMT:strftime.obj
 0002:0000048c       ??_C@_05DMJDNLEJ@April?$AA@ 110a948c     LIBCMT:strftime.obj
 0002:00000494       ??_C@_05HPCKOFNC@March?$AA@ 110a9494     LIBCMT:strftime.obj
 0002:0000049c       ??_C@_08GNJGEPFN@February?$AA@ 110a949c     LIBCMT:strftime.obj
 0002:000004a8       ??_C@_07CGJPFGJA@January?$AA@ 110a94a8     LIBCMT:strftime.obj
 0002:000004b0       ??_C@_08INBOOONO@Saturday?$AA@ 110a94b0     LIBCMT:strftime.obj
 0002:000004bc       ??_C@_06JECMNKMI@Friday?$AA@ 110a94bc     LIBCMT:strftime.obj
 0002:000004c4       ??_C@_08HACCIKIA@Thursday?$AA@ 110a94c4     LIBCMT:strftime.obj
 0002:000004d0       ??_C@_09DLIGFAKA@Wednesday?$AA@ 110a94d0     LIBCMT:strftime.obj
 0002:000004dc       ??_C@_07BAAGCFCM@Tuesday?$AA@ 110a94dc     LIBCMT:strftime.obj
 0002:000004e4       ??_C@_06JLEDEDGH@Monday?$AA@ 110a94e4     LIBCMT:strftime.obj
 0002:000004ec       ??_C@_06OOPIFAJ@Sunday?$AA@ 110a94ec     LIBCMT:strftime.obj
 0002:000004f4       ??_C@_03FEFJNEK@Sat?$AA@   110a94f4     LIBCMT:strftime.obj
 0002:000004f8       ??_C@_03IDIOELNC@Fri?$AA@  110a94f8     LIBCMT:strftime.obj
 0002:000004fc       ??_C@_03IOFIKPDN@Thu?$AA@  110a94fc     LIBCMT:strftime.obj
 0002:00000500       ??_C@_03MHOMLAJA@Wed?$AA@  110a9500     LIBCMT:strftime.obj
 0002:00000504       ??_C@_03NAGEINEP@Tue?$AA@  110a9504     LIBCMT:strftime.obj
 0002:00000508       ??_C@_03PDAGKDH@Mon?$AA@   110a9508     LIBCMT:strftime.obj
 0002:0000050c       ??_C@_03KOEHGMDN@Sun?$AA@  110a950c     LIBCMT:strftime.obj
 0002:00000510       ??_C@_03EBAPMIKO@a?1p?$AA@ 110a9510     LIBCMT:strftime.obj
 0002:00000514       ??_C@_05JAMEPDIN@am?1pm?$AA@ 110a9514     LIBCMT:strftime.obj
 0002:0000051c       ??_C@_07LCBHPJJN@LC_TIME?$AA@ 110a951c     LIBCMT:setlocal.obj
 0002:00000524       ??_C@_0L@DLHIECNL@LC_NUMERIC?$AA@ 110a9524     LIBCMT:setlocal.obj
 0002:00000530       ??_C@_0M@MIENIKLA@LC_MONETARY?$AA@ 110a9530     LIBCMT:setlocal.obj
 0002:0000053c       ??_C@_08EADHIDAD@LC_CTYPE?$AA@ 110a953c     LIBCMT:setlocal.obj
 0002:00000548       ??_C@_0L@KFJHEKIK@LC_COLLATE?$AA@ 110a9548     LIBCMT:setlocal.obj
 0002:00000554       ??_C@_06NEFDFEKB@LC_ALL?$AA@ 110a9554     LIBCMT:setlocal.obj
 0002:00000560       ___lc_category             110a9560     LIBCMT:setlocal.obj
 0002:00000628       ??_C@_03EGDHDPFD@_?4?0?$AA@ 110a9628     LIBCMT:setlocal.obj
 0002:0000062c       ??_C@_01NEMOKFLO@?$DN?$AA@ 110a962c     LIBCMT:setlocal.obj
 0002:00000630       ??_C@_02BALPLPBG@?$DN?$DL?$AA@ 110a9630     LIBCMT:setlocal.obj
 0002:00000634       __pRawDllMain              110a9634     LIBCMT:dllcrt0.obj
 0002:00000634       __pDefaultRawDllMain       110a9634     LIBCMT:dllcrt0.obj
 0002:00000638       ??_C@_1O@CEDCILHN@?$AA?$CI?$AAn?$AAu?$AAl?$AAl?$AA?$CJ?$AA?$AA@ 110a9638     LIBCMT:output.obj
 0002:00000648       ___lookuptable             110a9648     LIBCMT:output.obj
 0002:000006a4       ??_C@_02CLFPBFFP@TZ?$AA@   110a96a4     LIBCMT:tzset.obj
 0002:000006a8       ___dnames                  110a96a8     LIBCMT:timeset.obj
 0002:000006c0       ___mnames                  110a96c0     LIBCMT:timeset.obj
 0002:000006e8       ??_C@_0O@NLDKAIKN@EncodePointer?$AA@ 110a96e8     LIBCMT:tidtable.obj
 0002:000006f8       ??_C@_1BK@DBDEIDLH@?$AAK?$AAE?$AAR?$AAN?$AAE?$AAL?$AA3?$AA2?$AA?4?$AAD?$AAL?$AAL?$AA?$AA@ 110a96f8     LIBCMT:tidtable.obj
 0002:00000714       ??_C@_0O@KBPMFGHI@DecodePointer?$AA@ 110a9714     LIBCMT:tidtable.obj
 0002:00000724       ??_C@_07PEJMOBNF@FlsFree?$AA@ 110a9724     LIBCMT:tidtable.obj
 0002:0000072c       ??_C@_0M@JCPCPOEF@FlsSetValue?$AA@ 110a972c     LIBCMT:tidtable.obj
 0002:00000738       ??_C@_0M@GDNOONDI@FlsGetValue?$AA@ 110a9738     LIBCMT:tidtable.obj
 0002:00000744       ??_C@_08KNHFBNJ@FlsAlloc?$AA@ 110a9744     LIBCMT:tidtable.obj
 0002:00000770       ??_C@_13NOLLCAOD@?$AA?$AA?$AA?$AA@ 110a9770     LIBCMT:a_map.obj
 0002:00000770       __real@00000000            110a9770      CIL library: CIL module
 0002:00000798       ___lookuptable_s           110a9798     LIBCMT:outputs.obj
 0002:000007f4       ??_C@_0P@GGKDKEEG@runtime?5error?5?$AA@ 110a97f4     LIBCMT:crt0msg.obj
 0002:00000804       ??_C@_02PCIJFNDE@?$AN?6?$AA@ 110a9804     LIBCMT:crt0msg.obj
 0002:00000808       ??_C@_0O@MJNIPGOH@TLOSS?5error?$AN?6?$AA@ 110a9808     LIBCMT:crt0msg.obj
 0002:00000818       ??_C@_0N@BONNPDHF@SING?5error?$AN?6?$AA@ 110a9818     LIBCMT:crt0msg.obj
 0002:00000828       ??_C@_0P@MBDAJNE@DOMAIN?5error?$AN?6?$AA@ 110a9828     LIBCMT:crt0msg.obj
 0002:00000838       ??_C@_0JL@DFDOOABL@R6034?$AN?6An?5application?5has?5made?5a@ 110a9838     LIBCMT:crt0msg.obj
 0002:000008d8       ??_C@_0PH@EPAFIJ@R6033?$AN?6?9?5Attempt?5to?5use?5MSIL?5cod@ 110a98d8     LIBCMT:crt0msg.obj
 0002:000009d0       ??_C@_0DD@BKEEABMM@R6032?$AN?6?9?5not?5enough?5space?5for?5lo@ 110a99d0     LIBCMT:crt0msg.obj
 0002:00000a08       ??_C@_0GD@OFKILIED@R6031?$AN?6?9?5Attempt?5to?5initialize?5t@ 110a9a08     LIBCMT:crt0msg.obj
 0002:00000a6c       ??_C@_0BP@LPMHJOKI@R6030?$AN?6?9?5CRT?5not?5initialized?$AN?6?$AA@ 110a9a6c     LIBCMT:crt0msg.obj
 0002:00000a8c       ??_C@_0CF@KJDAIALP@R6028?$AN?6?9?5unable?5to?5initialize?5he@ 110a9a8c     LIBCMT:crt0msg.obj
 0002:00000ab4       ??_C@_0DF@GAKBPDFP@R6027?$AN?6?9?5not?5enough?5space?5for?5lo@ 110a9ab4     LIBCMT:crt0msg.obj
 0002:00000aec       ??_C@_0DF@IBLNNAIG@R6026?$AN?6?9?5not?5enough?5space?5for?5st@ 110a9aec     LIBCMT:crt0msg.obj
 0002:00000b24       ??_C@_0CG@IOHKGFNJ@R6025?$AN?6?9?5pure?5virtual?5function?5c@ 110a9b24     LIBCMT:crt0msg.obj
 0002:00000b4c       ??_C@_0DF@JIJJFJDC@R6024?$AN?6?9?5not?5enough?5space?5for?5_o@ 110a9b4c     LIBCMT:crt0msg.obj
 0002:00000b84       ??_C@_0CJ@EGEJHFME@R6019?$AN?6?9?5unable?5to?5open?5console?5@ 110a9b84     LIBCMT:crt0msg.obj
 0002:00000bb0       ??_C@_0CB@GNHNIELH@R6018?$AN?6?9?5unexpected?5heap?5error?$AN?6@ 110a9bb0     LIBCMT:crt0msg.obj
 0002:00000bd4       ??_C@_0CN@FOLDKNG@R6017?$AN?6?9?5unexpected?5multithread?5@ 110a9bd4     LIBCMT:crt0msg.obj
 0002:00000c04       ??_C@_0CM@FAHFJNHO@R6016?$AN?6?9?5not?5enough?5space?5for?5th@ 110a9c04     LIBCMT:crt0msg.obj
 0002:00000c30       ??_C@_0JG@LBKMGKLD@?$AN?6This?5application?5has?5requested@ 110a9c30     LIBCMT:crt0msg.obj
 0002:00000cc8       ??_C@_0CM@FLCNIPKK@R6009?$AN?6?9?5not?5enough?5space?5for?5en@ 110a9cc8     LIBCMT:crt0msg.obj
 0002:00000cf4       ??_C@_0CK@KMMJOAPP@R6008?$AN?6?9?5not?5enough?5space?5for?5ar@ 110a9cf4     LIBCMT:crt0msg.obj
 0002:00000d20       ??_C@_0CN@LEKKICBM@R6002?$AN?6?9?5floating?5point?5support?5@ 110a9d20     LIBCMT:crt0msg.obj
 0002:00000d50       ??_C@_0CF@GOGNBNAK@Microsoft?5Visual?5C?$CL?$CL?5Runtime?5Lib@ 110a9d50     LIBCMT:crt0msg.obj
 0002:00000d78       ??_C@_02PHMGELLB@?6?6?$AA@ 110a9d78     LIBCMT:crt0msg.obj
 0002:00000d7c       ??_C@_0BH@DNAGHKFM@?$DMprogram?5name?5unknown?$DO?$AA@ 110a9d7c     LIBCMT:crt0msg.obj
 0002:00000d94       ??_C@_0BK@OFGJDLJJ@Runtime?5Error?$CB?6?6Program?3?5?$AA@ 110a9d94     LIBCMT:crt0msg.obj
 0002:00000db0       __FPinit                   110a9db0     LIBCMT:_fpinit_.obj
 0002:00000db4       __FPmtinit                 110a9db4     LIBCMT:_fpinit_.obj
 0002:00000db8       __FPmtterm                 110a9db8     LIBCMT:_fpinit_.obj
 0002:00000dbc       ??_C@_0BG@KLEAJEFJ@Illegal?5byte?5sequence?$AA@ 110a9dbc     LIBCMT:syserr.obj
 0002:00000dd4       ??_C@_0BE@ICMCHPHH@Directory?5not?5empty?$AA@ 110a9dd4     LIBCMT:syserr.obj
 0002:00000de8       ??_C@_0BJ@IHEHINLI@Function?5not?5implemented?$AA@ 110a9de8     LIBCMT:syserr.obj
 0002:00000e04       ??_C@_0BD@CLHBCGPB@No?5locks?5available?$AA@ 110a9e04     LIBCMT:syserr.obj
 0002:00000e18       ??_C@_0BC@BEDIHIDK@Filename?5too?5long?$AA@ 110a9e18     LIBCMT:syserr.obj
 0002:00000e2c       ??_C@_0BK@JAEBMJJM@Resource?5deadlock?5avoided?$AA@ 110a9e2c     LIBCMT:syserr.obj
 0002:00000e48       ??_C@_0BB@FCBJFCAJ@Result?5too?5large?$AA@ 110a9e48     LIBCMT:syserr.obj
 0002:00000e5c       ??_C@_0N@MMJPGLJK@Domain?5error?$AA@ 110a9e5c     LIBCMT:syserr.obj
 0002:00000e6c       ??_C@_0M@LHEPIIOM@Broken?5pipe?$AA@ 110a9e6c     LIBCMT:syserr.obj
 0002:00000e78       ??_C@_0P@PKCJJLLM@Too?5many?5links?$AA@ 110a9e78     LIBCMT:syserr.obj
 0002:00000e88       ??_C@_0BG@DDBFNKBH@Read?9only?5file?5system?$AA@ 110a9e88     LIBCMT:syserr.obj
 0002:00000ea0       ??_C@_0N@FEHLOILP@Invalid?5seek?$AA@ 110a9ea0     LIBCMT:syserr.obj
 0002:00000eb0       ??_C@_0BI@FEALHKLD@No?5space?5left?5on?5device?$AA@ 110a9eb0     LIBCMT:syserr.obj
 0002:00000ec8       ??_C@_0P@LFMMIPAE@File?5too?5large?$AA@ 110a9ec8     LIBCMT:syserr.obj
 0002:00000ed8       ??_C@_0CE@ONOKNLPF@Inappropriate?5I?1O?5control?5operat@ 110a9ed8     LIBCMT:syserr.obj
 0002:00000efc       ??_C@_0BE@INBJMKGG@Too?5many?5open?5files?$AA@ 110a9efc     LIBCMT:syserr.obj
 0002:00000f10       ??_C@_0BO@IIFBODJE@Too?5many?5open?5files?5in?5system?$AA@ 110a9f10     LIBCMT:syserr.obj
 0002:00000f30       ??_C@_0BB@HMGGCEBG@Invalid?5argument?$AA@ 110a9f30     LIBCMT:syserr.obj
 0002:00000f44       ??_C@_0P@NDHGCGKE@Is?5a?5directory?$AA@ 110a9f44     LIBCMT:syserr.obj
 0002:00000f54       ??_C@_0BA@CJBACOOL@Not?5a?5directory?$AA@ 110a9f54     LIBCMT:syserr.obj
 0002:00000f64       ??_C@_0P@NLEIANHE@No?5such?5device?$AA@ 110a9f64     LIBCMT:syserr.obj
 0002:00000f74       ??_C@_0O@OAMDNOCP@Improper?5link?$AA@ 110a9f74     LIBCMT:syserr.obj
 0002:00000f84       ??_C@_0M@NAAJNNGH@File?5exists?$AA@ 110a9f84     LIBCMT:syserr.obj
 0002:00000f90       ??_C@_0BA@BIBLIOEK@Resource?5device?$AA@ 110a9f90     LIBCMT:syserr.obj
 0002:00000fa0       ??_C@_0O@NIPGCINC@Unknown?5error?$AA@ 110a9fa0     LIBCMT:syserr.obj
 0002:00000fb0       ??_C@_0M@LOEHLCJD@Bad?5address?$AA@ 110a9fb0     LIBCMT:syserr.obj
 0002:00000fbc       ??_C@_0BC@HFNFNKAI@Permission?5denied?$AA@ 110a9fbc     LIBCMT:syserr.obj
 0002:00000fd0       ??_C@_0BB@IMDKMPFB@Not?5enough?5space?$AA@ 110a9fd0     LIBCMT:syserr.obj
 0002:00000fe4       ??_C@_0CB@EPFKGNAK@Resource?5temporarily?5unavailable@ 110a9fe4     LIBCMT:syserr.obj
 0002:00001008       ??_C@_0BD@LOHELEP@No?5child?5processes?$AA@ 110aa008     LIBCMT:syserr.obj
 0002:0000101c       ??_C@_0BE@NFGDDCEF@Bad?5file?5descriptor?$AA@ 110aa01c     LIBCMT:syserr.obj
 0002:00001030       ??_C@_0BC@HKPNECK@Exec?5format?5error?$AA@ 110aa030     LIBCMT:syserr.obj
 0002:00001044       ??_C@_0BC@MFFGCDFL@Arg?5list?5too?5long?$AA@ 110aa044     LIBCMT:syserr.obj
 0002:00001058       ??_C@_0BK@DPKMCKJ@No?5such?5device?5or?5address?$AA@ 110aa058     LIBCMT:syserr.obj
 0002:00001074       ??_C@_0BD@KKNFOBBD@Input?1output?5error?$AA@ 110aa074     LIBCMT:syserr.obj
 0002:00001088       ??_C@_0BK@FJBOAFDK@Interrupted?5function?5call?$AA@ 110aa088     LIBCMT:syserr.obj
 0002:000010a4       ??_C@_0BA@FKIAIBGA@No?5such?5process?$AA@ 110aa0a4     LIBCMT:syserr.obj
 0002:000010b4       ??_C@_0BK@FMDHKPNF@No?5such?5file?5or?5directory?$AA@ 110aa0b4     LIBCMT:syserr.obj
 0002:000010d0       ??_C@_0BI@BJFCGOHL@Operation?5not?5permitted?$AA@ 110aa0d0     LIBCMT:syserr.obj
 0002:000010e8       ??_C@_08INEPGKHH@No?5error?$AA@ 110aa0e8     LIBCMT:syserr.obj
 0002:000010f8       __XcptActTab               110aa0f8     LIBCMT:winxfltr.obj
 0002:000011d8       ??_C@_05EOHGHCHD@exp10?$AA@ 110aa1d8     LIBCMT:_libm_error_.obj
 0002:000011e0       ??_C@_0L@KDOEJCKC@_nextafter?$AA@ 110aa1e0     LIBCMT:_fpexcept_.obj
 0002:000011ec       ??_C@_05JGDBENOH@_logb?$AA@ 110aa1ec     LIBCMT:_fpexcept_.obj
 0002:000011f4       ??_C@_03ONILCKOB@_yn?$AA@  110aa1f4     LIBCMT:_fpexcept_.obj
 0002:000011f8       ??_C@_03NAKIGLHK@_y1?$AA@  110aa1f8     LIBCMT:_fpexcept_.obj
 0002:000011fc       ??_C@_03MJLDFKDL@_y0?$AA@  110aa1fc     LIBCMT:_fpexcept_.obj
 0002:00001200       ??_C@_06MEIMCGCF@_hypot?$AA@ 110aa200     LIBCMT:_fpexcept_.obj
 0002:00001208       ??_C@_05KBKMEMPO@_cabs?$AA@ 110aa208     LIBCMT:_fpexcept_.obj
 0002:00001210       ??_C@_04ODHECPBC@fabs?$AA@ 110aa210     LIBCMT:_fpexcept_.obj
 0002:00001218       ??_C@_04PNGHFIJN@?4com?$AA@ 110aa218     LIBCMT:spawnve.obj
 0002:00001220       ??_C@_04JLMDILM@?4exe?$AA@ 110aa220     LIBCMT:spawnve.obj
 0002:00001228       ??_C@_04NEEFLLOK@?4bat?$AA@ 110aa228     LIBCMT:spawnve.obj
 0002:00001230       ??_C@_04CPCBDHLK@?4cmd?$AA@ 110aa230     LIBCMT:spawnve.obj
 0002:00001238       ??_C@_02CEGDFPFP@?4?2?$AA@ 110aa238     LIBCMT:spawnve.obj
 0002:00001240       ___newctype                110aa240     LIBCMT:ctype.obj
 0002:00001540       __wctype                   110aa540     LIBCMT:ctype.obj
 0002:00001748       ___newclmap                110aa748     LIBCMT:ctype.obj
 0002:000018c8       ___newcumap                110aa8c8     LIBCMT:ctype.obj
 0002:00001a48       ??_C@_0O@FMJNFNKE@united?9states?$AA@ 110aaa48     LIBCMT:getqloc.obj
 0002:00001a58       ??_C@_0P@NDHFFKCA@united?9kingdom?$AA@ 110aaa58     LIBCMT:getqloc.obj
 0002:00001a68       ??_C@_0BC@HHDADLGF@trinidad?5?$CG?5tobago?$AA@ 110aaa68     LIBCMT:getqloc.obj
 0002:00001a7c       ??_C@_0M@IOAEBDAC@south?9korea?$AA@ 110aaa7c     LIBCMT:getqloc.obj
 0002:00001a88       ??_C@_0N@FIELFKIJ@south?9africa?$AA@ 110aaa88     LIBCMT:getqloc.obj
 0002:00001a98       ??_C@_0M@OPNDHCMC@south?5korea?$AA@ 110aaa98     LIBCMT:getqloc.obj
 0002:00001aa4       ??_C@_0N@MDEOEPFI@south?5africa?$AA@ 110aaaa4     LIBCMT:getqloc.obj
 0002:00001ab4       ??_C@_06FKAPCJLB@slovak?$AA@ 110aaab4     LIBCMT:getqloc.obj
 0002:00001abc       ??_C@_0M@EFJANOAL@puerto?9rico?$AA@ 110aaabc     LIBCMT:getqloc.obj
 0002:00001ac8       ??_C@_08PGOJKDAI@pr?9china?$AA@ 110aaac8     LIBCMT:getqloc.obj
 0002:00001ad4       ??_C@_08JHDOMCMI@pr?5china?$AA@ 110aaad4     LIBCMT:getqloc.obj
 0002:00001ae0       ??_C@_02JHCHFBLL@nz?$AA@   110aaae0     LIBCMT:getqloc.obj
 0002:00001ae4       ??_C@_0M@LINHDHKP@new?9zealand?$AA@ 110aaae4     LIBCMT:getqloc.obj
 0002:00001af0       ??_C@_09IIIPPBDB@hong?9kong?$AA@ 110aaaf0     LIBCMT:getqloc.obj
 0002:00001afc       ??_C@_07HJLCKBG@holland?$AA@ 110aaafc     LIBCMT:getqloc.obj
 0002:00001b04       ??_C@_0O@LEHGMHAG@great?5britain?$AA@ 110aab04     LIBCMT:getqloc.obj
 0002:00001b14       ??_C@_07FACOMELA@england?$AA@ 110aab14     LIBCMT:getqloc.obj
 0002:00001b1c       ??_C@_05JIHCEICB@czech?$AA@ 110aab1c     LIBCMT:getqloc.obj
 0002:00001b24       ??_C@_05BBJOBLGB@china?$AA@ 110aab24     LIBCMT:getqloc.obj
 0002:00001b2c       ??_C@_07GPKPHICP@britain?$AA@ 110aab2c     LIBCMT:getqloc.obj
 0002:00001b34       ??_C@_07MHIPBHMG@america?$AA@ 110aab34     LIBCMT:getqloc.obj
 0002:00001b3c       ??_C@_03KIALPMKC@usa?$AA@  110aab3c     LIBCMT:getqloc.obj
 0002:00001b40       ??_C@_02FGJGKGGD@us?$AA@   110aab40     LIBCMT:getqloc.obj
 0002:00001b44       ??_C@_02NEINDODK@uk?$AA@   110aab44     LIBCMT:getqloc.obj
 0002:00001b48       ??_C@_05JMPCFJFJ@swiss?$AA@ 110aab48     LIBCMT:getqloc.obj
 0002:00001b50       ??_C@_0BA@HLOCPIOD@swedish?9finland?$AA@ 110aab50     LIBCMT:getqloc.obj
 0002:00001b60       ??_C@_0BC@PKCNIABK@spanish?9venezuela?$AA@ 110aab60     LIBCMT:getqloc.obj
 0002:00001b74       ??_C@_0BA@GBHHMIJI@spanish?9uruguay?$AA@ 110aab74     LIBCMT:getqloc.obj
 0002:00001b84       ??_C@_0BE@BHDOHPMC@spanish?9puerto?5rico?$AA@ 110aab84     LIBCMT:getqloc.obj
 0002:00001b98       ??_C@_0N@KMOIDGGN@spanish?9peru?$AA@ 110aab98     LIBCMT:getqloc.obj
 0002:00001ba8       ??_C@_0BB@HMHLPGPH@spanish?9paraguay?$AA@ 110aaba8     LIBCMT:getqloc.obj
 0002:00001bbc       ??_C@_0P@MCPKNGFD@spanish?9panama?$AA@ 110aabbc     LIBCMT:getqloc.obj
 0002:00001bcc       ??_C@_0BC@IHOHGAIL@spanish?9nicaragua?$AA@ 110aabcc     LIBCMT:getqloc.obj
 0002:00001be0       ??_C@_0P@KLMJDNFJ@spanish?9modern?$AA@ 110aabe0     LIBCMT:getqloc.obj
 0002:00001bf0       ??_C@_0BA@BPAPGBCM@spanish?9mexican?$AA@ 110aabf0     LIBCMT:getqloc.obj
 0002:00001c00       ??_C@_0BB@PDECHHHE@spanish?9honduras?$AA@ 110aac00     LIBCMT:getqloc.obj
 0002:00001c14       ??_C@_0BC@KLHKFGDB@spanish?9guatemala?$AA@ 110aac14     LIBCMT:getqloc.obj
 0002:00001c28       ??_C@_0BE@MFOOKJAI@spanish?9el?5salvador?$AA@ 110aac28     LIBCMT:getqloc.obj
 0002:00001c3c       ??_C@_0BA@FCOKFPFC@spanish?9ecuador?$AA@ 110aac3c     LIBCMT:getqloc.obj
 0002:00001c4c       ??_C@_0BL@PLMGIMOO@spanish?9dominican?5republic?$AA@ 110aac4c     LIBCMT:getqloc.obj
 0002:00001c68       ??_C@_0BD@HLGDNMHB@spanish?9costa?5rica?$AA@ 110aac68     LIBCMT:getqloc.obj
 0002:00001c7c       ??_C@_0BB@PKCBKCPE@spanish?9colombia?$AA@ 110aac7c     LIBCMT:getqloc.obj
 0002:00001c90       ??_C@_0O@MCBIJGNE@spanish?9chile?$AA@ 110aac90     LIBCMT:getqloc.obj
 0002:00001ca0       ??_C@_0BA@BEFEIGJJ@spanish?9bolivia?$AA@ 110aaca0     LIBCMT:getqloc.obj
 0002:00001cb0       ??_C@_0BC@EMECMPD@spanish?9argentina?$AA@ 110aacb0     LIBCMT:getqloc.obj
 0002:00001cc4       ??_C@_0BF@EALFLENP@portuguese?9brazilian?$AA@ 110aacc4     LIBCMT:getqloc.obj
 0002:00001cdc       ??_C@_0BC@HBLEBLNN@norwegian?9nynorsk?$AA@ 110aacdc     LIBCMT:getqloc.obj
 0002:00001cf0       ??_C@_0BB@HMACDDCK@norwegian?9bokmal?$AA@ 110aacf0     LIBCMT:getqloc.obj
 0002:00001d04       ??_C@_09BAFFPPHE@norwegian?$AA@ 110aad04     LIBCMT:getqloc.obj
 0002:00001d10       ??_C@_0O@EAJFJDFG@italian?9swiss?$AA@ 110aad10     LIBCMT:getqloc.obj
 0002:00001d20       ??_C@_0O@CNOMPGD@irish?9english?$AA@ 110aad20     LIBCMT:getqloc.obj
 0002:00001d30       ??_C@_0N@EDHBGCKG@german?9swiss?$AA@ 110aad30     LIBCMT:getqloc.obj
 0002:00001d40       ??_C@_0BC@JACMHNBP@german?9luxembourg?$AA@ 110aad40     LIBCMT:getqloc.obj
 0002:00001d54       ??_C@_0BE@HBGMGFEG@german?9lichtenstein?$AA@ 110aad54     LIBCMT:getqloc.obj
 0002:00001d68       ??_C@_0BA@HKKBIBKL@german?9austrian?$AA@ 110aad68     LIBCMT:getqloc.obj
 0002:00001d78       ??_C@_0N@GCAEPEBK@french?9swiss?$AA@ 110aad78     LIBCMT:getqloc.obj
 0002:00001d88       ??_C@_0BC@DJFJJCK@french?9luxembourg?$AA@ 110aad88     LIBCMT:getqloc.obj
 0002:00001d9c       ??_C@_0BA@NNCEDFIC@french?9canadian?$AA@ 110aad9c     LIBCMT:getqloc.obj
 0002:00001dac       ??_C@_0P@CMPOCLM@french?9belgian?$AA@ 110aadac     LIBCMT:getqloc.obj
 0002:00001dbc       ??_C@_0M@GHHDJOK@english?9usa?$AA@ 110aadbc     LIBCMT:getqloc.obj
 0002:00001dc8       ??_C@_0L@PLDJKEIL@english?9us?$AA@ 110aadc8     LIBCMT:getqloc.obj
 0002:00001dd4       ??_C@_0L@HJCCDMNC@english?9uk?$AA@ 110aadd4     LIBCMT:getqloc.obj
 0002:00001de0       ??_C@_0BK@CKLIAGJB@english?9trinidad?5y?5tobago?$AA@ 110aade0     LIBCMT:getqloc.obj
 0002:00001dfc       ??_C@_0BF@JMJMGNNF@english?9south?5africa?$AA@ 110aadfc     LIBCMT:getqloc.obj
 0002:00001e14       ??_C@_0L@DKIIFDFD@english?9nz?$AA@ 110aae14     LIBCMT:getqloc.obj
 0002:00001e20       ??_C@_0BA@ONHGJCLH@english?9jamaica?$AA@ 110aae20     LIBCMT:getqloc.obj
 0002:00001e30       ??_C@_0M@HJBGHOPO@english?9ire?$AA@ 110aae30     LIBCMT:getqloc.obj
 0002:00001e3c       ??_C@_0BC@LFEKMIFB@english?9caribbean?$AA@ 110aae3c     LIBCMT:getqloc.obj
 0002:00001e50       ??_C@_0M@OLDPFKHI@english?9can?$AA@ 110aae50     LIBCMT:getqloc.obj
 0002:00001e5c       ??_C@_0P@OMDEHBMP@english?9belize?$AA@ 110aae5c     LIBCMT:getqloc.obj
 0002:00001e6c       ??_C@_0M@KFHFPFED@english?9aus?$AA@ 110aae6c     LIBCMT:getqloc.obj
 0002:00001e78       ??_C@_0BB@MNMBKDFE@english?9american?$AA@ 110aae78     LIBCMT:getqloc.obj
 0002:00001e8c       ??_C@_0O@KIDLNNBA@dutch?9belgian?$AA@ 110aae8c     LIBCMT:getqloc.obj
 0002:00001e9c       ??_C@_0BE@JBKABBMH@chinese?9traditional?$AA@ 110aae9c     LIBCMT:getqloc.obj
 0002:00001eb0       ??_C@_0BC@MJJMPKCG@chinese?9singapore?$AA@ 110aaeb0     LIBCMT:getqloc.obj
 0002:00001ec4       ??_C@_0BD@FDKADDCP@chinese?9simplified?$AA@ 110aaec4     LIBCMT:getqloc.obj
 0002:00001ed8       ??_C@_0BB@DBEFDDME@chinese?9hongkong?$AA@ 110aaed8     LIBCMT:getqloc.obj
 0002:00001eec       ??_C@_07DHNMFMCI@chinese?$AA@ 110aaeec     LIBCMT:getqloc.obj
 0002:00001ef4       ??_C@_03FNDDCHI@chi?$AA@   110aaef4     LIBCMT:getqloc.obj
 0002:00001ef8       ??_C@_03BMMIADDJ@chh?$AA@  110aaef8     LIBCMT:getqloc.obj
 0002:00001efc       ??_C@_08OAIPJDGI@canadian?$AA@ 110aaefc     LIBCMT:getqloc.obj
 0002:00001f08       ??_C@_07HBPMNPNJ@belgian?$AA@ 110aaf08     LIBCMT:getqloc.obj
 0002:00001f10       ??_C@_0L@OEKOPBEL@australian?$AA@ 110aaf10     LIBCMT:getqloc.obj
 0002:00001f1c       ??_C@_0BB@MEIMBEDG@american?9english?$AA@ 110aaf1c     LIBCMT:getqloc.obj
 0002:00001f30       ??_C@_0BB@DFMDPDGB@american?5english?$AA@ 110aaf30     LIBCMT:getqloc.obj
 0002:00001f44       ??_C@_08IJLOKOLL@american?$AA@ 110aaf44     LIBCMT:getqloc.obj
 0002:00001f50       ___rg_language             110aaf50     LIBCMT:getqloc.obj
 0002:00002158       ___rg_country              110ab158     LIBCMT:getqloc.obj
 0002:00002210       ___rglangidNotDefault      110ab210     LIBCMT:getqloc.obj
 0002:00002224       ??_C@_03NFKLAGEF@OCP?$AA@  110ab224     LIBCMT:getqloc.obj
 0002:00002228       ??_C@_03DFHEHBHG@ACP?$AA@  110ab228     LIBCMT:getqloc.obj
 0002:0000222c       ??_C@_0BC@NFIEMBLL@Norwegian?9Nynorsk?$AA@ 110ab22c     LIBCMT:getqloc.obj
 0002:00002248       ??_C@_0BK@CFCOFLF@?5Complete?5Object?5Locator?8?$AA@ 110ab248     LIBCMT:undname.obj
 0002:00002264       ??_C@_0BN@MECKDCOJ@?5Class?5Hierarchy?5Descriptor?8?$AA@ 110ab264     LIBCMT:undname.obj
 0002:00002284       ??_C@_0BD@LGICGFMM@?5Base?5Class?5Array?8?$AA@ 110ab284     LIBCMT:undname.obj
 0002:00002298       ??_C@_0BM@LDKODKLH@?5Base?5Class?5Descriptor?5at?5?$CI?$AA@ 110ab298     LIBCMT:undname.obj
 0002:000022b4       ??_C@_0BC@DAFEJGAK@?5Type?5Descriptor?8?$AA@ 110ab2b4     LIBCMT:undname.obj
 0002:000022c8       ??_C@_0BM@PMGGMLDN@?$GAlocal?5static?5thread?5guard?8?$AA@ 110ab2c8     LIBCMT:undname.obj
 0002:000022e4       ??_C@_0CL@FGIJHLCE@?$GAmanaged?5vector?5copy?5constructor@ 110ab2e4     LIBCMT:undname.obj
 0002:00002310       ??_C@_0CJ@GJELGAMM@?$GAvector?5vbase?5copy?5constructor?5i@ 110ab310     LIBCMT:undname.obj
 0002:0000233c       ??_C@_0CD@CGAJBKEJ@?$GAvector?5copy?5constructor?5iterato@ 110ab33c     LIBCMT:undname.obj
 0002:00002360       ??_C@_0CB@PDBIFEP@?$GAdynamic?5atexit?5destructor?5for?5?8@ 110ab360     LIBCMT:undname.obj
 0002:00002384       ??_C@_0BL@CLIPGLGB@?$GAdynamic?5initializer?5for?5?8?$AA@ 110ab384     LIBCMT:undname.obj
 0002:000023a0       ??_C@_0CM@FCBBDIGB@?$GAeh?5vector?5vbase?5copy?5constructo@ 110ab3a0     LIBCMT:undname.obj
 0002:000023cc       ??_C@_0CG@HLDDJMAG@?$GAeh?5vector?5copy?5constructor?5iter@ 110ab3cc     LIBCMT:undname.obj
 0002:000023f4       ??_C@_0CF@IMGKMJNO@?$GAmanaged?5vector?5destructor?5itera@ 110ab3f4     LIBCMT:undname.obj
 0002:0000241c       ??_C@_0CG@CFDHKGGD@?$GAmanaged?5vector?5constructor?5iter@ 110ab41c     LIBCMT:undname.obj
 0002:00002444       ??_C@_0BN@CKNJLHMB@?$GAplacement?5delete?$FL?$FN?5closure?8?$AA@ 110ab444     LIBCMT:undname.obj
 0002:00002464       ??_C@_0BL@CNOONJFP@?$GAplacement?5delete?5closure?8?$AA@ 110ab464     LIBCMT:undname.obj
 0002:00002480       ??_C@_0P@HJKNJFNN@?$GAomni?5callsig?8?$AA@ 110ab480     LIBCMT:undname.obj
 0002:00002490       ??_C@_09LBNFPBCA@?5delete?$FL?$FN?$AA@ 110ab490     LIBCMT:undname.obj
 0002:0000249c       ??_C@_06FHBGPFGH@?5new?$FL?$FN?$AA@ 110ab49c     LIBCMT:undname.obj
 0002:000024a4       ??_C@_0CE@IIHCMGGL@?$GAlocal?5vftable?5constructor?5closu@ 110ab4a4     LIBCMT:undname.obj
 0002:000024c8       ??_C@_0BA@KKLDJDLB@?$GAlocal?5vftable?8?$AA@ 110ab4c8     LIBCMT:undname.obj
 0002:000024d8       ??_C@_05KHLCHHI@?$GARTTI?$AA@ 110ab4d8     LIBCMT:undname.obj
 0002:000024e0       ??_C@_03KLGMFNMG@?$GAEH?$AA@ 110ab4e0     LIBCMT:undname.obj
 0002:000024e4       ??_C@_0BA@KBCDOMBN@?$GAudt?5returning?8?$AA@ 110ab4e4     LIBCMT:undname.obj
 0002:000024f4       ??_C@_0BL@LLKPOHJI@?$GAcopy?5constructor?5closure?8?$AA@ 110ab4f4     LIBCMT:undname.obj
 0002:00002510       ??_C@_0CH@OOJPLCPH@?$GAeh?5vector?5vbase?5constructor?5ite@ 110ab510     LIBCMT:undname.obj
 0002:00002538       ??_C@_0CA@GCEOPDGL@?$GAeh?5vector?5destructor?5iterator?8?$AA@ 110ab538     LIBCMT:undname.obj
 0002:00002558       ??_C@_0CB@JONCMFFK@?$GAeh?5vector?5constructor?5iterator?8@ 110ab558     LIBCMT:undname.obj
 0002:0000257c       ??_C@_0BL@NILFHHPC@?$GAvirtual?5displacement?5map?8?$AA@ 110ab57c     LIBCMT:undname.obj
 0002:00002598       ??_C@_0CE@IKBNEHA@?$GAvector?5vbase?5constructor?5iterat@ 110ab598     LIBCMT:undname.obj
 0002:000025bc       ??_C@_0BN@LFPFMEDL@?$GAvector?5destructor?5iterator?8?$AA@ 110ab5bc     LIBCMT:undname.obj
 0002:000025dc       ??_C@_0BO@PFGOCPJJ@?$GAvector?5constructor?5iterator?8?$AA@ 110ab5dc     LIBCMT:undname.obj
 0002:000025fc       ??_C@_0BN@IMDCHIKM@?$GAscalar?5deleting?5destructor?8?$AA@ 110ab5fc     LIBCMT:undname.obj
 0002:0000261c       ??_C@_0BO@OBMKPJIG@?$GAdefault?5constructor?5closure?8?$AA@ 110ab61c     LIBCMT:undname.obj
 0002:0000263c       ??_C@_0BN@DEGPLNFK@?$GAvector?5deleting?5destructor?8?$AA@ 110ab63c     LIBCMT:undname.obj
 0002:0000265c       ??_C@_0BD@JDLKDPAB@?$GAvbase?5destructor?8?$AA@ 110ab65c     LIBCMT:undname.obj
 0002:00002670       ??_C@_08OBABFOLI@?$GAstring?8?$AA@ 110ab670     LIBCMT:undname.obj
 0002:0000267c       ??_C@_0BF@KDPPACIK@?$GAlocal?5static?5guard?8?$AA@ 110ab67c     LIBCMT:undname.obj
 0002:00002694       ??_C@_08LLFFHHDJ@?$GAtypeof?8?$AA@ 110ab694     LIBCMT:undname.obj
 0002:000026a0       ??_C@_07FEEIOKP@?$GAvcall?8?$AA@ 110ab6a0     LIBCMT:undname.obj
 0002:000026a8       ??_C@_09BLBHBJP@?$GAvbtable?8?$AA@ 110ab6a8     LIBCMT:undname.obj
 0002:000026b4       ??_C@_09IFPLHPGF@?$GAvftable?8?$AA@ 110ab6b4     LIBCMT:undname.obj
 0002:000026c0       ??_C@_02MHEGNOJ@?$FO?$DN?$AA@ 110ab6c0     LIBCMT:undname.obj
 0002:000026c4       ??_C@_02DHLNPPGH@?$HM?$DN?$AA@ 110ab6c4     LIBCMT:undname.obj
 0002:000026c8       ??_C@_02FGJGFEAB@?$CG?$DN?$AA@ 110ab6c8     LIBCMT:undname.obj
 0002:000026cc       ??_C@_03CDNPDDLA@?$DM?$DM?$DN?$AA@ 110ab6cc     LIBCMT:undname.obj
 0002:000026d0       ??_C@_03IKFCCPFF@?$DO?$DO?$DN?$AA@ 110ab6d0     LIBCMT:undname.obj
 0002:000026d4       ??_C@_02FENAOKFI@?$CF?$DN?$AA@ 110ab6d4     LIBCMT:undname.obj
 0002:000026d8       ??_C@_02FJEHGPIO@?1?$DN?$AA@ 110ab6d8     LIBCMT:undname.obj
 0002:000026dc       ??_C@_02FKMDLLOA@?9?$DN?$AA@ 110ab6dc     LIBCMT:undname.obj
 0002:000026e0       ??_C@_02FOEOMHFC@?$CL?$DN?$AA@ 110ab6e0     LIBCMT:undname.obj
 0002:000026e4       ??_C@_02FPIMKNGF@?$CK?$DN?$AA@ 110ab6e4     LIBCMT:undname.obj
 0002:000026e8       ??_C@_02NONPIBCD@?$HM?$HM?$AA@ 110ab6e8     LIBCMT:undname.obj
 0002:000026ec       ??_C@_02PPKAJPJL@?$CG?$CG?$AA@ 110ab6ec     LIBCMT:undname.obj
 0002:000026f0       ??_C@_01DNKMNLPK@?$HM?$AA@ 110ab6f0     LIBCMT:undname.obj
 0002:000026f4       ??_C@_01JKBOJNNK@?$FO?$AA@ 110ab6f4     LIBCMT:undname.obj
 0002:000026f8       ??_C@_01PJKLJHI@?$HO?$AA@  110ab6f8     LIBCMT:undname.obj
 0002:000026fc       ??_C@_02HCKGKOFO@?$CI?$CJ?$AA@ 110ab6fc     LIBCMT:undname.obj
 0002:00002700       ??_C@_01PPODPGHN@?$DO?$AA@ 110ab700     LIBCMT:undname.obj
 0002:00002704       ??_C@_01MNNFJEPP@?$DM?$AA@ 110ab704     LIBCMT:undname.obj
 0002:00002708       ??_C@_01KMDKNFGN@?1?$AA@   110ab708     LIBCMT:undname.obj
 0002:0000270c       ??_C@_03MNHNFDLC@?9?$DO?$CK?$AA@ 110ab70c     LIBCMT:undname.obj
 0002:00002710       ??_C@_01HNPIGOCE@?$CG?$AA@ 110ab710     LIBCMT:undname.obj
 0002:00002714       ??_C@_02BAABKJLB@?9?9?$AA@ 110ab714     LIBCMT:undname.obj
 0002:00002718       ??_C@_02ECNGHCIF@?$CL?$CL?$AA@ 110ab718     LIBCMT:undname.obj
 0002:0000271c       ??_C@_01NBENCBCI@?$CK?$AA@ 110ab71c     LIBCMT:undname.obj
 0002:00002720       ??_C@_02HBOOOICD@?9?$DO?$AA@ 110ab720     LIBCMT:undname.obj
 0002:00002724       ??_C@_08LHJFAFGD@operator?$AA@ 110ab724     LIBCMT:undname.obj
 0002:00002730       ??_C@_02GPECMEKF@?$FL?$FN?$AA@ 110ab730     LIBCMT:undname.obj
 0002:00002734       ??_C@_02FDNJECIE@?$CB?$DN?$AA@ 110ab734     LIBCMT:undname.obj
 0002:00002738       ??_C@_02FODMEDOG@?$DM?$DM?$AA@ 110ab738     LIBCMT:undname.obj
 0002:0000273c       ??_C@_02GPIOPFAK@?$DO?$DO?$AA@ 110ab73c     LIBCMT:undname.obj
 0002:00002740       ??_C@_07FPCDHGMM@?5delete?$AA@ 110ab740     LIBCMT:undname.obj
 0002:00002748       ??_C@_04NIHEBCM@?5new?$AA@ 110ab748     LIBCMT:undname.obj
 0002:00002750       ??_C@_0M@GFIIJFMG@__unaligned?$AA@ 110ab750     LIBCMT:undname.obj
 0002:0000275c       ??_C@_0L@PILCLIHE@__restrict?$AA@ 110ab75c     LIBCMT:undname.obj
 0002:00002768       ??_C@_07JOMMBBKO@__ptr64?$AA@ 110ab768     LIBCMT:undname.obj
 0002:00002770       ??_C@_09HIJEGCPM@__clrcall?$AA@ 110ab770     LIBCMT:undname.obj
 0002:0000277c       ??_C@_0L@JMKHOMEK@__fastcall?$AA@ 110ab77c     LIBCMT:undname.obj
 0002:00002788       ??_C@_0L@NPHFGOKO@__thiscall?$AA@ 110ab788     LIBCMT:undname.obj
 0002:00002794       ??_C@_09IFJBGAPI@__stdcall?$AA@ 110ab794     LIBCMT:undname.obj
 0002:000027a0       ??_C@_08GHMPAG@__pascal?$AA@ 110ab7a0     LIBCMT:undname.obj
 0002:000027ac       ??_C@_07KOLFKCDI@__cdecl?$AA@ 110ab7ac     LIBCMT:undname.obj
 0002:000027b4       ??_C@_08EHJDFFNH@__based?$CI?$AA@ 110ab7b4     LIBCMT:undname.obj
 0002:00002940       ??_C@_0BI@DFKBFLJE@GetProcessWindowStation?$AA@ 110ab940     LIBCMT:crtmbox.obj
 0002:00002958       ??_C@_0BK@CIDNPOGP@GetUserObjectInformationA?$AA@ 110ab958     LIBCMT:crtmbox.obj
 0002:00002974       ??_C@_0BD@HHGDFDBJ@GetLastActivePopup?$AA@ 110ab974     LIBCMT:crtmbox.obj
 0002:00002988       ??_C@_0BA@HNOPNCHB@GetActiveWindow?$AA@ 110ab988     LIBCMT:crtmbox.obj
 0002:00002998       ??_C@_0M@CHKKJDAI@MessageBoxA?$AA@ 110ab998     LIBCMT:crtmbox.obj
 0002:000029a4       ??_C@_0L@NDEGIDAG@USER32?4DLL?$AA@ 110ab9a4     LIBCMT:crtmbox.obj
 0002:000029b0       ??_C@_05KLBDPFGC@e?$CL000?$AA@ 110ab9b0     LIBCMT:cvt.obj
 0002:000029b8       __real@4150017ec0000000    110ab9b8     LIBCMT:_testfdiv_.obj
 0002:000029c0       __real@4147ffff80000000    110ab9c0     LIBCMT:_testfdiv_.obj
 0002:000029c8       ??_C@_0BK@NHEOCAHP@IsProcessorFeaturePresent?$AA@ 110ab9c8     LIBCMT:_testfdiv_.obj
 0002:000029e4       ??_C@_08CPNIBGIE@KERNEL32?$AA@ 110ab9e4     LIBCMT:_testfdiv_.obj
 0002:000029f0       ??_C@_0L@NKOGAPMJ@SystemRoot?$AA@ 110ab9f0     LIBCMT:cenvarg.obj
 0002:000029fc       ??_C@_07GPDNMNG@CONOUT$?$AA@ 110ab9fc     LIBCMT:initcon.obj
 0002:00002a04       ??_C@_06IMKFLFPG@1?$CDQNAN?$AA@ 110aba04     LIBCMT:_x10fout_.obj
 0002:00002a0c       ??_C@_05DNEBIAHO@1?$CDINF?$AA@ 110aba0c     LIBCMT:_x10fout_.obj
 0002:00002a14       ??_C@_05PHHOCPM@1?$CDIND?$AA@ 110aba14     LIBCMT:_x10fout_.obj
 0002:00002a1c       ??_C@_06PGGFOGJG@1?$CDSNAN?$AA@ 110aba1c     LIBCMT:_x10fout_.obj
 0002:00002a28       ??_7logic_error@std@@6B@   110aba28     libcpmt:string.obj
 0002:00002a34       ??_7length_error@std@@6B@  110aba34     libcpmt:string.obj
 0002:00002a40       ??_7out_of_range@std@@6B@  110aba40     libcpmt:string.obj
 0002:00002a48       ??_C@_0BA@JFNIOLAK@string?5too?5long?$AA@ 110aba48     libcpmt:string.obj
 0002:00002a58       ??_C@_0BI@CFPLBAOH@invalid?5string?5position?$AA@ 110aba58     libcpmt:string.obj
 0002:00002a70       ?_BADOFF@std@@3JB          110aba70     libcpmt:ios.obj
 0002:00002a74       __pDestructExceptionObject 110aba74     LIBCMT:frame.obj
 0002:00002a7c       ??_7bad_exception@std@@6B@ 110aba7c     LIBCMT:frame.obj
 0002:00002a84       ??_C@_0O@DPKOEFFH@bad?5exception?$AA@ 110aba84     LIBCMT:frame.obj
 0002:00002acc       ??_C@_03MKABNOCG@Dec?$AA@  110abacc     date.obj
 0002:00002ad0       ??_C@_03JPJOFNIA@Nov?$AA@  110abad0     date.obj
 0002:00002ad4       ??_C@_03BMAOKBAD@Oct?$AA@  110abad4     date.obj
 0002:00002ad8       ??_C@_03GGCAPAJC@Sep?$AA@  110abad8     date.obj
 0002:00002adc       ??_C@_03IFJFEIGA@Aug?$AA@  110abadc     date.obj
 0002:00002ae0       ??_C@_03LBGABGKK@Jul?$AA@  110abae0     date.obj
 0002:00002ae4       ??_C@_03IDFGHECI@Jun?$AA@  110abae4     date.obj
 0002:00002ae8       ??_C@_03CNMDKL@May?$AA@    110abae8     date.obj
 0002:00002aec       ??_C@_03LEOLGMJP@Apr?$AA@  110abaec     date.obj
 0002:00002af0       ??_C@_03ODNJBKGA@Mar?$AA@  110abaf0     date.obj
 0002:00002af4       ??_C@_03HJBDCHOM@Feb?$AA@  110abaf4     date.obj
 0002:00002af8       ??_C@_03JIHJHPIE@Jan?$AA@  110abaf8     date.obj
 0002:00002afc       ??_C@_01CLKCMJKC@?5?$AA@   110abafc     date.obj
 0002:00002b00       ??_C@_0P@GHFPNOJB@bad?5allocation?$AA@ 110abb00     engine_gm.obj
 0002:00002b0f       ??_C@_00CNPNBAHC@?$AA@     110abb0f     engine_gm.obj
 0002:00002b10       ??_C@_04OHJIHAFH@None?$AA@ 110abb10     engine_gm.obj
 0002:00002b18       ??_C@_1BE@PJAIDCO@?$AAN?$AAo?$AA?5?$AAS?$AAt?$AAr?$AAi?$AAn?$AAg?$AA?$AA@ 110abb18     engine_gm.obj
 0002:00002b2c       ??_C@_05LAPONLG@false?$AA@ 110abb2c     gmfunc.obj
 0002:00002b34       ??_C@_04LOAJBDKD@true?$AA@ 110abb34     gmfunc.obj
 0002:00002b3c       ??_C@_06LGMEBDBC@Server?$AA@ 110abb3c     gmfunc.obj
 0002:00002b44       ??_C@_04MLLLIHIP@null?$AA@ 110abb44     gmfunc.obj
 0002:00002b4c       ??_C@_01GBGANLPD@0?$AA@    110abb4c     gmfunc.obj
 0002:00002b50       ??_C@_09MJONCACI@No?5String?$AA@ 110abb50     gmfunc.obj
 0002:00002b5c       ??_C@_0BB@NHJNEILC@Invisible_Object?$AA@ 110abb5c     gmfunc.obj
 0002:00002b70       ??_C@_03OFAPEBGM@?$CFs?6?$AA@ 110abb70     gmfunc.obj
 0002:00002b74       ??_C@_02BBAHNLBA@?$CFp?$AA@ 110abb74     gmfunc.obj
 0002:00002b78       ??_C@_04HIBGFPH@NULL?$AA@  110abb78     gmsettingsclass.obj
 0002:00002b80       ??_C@_04OGKJMPGK@?$CF02d?$AA@ 110abb80     gmsettingsclass.obj
 0002:00002b88       ??_C@_0BD@NIHJDDGB@Error?5loading?5?$CC?$CFs?$CC?$AA@ 110abb88     Hooks.obj
 0002:00002b9c       ??_C@_01LFCBOECM@?4?$AA@   110abb9c     Hooks.obj
 0002:00002ba0       ??_C@_09FNDOKMBB@Hooks?4dll?$AA@ 110abba0     Hooks.obj
 0002:00002bac       ??_C@_0BJ@LBAHEJEJ@Error?5loading?5Hooks?4dll?6?$AA@ 110abbac     Hooks.obj
 0002:00002bc8       ??_C@_0O@BCPIJPHI@RequestSerial?$AA@ 110abbc8     Hooks.obj
 0002:00002bd8       ??_C@_0O@EMDMBBAO@AddSerialHook?$AA@ 110abbd8     Hooks.obj
 0002:00002be8       ??_C@_0BA@BAKHGDMG@AddLoadingEHook?$AA@ 110abbe8     Hooks.obj
 0002:00002bf8       ??_C@_0O@CGFJJCNL@AddDamageHook?$AA@ 110abbf8     Hooks.obj
 0002:00002c08       ??_C@_0M@IAMKMFFJ@AddChatHook?$AA@ 110abc08     Hooks.obj
 0002:00002c14       ??_C@_0M@KKCHLLKP@AddPingHook?$AA@ 110abc14     Hooks.obj
 0002:00002c20       ??_C@_0P@KKLLIPMC@AddSuicideHook?$AA@ 110abc20     Hooks.obj
 0002:00002c30       ??_C@_0N@NAFJFAFI@AddRadioHook?$AA@ 110abc30     Hooks.obj
 0002:00002c40       ??_C@_0N@LENHPPAN@AddThinkHook?$AA@ 110abc40     Hooks.obj
 0002:00002c50       ??_C@_0BA@LNCFPFLP@?$CFs?2LuaPlugins?2?$CK?$AA@ 110abc50     plugin.obj
 0002:00002c60       ??_C@_0BB@FECNOGOA@?$CFs?2LuaPlugins?2?$CFs?$AA@ 110abc60     plugin.obj
 0002:00002c74       ??_C@_0BE@OLLJHALI@OnCharacterPurchase?$AA@ 110abc74     plugin.obj
 0002:00002c88       ??_C@_0BC@PBIKCCF@OnVehiclePurchase?$AA@ 110abc88     plugin.obj
 0002:00002c9c       ??_C@_0BC@BCJLJGMH@OnPowerupPurchase?$AA@ 110abc9c     plugin.obj
 0002:00002cb0       ??_C@_0CM@MKMOBENL@Error?5getting?5function?5address?5f@ 110abcb0     dllmain.obj
 0002:00002cdc       ??_C@_0BD@CEDCHKBB@New_Enable_Stealth?$AA@ 110abcdc     dllmain.obj
 0002:00002cf0       ??_C@_0BF@LANEKPIK@New_Create_Explosion?$AA@ 110abcf0     dllmain.obj
 0002:00002d08       ??_C@_0BN@FMOGPLMC@New_Create_Explosion_At_Bone?$AA@ 110abd08     dllmain.obj
 0002:00002d28       ??_C@_0BD@LMPMLNOO@New_Set_Fog_Enable?$AA@ 110abd28     dllmain.obj
 0002:00002d3c       ??_C@_0BC@LEAPKNGA@New_Set_Fog_Range?$AA@ 110abd3c     dllmain.obj
 0002:00002d50       ??_C@_0BC@DFFBEOEP@New_Set_War_Blitz?$AA@ 110abd50     dllmain.obj
 0002:00002d64       ??_C@_0BK@FMEFIGMJ@New_Fade_Background_Music?$AA@ 110abd64     dllmain.obj
 0002:00002d80       ??_C@_0BJ@CHDMIIDC@New_Set_Background_Music?$AA@ 110abd80     dllmain.obj
 0002:00002d9c       ??_C@_0BK@GHEGIDEJ@New_Stop_Background_Music?$AA@ 110abd9c     dllmain.obj
 0002:00002db8       ??_C@_0BB@DMKAPJOM@New_Create_Sound?$AA@ 110abdb8     dllmain.obj
 0002:00002dcc       ??_C@_0BE@OHJEGAJE@New_Create_2D_Sound?$AA@ 110abdcc     dllmain.obj
 0002:00002de0       ??_C@_0BI@HGKHHIKA@New_Create_2D_WAV_Sound?$AA@ 110abde0     dllmain.obj
 0002:00002df8       ??_C@_0CA@COANFJBN@New_Create_3D_WAV_Sound_At_Bone?$AA@ 110abdf8     dllmain.obj
 0002:00002e18       ??_C@_0BM@NEPOFEN@New_Create_3D_Sound_At_Bone?$AA@ 110abe18     dllmain.obj
 0002:00002e34       ??_C@_0BP@JPAENPMP@New_Play_Building_Announcement?$AA@ 110abe34     dllmain.obj
 0002:00002e54       ??_C@_0BC@KOFDDJA@New_Clear_Weapons?$AA@ 110abe54     dllmain.obj
 0002:00002e68       ??_C@_0BP@HAHCDGEG@New_Enable_Vehicle_Transitions?$AA@ 110abe68     dllmain.obj
 0002:00002e88       ??_C@_0BE@ONIFHAHC@New_Set_Player_Type?$AA@ 110abe88     dllmain.obj
 0002:00002e9c       ??_C@_0BK@FDMKHFBH@New_Set_Screen_Fade_Color?$AA@ 110abe9c     dllmain.obj
 0002:00002eb8       ??_C@_0BM@LAKGIHPF@New_Set_Screen_Fade_Opacity?$AA@ 110abeb8     dllmain.obj
 0002:00002ed4       ??_C@_0BG@IEMOFMGB@New_Set_Display_Color?$AA@ 110abed4     dllmain.obj
 0002:00002eec       ??_C@_0BB@COAKGDMN@New_Display_Text?$AA@ 110abeec     dllmain.obj
 0002:00002f00       ??_C@_0BC@DKIFMHMA@New_Display_Float?$AA@ 110abf00     dllmain.obj
 0002:00002f14       ??_C@_0BA@OLJFNGPH@New_Display_Int?$AA@ 110abf14     dllmain.obj
 0002:00002f24       ??_C@_0BC@NCKGKIKH@New_Select_Weapon?$AA@ 110abf24     dllmain.obj
 0002:00002f38       ??_C@_0BB@MNJLFKNF@New_Shake_Camera?$AA@ 110abf38     dllmain.obj
 0002:00002f4c       ??_C@_0O@COMKEHBD@New_Set_Model?$AA@ 110abf4c     dllmain.obj
 0002:00002f5c       ??_C@_0BK@KODEAOPK@New_Enable_Stealth_Player?$AA@ 110abf5c     dllmain.obj
 0002:00002f78       ??_C@_0BK@BODOPFDH@New_Set_Fog_Enable_Player?$AA@ 110abf78     dllmain.obj
 0002:00002f94       ??_C@_0BJ@POBGEGB@New_Set_Fog_Range_Player?$AA@ 110abf94     dllmain.obj
 0002:00002fb0       ??_C@_0CA@KFLOIEGG@New_Set_Background_Music_Player?$AA@ 110abfb0     dllmain.obj
 0002:00002fd0       ??_C@_0CB@LBDBCOBG@New_Fade_Background_Music_Player@ 110abfd0     dllmain.obj
 0002:00002ff4       ??_C@_0CB@JGAFACH@New_Stop_Background_Music_Player@ 110abff4     dllmain.obj
 0002:00003018       ??_C@_0BI@MCHCNCJI@New_Enable_Radar_Player?$AA@ 110ac018     dllmain.obj
 0002:00003030       ??_C@_0CH@GGHFFKPO@New_Display_GDI_Player_Terminal_@ 110ac030     dllmain.obj
 0002:00003058       ??_C@_0CH@BPDIBODD@New_Display_NOD_Player_Terminal_@ 110ac058     dllmain.obj
 0002:00003080       ??_C@_0CB@LCBOAKKM@New_Set_Screen_Fade_Color_Player@ 110ac080     dllmain.obj
 0002:000030a4       ??_C@_0CD@OGHDHBBK@New_Set_Screen_Fade_Opacity_Play@ 110ac0a4     dllmain.obj
 0002:000030c8       ??_C@_0BN@MANAFNCH@New_Force_Camera_Look_Player?$AA@ 110ac0c8     dllmain.obj
 0002:000030e8       ??_C@_0BG@OABCCFFJ@New_Enable_HUD_Player?$AA@ 110ac0e8     dllmain.obj
 0002:00003100       ??_C@_0BI@NNCDIJF@New_Create_Sound_Player?$AA@ 110ac100     dllmain.obj
 0002:00003118       ??_C@_0BL@ENMIMBIM@New_Create_2D_Sound_Player?$AA@ 110ac118     dllmain.obj
 0002:00003134       ??_C@_0BP@BNBMIEKM@New_Create_2D_WAV_Sound_Player?$AA@ 110ac134     dllmain.obj
 0002:00003154       ??_C@_0CH@KEGANMCF@New_Create_3D_WAV_Sound_At_Bone_@ 110ac154     dllmain.obj
 0002:0000317c       ??_C@_0CD@HKAJONGF@New_Create_3D_Sound_At_Bone_Play@ 110ac17c     dllmain.obj
 0002:000031a0       ??_C@_0BN@FDAGJMKD@New_Set_Display_Color_Player?$AA@ 110ac1a0     dllmain.obj
 0002:000031c0       ??_C@_0BI@BIGCCHLL@New_Display_Text_Player?$AA@ 110ac1c0     dllmain.obj
 0002:000031d8       ??_C@_0BH@EMLDPBJE@New_Display_Int_Player?$AA@ 110ac1d8     dllmain.obj
 0002:000031f0       ??_C@_0BJ@BHPFPCAI@New_Display_Float_Player?$AA@ 110ac1f0     dllmain.obj
 0002:0000320c       ??_C@_0BN@ICDIBFBA@New_Set_Obj_Radar_Blip_Shape?$AA@ 110ac20c     dllmain.obj
 0002:0000322c       ??_C@_0BN@NDFNHDJN@New_Set_Obj_Radar_Blip_Color?$AA@ 110ac22c     dllmain.obj
 0002:0000324c       ??_C@_0CE@NDFBOGLJ@New_Set_Obj_Radar_Blip_Shape_Pla@ 110ac24c     dllmain.obj
 0002:00003270       ??_C@_0CE@MGFOBBDG@New_Set_Obj_Radar_Blip_Color_Pla@ 110ac270     dllmain.obj
 0002:00003294       ??_C@_0BH@LGGKJPMB@NewAddObjectCreateHook?$AA@ 110ac294     dllmain.obj
 0002:000032ac       ??_C@_0BK@GKCDPKE@NewRemoveObjectCreateHook?$AA@ 110ac2ac     dllmain.obj
 0002:000032c8       ??_C@_0L@BFCNNHMC@AddKeyHook?$AA@ 110ac2c8     dllmain.obj
 0002:000032d4       ??_C@_0O@CMJPPFDF@RemoveKeyHook?$AA@ 110ac2d4     dllmain.obj
 0002:000032e4       ??_C@_09NOJDAPDO@Set_Scope?$AA@ 110ac2e4     dllmain.obj
 0002:000032f0       ??_C@_0BA@KLLGFAPE@Set_HUD_Texture?$AA@ 110ac2f0     dllmain.obj
 0002:00003300       ??_C@_0M@PIBLNPHK@AddHostHook?$AA@ 110ac300     dllmain.obj
 0002:0000330c       ??_C@_0BB@EIEGDAAC@AddLoadLevelHook?$AA@ 110ac30c     dllmain.obj
 0002:00003320       ??_C@_0BA@CLNCABAJ@AddGameOverHook?$AA@ 110ac320     dllmain.obj
 0002:00003330       ??_C@_0BC@BBENPMJL@AddPlayerJoinHook?$AA@ 110ac330     dllmain.obj
 0002:00003344       ??_C@_0BF@LBJICEGB@GetCurrentMusicTrack?$AA@ 110ac344     dllmain.obj
 0002:0000335c       ??_C@_0BB@KPPILEKB@Set_Info_Texture?$AA@ 110ac35c     dllmain.obj
 0002:00003370       ??_C@_0BD@MBHONDFC@Clear_Info_Texture?$AA@ 110ac370     dllmain.obj
 0002:00003384       ??_C@_0BC@JNCDLPNM@Set_Vehicle_Limit?$AA@ 110ac384     dllmain.obj
 0002:00003398       ??_C@_0BC@LICIDEMC@Get_Vehicle_Limit?$AA@ 110ac398     dllmain.obj
 0002:000033ac       ??_C@_0N@NCFONGG@Send_Message?$AA@ 110ac3ac     dllmain.obj
 0002:000033bc       ??_C@_0BE@IIGCGNIC@Send_Message_Player?$AA@ 110ac3bc     dllmain.obj
 0002:000033d0       ??_C@_0BH@GJJAIAB@New_Display_Health_Bar?$AA@ 110ac3d0     dllmain.obj
 0002:000033e8       ??_C@_0P@IHKAKAEO@AddVersionHook?$AA@ 110ac3e8     dllmain.obj
 0002:000033f8       ??_C@_0BD@CNJALGFI@Set_Wireframe_Mode?$AA@ 110ac3f8     dllmain.obj
 0002:0000340c       ??_C@_0BL@DCIMBMAN@New_Disable_All_Collisions?$AA@ 110ac40c     dllmain.obj
 0002:00003428       ??_C@_0CA@LBEEGJKG@New_Disable_Physical_Collisions?$AA@ 110ac428     dllmain.obj
 0002:00003448       ??_C@_0BG@BBLOAJCE@New_Enable_Collisions?$AA@ 110ac448     dllmain.obj
 0002:00003460       ??_C@_0BB@FALIJHOM@Load_New_HUD_INI?$AA@ 110ac460     dllmain.obj
 0002:00003474       ??_C@_0O@CGFKECIG@Remove_Weapon?$AA@ 110ac474     dllmain.obj
 0002:00003484       ??_C@_0P@KIKNJFGM@Update_PT_Data?$AA@ 110ac484     dllmain.obj
 0002:00003494       ??_C@_0BB@JKEOAOPH@Change_Radar_Map?$AA@ 110ac494     dllmain.obj
 0002:000034a8       ??_C@_0BH@DAOOINAA@AddPowerupPurchaseHook?$AA@ 110ac4a8     dllmain.obj
 0002:000034c0       ??_C@_0BH@BMFCOOKO@AddVehiclePurchaseHook?$AA@ 110ac4c0     dllmain.obj
 0002:000034d8       ??_C@_0BJ@INOONOPD@AddCharacterPurchaseHook?$AA@ 110ac4d8     dllmain.obj
 0002:000034f4       ??_C@_0BK@GKIFHIHI@AddPowerupPurchaseMonHook?$AA@ 110ac4f4     dllmain.obj
 0002:00003510       ??_C@_0BK@DFGEMPPN@AddVehiclePurchaseMonHook?$AA@ 110ac510     dllmain.obj
 0002:0000352c       ??_C@_0BM@EMJBLLNL@AddCharacterPurchaseMonHook?$AA@ 110ac52c     dllmain.obj
 0002:00003548       ??_C@_0BK@NGJKJBAA@RemovePowerupPurchaseHook?$AA@ 110ac548     dllmain.obj
 0002:00003564       ??_C@_0BK@PKCGPCKO@RemoveVehiclePurchaseHook?$AA@ 110ac564     dllmain.obj
 0002:00003580       ??_C@_0BM@JJOPGEMI@RemoveCharacterPurchaseHook?$AA@ 110ac580     dllmain.obj
 0002:0000359c       ??_C@_0BN@NLJKJAOG@RemovePowerupPurchaseMonHook?$AA@ 110ac59c     dllmain.obj
 0002:000035bc       ??_C@_0BN@IEHLCHGD@RemoveVehiclePurchaseMonHook?$AA@ 110ac5bc     dllmain.obj
 0002:000035dc       ??_C@_0BP@NICMHBK@RemoveCharacterPurchaseMonHook?$AA@ 110ac5dc     dllmain.obj
 0002:000035fc       ??_C@_0BK@FFCPOFBA@Get_Build_Time_Multiplier?$AA@ 110ac5fc     dllmain.obj
 0002:00003618       ??_C@_0BH@NFHCMOHH@Set_Currently_Building?$AA@ 110ac618     dllmain.obj
 0002:00003630       ??_C@_0BG@HJDMFMAJ@Is_Currently_Building?$AA@ 110ac630     dllmain.obj
 0002:00003648       ??_C@_0BF@JHNKODII@AddConsoleOutputHook?$AA@ 110ac648     dllmain.obj
 0002:00003660       ??_C@_0L@OONHDGA@AddCRCHook?$AA@ 110ac660     dllmain.obj
 0002:0000366c       ??_C@_0M@JNBJJDPK@AddDataHook?$AA@ 110ac66c     dllmain.obj
 0002:00003678       ??_C@_0BF@IJDIAGHM@Set_Reticle_Texture1?$AA@ 110ac678     dllmain.obj
 0002:00003690       ??_C@_0BF@KCBFFFLP@Set_Reticle_Texture2?$AA@ 110ac690     dllmain.obj
 0002:000036a8       ??_C@_0BC@GCCMNPJK@New_Set_Fog_Color?$AA@ 110ac6a8     dllmain.obj
 0002:000036bc       ??_C@_0BF@KHIDDEHK@Set_Fog_Color_Player?$AA@ 110ac6bc     dllmain.obj
 0002:000036d4       ??_C@_0BB@EAFFCBP@New_Set_Fog_Mode?$AA@ 110ac6d4     dllmain.obj
 0002:000036e8       ??_C@_0BE@KPNALHHL@Set_Fog_Mode_Player?$AA@ 110ac6e8     dllmain.obj
 0002:000036fc       ??_C@_0BC@GFPPEJCD@Set_Shader_Number?$AA@ 110ac6fc     dllmain.obj
 0002:00003710       ??_C@_0BE@PBLCJAIL@New_Set_Fog_Density?$AA@ 110ac710     dllmain.obj
 0002:00003724       ??_C@_0BH@OHPNNHID@Set_Fog_Density_Player?$AA@ 110ac724     dllmain.obj
 0002:0000373c       ??_C@_0BK@FGLGICLJ@New_Change_Time_Remaining?$AA@ 110ac73c     dllmain.obj
 0002:00003758       ??_C@_0BG@OOEEFDBO@New_Change_Time_Limit?$AA@ 110ac758     dllmain.obj
 0002:00003770       ??_C@_0BE@FJOCJKNG@Display_GDI_Sidebar?$AA@ 110ac770     dllmain.obj
 0002:00003784       ??_C@_0BE@BCJEKMLD@Display_NOD_Sidebar?$AA@ 110ac784     dllmain.obj
 0002:00003798       ??_C@_0BI@KABJNJEM@Display_Security_Dialog?$AA@ 110ac798     dllmain.obj
 0002:000037b0       ??_C@_0BD@DBPLMLLJ@AddPlayerLeaveHook?$AA@ 110ac7b0     dllmain.obj
 0002:000037c4       ??_C@_0BA@ICBJGPDH@GetExplosionObj?$AA@ 110ac7c4     dllmain.obj
 0002:000037d4       ??_C@_05FGPGKOKF@2?40?42?$AA@ 110ac7d4     dllmain.obj
 0002:000037dc       ??_C@_09EJNOGGAN@LuaPlugin?$AA@ 110ac7dc     dllmain.obj
 0002:000037e8       ??_C@_03EMGHBCAM@4?40?$AA@ 110ac7e8     dllmain.obj
 0002:000037f0       ??_7?$VectorClass@PAE@@6B@ 110ac7f0     engine_bhs.obj
 0002:00004068       _sqlite3_apis              110ad068     sqlite3.obj
 0002:0000659c       _luaT_typenames            110af59c     ltm.obj
 0002:000067d8       _sqlite3_version           110af7d8     sqlite3.obj
 0002:00006a20       _luaP_opnames              110afa20     lopcodes.obj
 0002:00006abc       _luaP_opmodes              110afabc     lopcodes.obj
 0002:00006ae8       _luaO_nilobject_           110afae8     lobject.obj
 0002:00006d28       _luaX_tokens               110afd28     llex.obj
 0002:000070c0       _lua_ident                 110b00c0     lapi.obj
 0002:00007150       ?methods@Lua_sqlite_wrapper@@0QBUluaL_Reg@@B 110b0150     Lua_Class.obj
 0002:00007174       ??_C@_04CGFJFPFD@none?$AA@ 110b0174     engine_def.obj
 0002:0000717c       ??_C@_02CPIDLAI@at?$AA@    110b017c     engine_diagnostics.obj
 0002:00007180       ??_C@_03KPGLNNAM@WOL?$AA@  110b0180     engine_game.obj
 0002:00007184       ??_C@_03BANLECBK@LAN?$AA@  110b0184     engine_game.obj
 0002:0000718c       ??_7_Vector3MathFunctions@@6B@ 110b018c     engine_math.obj
 0002:000071d8       ??_7_Vector4MathFunctions@@6B@ 110b01d8     engine_math.obj
 0002:0000720c       ??_7_Vector4MathFunctionsSSE@@6B@ 110b020c     engine_math.obj
 0002:0000723c       ??_C@_0M@PCENNPGA@?$CFd?4?$CFd?4?$CFd?4?$CFd?$AA@ 110b023c     engine_net.obj
 0002:00007248       ??_C@_0P@FOCHHKCH@?$CFd?4?$CFd?4?$CFd?4?$CFd?$DL?$CFd?$AA@ 110b0248     engine_net.obj
 0002:00007258       ??_C@_0O@HNNKEAKD@Is_PowerPlant?$AA@ 110b0258     engine_obj.obj
 0002:00007268       ??_C@_0BC@BJIJEBBO@Is_SoldierFactory?$AA@ 110b0268     engine_obj.obj
 0002:0000727c       ??_C@_0M@FDGOOIDO@Is_Airstrip?$AA@ 110b027c     engine_obj.obj
 0002:00007288       ??_C@_0O@LDEDDJBA@Is_WarFactory?$AA@ 110b0288     engine_obj.obj
 0002:00007298       ??_C@_0M@IGHPANDI@Is_Refinery?$AA@ 110b0298     engine_obj.obj
 0002:000072a4       ??_C@_0N@HDCIACDB@Is_ComCenter?$AA@ 110b02a4     engine_obj.obj
 0002:000072b4       ??_C@_0N@HCJJACKE@Is_RepairBay?$AA@ 110b02b4     engine_obj.obj
 0002:000072c4       ??_C@_06OJHGLDPL@?$CInull?$CJ?$AA@ 110b02c4     engine_obj.obj
 0002:000072cc       ??_C@_05FAECCOPD@DUMMY?$AA@ 110b02cc     engine_phys.obj
 0002:000072d4       ??_C@_07BMODAHHB@Is_Door?$AA@ 110b02d4     engine_phys.obj
 0002:000072dc       ??_C@_0M@PAGNNLL@Is_Elevator?$AA@ 110b02dc     engine_phys.obj
 0002:000072e8       ??_C@_0BI@MILEOEOM@Is_DamageableStaticPhys?$AA@ 110b02e8     engine_phys.obj
 0002:00007300       ??_C@_0BC@FHHCMIE@Is_AccessablePhys?$AA@ 110b0300     engine_phys.obj
 0002:00007314       ??_C@_0BC@CGMCEOPL@Is_DecorationPhys?$AA@ 110b0314     engine_phys.obj
 0002:00007328       ??_C@_0N@IIDKGMMK@Is_HumanPhys?$AA@ 110b0328     engine_phys.obj
 0002:00007338       ??_C@_0BA@NMEMOAAA@Is_MotorVehicle?$AA@ 110b0338     engine_phys.obj
 0002:00007348       ??_C@_08INKCDJHE@Is_Phys3?$AA@ 110b0348     engine_phys.obj
 0002:00007354       ??_C@_0N@JIBAJJLF@Is_RigidBody?$AA@ 110b0354     engine_phys.obj
 0002:00007364       ??_C@_0BI@IDFOMLA@Is_ShakeableStatricPhys?$AA@ 110b0364     engine_phys.obj
 0002:0000737c       ??_C@_0BC@BNMPKHKP@Is_StaticAnimPhys?$AA@ 110b037c     engine_phys.obj
 0002:00007390       ??_C@_0O@PMHLNCPL@Is_StaticPhys?$AA@ 110b0390     engine_phys.obj
 0002:000073a0       ??_C@_0BH@OPGDFLJA@Is_TimedDecorationPhys?$AA@ 110b03a0     engine_phys.obj
 0002:000073b8       ??_C@_0P@DPJMCENA@Is_VehiclePhys?$AA@ 110b03b8     engine_phys.obj
 0002:000073c8       ??_C@_0BD@JPEOMMEF@Is_DynamicAnimPhys?$AA@ 110b03c8     engine_phys.obj
 0002:000073dc       ??_C@_0BF@LGMFACPH@Is_BuildingAggregate?$AA@ 110b03dc     engine_phys.obj
 0002:000073f4       ??_C@_0O@IEFMGMKP@Is_Projectile?$AA@ 110b03f4     engine_phys.obj
 0002:00007404       ??_C@_0BG@HDNGLABG@msg?5?$CFs?5switched?5teams?$AA@ 110b0404     engine_player.obj
 0002:0000741c       ??_C@_07GJJCKENN@Neutral?$AA@ 110b041c     engine_tdb.obj
 0002:00007424       ??_C@_1BA@KOPEKOGK@?$AAV?$AAe?$AAh?$AAi?$AAc?$AAl?$AAe?$AA?$AA@ 110b0424     engine_tdb.obj
 0002:00007438       ??_7ScriptFactory@@6B@     110b0438     scriptfactory.obj
 0002:00007440       ??_C@_01IHBHIGKO@?0?$AA@   110b0440     scripts.obj
 0002:00007444       ??_C@_03POJIIFD@?$DN?3?6?$AA@ 110b0444     scripts.obj
 0002:00007448       ??_C@_0N@CILGKGLK@critical?4txt?$AA@ 110b0448     scripts.obj
 0002:00007458       ??_C@_0CM@KMOCPEFC@Critical?5Scripts?4dll?5error?0param@ 110b0458     scripts.obj
 0002:0000748c       ??_7GameObjObserverClass@@6B@ 110b048c     scripts.obj
 0002:000074d4       ??_7ScriptImpClass@@6B@    110b04d4     scripts.obj
 0002:0000753c       ??_C@_05BNKNJDAB@Query?$AA@ 110b053c     Lua_Class.obj
 0002:00007544       ??_C@_06COPDEJPI@sqlite?$AA@ 110b0544     Lua_Class.obj
 0002:0000754c       ??_C@_05GGFCIFOJ@db?4db?$AA@ 110b054c     LuaFunctions.obj
 0002:00007554       ??_C@_0M@OKDMMFBL@__metatable?$AA@ 110b0554     LuaFunctions.obj
 0002:00007560       ??_C@_07NHABFFHN@__index?$AA@ 110b0560     LuaFunctions.obj
 0002:00007568       ??_C@_04BDLIKKMN@__gc?$AA@ 110b0568     LuaFunctions.obj
 0002:00007570       ??_C@_01MMEEDKFM@X?$AA@    110b0570     LuaFunctions.obj
 0002:00007574       ??_C@_01NFFPALBN@Y?$AA@    110b0574     LuaFunctions.obj
 0002:00007578       ??_C@_01POHCFINO@Z?$AA@    110b0578     LuaFunctions.obj
 0002:0000757c       ??_C@_0CE@JPEJFGLC@Invalid?5argument?0?5expected?5a?5tab@ 110b057c     LuaFunctions.obj
 0002:000075a0       ??_C@_0CH@OBMHCNHM@Invalid?5argument?5?$CD1?4?5Expected?5a?5@ 110b05a0     LuaFunctions.obj
 0002:000075c8       ??_C@_0CB@IMEINMNJ@Bad?5argument?5?$CD2?0?5expected?5table?4@ 110b05c8     LuaFunctions.obj
 0002:000075ec       ??_C@_0DK@FOONMHPB@Invalid?5argument?5?$CD3?5to?5Create_Sc@ 110b05ec     LuaFunctions.obj
 0002:00007628       ??_C@_0DK@PBKJFFLG@Invalid?5argument?5?$CD2?5to?5Create_Sc@ 110b0628     LuaFunctions.obj
 0002:00007664       ??_C@_02DPKJAMEF@?$CFd?$AA@ 110b0664     LuaFunctions.obj
 0002:00007668       ??_C@_03FKNCMABI@?$CFlu?$AA@ 110b0668     LuaFunctions.obj
 0002:0000766c       ??_C@_0BH@EAGJOFBI@Not?5a?5valid?5GameObject?$AA@ 110b066c     LuaFunctions.obj
 0002:00007684       ??_C@_0N@PFJHKDIJ@AlliesKilled?$AA@ 110b0684     LuaFunctions.obj
 0002:00007694       ??_C@_06PFFCHNPF@ArmHit?$AA@ 110b0694     LuaFunctions.obj
 0002:0000769c       ??_C@_08MDPMAMOE@ArmShots?$AA@ 110b069c     LuaFunctions.obj
 0002:000076a8       ??_C@_0BC@EPKCIPIL@BuildingDestroyed?$AA@ 110b06a8     LuaFunctions.obj
 0002:000076bc       ??_C@_0BG@JFOMGKPN@ClientUpdateFrequency?$AA@ 110b06bc     LuaFunctions.obj
 0002:000076d4       ??_C@_0N@NJMIGDDL@CreationTime?$AA@ 110b06d4     LuaFunctions.obj
 0002:000076e4       ??_C@_0M@JPJEKEFD@CreditGrant?$AA@ 110b06e4     LuaFunctions.obj
 0002:000076f0       ??_C@_09NDJGPLKB@CrotchHit?$AA@ 110b06f0     LuaFunctions.obj
 0002:000076fc       ??_C@_0M@BJPAJEGF@CrotchShots?$AA@ 110b06fc     LuaFunctions.obj
 0002:00007708       ??_C@_0BC@PCBEOMIP@DamageScaleFactor?$AA@ 110b0708     LuaFunctions.obj
 0002:0000771c       ??_C@_06IIDHDGJJ@Deaths?$AA@ 110b071c     LuaFunctions.obj
 0002:00007724       ??_C@_0O@CGGLHOMB@EnemiesKilled?$AA@ 110b0724     LuaFunctions.obj
 0002:00007734       ??_C@_0M@HHDMAFHP@FinalHealth?$AA@ 110b0734     LuaFunctions.obj
 0002:00007740       ??_C@_03DACHGFGH@Fps?$AA@  110b0740     LuaFunctions.obj
 0002:00007744       ??_C@_08NOCEIAGF@GameTime?$AA@ 110b0744     LuaFunctions.obj
 0002:00007750       ??_C@_07EEMEKLHB@HeadHit?$AA@ 110b0750     LuaFunctions.obj
 0002:00007758       ??_C@_09PDKDJHNM@HeadShots?$AA@ 110b0758     LuaFunctions.obj
 0002:00007764       ??_C@_09FKJNNHFN@IpAddress?$AA@ 110b0764     LuaFunctions.obj
 0002:00007770       ??_C@_08CHIOLOMB@IsActive?$AA@ 110b0770     LuaFunctions.obj
 0002:0000777c       ??_C@_07NIJBBMLI@IsHuman?$AA@ 110b077c     LuaFunctions.obj
 0002:00007784       ??_C@_08JLLJEFFA@IsInGame?$AA@ 110b0784     LuaFunctions.obj
 0002:00007790       ??_C@_0BJ@BIPGKJHL@IsWaitingForIntermission?$AA@ 110b0790     LuaFunctions.obj
 0002:000077ac       ??_C@_08KEGJKBNA@JoinTime?$AA@ 110b07ac     LuaFunctions.obj
 0002:000077b8       ??_C@_05ILKPOBAF@Kills?$AA@ 110b07b8     LuaFunctions.obj
 0002:000077c0       ??_C@_0BB@CCHNCKND@KillsFromVehicle?$AA@ 110b07c0     LuaFunctions.obj
 0002:000077d4       ??_C@_0M@OJHKIHLG@LastDamaged?$AA@ 110b07d4     LuaFunctions.obj
 0002:000077e0       ??_C@_0M@PFOCDCGB@LastDamager?$AA@ 110b07e0     LuaFunctions.obj
 0002:000077ec       ??_C@_06MAOGDGLH@LegHit?$AA@ 110b07ec     LuaFunctions.obj
 0002:000077f4       ??_C@_08OALNIMMP@LegShots?$AA@ 110b07f4     LuaFunctions.obj
 0002:00007800       ??_C@_05INIBOMDG@Money?$AA@ 110b0800     LuaFunctions.obj
 0002:00007808       ??_C@_04CPBFGEOK@Ping?$AA@ 110b0808     LuaFunctions.obj
 0002:00007810       ??_C@_08DDCIMEN@PlayerId?$AA@ 110b0810     LuaFunctions.obj
 0002:0000781c       ??_C@_02KPKOKMHB@?$CFS?$AA@ 110b081c     LuaFunctions.obj
 0002:00007820       ??_C@_0L@HMKCBGMC@PlayerName?$AA@ 110b0820     LuaFunctions.obj
 0002:0000782c       ??_C@_0L@NHKBNGLC@PlayerType?$AA@ 110b082c     LuaFunctions.obj
 0002:00007838       ??_C@_0BC@BFKFKHAI@PowerupsCollected?$AA@ 110b0838     LuaFunctions.obj
 0002:0000784c       ??_C@_04EPBKNPKN@Rung?$AA@ 110b084c     LuaFunctions.obj
 0002:00007854       ??_C@_05DGAPONBB@Score?$AA@ 110b0854     LuaFunctions.obj
 0002:0000785c       ??_C@_0M@GJIALFDI@SessionTime?$AA@ 110b085c     LuaFunctions.obj
 0002:00007868       ??_C@_0L@CMMJJCJ@ShotsFired?$AA@ 110b0868     LuaFunctions.obj
 0002:00007874       ??_C@_08KJJGMAPP@Squishes?$AA@ 110b0874     LuaFunctions.obj
 0002:00007880       ??_C@_08IAFFCLEC@TorsoHit?$AA@ 110b0880     LuaFunctions.obj
 0002:0000788c       ??_C@_0L@OKHALFFN@TorsoShots?$AA@ 110b088c     LuaFunctions.obj
 0002:00007898       ??_C@_09IGIFPOMH@TotalTime?$AA@ 110b0898     LuaFunctions.obj
 0002:000078a4       ??_C@_0BC@PHEILIGG@VehiclesDestroyed?$AA@ 110b08a4     LuaFunctions.obj
 0002:000078b8       ??_C@_0M@NNGMIGEO@VehicleTime?$AA@ 110b08b8     LuaFunctions.obj
 0002:000078c4       ??_C@_0BD@NDPDHFLE@CanRepairBuildings?$AA@ 110b08c4     LuaFunctions.obj
 0002:000078d8       ??_C@_0L@HNLOJILL@CFGModTime?$AA@ 110b08d8     LuaFunctions.obj
 0002:000078e4       ??_C@_0P@LNJIGANM@CurrentPlayers?$AA@ 110b08e4     LuaFunctions.obj
 0002:000078f4       ??_C@_0L@BCLFDHEE@DoMapsLoop?$AA@ 110b08f4     LuaFunctions.obj
 0002:00007900       ??_C@_0BF@HEDDIIJA@DriverIsAlwaysGunner?$AA@ 110b0900     LuaFunctions.obj
 0002:00007918       ??_C@_0L@EGBEBJPN@FrameCount?$AA@ 110b0918     LuaFunctions.obj
 0002:00007924       ??_C@_0BF@GLDOOLID@GameDuration_Seconds?$AA@ 110b0924     LuaFunctions.obj
 0002:0000793c       ??_C@_0BC@BNIFAPOJ@GameplayPermitted?$AA@ 110b093c     LuaFunctions.obj
 0002:00007950       ??_C@_0O@JFHKBIDP@GameStartTime?$AA@ 110b0950     LuaFunctions.obj
 0002:00007960       ??_C@_09HEMANCP@GameTitle?$AA@ 110b0960     LuaFunctions.obj
 0002:0000796c       ??_C@_0N@JCDGFAOA@GrantWeapons?$AA@ 110b096c     LuaFunctions.obj
 0002:0000797c       ??_C@_03GDBIGDNC@INI?$AA@  110b097c     LuaFunctions.obj
 0002:00007980       ??_C@_0BJ@KKNKKMDM@IntermissionTime_Seconds?$AA@ 110b0980     LuaFunctions.obj
 0002:0000799c       ??_C@_0BF@MOPKHNN@IntermissionTimeLeft?$AA@ 110b099c     LuaFunctions.obj
 0002:000079b4       ??_C@_02MFEOMNPG@IP?$AA@   110b09b4     LuaFunctions.obj
 0002:000079b8       ??_C@_0O@EOILMOEJ@IsAutoRestart?$AA@ 110b09b8     LuaFunctions.obj
 0002:000079c8       ??_C@_0L@GKKLCHAB@IsClanGame?$AA@ 110b09c8     LuaFunctions.obj
 0002:000079d4       ??_C@_0M@EOIPHOP@IsDedicated?$AA@ 110b09d4     LuaFunctions.obj
 0002:000079e0       ??_C@_0BI@EFFODFJL@IsFriendlyFirePermitted?$AA@ 110b09e0     LuaFunctions.obj
 0002:000079f8       ??_C@_0L@DDBBBFCM@IsLaddered?$AA@ 110b09f8     LuaFunctions.obj
 0002:00007a04       ??_C@_0N@JMJLINIK@IsPassworded?$AA@ 110b0a04     LuaFunctions.obj
 0002:00007a14       ??_C@_0N@DHOFBOI@IsQuickMatch?$AA@ 110b0a14     LuaFunctions.obj
 0002:00007a24       ??_C@_0BG@FMJONICE@IsTeamChangingAllowed?$AA@ 110b0a24     LuaFunctions.obj
 0002:00007a3c       ??_C@_0N@ODNLMOFG@MapCycleOver?$AA@ 110b0a3c     LuaFunctions.obj
 0002:00007a4c       ??_C@_07DCHKAMOF@MapName?$AA@ 110b0a4c     LuaFunctions.obj
 0002:00007a54       ??_C@_09HMDKBDHD@MapNumber?$AA@ 110b0a54     LuaFunctions.obj
 0002:00007a60       ??_C@_0L@INDPAOFE@MaxPlayers?$AA@ 110b0a60     LuaFunctions.obj
 0002:00007a6c       ??_C@_0BB@CKLLELJN@MaxWorldDistance?$AA@ 110b0a6c     LuaFunctions.obj
 0002:00007a80       ??_C@_0BK@IMOMEAAO@MinQualifyingTime_Minutes?$AA@ 110b0a80     LuaFunctions.obj
 0002:00007a9c       ??_C@_07PKACDHDF@ModName?$AA@ 110b0a9c     LuaFunctions.obj
 0002:00007aa4       ??_C@_04KIJCBNGA@Motd?$AA@ 110b0aa4     LuaFunctions.obj
 0002:00007aac       ??_C@_08EBOCIONP@MVPCount?$AA@ 110b0aac     LuaFunctions.obj
 0002:00007ab8       ??_C@_07FIBCJCAP@MVPName?$AA@ 110b0ab8     LuaFunctions.obj
 0002:00007ac0       ??_C@_05HDCNEILF@Owner?$AA@ 110b0ac0     LuaFunctions.obj
 0002:00007ac8       ??_C@_08FJIAHGMM@Password?$AA@ 110b0ac8     LuaFunctions.obj
 0002:00007ad4       ??_C@_04HOKNCALA@Port?$AA@ 110b0ad4     LuaFunctions.obj
 0002:00007adc       ??_C@_09EBHEJGHC@RadarMode?$AA@ 110b0adc     LuaFunctions.obj
 0002:00007ae8       ??_C@_0L@DPCBPGBB@RemixTeams?$AA@ 110b0ae8     LuaFunctions.obj
 0002:00007af4       ??_C@_0BE@MMBIOHDE@SettingsDescription?$AA@ 110b0af4     LuaFunctions.obj
 0002:00007b08       ??_C@_0N@OIOGGAPO@SpawnWeapons?$AA@ 110b0b08     LuaFunctions.obj
 0002:00007b18       ??_C@_0BE@MEBJKMMP@StringVersionsMatch?$AA@ 110b0b18     LuaFunctions.obj
 0002:00007b2c       ??_C@_0BC@HIKNDPHH@TimeLimit_Minutes?$AA@ 110b0b2c     LuaFunctions.obj
 0002:00007b40       ??_C@_0BG@FIOEAFLK@TimeRemaining_Seconds?$AA@ 110b0b40     LuaFunctions.obj
 0002:00007b58       ??_C@_0BA@GODJPBNA@UseLagReduction?$AA@ 110b0b58     LuaFunctions.obj
 0002:00007b68       ??_C@_08FCKMIJII@WinnerID?$AA@ 110b0b68     LuaFunctions.obj
 0002:00007b74       ??_C@_07HODBMMPK@WinType?$AA@ 110b0b74     LuaFunctions.obj
 0002:00007b7c       ??_C@_0DG@MCBGHCJD@Invalid?5argument?5?$CD2?5to?5Set_cPlay@ 110b0b7c     LuaFunctions.obj
 0002:00007bb4       ??_C@_0DF@NLCPHGNC@Invalid?5argument?5?$CD1?5to?5Set_The_G@ 110b0bb4     LuaFunctions.obj
 0002:00007bec       ??_C@_0O@DHJCOOAM@Console_Input?$AA@ 110b0bec     LuaFunctions.obj
 0002:00007bfc       ??_C@_0P@ILIPJJJA@Console_Output?$AA@ 110b0bfc     LuaFunctions.obj
 0002:00007c0c       ??_C@_0BE@LPJECHLL@Get_Definition_Name?$AA@ 110b0c0c     LuaFunctions.obj
 0002:00007c20       ??_C@_0BC@JMDPJLIO@Get_Definition_ID?$AA@ 110b0c20     LuaFunctions.obj
 0002:00007c34       ??_C@_0BI@HKFLICM@Get_Definition_Class_ID?$AA@ 110b0c34     LuaFunctions.obj
 0002:00007c4c       ??_C@_0BD@JIAHLMJB@Is_Valid_Preset_ID?$AA@ 110b0c4c     LuaFunctions.obj
 0002:00007c60       ??_C@_0BA@COPKFGHH@Is_Valid_Preset?$AA@ 110b0c60     LuaFunctions.obj
 0002:00007c70       ??_C@_0P@GLDDGJOL@Set_Max_Health?$AA@ 110b0c70     LuaFunctions.obj
 0002:00007c80       ??_C@_0BI@OHENJIG@Set_Max_Shield_Strength?$AA@ 110b0c80     LuaFunctions.obj
 0002:00007c98       ??_C@_0BA@GEANJNAI@Get_Shield_Type?$AA@ 110b0c98     LuaFunctions.obj
 0002:00007ca8       ??_C@_08PBBNBGMF@Get_Skin?$AA@ 110b0ca8     LuaFunctions.obj
 0002:00007cb4       ??_C@_08DBAFLI@Set_Skin?$AA@ 110b0cb4     LuaFunctions.obj
 0002:00007cc0       ??_C@_0L@KJFIGFIN@Power_Base?$AA@ 110b0cc0     LuaFunctions.obj
 0002:00007ccc       ??_C@_0BK@HFDGOJPL@Set_Can_Generate_Soldiers?$AA@ 110b0ccc     LuaFunctions.obj
 0002:00007ce8       ??_C@_0BK@MIGBGFGP@Set_Can_Generate_Vehicles?$AA@ 110b0ce8     LuaFunctions.obj
 0002:00007d04       ??_C@_0N@BJAOOMHC@Destroy_Base?$AA@ 110b0d04     LuaFunctions.obj
 0002:00007d14       ??_C@_0BG@PNCKMKBB@Beacon_Destroyed_Base?$AA@ 110b0d14     LuaFunctions.obj
 0002:00007d2c       ??_C@_0BC@EDCNPODK@Enable_Base_Radar?$AA@ 110b0d2c     LuaFunctions.obj
 0002:00007d40       ??_C@_0N@IELKNIBF@Is_Harvester?$AA@ 110b0d40     LuaFunctions.obj
 0002:00007d50       ??_C@_0BB@HCNFOKHJ@Is_Radar_Enabled?$AA@ 110b0d50     LuaFunctions.obj
 0002:00007d64       ??_C@_0O@PMGLAAP@Building_Type?$AA@ 110b0d64     LuaFunctions.obj
 0002:00007d74       ??_C@_0BB@HJANHOLL@Is_Building_Dead?$AA@ 110b0d74     LuaFunctions.obj
 0002:00007d88       ??_C@_0O@EAINGNIM@Find_Building?$AA@ 110b0d88     LuaFunctions.obj
 0002:00007d98       ??_C@_0BC@GDHJAIFB@Find_Base_Defense?$AA@ 110b0d98     LuaFunctions.obj
 0002:00007dac       ??_C@_0O@FFNCOMLI@Is_Map_Flying?$AA@ 110b0dac     LuaFunctions.obj
 0002:00007dbc       ??_C@_0P@CABKALEI@Find_Harvester?$AA@ 110b0dbc     LuaFunctions.obj
 0002:00007dcc       ??_C@_0BA@PEKKDHCH@Is_Base_Powered?$AA@ 110b0dcc     LuaFunctions.obj
 0002:00007ddc       ??_C@_0BG@LKJBBFJH@Can_Generate_Vehicles?$AA@ 110b0ddc     LuaFunctions.obj
 0002:00007df4       ??_C@_0BG@EDMIEOGM@Can_Generate_Soliders?$AA@ 110b0df4     LuaFunctions.obj
 0002:00007e0c       ??_C@_0O@OAAGEAHI@Is_A_Building?$AA@ 110b0e0c     LuaFunctions.obj
 0002:00007e1c       ??_C@_0BI@NNPONLPD@Get_Building_Count_Team?$AA@ 110b0e1c     LuaFunctions.obj
 0002:00007e34       ??_C@_0BG@OHOFMNF@Find_Building_By_Team?$AA@ 110b0e34     LuaFunctions.obj
 0002:00007e4c       ??_C@_0BG@GKIPDHMN@Find_Building_By_Name?$AA@ 110b0e4c     LuaFunctions.obj
 0002:00007e64       ??_C@_0BB@CAIMNFEJ@Find_Power_Plant?$AA@ 110b0e64     LuaFunctions.obj
 0002:00007e78       ??_C@_0O@PHGIDNFO@Find_Refinery?$AA@ 110b0e78     LuaFunctions.obj
 0002:00007e88       ??_C@_0BA@CIIBAPN@Find_Repair_Bay?$AA@ 110b0e88     LuaFunctions.obj
 0002:00007e98       ??_C@_0BF@CKDOPONL@Find_Soldier_Factory?$AA@ 110b0e98     LuaFunctions.obj
 0002:00007eb0       ??_C@_0O@CCHJNIFI@Find_Airstrip?$AA@ 110b0eb0     LuaFunctions.obj
 0002:00007ec0       ??_C@_0BB@DALMOPGK@Find_War_Factory?$AA@ 110b0ec0     LuaFunctions.obj
 0002:00007ed4       ??_C@_0BF@DNOAPNML@Find_Vehicle_Factory?$AA@ 110b0ed4     LuaFunctions.obj
 0002:00007eec       ??_C@_0BA@GPPIGMPL@Find_Com_Center?$AA@ 110b0eec     LuaFunctions.obj
 0002:00007efc       ??_C@_0BG@OGFEDFNC@Is_Gameplay_Permitted?$AA@ 110b0efc     LuaFunctions.obj
 0002:00007f14       ??_C@_0N@DIMJCPDE@Is_Dedicated?$AA@ 110b0f14     LuaFunctions.obj
 0002:00007f24       ??_C@_08BOBIFHHO@Is_Linux?$AA@ 110b0f24     LuaFunctions.obj
 0002:00007f30       ??_C@_0BG@EAGJPJOH@Get_Current_Game_Mode?$AA@ 110b0f30     LuaFunctions.obj
 0002:00007f48       ??_C@_0BI@BBJMIFAE@Get_Harvester_Preset_ID?$AA@ 110b0f48     LuaFunctions.obj
 0002:00007f60       ??_C@_0BE@DHOJPKJD@Is_Harvester_Preset?$AA@ 110b0f60     LuaFunctions.obj
 0002:00007f74       ??_C@_0BD@CCCDBFNP@Destroy_Connection?$AA@ 110b0f74     LuaFunctions.obj
 0002:00007f88       ??_C@_0P@CIBEDKLK@Get_IP_Address?$AA@ 110b0f88     LuaFunctions.obj
 0002:00007f98       ??_C@_0M@BMLEFENB@Get_IP_Port?$AA@ 110b0f98     LuaFunctions.obj
 0002:00007fa4       ??_C@_0O@HGLENABK@Get_Bandwidth?$AA@ 110b0fa4     LuaFunctions.obj
 0002:00007fb4       ??_C@_08MIDJAJFC@Get_Ping?$AA@ 110b0fb4     LuaFunctions.obj
 0002:00007fc0       ??_C@_09BMMJMFDN@Get_Kbits?$AA@ 110b0fc0     LuaFunctions.obj
 0002:00007fcc       ??_C@_0BA@NKHJFAJA@Get_Object_Type?$AA@ 110b0fcc     LuaFunctions.obj
 0002:00007fdc       ??_C@_0BA@OIGPCCIJ@Set_Object_Type?$AA@ 110b0fdc     LuaFunctions.obj
 0002:00007fec       ??_C@_0M@DBJKFNOK@Is_Building?$AA@ 110b0fec     LuaFunctions.obj
 0002:00007ff8       ??_C@_0L@CJAAKFPG@Is_Soldier?$AA@ 110b0ff8     LuaFunctions.obj
 0002:00008004       ??_C@_0L@MDHOCNAG@Is_Vehicle?$AA@ 110b1004     LuaFunctions.obj
 0002:00008010       ??_C@_0N@BGBALPDG@Is_Cinematic?$AA@ 110b1010     LuaFunctions.obj
 0002:00008020       ??_C@_0O@HFPJNJCA@Is_ScriptZone?$AA@ 110b1020     LuaFunctions.obj
 0002:00008030       ??_C@_0L@FKPGGIJB@Is_Powerup?$AA@ 110b1030     LuaFunctions.obj
 0002:0000803c       ??_C@_05ICIAEAHN@Is_C4?$AA@ 110b103c     LuaFunctions.obj
 0002:00008044       ??_C@_09IFGLJDAE@Is_Beacon?$AA@ 110b1044     LuaFunctions.obj
 0002:00008050       ??_C@_08FNFCLDPA@Is_Armed?$AA@ 110b1050     LuaFunctions.obj
 0002:0000805c       ??_C@_09FFOOLGOH@Is_Simple?$AA@ 110b105c     LuaFunctions.obj
 0002:00008068       ??_C@_0BC@HADEBCIA@Is_VehicleFactory?$AA@ 110b1068     LuaFunctions.obj
 0002:0000807c       ??_C@_0O@FCOGFMAE@Is_Scriptable?$AA@ 110b107c     LuaFunctions.obj
 0002:0000808c       ??_C@_0BC@LEMIBPDC@Get_Building_Type?$AA@ 110b108c     LuaFunctions.obj
 0002:000080a0       ??_C@_0BB@HBHOBJDE@Get_Object_Count?$AA@ 110b10a0     LuaFunctions.obj
 0002:000080b4       ??_C@_0BD@JCMLMBAJ@Find_Random_Preset?$AA@ 110b10b4     LuaFunctions.obj
 0002:000080c8       ??_C@_0BO@PNBOICAN@Send_Custom_To_Team_Buildings?$AA@ 110b10c8     LuaFunctions.obj
 0002:000080e8       ??_C@_0BL@ILOBIBGA@Send_Custom_To_Team_Preset?$AA@ 110b10e8     LuaFunctions.obj
 0002:00008104       ??_C@_0BI@JBDDINHK@Send_Custom_All_Objects?$AA@ 110b1104     LuaFunctions.obj
 0002:0000811c       ??_C@_0BM@BGIMAAAL@Send_Custom_Event_To_Object?$AA@ 110b111c     LuaFunctions.obj
 0002:00008138       ??_C@_0BK@OBMKNCPF@Get_Is_Powerup_Persistant?$AA@ 110b1138     LuaFunctions.obj
 0002:00008154       ??_C@_0BK@GBAMBPFD@Set_Is_Powerup_Persistant?$AA@ 110b1154     LuaFunctions.obj
 0002:00008170       ??_C@_0BP@HNEGLABL@Get_Powerup_Always_Allow_Grant?$AA@ 110b1170     LuaFunctions.obj
 0002:00008190       ??_C@_0BP@KIKHJOEP@Set_Powerup_Always_Allow_Grant?$AA@ 110b1190     LuaFunctions.obj
 0002:000081b0       ??_C@_0BI@FDDCJLFE@Get_Powerup_Grant_Sound?$AA@ 110b11b0     LuaFunctions.obj
 0002:000081c8       ??_C@_0BI@EFFPHKDG@Set_Powerup_Grant_Sound?$AA@ 110b11c8     LuaFunctions.obj
 0002:000081e0       ??_C@_0O@OAJKJFAO@Grant_Powerup?$AA@ 110b11e0     LuaFunctions.obj
 0002:000081f0       ??_C@_0M@PJINACJD@Get_Vehicle?$AA@ 110b11f0     LuaFunctions.obj
 0002:000081fc       ??_C@_0N@LDJDHFJB@Grant_Refill?$AA@ 110b11fc     LuaFunctions.obj
 0002:0000820c       ??_C@_0BB@LJNIICIK@Change_Character?$AA@ 110b120c     LuaFunctions.obj
 0002:00008220       ??_C@_0P@MGMIEHHP@Create_Vehicle?$AA@ 110b1220     LuaFunctions.obj
 0002:00008230       ??_C@_0BA@PNFIOOPO@Toggle_Fly_Mode?$AA@ 110b1230     LuaFunctions.obj
 0002:00008240       ??_C@_0BL@INEMFOGD@Get_Vehicle_Occupant_Count?$AA@ 110b1240     LuaFunctions.obj
 0002:0000825c       ??_C@_0BF@OPNCOMFF@Get_Vehicle_Occupant?$AA@ 110b125c     LuaFunctions.obj
 0002:00008274       ??_C@_0BD@NCDLAEKN@Get_Vehicle_Driver?$AA@ 110b1274     LuaFunctions.obj
 0002:00008288       ??_C@_0BD@NJFLINOI@Get_Vehicle_Gunner?$AA@ 110b1288     LuaFunctions.obj
 0002:0000829c       ??_C@_0BE@MHIHJLBJ@Force_Occupant_Exit?$AA@ 110b129c     LuaFunctions.obj
 0002:000082b0       ??_C@_0BF@CAEFJNFC@Force_Occupants_Exit?$AA@ 110b12b0     LuaFunctions.obj
 0002:000082c8       ??_C@_0BD@LNDNILAP@Get_Vehicle_Return?$AA@ 110b12c8     LuaFunctions.obj
 0002:000082dc       ??_C@_0L@DJCBHANE@Is_Stealth?$AA@ 110b12dc     LuaFunctions.obj
 0002:000082e8       ??_C@_0N@LMPGKODC@Get_Fly_Mode?$AA@ 110b12e8     LuaFunctions.obj
 0002:000082f8       ??_C@_0BH@NKIJBPIG@Get_Vehicle_Seat_Count?$AA@ 110b12f8     LuaFunctions.obj
 0002:00008310       ??_C@_0P@CMBOEDAL@Get_Spawn_Char?$AA@ 110b1310     LuaFunctions.obj
 0002:00008320       ??_C@_0BC@LIEJLECG@Change_Spawn_Char?$AA@ 110b1320     LuaFunctions.obj
 0002:00008334       ??_C@_0BL@HGPCADIO@Soldier_Transition_Vehicle?$AA@ 110b1334     LuaFunctions.obj
 0002:00008350       ??_C@_0BB@HJJGHKPN@Get_Vehicle_Mode?$AA@ 110b1350     LuaFunctions.obj
 0002:00008364       ??_C@_0BH@NDNCNIB@Get_Team_Vehicle_Count?$AA@ 110b1364     LuaFunctions.obj
 0002:0000837c       ??_C@_0BC@KMJJJOID@Get_Vehicle_Owner?$AA@ 110b137c     LuaFunctions.obj
 0002:00008390       ??_C@_0BK@ELNJKOLO@Force_Occupants_Exit_Team?$AA@ 110b1390     LuaFunctions.obj
 0002:000083ac       ??_C@_0BM@DGHMDNCD@Get_Vehicle_Definition_Mode?$AA@ 110b13ac     LuaFunctions.obj
 0002:000083c8       ??_C@_0N@JBADJJPL@IsInsideZone?$AA@ 110b13c8     LuaFunctions.obj
 0002:000083d8       ??_C@_0CC@MCHJBOJE@Get_Vehicle_Definition_Mode_By_I@ 110b13d8     LuaFunctions.obj
 0002:000083fc       ??_C@_0O@IOOCGDJP@Get_Zone_Type?$AA@ 110b13fc     LuaFunctions.obj
 0002:0000840c       ??_C@_0BH@IFLLPNGL@IsAvailableForPurchase?$AA@ 110b140c     LuaFunctions.obj
 0002:00008424       ??_C@_0BC@IOJHPNHG@Check_Transitions?$AA@ 110b1424     LuaFunctions.obj
 0002:00008438       ??_C@_0BH@GKLBPOHL@Get_Vehicle_Gunner_Pos?$AA@ 110b1438     LuaFunctions.obj
 0002:00008450       ??_C@_0BH@DNPENBOP@Set_Vehicle_Is_Visible?$AA@ 110b1450     LuaFunctions.obj
 0002:00008468       ??_C@_0BD@CDHBLLAA@Set_Vehicle_Gunner?$AA@ 110b1468     LuaFunctions.obj
 0002:0000847c       ??_C@_09BANEPNJF@Get_Model?$AA@ 110b147c     LuaFunctions.obj
 0002:00008488       ??_C@_0BE@LJBOEPPA@Get_Animation_Frame?$AA@ 110b1488     LuaFunctions.obj
 0002:0000849c       ??_C@_0BC@CHJINDKP@Is_TrackedVehicle?$AA@ 110b149c     LuaFunctions.obj
 0002:000084b0       ??_C@_0P@CKPBONOH@Is_VTOLVehicle?$AA@ 110b14b0     LuaFunctions.obj
 0002:000084c0       ??_C@_0BC@IENPIFNE@Is_WheeledVehicle?$AA@ 110b14c0     LuaFunctions.obj
 0002:000084d4       ??_C@_0O@GAEPLLGG@Is_Motorcycle?$AA@ 110b14d4     LuaFunctions.obj
 0002:000084e4       ??_C@_0M@MEJGCGEH@Get_Physics?$AA@ 110b14e4     LuaFunctions.obj
 0002:000084f0       ??_C@_0P@BHHHNBDP@Copy_Transform?$AA@ 110b14f0     LuaFunctions.obj
 0002:00008500       ??_C@_08KPKNJFPI@Get_Mass?$AA@ 110b1500     LuaFunctions.obj
 0002:0000850c       ??_C@_0P@IIPHEKCP@Get_Htree_Name?$AA@ 110b150c     LuaFunctions.obj
 0002:0000851c       ??_C@_07DKLJMFJE@Get_Sex?$AA@ 110b151c     LuaFunctions.obj
 0002:00008524       ??_C@_0BM@JEPILEHJ@Create_Effect_All_Of_Preset?$AA@ 110b1524     LuaFunctions.obj
 0002:00008540       ??_C@_0M@EPAMEKME@Get_GameObj?$AA@ 110b1540     LuaFunctions.obj
 0002:0000854c       ??_C@_0O@BAAPOOPE@Get_Player_ID?$AA@ 110b154c     LuaFunctions.obj
 0002:0000855c       ??_C@_0BA@EKCLLPEE@Get_Player_Name?$AA@ 110b155c     LuaFunctions.obj
 0002:0000856c       ??_C@_0BG@BHJPGEKL@Get_Player_Name_By_ID?$AA@ 110b156c     LuaFunctions.obj
 0002:00008584       ??_C@_0M@CFBBLEJA@Change_Team?$AA@ 110b1584     LuaFunctions.obj
 0002:00008590       ??_C@_0BC@DFPNJPFL@Change_Team_By_ID?$AA@ 110b1590     LuaFunctions.obj
 0002:000085a4       ??_C@_0BB@KAPOCPOK@Get_Player_Count?$AA@ 110b15a4     LuaFunctions.obj
 0002:000085b8       ??_C@_0BG@JPGHPBFF@Get_Team_Player_Count?$AA@ 110b15b8     LuaFunctions.obj
 0002:000085d0       ??_C@_08IGNMLPJN@Get_Team?$AA@ 110b15d0     LuaFunctions.obj
 0002:000085dc       ??_C@_08NLPIDNNB@Get_Rank?$AA@ 110b15dc     LuaFunctions.obj
 0002:000085e8       ??_C@_09EOPCPGNG@Get_Kills?$AA@ 110b15e8     LuaFunctions.obj
 0002:000085f4       ??_C@_0L@JHCIOIOA@Get_Deaths?$AA@ 110b15f4     LuaFunctions.obj
 0002:00008600       ??_C@_09PDFCPKMC@Get_Score?$AA@ 110b1600     LuaFunctions.obj
 0002:0000860c       ??_C@_09EINMPLOF@Get_Money?$AA@ 110b160c     LuaFunctions.obj
 0002:00008618       ??_C@_0BI@HJDHHFKF@Get_Kill_To_Death_Ratio?$AA@ 110b1618     LuaFunctions.obj
 0002:00008630       ??_C@_0O@BALMFLKK@Get_Part_Name?$AA@ 110b1630     LuaFunctions.obj
 0002:00008640       ??_C@_0P@DCABNMJI@Get_Part_Names?$AA@ 110b1640     LuaFunctions.obj
 0002:00008650       ??_C@_0BL@CNKGLJFF@Get_GameObj_By_Player_Name?$AA@ 110b1650     LuaFunctions.obj
 0002:0000866c       ??_C@_0O@PIDOCMC@Purchase_Item?$AA@ 110b166c     LuaFunctions.obj
 0002:0000867c       ??_C@_0BC@GEOKJLFB@Set_Ladder_Points?$AA@ 110b167c     LuaFunctions.obj
 0002:00008690       ??_C@_08FJBKKBGI@Set_Rung?$AA@ 110b1690     LuaFunctions.obj
 0002:0000869c       ??_C@_09GGJJNKHH@Set_Money?$AA@ 110b169c     LuaFunctions.obj
 0002:000086a8       ??_C@_09NNBHNLFA@Set_Score?$AA@ 110b16a8     LuaFunctions.obj
 0002:000086b4       ??_C@_0BC@BBCBDAHE@Find_First_Player?$AA@ 110b16b4     LuaFunctions.obj
 0002:000086c8       ??_C@_0BD@GLJBNPNO@Change_Player_Team?$AA@ 110b16c8     LuaFunctions.obj
 0002:000086dc       ??_C@_0BA@EBKPOLGJ@Tally_Team_Size?$AA@ 110b16dc     LuaFunctions.obj
 0002:000086ec       ??_C@_0P@BHPKNBFI@Get_Team_Score?$AA@ 110b16ec     LuaFunctions.obj
 0002:000086fc       ??_C@_0BI@IKKGHMIO@Send_Custom_All_Players?$AA@ 110b16fc     LuaFunctions.obj
 0002:00008714       ??_C@_0BD@OENNAHJF@Steal_Team_Credits?$AA@ 110b1714     LuaFunctions.obj
 0002:00008728       ??_C@_0BB@GNKDJAPA@Get_Team_Credits?$AA@ 110b1728     LuaFunctions.obj
 0002:0000873c       ??_C@_0O@DHNNOFGC@Change_Team_2?$AA@ 110b173c     LuaFunctions.obj
 0002:0000874c       ??_C@_0BA@OBCIHPDE@Get_Player_Type?$AA@ 110b174c     LuaFunctions.obj
 0002:0000875c       ??_C@_0O@BJOHFLOB@Get_Team_Cost?$AA@ 110b175c     LuaFunctions.obj
 0002:0000876c       ??_C@_08LPADMKGN@Get_Cost?$AA@ 110b176c     LuaFunctions.obj
 0002:00008778       ??_C@_0N@NFPFIDBA@Set_Enlisted?$AA@ 110b1778     LuaFunctions.obj
 0002:00008788       ??_C@_0L@NNDKHPCM@Set_Beacon?$AA@ 110b1788     LuaFunctions.obj
 0002:00008794       ??_C@_0L@FHAJADEN@Set_Refill?$AA@ 110b1794     LuaFunctions.obj
 0002:000087a0       ??_C@_0L@CLILEOLK@Set_Preset?$AA@ 110b17a0     LuaFunctions.obj
 0002:000087ac       ??_C@_0O@DIEDNKLC@Set_Alternate?$AA@ 110b17ac     LuaFunctions.obj
 0002:000087bc       ??_C@_0BB@PHNHDOPH@Disable_Enlisted?$AA@ 110b17bc     LuaFunctions.obj
 0002:000087d0       ??_C@_0P@OPFAELMP@Disable_Preset?$AA@ 110b17d0     LuaFunctions.obj
 0002:000087e0       ??_C@_0BJ@IGHKLGLE@Disable_Enlisted_By_Name?$AA@ 110b17e0     LuaFunctions.obj
 0002:000087fc       ??_C@_0BH@DNCHPJND@Disable_Preset_By_Name?$AA@ 110b17fc     LuaFunctions.obj
 0002:00008814       ??_C@_0BM@MJBMFDDA@Disable_All_Ground_Vehicles?$AA@ 110b1814     LuaFunctions.obj
 0002:00008830       ??_C@_0BM@OHEKELGB@Disable_All_Flying_Vehicles?$AA@ 110b1830     LuaFunctions.obj
 0002:0000884c       ??_C@_0O@LMJAFMDH@Get_Team_Icon?$AA@ 110b184c     LuaFunctions.obj
 0002:0000885c       ??_C@_08BKHEMNLL@Get_Icon?$AA@ 110b185c     LuaFunctions.obj
 0002:00008868       ??_C@_0O@KJEKGOFJ@Remove_Script?$AA@ 110b1868     LuaFunctions.obj
 0002:00008878       ??_C@_0BD@MADIJJLM@Remove_All_Scripts?$AA@ 110b1878     LuaFunctions.obj
 0002:0000888c       ??_C@_0BF@OJHPLBNC@Attach_Script_Preset?$AA@ 110b188c     LuaFunctions.obj
 0002:000088a4       ??_C@_0BD@GBKKAEHP@Attach_Script_Type?$AA@ 110b18a4     LuaFunctions.obj
 0002:000088b8       ??_C@_0BF@GCLNDCEI@Remove_Script_Preset?$AA@ 110b18b8     LuaFunctions.obj
 0002:000088d0       ??_C@_0BD@IGDFOJLB@Remove_Script_Type?$AA@ 110b18d0     LuaFunctions.obj
 0002:000088e4       ??_C@_0BD@FOCNJNPB@Is_Script_Attached?$AA@ 110b18e4     LuaFunctions.obj
 0002:000088f8       ??_C@_0BD@KFDENAOD@Attach_Script_Once?$AA@ 110b18f8     LuaFunctions.obj
 0002:0000890c       ??_C@_0BK@CIHDHNBP@Attach_Script_Preset_Once?$AA@ 110b190c     LuaFunctions.obj
 0002:00008928       ??_C@_0BI@PCHAHNAI@Attach_Script_Type_Once?$AA@ 110b1928     LuaFunctions.obj
 0002:00008940       ??_C@_0BH@EFFNMJJE@Attach_Script_Building?$AA@ 110b1940     LuaFunctions.obj
 0002:00008958       ??_C@_0BI@KKGHPGGM@Attach_Script_Is_Preset?$AA@ 110b1958     LuaFunctions.obj
 0002:00008970       ??_C@_0BG@HOPLOFDL@Attach_Script_Is_Type?$AA@ 110b1970     LuaFunctions.obj
 0002:00008988       ??_C@_0BK@CLOGINAM@Attach_Script_Player_Once?$AA@ 110b1988     LuaFunctions.obj
 0002:000089a4       ??_C@_0BI@OMEFGCBM@Remove_Duplicate_Script?$AA@ 110b19a4     LuaFunctions.obj
 0002:000089bc       ??_C@_0CB@EMCAIIDE@Attach_Script_All_Buildings_Team@ 110b19bc     LuaFunctions.obj
 0002:000089e0       ??_C@_0BP@HDCBLIED@Attach_Script_All_Turrets_Team?$AA@ 110b19e0     LuaFunctions.obj
 0002:00008a00       ??_C@_0BK@KMLIDHPM@Find_Building_With_Script?$AA@ 110b1a00     LuaFunctions.obj
 0002:00008a1c       ??_C@_0BI@NGKNKGEH@Find_Object_With_Script?$AA@ 110b1a1c     LuaFunctions.obj
 0002:00008a34       ??_C@_0BG@PHJAAPBJ@Get_Translated_String?$AA@ 110b1a34     LuaFunctions.obj
 0002:00008a4c       ??_C@_0BL@DKJCPBBK@Get_Translated_Preset_Name?$AA@ 110b1a4c     LuaFunctions.obj
 0002:00008a68       ??_C@_0BG@BBAENOAN@Get_Translated_Weapon?$AA@ 110b1a68     LuaFunctions.obj
 0002:00008a80       ??_C@_0BO@HMCHEDAL@Get_Current_Translated_Weapon?$AA@ 110b1a80     LuaFunctions.obj
 0002:00008aa0       ??_C@_0O@EEMJEFAJ@Get_Team_Name?$AA@ 110b1aa0     LuaFunctions.obj
 0002:00008ab0       ??_C@_0BB@NBDIEMJB@Get_Vehicle_Name?$AA@ 110b1ab0     LuaFunctions.obj
 0002:00008ac4       ??_C@_0BP@OJBHDPGJ@Get_Translated_Definition_Name?$AA@ 110b1ac4     LuaFunctions.obj
 0002:00008ae4       ??_C@_0BE@JBBFOOPB@Get_Current_Bullets?$AA@ 110b1ae4     LuaFunctions.obj
 0002:00008af8       ??_C@_0BJ@NCCKMLID@Get_Current_Clip_Bullets?$AA@ 110b1af8     LuaFunctions.obj
 0002:00008b14       ??_C@_0BK@HAPEIEHF@Get_Current_Total_Bullets?$AA@ 110b1b14     LuaFunctions.obj
 0002:00008b30       ??_C@_0BC@PPEGHJDL@Get_Total_Bullets?$AA@ 110b1b30     LuaFunctions.obj
 0002:00008b44       ??_C@_0BB@FEJHKFP@Get_Clip_Bullets?$AA@ 110b1b44     LuaFunctions.obj
 0002:00008b58       ??_C@_0M@BOBFHECJ@Get_Bullets?$AA@ 110b1b58     LuaFunctions.obj
 0002:00008b64       ??_C@_0BI@NIMNJLGC@Get_Current_Max_Bullets?$AA@ 110b1b64     LuaFunctions.obj
 0002:00008b7c       ??_C@_0BN@JAHGENGI@Get_Current_Clip_Max_Bullets?$AA@ 110b1b7c     LuaFunctions.obj
 0002:00008b9c       ??_C@_0BO@GPNOOELL@Get_Current_Total_Max_Bullets?$AA@ 110b1b9c     LuaFunctions.obj
 0002:00008bbc       ??_C@_0BG@CLLMDFBI@Get_Max_Total_Bullets?$AA@ 110b1bbc     LuaFunctions.obj
 0002:00008bd4       ??_C@_0BF@EEDFLLDM@Get_Max_Clip_Bullets?$AA@ 110b1bd4     LuaFunctions.obj
 0002:00008bec       ??_C@_0BA@LGKOKJID@Get_Max_Bullets?$AA@ 110b1bec     LuaFunctions.obj
 0002:00008bfc       ??_C@_0BL@INDBFGAN@Get_Position_Total_Bullets?$AA@ 110b1bfc     LuaFunctions.obj
 0002:00008c18       ??_C@_0BF@NPMDDJHL@Get_Position_Bullets?$AA@ 110b1c18     LuaFunctions.obj
 0002:00008c30       ??_C@_0BK@HFABMJJJ@Get_Position_Clip_Bullets?$AA@ 110b1c30     LuaFunctions.obj
 0002:00008c4c       ??_C@_0BP@DKNJCADM@Get_Position_Total_Max_Bullets?$AA@ 110b1c4c     LuaFunctions.obj
 0002:00008c6c       ??_C@_0BJ@JEOJOAIG@Get_Position_Max_Bullets?$AA@ 110b1c6c     LuaFunctions.obj
 0002:00008c88       ??_C@_0BO@JCJEOFNP@Get_Position_Clip_Max_Bullets?$AA@ 110b1c88     LuaFunctions.obj
 0002:00008ca8       ??_C@_0BE@DPDOKOIN@Set_Current_Bullets?$AA@ 110b1ca8     LuaFunctions.obj
 0002:00008cbc       ??_C@_0BJ@HBIAKGBG@Set_Current_Clip_Bullets?$AA@ 110b1cbc     LuaFunctions.obj
 0002:00008cd8       ??_C@_0BF@IGNOCPCM@Set_Position_Bullets?$AA@ 110b1cd8     LuaFunctions.obj
 0002:00008cf0       ??_C@_0BK@PFMHAEDP@Set_Position_Clip_Bullets?$AA@ 110b1cf0     LuaFunctions.obj
 0002:00008d0c       ??_C@_0M@BBALKCKK@Set_Bullets?$AA@ 110b1d0c     LuaFunctions.obj
 0002:00008d18       ??_C@_0BB@GBBAMEON@Set_Clip_Bullets?$AA@ 110b1d18     LuaFunctions.obj
 0002:00008d2c       ??_C@_0BD@FAABPKFL@Get_Powerup_Weapon?$AA@ 110b1d2c     LuaFunctions.obj
 0002:00008d40       ??_C@_0BK@LNHMPEAB@Get_Powerup_Weapon_By_Obj?$AA@ 110b1d40     LuaFunctions.obj
 0002:00008d5c       ??_C@_0BJ@NLAFMLAB@Get_Current_Weapon_Style?$AA@ 110b1d5c     LuaFunctions.obj
 0002:00008d78       ??_C@_0O@FALGNADJ@Disarm_Beacon?$AA@ 110b1d78     LuaFunctions.obj
 0002:00008d88       ??_C@_0P@FLEHBEON@Disarm_Beacons?$AA@ 110b1d88     LuaFunctions.obj
 0002:00008d98       ??_C@_0BG@LIKGGLDF@Disarm_Nearest_Beacon?$AA@ 110b1d98     LuaFunctions.obj
 0002:00008db0       ??_C@_09JCKBGCC@Disarm_C4?$AA@ 110b1db0     LuaFunctions.obj
 0002:00008dbc       ??_C@_0BE@IJFEKKMH@Disarm_All_Proxy_C4?$AA@ 110b1dbc     LuaFunctions.obj
 0002:00008dd0       ??_C@_0O@HFDPBCJO@Disarm_All_C4?$AA@ 110b1dd0     LuaFunctions.obj
 0002:00008de0       ??_C@_0BD@NBFLKEKB@Get_Current_Weapon?$AA@ 110b1de0     LuaFunctions.obj
 0002:00008df4       ??_C@_0BB@CALJGBD@Get_Weapon_Count?$AA@ 110b1df4     LuaFunctions.obj
 0002:00008e08       ??_C@_0L@LEFPIDHN@Get_Weapon?$AA@ 110b1e08     LuaFunctions.obj
 0002:00008e14       ??_C@_0L@EKCNLKAI@Has_Weapon?$AA@ 110b1e14     LuaFunctions.obj
 0002:00008e20       ??_C@_0M@IMNDLAKB@Find_Beacon?$AA@ 110b1e20     LuaFunctions.obj
 0002:00008e2c       ??_C@_0N@HCDAKABB@Get_C4_Count?$AA@ 110b1e2c     LuaFunctions.obj
 0002:00008e3c       ??_C@_0BB@GHLKLJDB@Get_Beacon_Count?$AA@ 110b1e3c     LuaFunctions.obj
 0002:00008e50       ??_C@_0P@IFLCBABJ@Get_Mine_Limit?$AA@ 110b1e50     LuaFunctions.obj
 0002:00008e60       ??_C@_0M@CBIPIPAO@Get_C4_Mode?$AA@ 110b1e60     LuaFunctions.obj
 0002:00008e6c       ??_C@_0BH@CNMLMFDD@Get_C4_Count_Proximity?$AA@ 110b1e6c     LuaFunctions.obj
 0002:00008e84       ??_C@_0BE@JBECNKNP@Get_C4_Count_Remote?$AA@ 110b1e84     LuaFunctions.obj
 0002:00008e98       ??_C@_0P@INIBIMKP@Get_C4_Planter?$AA@ 110b1e98     LuaFunctions.obj
 0002:00008ea8       ??_C@_0BA@KOODMKPM@Get_C4_Attached?$AA@ 110b1ea8     LuaFunctions.obj
 0002:00008eb8       ??_C@_0BD@HMGOBFEH@Get_Beacon_Planter?$AA@ 110b1eb8     LuaFunctions.obj
 0002:00008ecc       ??_C@_0O@KEAIMFMJ@Create_Object?$AA@ 110b1ecc     LuaFunctions.obj
 0002:00008edc       ??_C@_0P@DPMEIDDP@Destroy_Object?$AA@ 110b1edc     LuaFunctions.obj
 0002:00008eec       ??_C@_0BA@EJLOEPFH@Get_Preset_Name?$AA@ 110b1eec     LuaFunctions.obj
 0002:00008efc       ??_C@_0N@PNALJKNF@Get_Position?$AA@ 110b1efc     LuaFunctions.obj
 0002:00008f0c       ??_C@_0BL@MCPFAOID@Enable_Vehicle_Transitions?$AA@ 110b1f0c     LuaFunctions.obj
 0002:00008f28       ??_C@_09DOJBNMAH@Set_Model?$AA@ 110b1f28     LuaFunctions.obj
 0002:00008f34       ??_C@_0O@DFNOCNOD@Goto_Location?$AA@ 110b1f34     LuaFunctions.obj
 0002:00008f44       ??_C@_0M@NKEEIFHL@Goto_Object?$AA@ 110b1f44     LuaFunctions.obj
 0002:00008f50       ??_C@_0BM@FKPINIKB@Disable_Physical_Collisions?$AA@ 110b1f50     LuaFunctions.obj
 0002:00008f6c       ??_C@_0BC@CCJHLIF@Enable_Collisions?$AA@ 110b1f6c     LuaFunctions.obj
 0002:00008f80       ??_C@_0BA@JAEIFIGI@Random_Building?$AA@ 110b1f80     LuaFunctions.obj
 0002:00008f90       ??_C@_0BA@OOAEGMLL@Get_Current_Map?$AA@ 110b1f90     LuaFunctions.obj
 0002:00008fa0       ??_C@_0N@PCBIGOOI@Get_Next_Map?$AA@ 110b1fa0     LuaFunctions.obj
 0002:00008fb0       ??_C@_0N@IJLFFGJJ@Set_Position?$AA@ 110b1fb0     LuaFunctions.obj
 0002:00008fc0       ??_C@_0N@JFODLOAG@Apply_Damage?$AA@ 110b1fc0     LuaFunctions.obj
 0002:00008fd0       ??_C@_0L@GJLGMMBK@Get_Facing?$AA@ 110b1fd0     LuaFunctions.obj
 0002:00008fdc       ??_C@_0L@HHJJHLFD@Set_Facing?$AA@ 110b1fdc     LuaFunctions.obj
 0002:00008fe8       ??_C@_0L@GFDJBAIP@Set_Clouds?$AA@ 110b1fe8     LuaFunctions.obj
 0002:00008ff4       ??_C@_07GKDBKIMC@Set_Ash?$AA@ 110b1ff4     LuaFunctions.obj
 0002:00008ffc       ??_C@_08FCOMMMGM@Set_Rain?$AA@ 110b1ffc     LuaFunctions.obj
 0002:00009008       ??_C@_08KIGCCACA@Set_Snow?$AA@ 110b2008     LuaFunctions.obj
 0002:00009014       ??_C@_08KABIJFPM@Set_Wind?$AA@ 110b2014     LuaFunctions.obj
 0002:00009020       ??_C@_0O@CJAHFJCB@Attach_Script?$AA@ 110b2020     LuaFunctions.obj
 0002:00009030       ??_C@_0BG@CEKOMAHB@Create_Object_At_Bone?$AA@ 110b2030     LuaFunctions.obj
 0002:00009048       ??_C@_0BG@JJMIAMIJ@Attach_To_Object_Bone?$AA@ 110b2048     LuaFunctions.obj
 0002:00009060       ??_C@_0BD@KHFLAMAN@Display_Health_Bar?$AA@ 110b2060     LuaFunctions.obj
 0002:00009074       ??_C@_0BD@DPPGDEGD@Create_Script_Zone?$AA@ 110b2074     LuaFunctions.obj
 0002:00009088       ??_C@_06MPGEJACK@Get_ID?$AA@ 110b2088     LuaFunctions.obj
 0002:00009090       ??_C@_06GHBGHH@tClock?$AA@ 110b2090     LuaFunctions.obj
 0002:00009098       ??_C@_06MICBDHBI@Invoke?$AA@ 110b2098     LuaFunctions.obj
 0002:000090a0       ??_C@_0BB@EOFLGPNH@GetTimeRemaining?$AA@ 110b20a0     LuaFunctions.obj
 0002:000090b4       ??_C@_0L@HJCPGMGK@Get_Health?$AA@ 110b20b4     LuaFunctions.obj
 0002:000090c0       ??_C@_0P@KFCNJDMH@Get_Max_Health?$AA@ 110b20c0     LuaFunctions.obj
 0002:000090d0       ??_C@_0BE@NJNKJGME@Get_Shield_Strength?$AA@ 110b20d0     LuaFunctions.obj
 0002:000090e4       ??_C@_0BI@BIBJDIOE@Get_Max_Shield_Strength?$AA@ 110b20e4     LuaFunctions.obj
 0002:000090fc       ??_C@_08INMFMEEK@LongToIP?$AA@ 110b20fc     LuaFunctions.obj
 0002:00009108       ??_C@_08IGGKJELH@IPToLong?$AA@ 110b2108     LuaFunctions.obj
 0002:00009114       ??_C@_09OLKEFJMF@Is_A_Star?$AA@ 110b2114     LuaFunctions.obj
 0002:00009120       ??_C@_0P@PBDIPOPG@Enable_Stealth?$AA@ 110b2120     LuaFunctions.obj
 0002:00009130       ??_C@_0N@PKAJAOLA@Get_Rotation?$AA@ 110b2130     LuaFunctions.obj
 0002:00009140       ??_C@_0BA@IKLOBAEC@Get_All_Players?$AA@ 110b2140     LuaFunctions.obj
 0002:00009150       ??_C@_0BB@EBHMJLLO@Get_All_Vehicles?$AA@ 110b2150     LuaFunctions.obj
 0002:00009164       ??_C@_0BC@CNFGLHJK@Get_All_Buildings?$AA@ 110b2164     LuaFunctions.obj
 0002:00009178       ??_C@_0BA@JBCLOBLG@Get_All_Objects?$AA@ 110b2178     LuaFunctions.obj
 0002:00009188       ??_C@_0CD@OALLDNCM@Display_Nod_Player_Terminal_Play@ 110b2188     LuaFunctions.obj
 0002:000091ac       ??_C@_0CD@KGANIHIM@Display_GDI_Player_Terminal_Play@ 110b21ac     LuaFunctions.obj
 0002:000091d0       ??_C@_0BD@ODKAOELM@Reload_All_Plugins?$AA@ 110b21d0     LuaFunctions.obj
 0002:000091e4       ??_C@_0BE@HHPBNGLI@Set_Shield_Strength?$AA@ 110b21e4     LuaFunctions.obj
 0002:000091f8       ??_C@_0L@GHAANLCD@Set_Health?$AA@ 110b21f8     LuaFunctions.obj
 0002:00009204       ??_C@_07HJCKACAM@cPlayer?$AA@ 110b2204     LuaFunctions.obj
 0002:0000920c       ??_C@_08CANMEKOL@The_Game?$AA@ 110b220c     LuaFunctions.obj
 0002:00009218       ??_C@_0M@FPPCACMJ@Set_cPlayer?$AA@ 110b2218     LuaFunctions.obj
 0002:00009224       ??_C@_0N@MLPEKENE@Set_The_Game?$AA@ 110b2224     LuaFunctions.obj
 0002:00009234       ??_C@_0M@KEOGBLFD@MemoryWrite?$AA@ 110b2234     LuaFunctions.obj
 0002:00009240       ??_C@_0L@ELPIAIAO@MemoryRead?$AA@ 110b2240     LuaFunctions.obj
 0002:0000924c       ??_C@_0BA@FGBLOPBB@Set_Shield_Type?$AA@ 110b224c     LuaFunctions.obj
 0002:0000925c       ??_C@_0DE@IEEDHFKJ@Bad?5argument?5?$CD1?5to?5Register_Scri@ 110b225c     LuaManager.obj
 0002:00009290       ??_C@_0DN@JPDPLOHD@You?5cannot?5register?5more?5than?5on@ 110b2290     LuaManager.obj
 0002:000092d0       ??_C@_0O@PMBICFNL@DestroyScript?$AA@ 110b22d0     LuaManager.obj
 0002:000092e0       ??_C@_0BE@ODIPCCMJ@Get_Float_Parameter?$AA@ 110b22e0     LuaManager.obj
 0002:000092f4       ??_C@_0BC@CBPCGHON@Get_Int_Parameter?$AA@ 110b22f4     LuaManager.obj
 0002:00009308       ??_C@_0BF@GKNOMPIJ@Get_String_Parameter?$AA@ 110b2308     LuaManager.obj
 0002:00009320       ??_C@_0M@FKHHAII@Start_Timer?$AA@ 110b2320     LuaManager.obj
 0002:0000932c       ??_C@_0BA@HDADLBLI@Register_Script?$AA@ 110b232c     LuaManager.obj
 0002:0000933c       ??_C@_07BBIDHECN@Created?$AA@ 110b233c     LuaManager.obj
 0002:00009344       ??_C@_09KDBKJCNL@Destroyed?$AA@ 110b2344     LuaManager.obj
 0002:00009350       ??_C@_06GJNLCKAP@Killed?$AA@ 110b2350     LuaManager.obj
 0002:00009358       ??_C@_07ODIPIBHL@Damaged?$AA@ 110b2358     LuaManager.obj
 0002:00009360       ??_C@_06IFGIOHDE@Custom?$AA@ 110b2360     LuaManager.obj
 0002:00009368       ??_C@_0L@ODFCGMOO@Enemy_Seen?$AA@ 110b2368     LuaManager.obj
 0002:00009374       ??_C@_0BA@LOBAOMBD@Action_Complete?$AA@ 110b2374     LuaManager.obj
 0002:00009384       ??_C@_0O@POONBLNB@Timer_Expired?$AA@ 110b2384     LuaManager.obj
 0002:00009394       ??_C@_0BD@OGGHBCHH@Animation_Complete?$AA@ 110b2394     LuaManager.obj
 0002:000093a8       ??_C@_05PKHLGBFN@Poked?$AA@ 110b23a8     LuaManager.obj
 0002:000093b0       ??_C@_07GPPDKDDC@Entered?$AA@ 110b23b0     LuaManager.obj
 0002:000093b8       ??_C@_06KMCDHAGM@Exited?$AA@ 110b23b8     LuaManager.obj
 0002:000093c0       ??_C@_0DH@JAPFGAIF@?$HM?9?9?9?9?9?9?9?9?9?9?9?9?9?9?9?9?9?9?9?9?9?9?9?9?9?9?9?9?9?9?9@ 110b23c0     LuaManager.obj
 0002:000093f8       ??_C@_0DH@BOBJNDFI@?$HM?5Lua?55?40?5Copyright?5?$CIC?$CJ?51994?9200@ 110b23f8     LuaManager.obj
 0002:00009430       ??_C@_0DH@IDMJHBPB@?$HM?5R?4?5Ierusalimschy?0?5L?4?5H?4?5de?5Fig@ 110b2430     LuaManager.obj
 0002:00009468       ??_C@_0DH@JIDGIEHA@?$HM?5www?4lua?4org?5?5?5?5?5?5?5?5?5?5?5?5?5?5?5?5?5?5?5@ 110b2468     LuaManager.obj
 0002:000094a0       ??_C@_0DH@IHAKMOMC@?$HM?5Embedded?5with?5scripts?4dll?5by?5j@ 110b24a0     LuaManager.obj
 0002:000094d8       ??_C@_0DH@DDHKAMMP@?$HM?5www?4dcomproductions?4com?5?5?5?5?5?5?5@ 110b24d8     LuaManager.obj
 0002:00009510       ??_C@_0BL@MGOOMGEF@Failed?5to?5load?5plugin?3?5?$CFs?6?$AA@ 110b2510     LuaManager.obj
 0002:0000952c       ??_C@_06FEOMBGJC@OnLoad?$AA@ 110b252c     LuaManager.obj
 0002:00009534       ??_C@_0BD@MKFIIKNH@Loaded?5plugin?3?5?$CFs?6?$AA@ 110b2534     LuaManager.obj
 0002:00009548       ??_C@_0BF@HGKBFGFL@Unloaded?5a?5lua?5file?6?$AA@ 110b2548     LuaManager.obj
 0002:00009560       ??_C@_07PCNKBAGB@OnError?$AA@ 110b2560     LuaManager.obj
 0002:00009568       ??_C@_0CD@FPAKOKNH@?$FLError?$FN?5Could?5not?5call?5OnError?6?$CF@ 110b2568     LuaManager.obj
 0002:0000958c       ??_C@_0M@HKGMOKHO@?$FLError?$FN?5?$CFs?6?$AA@ 110b258c     LuaManager.obj
 0002:00009598       ??_C@_08OJKMEPJJ@OnUnload?$AA@ 110b2598     LuaManager.obj
 0002:000095a4       ??_C@_06BKJKLKL@OnChat?$AA@ 110b25a4     LuaManager.obj
 0002:000095ac       ??_C@_0O@GFEJPEM@OnHostMessage?$AA@ 110b25ac     LuaManager.obj
 0002:000095bc       ??_C@_0N@LCGNLKMA@OnPlayerJoin?$AA@ 110b25bc     LuaManager.obj
 0002:000095cc       ??_C@_0O@MIDEBBHD@OnPlayerLeave?$AA@ 110b25cc     LuaManager.obj
 0002:000095dc       ??_C@_0O@JGODGMFJ@OnLevelLoaded?$AA@ 110b25dc     LuaManager.obj
 0002:000095ec       ??_C@_0L@MNOOMILJ@OnGameOver?$AA@ 110b25ec     LuaManager.obj
 0002:000095f8       ??_C@_0BA@DLHNMEPD@OnConsoleOutput?$AA@ 110b25f8     LuaManager.obj
 0002:00009608       ??_C@_0BA@DMFIGFNJ@OnPlayerVersion?$AA@ 110b2608     LuaManager.obj
 0002:00009618       ??_C@_0P@MNPPPPMA@OnObjectCreate?$AA@ 110b2618     LuaManager.obj
 0002:00009628       ??_C@_05HINKHOPP@OnDDE?$AA@ 110b2628     LuaManager.obj
 0002:00009630       ??_C@_07NNKFNMN@OnThink?$AA@ 110b2630     LuaManager.obj
 0002:00009638       ??_C@_0M@IPPLBPHG@Serial_Hook?$AA@ 110b2638     LuaManager.obj
 0002:00009644       ??_C@_0N@IMAAAIDF@Loading_Hook?$AA@ 110b2644     LuaManager.obj
 0002:00009654       ??_C@_0M@HJCIFMKO@Damage_Hook?$AA@ 110b2654     LuaManager.obj
 0002:00009660       ??_C@_09ONENJGFC@Ping_Hook?$AA@ 110b2660     LuaManager.obj
 0002:0000966c       ??_C@_0N@KHBIIJJK@Suicide_Hook?$AA@ 110b266c     LuaManager.obj
 0002:0000967c       ??_C@_0L@KMGGCAC@Radio_Hook?$AA@ 110b267c     LuaManager.obj
 0002:00009688       ??_C@_0DB@MMHCKAAL@Error?5starting?5winsock?0?5LuaSocke@ 110b2688     LuaManager.obj
 0002:000096bc       ??_C@_06PJIGMIJB@Client?$AA@ 110b26bc     LuaManager.obj
 0002:000096c4       ??_C@_06MDEHPNLG@Accept?$AA@ 110b26c4     LuaManager.obj
 0002:000096cc       ??_C@_04EEACDIHB@Recv?$AA@ 110b26cc     LuaManager.obj
 0002:000096d4       ??_C@_04JEOPCEB@Send?$AA@  110b26d4     LuaManager.obj
 0002:000096dc       ??_C@_0O@PCHFMMEO@DataAvaliable?$AA@ 110b26dc     LuaManager.obj
 0002:000096ec       ??_C@_0O@OJMPLJO@ClientWaiting?$AA@ 110b26ec     LuaManager.obj
 0002:000096fc       ??_C@_0L@CMGJAGDM@Disconnect?$AA@ 110b26fc     LuaManager.obj
 0002:00009708       ??_C@_06GPFPJJPN@Upload?$AA@ 110b2708     LuaManager.obj
 0002:00009710       ??_C@_0N@JKDNJMII@Check_Upload?$AA@ 110b2710     LuaManager.obj
 0002:00009720       ??_C@_0BD@ICHOAPKO@Check_Upload_Error?$AA@ 110b2720     LuaManager.obj
 0002:00009734       ??_C@_03CBKFDHDL@Lua?$AA@  110b2734     LuaManager.obj
 0002:00009738       ??_C@_0CH@FPIIMIAC@There?5is?5already?5an?5upload?5in?5pr@ 110b2738     LuaManager.obj
 0002:00009760       ??_C@_0CL@PMBKKHCB@Bad?5argument?5?$CD1?5to?5Upload?4?5Expec@ 110b2760     LuaManager.obj
 0002:0000978c       ??_C@_04CPPPJGME@Host?$AA@ 110b278c     LuaManager.obj
 0002:00009794       ??_C@_0DI@FONLCJCF@Bad?5table?5passed?5to?5Upload?4?5Fiel@ 110b2794     LuaManager.obj
 0002:000097cc       ??_C@_0DI@OHCPLCOH@Bad?5table?5passed?5to?5Upload?4?5Fiel@ 110b27cc     LuaManager.obj
 0002:00009804       ??_C@_09NPGAKJDM@LocalFile?$AA@ 110b2804     LuaManager.obj
 0002:00009810       ??_C@_0DN@OGBDGGAA@Bad?5table?5passed?5to?5Upload?4?5Fiel@ 110b2810     LuaManager.obj
 0002:00009850       ??_C@_0L@KPEHODDB@RemoteFile?$AA@ 110b2850     LuaManager.obj
 0002:0000985c       ??_C@_0DO@BKBBFPDH@Bad?5table?5passed?5to?5Upload?4?5Fiel@ 110b285c     LuaManager.obj
 0002:0000989c       ??_C@_08GBJFCIEI@Username?$AA@ 110b289c     LuaManager.obj
 0002:000098a8       ??_C@_0DM@JEAEJMOL@Bad?5table?5passed?5to?5Upload?4?5Fiel@ 110b28a8     LuaManager.obj
 0002:000098e4       ??_C@_0DM@MAEJKNJM@Bad?5table?5passed?5to?5Upload?4?5Fiel@ 110b28e4     LuaManager.obj
 0002:00009924       ??_7LuaScript@LuaScriptManager@@6B@ 110b2924     LuaManager.obj
 0002:00009990       ??_7?$ScriptRegistrant@VLuaScript@LuaScriptManager@@@@6B@ 110b2990     LuaManager.obj
 0002:00009998       ??_C@_09PFCHIMEP@127?40?40?41?$AA@ 110b2998     Misc.obj
 0002:000099a4       ??_C@_0BH@CCGEKEGO@no?5calling?5environment?$AA@ 110b29a4     lapi.obj
 0002:000099bc       ??_C@_08JEIPHCP@no?5value?$AA@ 110b29bc     lapi.obj
 0002:000099c8       ??_C@_01OGPIMHDM@?$DP?$AA@ 110b29c8     lapi.obj
 0002:000099cc       ??_C@_0BG@CHJGEHJL@bad?5argument?5?$CD?$CFd?5?$CI?$CFs?$CJ?$AA@ 110b29cc     lauxlib.obj
 0002:000099e4       ??_C@_01EFFIKLCJ@n?$AA@    110b29e4     lauxlib.obj
 0002:000099e8       ??_C@_06GABBCIBA@method?$AA@ 110b29e8     lauxlib.obj
 0002:000099f0       ??_C@_0BO@LENGMNDF@calling?5?8?$CFs?8?5on?5bad?5self?5?$CI?$CFs?$CJ?$AA@ 110b29f0     lauxlib.obj
 0002:00009a10       ??_C@_0BO@GOMKJOAH@bad?5argument?5?$CD?$CFd?5to?5?8?$CFs?8?5?$CI?$CFs?$CJ?$AA@ 110b2a10     lauxlib.obj
 0002:00009a30       ??_C@_0BE@LDJANOJE@?$CFs?5expected?0?5got?5?$CFs?$AA@ 110b2a30     lauxlib.obj
 0002:00009a44       ??_C@_02KHAMJCKP@Sl?$AA@   110b2a44     lauxlib.obj
 0002:00009a48       ??_C@_07FCDHCGBN@?$CFs?3?$CFd?3?5?$AA@ 110b2a48     lauxlib.obj
 0002:00009a50       ??_C@_0BE@HBADPNMP@invalid?5option?5?8?$CFs?8?$AA@ 110b2a50     lauxlib.obj
 0002:00009a64       ??_C@_0BE@CBBDHBEP@stack?5overflow?5?$CI?$CFs?$CJ?$AA@ 110b2a64     lauxlib.obj
 0002:00009a78       ??_C@_0P@PDHEKNMA@value?5expected?$AA@ 110b2a78     lauxlib.obj
 0002:00009a88       ??_C@_07PINPBNPB@_LOADED?$AA@ 110b2a88     lauxlib.obj
 0002:00009a90       ??_C@_0BO@CBJIAGLF@name?5conflict?5for?5module?5?8?$CFs?8?$AA@ 110b2a90     lauxlib.obj
 0002:00009ab0       ??_C@_01EEMJAFIK@?6?$AA@   110b2ab0     lauxlib.obj
 0002:00009ab4       ??_C@_0BB@BJDGDOHH@cannot?5?$CFs?5?$CFs?3?5?$CFs?$AA@ 110b2ab4     lauxlib.obj
 0002:00009ac8       ??_C@_06CCPPALKB@?$DNstdin?$AA@ 110b2ac8     lauxlib.obj
 0002:00009ad0       ??_C@_03HPDLNGOA@?$EA?$CFs?$AA@ 110b2ad0     lauxlib.obj
 0002:00009ad4       ??_C@_01KDCPPGHE@r?$AA@    110b2ad4     lauxlib.obj
 0002:00009ad8       ??_C@_04PMOCAHAA@open?$AA@ 110b2ad8     lauxlib.obj
 0002:00009ae0       ??_C@_02JDPG@rb?$AA@       110b2ae0     lauxlib.obj
 0002:00009ae4       ??_C@_06IEGCHAII@reopen?$AA@ 110b2ae4     lauxlib.obj
 0002:00009aec       ??_C@_04POLDLDMI@read?$AA@ 110b2aec     lauxlib.obj
 0002:00009af4       ??_C@_0DC@EFOPIIKP@PANIC?3?5unprotected?5error?5in?5call@ 110b2af4     lauxlib.obj
 0002:00009b28       ??_C@_05LKJGIMLP@yield?$AA@ 110b2b28     lbaselib.obj
 0002:00009b30       ??_C@_04NFDDIEML@wrap?$AA@ 110b2b30     lbaselib.obj
 0002:00009b38       ??_C@_06DJIHEMFI@status?$AA@ 110b2b38     lbaselib.obj
 0002:00009b40       ??_C@_06PLELHCEK@resume?$AA@ 110b2b40     lbaselib.obj
 0002:00009b48       ??_C@_06HBNONAG@create?$AA@ 110b2b48     lbaselib.obj
 0002:00009b50       ??_C@_04BBBDNBOK@dead?$AA@ 110b2b50     lbaselib.obj
 0002:00009b58       ??_C@_06IKLLLDHL@normal?$AA@ 110b2b58     lbaselib.obj
 0002:00009b60       ??_C@_09PAHKPJCJ@suspended?$AA@ 110b2b60     lbaselib.obj
 0002:00009b6c       ??_C@_07PANPENDC@running?$AA@ 110b2b6c     lbaselib.obj
 0002:00009b74       ??_C@_06GDLLDIBI@xpcall?$AA@ 110b2b74     lbaselib.obj
 0002:00009b7c       ??_C@_06FIONAGJL@unpack?$AA@ 110b2b7c     lbaselib.obj
 0002:00009b84       ??_C@_04GPMDFGEJ@type?$AA@ 110b2b84     lbaselib.obj
 0002:00009b8c       ??_C@_08JOIMPOJO@tonumber?$AA@ 110b2b8c     lbaselib.obj
 0002:00009b98       ??_C@_0N@MCAAIDEK@setmetatable?$AA@ 110b2b98     lbaselib.obj
 0002:00009ba8       ??_C@_07NAJJCHPG@setfenv?$AA@ 110b2ba8     lbaselib.obj
 0002:00009bb0       ??_C@_06LGNCCACI@select?$AA@ 110b2bb0     lbaselib.obj
 0002:00009bb8       ??_C@_06ONPLLLOI@rawset?$AA@ 110b2bb8     lbaselib.obj
 0002:00009bc0       ??_C@_06DCIAHLCA@rawget?$AA@ 110b2bc0     lbaselib.obj
 0002:00009bc8       ??_C@_08LCBKMMAG@rawequal?$AA@ 110b2bc8     lbaselib.obj
 0002:00009bd4       ??_C@_05IJDJACGD@print?$AA@ 110b2bd4     lbaselib.obj
 0002:00009bdc       ??_C@_05JAJCNIIJ@pcall?$AA@ 110b2bdc     lbaselib.obj
 0002:00009be4       ??_C@_04CJGEDOF@next?$AA@  110b2be4     lbaselib.obj
 0002:00009bec       ??_C@_0L@BBBJLLLK@loadstring?$AA@ 110b2bec     lbaselib.obj
 0002:00009bf8       ??_C@_04EONOHKEP@load?$AA@ 110b2bf8     lbaselib.obj
 0002:00009c00       ??_C@_08BNNFLGCJ@loadfile?$AA@ 110b2c00     lbaselib.obj
 0002:00009c0c       ??_C@_0N@LGLOEPAG@getmetatable?$AA@ 110b2c0c     lbaselib.obj
 0002:00009c1c       ??_C@_07CIGIBICH@getfenv?$AA@ 110b2c1c     lbaselib.obj
 0002:00009c24       ??_C@_06EDAGHKOI@gcinfo?$AA@ 110b2c24     lbaselib.obj
 0002:00009c2c       ??_C@_05KKCIMGE@error?$AA@ 110b2c2c     lbaselib.obj
 0002:00009c34       ??_C@_06ONNDGCDK@dofile?$AA@ 110b2c34     lbaselib.obj
 0002:00009c3c       ??_C@_0P@CKFEAJJE@collectgarbage?$AA@ 110b2c3c     lbaselib.obj
 0002:00009c4c       ??_C@_06GMEIIFFN@assert?$AA@ 110b2c4c     lbaselib.obj
 0002:00009c54       ??_C@_0L@KABEJKKP@setstepmul?$AA@ 110b2c54     lbaselib.obj
 0002:00009c60       ??_C@_08ONFIAENP@setpause?$AA@ 110b2c60     lbaselib.obj
 0002:00009c6c       ??_C@_04CNBNFAL@step?$AA@  110b2c6c     lbaselib.obj
 0002:00009c74       ??_C@_05IOMEMJEC@count?$AA@ 110b2c74     lbaselib.obj
 0002:00009c7c       ??_C@_07JHIJCABF@collect?$AA@ 110b2c7c     lbaselib.obj
 0002:00009c84       ??_C@_07LDHOHMPD@restart?$AA@ 110b2c84     lbaselib.obj
 0002:00009c8c       ??_C@_04PEGFANN@stop?$AA@  110b2c8c     lbaselib.obj
 0002:00009c94       ??_C@_08FNIIFOJC@tostring?$AA@ 110b2c94     lbaselib.obj
 0002:00009ca0       ??_C@_0CL@KMHHCBJA@?8tostring?8?5must?5return?5a?5string?5@ 110b2ca0     lbaselib.obj
 0002:00009ccc       ??_C@_01GPOEFGEJ@?7?$AA@   110b2ccc     lbaselib.obj
 0002:00009cd0       ??_C@_0BC@GGLHLOMM@base?5out?5of?5range?$AA@ 110b2cd0     lbaselib.obj
 0002:00009ce4       ??_C@_0BG@HDIIKINN@nil?5or?5table?5expected?$AA@ 110b2ce4     lbaselib.obj
 0002:00009cfc       ??_C@_0CE@LJKICCEL@cannot?5change?5a?5protected?5metata@ 110b2cfc     lbaselib.obj
 0002:00009d20       ??_C@_0BL@NGAFCBHD@level?5must?5be?5non?9negative?$AA@ 110b2d20     lbaselib.obj
 0002:00009d3c       ??_C@_0O@OFBEOMLD@invalid?5level?$AA@ 110b2d3c     lbaselib.obj
 0002:00009d4c       ??_C@_01INIBCBCB@f?$AA@    110b2d4c     lbaselib.obj
 0002:00009d50       ??_C@_0DC@LPPOGBD@no?5function?5environment?5for?5tail@ 110b2d50     lbaselib.obj
 0002:00009d84       ??_C@_0DE@PIGGMBA@?8setfenv?8?5cannot?5change?5environm@ 110b2d84     lbaselib.obj
 0002:00009db8       ??_C@_0BK@NJPFPDBN@too?5many?5nested?5functions?$AA@ 110b2db8     lbaselib.obj
 0002:00009dd4       ??_C@_0CF@IPNALDCD@reader?5function?5must?5return?5a?5st@ 110b2dd4     lbaselib.obj
 0002:00009dfc       ??_C@_07JEBBFCAN@?$DN?$CIload?$CJ?$AA@ 110b2dfc     lbaselib.obj
 0002:00009e04       ??_C@_0BC@ONMFJPBH@assertion?5failed?$CB?$AA@ 110b2e04     lbaselib.obj
 0002:00009e18       ??_C@_02DKCKIIND@?$CFs?$AA@ 110b2e18     lbaselib.obj
 0002:00009e1c       ??_C@_0BL@EDBCOFHM@too?5many?5results?5to?5unpack?$AA@ 110b2e1c     lbaselib.obj
 0002:00009e38       ??_C@_0BD@ILOGJALA@index?5out?5of?5range?$AA@ 110b2e38     lbaselib.obj
 0002:00009e4c       ??_C@_0L@HDFPAPPH@__tostring?$AA@ 110b2e4c     lbaselib.obj
 0002:00009e58       ??_C@_03ILAMHENH@nil?$AA@  110b2e58     lbaselib.obj
 0002:00009e5c       ??_C@_06CILKLLDB@?$CFs?3?5?$CFp?$AA@ 110b2e5c     lbaselib.obj
 0002:00009e64       ??_C@_0BK@OMPDBBEM@boolean?5or?5proxy?5expected?$AA@ 110b2e64     lbaselib.obj
 0002:00009e80       ??_C@_0BD@LDCLGBHF@coroutine?5expected?$AA@ 110b2e80     lbaselib.obj
 0002:00009e94       ??_C@_0BN@CLPLGDGN@too?5many?5arguments?5to?5resume?$AA@ 110b2e94     lbaselib.obj
 0002:00009eb4       ??_C@_0BL@DGCALGPK@cannot?5resume?5?$CFs?5coroutine?$AA@ 110b2eb4     lbaselib.obj
 0002:00009ed0       ??_C@_0BL@OALEJBKN@too?5many?5results?5to?5resume?$AA@ 110b2ed0     lbaselib.obj
 0002:00009eec       ??_C@_0BG@EHJAKGKG@Lua?5function?5expected?$AA@ 110b2eec     lbaselib.obj
 0002:00009f04       ??_C@_02NIGGJGKC@_G?$AA@   110b2f04     lbaselib.obj
 0002:00009f08       ??_C@_07GLKNJPII@Lua?55?41?$AA@ 110b2f08     lbaselib.obj
 0002:00009f10       ??_C@_08PMLCGGEP@_VERSION?$AA@ 110b2f10     lbaselib.obj
 0002:00009f1c       ??_C@_06MGIEFEAJ@ipairs?$AA@ 110b2f1c     lbaselib.obj
 0002:00009f24       ??_C@_05PEAECDOC@pairs?$AA@ 110b2f24     lbaselib.obj
 0002:00009f2c       ??_C@_02DNFJNMFM@kv?$AA@   110b2f2c     lbaselib.obj
 0002:00009f30       ??_C@_06BPGFKLEK@__mode?$AA@ 110b2f30     lbaselib.obj
 0002:00009f38       ??_C@_08HDPJFDHB@newproxy?$AA@ 110b2f38     lbaselib.obj
 0002:00009f44       ??_C@_09HNKENHFC@coroutine?$AA@ 110b2f44     lbaselib.obj
 0002:00009f50       ??_C@_0BL@BDOLDOFI@control?5structure?5too?5long?$AA@ 110b2f50     lcode.obj
 0002:00009f6c       ??_C@_0CD@HGHHKJGL@function?5or?5expression?5too?5compl@ 110b2f6c     lcode.obj
 0002:00009f90       ??_C@_0BI@DGLMJHJB@constant?5table?5overflow?$AA@ 110b2f90     lcode.obj
 0002:00009fa8       ??_C@_0BD@LKJEPOHE@code?5size?5overflow?$AA@ 110b2fa8     lcode.obj
 0002:00009fbc       ??_C@_09GPFEECNC@traceback?$AA@ 110b2fbc     ldblib.obj
 0002:00009fc8       ??_C@_0L@CDIIKFBA@setupvalue?$AA@ 110b2fc8     ldblib.obj
 0002:00009fd4       ??_C@_08JNGOLMEK@setlocal?$AA@ 110b2fd4     ldblib.obj
 0002:00009fe0       ??_C@_07POLKHPNI@sethook?$AA@ 110b2fe0     ldblib.obj
 0002:00009fe8       ??_C@_0L@DNKHBCFJ@getupvalue?$AA@ 110b2fe8     ldblib.obj
 0002:00009ff4       ??_C@_0M@NCNCBJKP@getregistry?$AA@ 110b2ff4     ldblib.obj
 0002:0000a000       ??_C@_08GMECKPDH@getlocal?$AA@ 110b3000     ldblib.obj
 0002:0000a00c       ??_C@_07OICKPAFH@getinfo?$AA@ 110b300c     ldblib.obj
 0002:0000a014       ??_C@_07GELEAAJ@gethook?$AA@ 110b3014     ldblib.obj
 0002:0000a01c       ??_C@_05GFCDIDHO@debug?$AA@ 110b301c     ldblib.obj
 0002:0000a024       ??_C@_0M@IDJJEGOC@tail?5return?$AA@ 110b3024     ldblib.obj
 0002:0000a030       ??_C@_04HJPCFDOP@line?$AA@ 110b3030     ldblib.obj
 0002:0000a038       ??_C@_06LNOFJDNM@return?$AA@ 110b3038     ldblib.obj
 0002:0000a040       ??_C@_04OMFAIDPG@call?$AA@ 110b3040     ldblib.obj
 0002:0000a048       ??_C@_05CLBJLFDN@flnSu?$AA@ 110b3048     ldblib.obj
 0002:0000a050       ??_C@_03PENLABEP@?$DO?$CFs?$AA@ 110b3050     ldblib.obj
 0002:0000a054       ??_C@_0BL@NMONLLHA@function?5or?5level?5expected?$AA@ 110b3054     ldblib.obj
 0002:0000a070       ??_C@_0P@PJFAGLMH@invalid?5option?$AA@ 110b3070     ldblib.obj
 0002:0000a080       ??_C@_06OEKOLKIL@source?$AA@ 110b3080     ldblib.obj
 0002:0000a088       ??_C@_09NOFDGFFO@short_src?$AA@ 110b3088     ldblib.obj
 0002:0000a094       ??_C@_0M@IOFFDKM@linedefined?$AA@ 110b3094     ldblib.obj
 0002:0000a0a0       ??_C@_0BA@BGGOJOFO@lastlinedefined?$AA@ 110b30a0     ldblib.obj
 0002:0000a0b0       ??_C@_04IOPLPGDE@what?$AA@ 110b30b0     ldblib.obj
 0002:0000a0b8       ??_C@_0M@OLGEEKJC@currentline?$AA@ 110b30b8     ldblib.obj
 0002:0000a0c4       ??_C@_04BDNNNDAF@nups?$AA@ 110b30c4     ldblib.obj
 0002:0000a0cc       ??_C@_04MEMAJGDJ@name?$AA@ 110b30cc     ldblib.obj
 0002:0000a0d4       ??_C@_08JEGIFMFI@namewhat?$AA@ 110b30d4     ldblib.obj
 0002:0000a0e0       ??_C@_0M@DINLHJFF@activelines?$AA@ 110b30e0     ldblib.obj
 0002:0000a0ec       ??_C@_04HPNHAEOP@func?$AA@ 110b30ec     ldblib.obj
 0002:0000a0f4       ??_C@_0BD@EFMIJNPC@level?5out?5of?5range?$AA@ 110b30f4     ldblib.obj
 0002:0000a108       ??_C@_0O@POGBCBNN@external?5hook?$AA@ 110b3108     ldblib.obj
 0002:0000a118       ??_C@_0M@FBGICICO@lua_debug?$DO?5?$AA@ 110b3118     ldblib.obj
 0002:0000a124       ??_C@_05KJNBGLAC@cont?6?$AA@ 110b3124     ldblib.obj
 0002:0000a12c       ??_C@_0BB@BLKFCGLG@?$DN?$CIdebug?5command?$CJ?$AA@ 110b312c     ldblib.obj
 0002:0000a140       ??_C@_0BB@CJHIJJAH@stack?5traceback?3?$AA@ 110b3140     ldblib.obj
 0002:0000a154       ??_C@_05JLIPKFIA@?6?7?4?4?4?$AA@ 110b3154     ldblib.obj
 0002:0000a15c       ??_C@_02NMOLBIHC@?6?7?$AA@ 110b315c     ldblib.obj
 0002:0000a160       ??_C@_03IMACECCO@Snl?$AA@  110b3160     ldblib.obj
 0002:0000a164       ??_C@_03DKEJHHJP@?$CFs?3?$AA@ 110b3164     ldblib.obj
 0002:0000a168       ??_C@_03CDCAMCGK@?$CFd?3?$AA@ 110b3168     ldblib.obj
 0002:0000a16c       ??_C@_0BC@CPJFAADE@?5in?5function?5?8?$CFs?8?$AA@ 110b316c     ldblib.obj
 0002:0000a180       ??_C@_0P@IOLMPCPC@?5in?5main?5chunk?$AA@ 110b3180     ldblib.obj
 0002:0000a190       ??_C@_02GACNEKDB@?5?$DP?$AA@ 110b3190     ldblib.obj
 0002:0000a194       ??_C@_0BF@IDFBHDGL@?5in?5function?5?$DM?$CFs?3?$CFd?$DO?$AA@ 110b3194     ldblib.obj
 0002:0000a1ac       ??_C@_0N@NCKPGBEC@?$CI?$CKtemporary?$CJ?$AA@ 110b31ac     ldebug.obj
 0002:0000a1bc       ??_C@_04BKJOMPG@?$DN?$FLC?$FN?$AA@ 110b31bc     ldebug.obj
 0002:0000a1c4       ??_C@_01GFHCPBMG@C?$AA@    110b31c4     ldebug.obj
 0002:0000a1c8       ??_C@_04GHJNJNPO@main?$AA@ 110b31c8     ldebug.obj
 0002:0000a1d0       ??_C@_04DIFLAKIP@tail?$AA@ 110b31d0     ldebug.obj
 0002:0000a1d8       ??_C@_0N@DIENKKJP@?$DN?$CItail?5call?$CJ?$AA@ 110b31d8     ldebug.obj
 0002:0000a1e8       ??_C@_05IDKHKMLA@local?$AA@ 110b31e8     ldebug.obj
 0002:0000a1f0       ??_C@_06FJKEMHGD@global?$AA@ 110b31f0     ldebug.obj
 0002:0000a1f8       ??_C@_05EIBGDMPB@field?$AA@ 110b31f8     ldebug.obj
 0002:0000a200       ??_C@_07NAGMKCIK@upvalue?$AA@ 110b3200     ldebug.obj
 0002:0000a208       ??_C@_0CD@HAGFMPIP@attempt?5to?5?$CFs?5?$CFs?5?8?$CFs?8?5?$CIa?5?$CFs?5valu@ 110b3208     ldebug.obj
 0002:0000a22c       ??_C@_0BJ@HGCMIDJD@attempt?5to?5?$CFs?5a?5?$CFs?5value?$AA@ 110b322c     ldebug.obj
 0002:0000a248       ??_C@_0M@LPKAOE@concatenate?$AA@ 110b3248     ldebug.obj
 0002:0000a254       ??_C@_0BG@IOLALLOM@perform?5arithmetic?5on?$AA@ 110b3254     ldebug.obj
 0002:0000a26c       ??_C@_0CB@DEJMKNMB@attempt?5to?5compare?5two?5?$CFs?5values@ 110b326c     ldebug.obj
 0002:0000a290       ??_C@_0BO@DNBGDDFP@attempt?5to?5compare?5?$CFs?5with?5?$CFs?$AA@ 110b3290     ldebug.obj
 0002:0000a2b0       ??_C@_09BHPFBFOI@?$CFs?3?$CFd?3?5?$CFs?$AA@ 110b32b0     ldebug.obj
 0002:0000a2bc       ??_C@_0BC@ENOOLCNF@not?5enough?5memory?$AA@ 110b32bc     ldo.obj
 0002:0000a2d0       ??_C@_0BI@KGOCJOGJ@error?5in?5error?5handling?$AA@ 110b32d0     ldo.obj
 0002:0000a2e8       ??_C@_0P@EODJGPIM@stack?5overflow?$AA@ 110b32e8     ldo.obj
 0002:0000a2f8       ??_C@_0BB@EJOGNINL@C?5stack?5overflow?$AA@ 110b32f8     ldo.obj
 0002:0000a30c       ??_C@_0CG@NAAHDPPN@cannot?5resume?5non?9suspended?5coro@ 110b330c     ldo.obj
 0002:0000a334       ??_C@_0DD@CPKEKIFA@attempt?5to?5yield?5across?5metameth@ 110b3334     ldo.obj
 0002:0000a368       ??_C@_04CFDJAKFL@math?$AA@ 110b3368     linit.obj
 0002:0000a370       ??_C@_06ICGJLFIM@string?$AA@ 110b3370     linit.obj
 0002:0000a378       ??_C@_02EHCHIAMF@os?$AA@   110b3378     linit.obj
 0002:0000a37c       ??_C@_02KFNNKBCK@io?$AA@   110b337c     linit.obj
 0002:0000a380       ??_C@_05LCLENNFI@table?$AA@ 110b3380     linit.obj
 0002:0000a388       ??_C@_07KNEGBPNO@package?$AA@ 110b3388     linit.obj
 0002:0000a390       ??_C@_07HHBPNGAN@setvbuf?$AA@ 110b3390     liolib.obj
 0002:0000a398       ??_C@_04EDECCOGL@seek?$AA@ 110b3398     liolib.obj
 0002:0000a3a0       ??_C@_05NGFEDHGN@write?$AA@ 110b33a0     liolib.obj
 0002:0000a3a8       ??_C@_07FKJPAINK@tmpfile?$AA@ 110b33a8     liolib.obj
 0002:0000a3b0       ??_C@_05IACAFMHP@popen?$AA@ 110b33b0     liolib.obj
 0002:0000a3b8       ??_C@_05DENOCHIP@lines?$AA@ 110b33b8     liolib.obj
 0002:0000a3c0       ??_C@_05GLCAEPFP@flush?$AA@ 110b33c0     liolib.obj
 0002:0000a3c8       ??_C@_05LBOHBHFK@close?$AA@ 110b33c8     liolib.obj
 0002:0000a3d0       ??_C@_04PLMLMMEO@full?$AA@ 110b33d0     liolib.obj
 0002:0000a3d8       ??_C@_02KAJCLHKP@no?$AA@   110b33d8     liolib.obj
 0002:0000a3dc       ??_C@_03JBJLGPFL@end?$AA@  110b33dc     liolib.obj
 0002:0000a3e0       ??_C@_03LIBLMJMB@cur?$AA@  110b33e0     liolib.obj
 0002:0000a3e4       ??_C@_03KCHOJKKI@set?$AA@  110b33e4     liolib.obj
 0002:0000a3e8       ??_C@_06DKIGHACF@output?$AA@ 110b33e8     liolib.obj
 0002:0000a3f0       ??_C@_05DFJCHPDH@input?$AA@ 110b33f0     liolib.obj
 0002:0000a3f8       ??_C@_06DJHOIPC@?$CFs?3?5?$CFs?$AA@ 110b33f8     liolib.obj
 0002:0000a400       ??_C@_05KCHOJJD@FILE?$CK?$AA@ 110b3400     liolib.obj
 0002:0000a408       ??_C@_0M@IBKPHHKH@closed?5file?$AA@ 110b3408     liolib.obj
 0002:0000a414       ??_C@_04DAMGJPCA@file?$AA@ 110b3414     liolib.obj
 0002:0000a41c       ??_C@_0BN@LPOOHAOM@attempt?5to?5use?5a?5closed?5file?$AA@ 110b341c     liolib.obj
 0002:0000a43c       ??_C@_0BL@PEFGCPAG@cannot?5close?5standard?5file?$AA@ 110b343c     liolib.obj
 0002:0000a458       ??_C@_07DMJMBBKE@__close?$AA@ 110b3458     liolib.obj
 0002:0000a460       ??_C@_0O@PLFAPHPG@file?5?$CIclosed?$CJ?$AA@ 110b3460     liolib.obj
 0002:0000a470       ??_C@_09BPMAMLLD@file?5?$CI?$CFp?$CJ?$AA@ 110b3470     liolib.obj
 0002:0000a47c       ??_C@_0BL@JMNLNGCA@standard?5?$CFs?5file?5is?5closed?$AA@ 110b347c     liolib.obj
 0002:0000a498       ??_C@_01NOFIACDB@w?$AA@    110b3498     liolib.obj
 0002:0000a49c       ??_C@_03DLDNIBIK@?$CFlf?$AA@ 110b349c     liolib.obj
 0002:0000a4a0       ??_C@_0BD@IOJAAODF@too?5many?5arguments?$AA@ 110b34a0     liolib.obj
 0002:0000a4b4       ??_C@_0P@CENJCLHM@invalid?5format?$AA@ 110b34b4     liolib.obj
 0002:0000a4c4       ??_C@_0BH@PBGIDLEF@file?5is?5already?5closed?$AA@ 110b34c4     liolib.obj
 0002:0000a4dc       ??_C@_05CGOEHEFE@?$CF?414g?$AA@ 110b34dc     liolib.obj
 0002:0000a4e4       ??_C@_05MHOFLBOO@stdin?$AA@ 110b34e4     liolib.obj
 0002:0000a4ec       ??_C@_06DJDOIFHB@stdout?$AA@ 110b34ec     liolib.obj
 0002:0000a4f4       ??_C@_06FJGNEBG@stderr?$AA@ 110b34f4     liolib.obj
 0002:0000a4fc       ??_C@_05CINCKAN@?$DMeof?$DO?$AA@ 110b34fc     llex.obj
 0002:0000a504       ??_C@_08OOGHEFMC@?$DMstring?$DO?$AA@ 110b3504     llex.obj
 0002:0000a510       ??_C@_06FNGJOCBI@?$DMname?$DO?$AA@ 110b3510     llex.obj
 0002:0000a518       ??_C@_08OHBCANEJ@?$DMnumber?$DO?$AA@ 110b3518     llex.obj
 0002:0000a524       ??_C@_02DEDJCLAJ@?$HO?$DN?$AA@ 110b3524     llex.obj
 0002:0000a528       ??_C@_02EHCHHCKH@?$DM?$DN?$AA@ 110b3528     llex.obj
 0002:0000a52c       ??_C@_02EEKDKGMJ@?$DO?$DN?$AA@ 110b352c     llex.obj
 0002:0000a530       ??_C@_02EGOFBIJA@?$DN?$DN?$AA@ 110b3530     llex.obj
 0002:0000a534       ??_C@_03KHICJKCI@?4?4?4?$AA@ 110b3534     llex.obj
 0002:0000a538       ??_C@_02DJGKEECL@?4?4?$AA@ 110b3538     llex.obj
 0002:0000a53c       ??_C@_05OODBEKIG@while?$AA@ 110b353c     llex.obj
 0002:0000a544       ??_C@_05FJMDOIMN@until?$AA@ 110b3544     llex.obj
 0002:0000a54c       ??_C@_04HOHPNOOD@then?$AA@ 110b354c     llex.obj
 0002:0000a554       ??_C@_06LGDBIFHB@repeat?$AA@ 110b3554     llex.obj
 0002:0000a55c       ??_C@_02FODMLBIE@or?$AA@   110b355c     llex.obj
 0002:0000a560       ??_C@_03NJKJADM@not?$AA@   110b3560     llex.obj
 0002:0000a564       ??_C@_02LMMGJAGL@in?$AA@   110b3564     llex.obj
 0002:0000a568       ??_C@_02HEBPBKGD@if?$AA@   110b3568     llex.obj
 0002:0000a56c       ??_C@_08HFFPPCHF@function?$AA@ 110b356c     llex.obj
 0002:0000a578       ??_C@_03JOHEBPFF@for?$AA@  110b3578     llex.obj
 0002:0000a57c       ??_C@_06CAACNEC@elseif?$AA@ 110b357c     llex.obj
 0002:0000a584       ??_C@_04FHMCPBIP@else?$AA@ 110b3584     llex.obj
 0002:0000a58c       ??_C@_02KNAFDCHJ@do?$AA@   110b358c     llex.obj
 0002:0000a590       ??_C@_05ELPHFHOI@break?$AA@ 110b3590     llex.obj
 0002:0000a598       ??_C@_03BOPJPIAM@and?$AA@  110b3598     llex.obj
 0002:0000a59c       ??_C@_0BJ@JNKOFINI@lexical?5element?5too?5long?$AA@ 110b359c     llex.obj
 0002:0000a5b8       ??_C@_08HJPIMBHL@char?$CI?$CFd?$CJ?$AA@ 110b35b8     llex.obj
 0002:0000a5c4       ??_C@_02HAOIJKIC@?$CFc?$AA@ 110b35c4     llex.obj
 0002:0000a5c8       ??_C@_0N@FKCNMBAF@?$CFs?5near?5?8?$CFs?8?$AA@ 110b35c8     llex.obj
 0002:0000a5d8       ??_C@_0BJ@LAKGPFF@chunk?5has?5too?5many?5lines?$AA@ 110b35d8     llex.obj
 0002:0000a5f4       ??_C@_0BB@CFMNENCE@malformed?5number?$AA@ 110b35f4     llex.obj
 0002:0000a608       ??_C@_02GOGFPGCE@Ee?$AA@   110b3608     llex.obj
 0002:0000a60c       ??_C@_02BEIMNFAD@?$CL?9?$AA@ 110b360c     llex.obj
 0002:0000a610       ??_C@_0BH@BBMFLJJP@unfinished?5long?5string?$AA@ 110b3610     llex.obj
 0002:0000a628       ??_C@_0BI@ONEAKEIB@unfinished?5long?5comment?$AA@ 110b3628     llex.obj
 0002:0000a640       ??_C@_0CB@BALFDNPK@nesting?5of?5?$FL?$FL?4?4?4?$FN?$FN?5is?5deprecated@ 110b3640     llex.obj
 0002:0000a664       ??_C@_0BC@IBAFBKML@unfinished?5string?$AA@ 110b3664     llex.obj
 0002:0000a678       ??_C@_0BK@GLJFEJMO@escape?5sequence?5too?5large?$AA@ 110b3678     llex.obj
 0002:0000a694       ??_C@_0BO@DBNLNIBP@invalid?5long?5string?5delimiter?$AA@ 110b3694     llex.obj
 0002:0000a6b4       ??_C@_03IIINPABG@tan?$AA@  110b36b4     lmathlib.obj
 0002:0000a6b8       ??_C@_04FJHINJAO@tanh?$AA@ 110b36b8     lmathlib.obj
 0002:0000a6c0       ??_C@_04EIAKFFMI@sqrt?$AA@ 110b36c0     lmathlib.obj
 0002:0000a6c8       ??_C@_03BLEJJJBH@sin?$AA@  110b36c8     lmathlib.obj
 0002:0000a6cc       ??_C@_04COOMCNPB@sinh?$AA@ 110b36cc     lmathlib.obj
 0002:0000a6d4       ??_C@_0L@PIIACENG@randomseed?$AA@ 110b36d4     lmathlib.obj
 0002:0000a6e0       ??_C@_06NLFCANPD@random?$AA@ 110b36e0     lmathlib.obj
 0002:0000a6e8       ??_C@_03FHAJEHEA@rad?$AA@  110b36e8     lmathlib.obj
 0002:0000a6ec       ??_C@_03JGHBODFD@pow?$AA@  110b36ec     lmathlib.obj
 0002:0000a6f0       ??_C@_04EHEDPDJG@modf?$AA@ 110b36f0     lmathlib.obj
 0002:0000a6f8       ??_C@_03KLIPLJLL@min?$AA@  110b36f8     lmathlib.obj
 0002:0000a6fc       ??_C@_03LJAEFNNE@max?$AA@  110b36fc     lmathlib.obj
 0002:0000a700       ??_C@_03MGHMBJCF@log?$AA@  110b3700     lmathlib.obj
 0002:0000a704       ??_C@_05HGHHAHAP@log10?$AA@ 110b3704     lmathlib.obj
 0002:0000a70c       ??_C@_05CEJMAHNP@ldexp?$AA@ 110b370c     lmathlib.obj
 0002:0000a714       ??_C@_05GKKHEGJL@frexp?$AA@ 110b3714     lmathlib.obj
 0002:0000a71c       ??_C@_04KEPJIHGP@fmod?$AA@ 110b371c     lmathlib.obj
 0002:0000a724       ??_C@_05PBJFFIGL@floor?$AA@ 110b3724     lmathlib.obj
 0002:0000a72c       ??_C@_03KHJOGHMM@exp?$AA@  110b372c     lmathlib.obj
 0002:0000a730       ??_C@_03OFPLEBM@deg?$AA@   110b3730     lmathlib.obj
 0002:0000a734       ??_C@_03LALBNOCG@cos?$AA@  110b3734     lmathlib.obj
 0002:0000a738       ??_C@_04HPJJNFIM@cosh?$AA@ 110b3738     lmathlib.obj
 0002:0000a740       ??_C@_04GFPJNGEK@ceil?$AA@ 110b3740     lmathlib.obj
 0002:0000a748       ??_C@_04MLLJIGOK@atan?$AA@ 110b3748     lmathlib.obj
 0002:0000a750       ??_C@_05KNGEOGJB@atan2?$AA@ 110b3750     lmathlib.obj
 0002:0000a758       ??_C@_04FIHNOPOL@asin?$AA@ 110b3758     lmathlib.obj
 0002:0000a760       ??_C@_04PDIFKINK@acos?$AA@ 110b3760     lmathlib.obj
 0002:0000a768       ??_C@_03BCGAIFPO@abs?$AA@  110b3768     lmathlib.obj
 0002:0000a76c       ??_C@_0BC@JKHEKPDC@interval?5is?5empty?$AA@ 110b376c     lmathlib.obj
 0002:0000a780       ??_C@_0BK@KNAOOCNO@wrong?5number?5of?5arguments?$AA@ 110b3780     lmathlib.obj
 0002:0000a79c       ??_C@_02OAHAJOFD@pi?$AA@   110b379c     lmathlib.obj
 0002:0000a7a0       ??_C@_04JJGMCGIH@huge?$AA@ 110b37a0     lmathlib.obj
 0002:0000a7a8       ??_C@_03FFONCNID@mod?$AA@  110b37a8     lmathlib.obj
 0002:0000a7ac       ??_C@_0CH@LBFPMMCP@memory?5allocation?5error?3?5block?5t@ 110b37ac     lmem.obj
 0002:0000a7d4       ??_C@_07FFLLPPLH@require?$AA@ 110b37d4     loadlib.obj
 0002:0000a7dc       ??_C@_06BIEEJMKO@module?$AA@ 110b37dc     loadlib.obj
 0002:0000a7e4       ??_C@_06LNOHAKGK@seeall?$AA@ 110b37e4     loadlib.obj
 0002:0000a7ec       ??_C@_07KOEABFCN@loadlib?$AA@ 110b37ec     loadlib.obj
 0002:0000a7f4       ??_C@_0BN@GMPFCLAN@unable?5to?5get?5ModuleFileName?$AA@ 110b37f4     loadlib.obj
 0002:0000a814       ??_C@_01DCLJPIOD@?$CB?$AA@ 110b3814     loadlib.obj
 0002:0000a818       ??_C@_0BB@BLJKPILH@system?5error?5?$CFd?6?$AA@ 110b3818     loadlib.obj
 0002:0000a82c       ??_C@_09GMLHALBF@LOADLIB?3?5?$AA@ 110b382c     loadlib.obj
 0002:0000a838       ??_C@_04HDOCAJNK@?$CFs?$CFs?$AA@ 110b3838     loadlib.obj
 0002:0000a840       ??_C@_08HNNNOMMJ@_LOADLIB?$AA@ 110b3840     loadlib.obj
 0002:0000a84c       ??_C@_04HKFDNBLD@init?$AA@ 110b384c     loadlib.obj
 0002:0000a854       ??_C@_01ICJEACDI@?$DL?$AA@ 110b3854     loadlib.obj
 0002:0000a858       ??_C@_01KICIPPFI@?2?$AA@   110b3858     loadlib.obj
 0002:0000a85c       ??_C@_0BO@COFCKCAL@?8package?4?$CFs?8?5must?5be?5a?5string?$AA@ 110b385c     loadlib.obj
 0002:0000a87c       ??_C@_0P@NEBKIMDC@?6?7no?5file?5?8?$CFs?8?$AA@ 110b387c     loadlib.obj
 0002:0000a88c       ??_C@_0CO@KHMIPLKM@error?5loading?5module?5?8?$CFs?8?5from?5f@ 110b388c     loadlib.obj
 0002:0000a8bc       ??_C@_04LNEJFJGI@path?$AA@ 110b38bc     loadlib.obj
 0002:0000a8c4       ??_C@_01JOAMLHOP@?9?$AA@   110b38c4     loadlib.obj
 0002:0000a8c8       ??_C@_01IDAFKMJL@_?$AA@    110b38c8     loadlib.obj
 0002:0000a8cc       ??_C@_0L@KHKMBFOE@luaopen_?$CFs?$AA@ 110b38cc     loadlib.obj
 0002:0000a8d8       ??_C@_05EEMJHCCC@cpath?$AA@ 110b38d8     loadlib.obj
 0002:0000a8e0       ??_C@_0BO@KOILFIGK@?6?7no?5module?5?8?$CFs?8?5in?5file?5?8?$CFs?8?$AA@ 110b38e0     loadlib.obj
 0002:0000a900       ??_C@_07GCEAJMEA@preload?$AA@ 110b3900     loadlib.obj
 0002:0000a908       ??_C@_0CC@CCJHFBLH@?8package?4preload?8?5must?5be?5a?5tabl@ 110b3908     loadlib.obj
 0002:0000a92c       ??_C@_0CB@NPNABMBF@?6?7no?5field?5package?4preload?$FL?8?$CFs?8?$FN@ 110b392c     loadlib.obj
 0002:0000a950       ??_C@_0CL@DIEJCPFH@loop?5or?5previous?5error?5loading?5m@ 110b3950     loadlib.obj
 0002:0000a97c       ??_C@_07JAOCDFCG@loaders?$AA@ 110b397c     loadlib.obj
 0002:0000a984       ??_C@_0CC@IGEJMOFI@?8package?4loaders?8?5must?5be?5a?5tabl@ 110b3984     loadlib.obj
 0002:0000a9a8       ??_C@_0BJ@HFHHABH@module?5?8?$CFs?8?5not?5found?3?$CFs?$AA@ 110b39a8     loadlib.obj
 0002:0000a9c4       ??_C@_0CI@GKOMOAFD@?8module?8?5not?5called?5from?5a?5Lua?5f@ 110b39c4     loadlib.obj
 0002:0000a9ec       ??_C@_02CCIJHOCI@_M?$AA@   110b39ec     loadlib.obj
 0002:0000a9f0       ??_C@_05ICMCJINN@_NAME?$AA@ 110b39f0     loadlib.obj
 0002:0000a9f8       ??_C@_08HONLOGDK@_PACKAGE?$AA@ 110b39f8     loadlib.obj
 0002:0000aa04       ??_C@_03MEOBNKEM@?$DL?$AB?$DL?$AA@ 110b3a04     loadlib.obj
 0002:0000aa08       ??_C@_02BEDCMDKE@?$DL?$DL?$AA@ 110b3a08     loadlib.obj
 0002:0000aa0c       ??_C@_01KHDNNMEB@?$AB?$AA@ 110b3a0c     loadlib.obj
 0002:0000aa10       ??_C@_0DK@FOBKGJIE@?4?2?$DP?4lua?$DL?$CB?2lua?2?$DP?4lua?$DL?$CB?2lua?2?$DP?2init@ 110b3a10     loadlib.obj
 0002:0000aa4c       ??_C@_08GLJMJBPN@LUA_PATH?$AA@ 110b3a4c     loadlib.obj
 0002:0000aa58       ??_C@_0BO@DBNDCFPP@?4?2?$DP?4dll?$DL?$CB?2?$DP?4dll?$DL?$CB?2loadall?4dll?$AA@ 110b3a58     loadlib.obj
 0002:0000aa78       ??_C@_09FBPOOEID@LUA_CPATH?$AA@ 110b3a78     loadlib.obj
 0002:0000aa84       ??_C@_09NMALNBAP@?2?6?$DL?6?$DP?6?$CB?6?9?$AA@ 110b3a84     loadlib.obj
 0002:0000aa90       ??_C@_06HEJKKHEK@config?$AA@ 110b3a90     loadlib.obj
 0002:0000aa98       ??_C@_06IILMCCFO@loaded?$AA@ 110b3a98     loadlib.obj
 0002:0000aaa0       ??_C@_01FGNFDNOH@?$CF?$AA@ 110b3aa0     lobject.obj
 0002:0000aaa4       ??_C@_02LIIHNNHG@?6?$AN?$AA@ 110b3aa4     lobject.obj
 0002:0000aaa8       ??_C@_09PHLFBDIK@?$FLstring?5?$CC?$AA@ 110b3aa8     lobject.obj
 0002:0000aab4       ??_C@_02DEGCJHHK@?$CC?$FN?$AA@ 110b3ab4     lobject.obj
 0002:0000aab8       ??_C@_06FHOJKFCK@VARARG?$AA@ 110b3ab8     lopcodes.obj
 0002:0000aac0       ??_C@_07CBDMEJDJ@CLOSURE?$AA@ 110b3ac0     lopcodes.obj
 0002:0000aac8       ??_C@_05HKHBPABE@CLOSE?$AA@ 110b3ac8     lopcodes.obj
 0002:0000aad0       ??_C@_07LGKGOMK@SETLIST?$AA@ 110b3ad0     lopcodes.obj
 0002:0000aad8       ??_C@_08LFLGPGKH@TFORLOOP?$AA@ 110b3ad8     lopcodes.obj
 0002:0000aae4       ??_C@_07BDNHFNAN@FORPREP?$AA@ 110b3ae4     lopcodes.obj
 0002:0000aaec       ??_C@_07BJCDCNBK@FORLOOP?$AA@ 110b3aec     lopcodes.obj
 0002:0000aaf4       ??_C@_06LJMOENAO@RETURN?$AA@ 110b3af4     lopcodes.obj
 0002:0000aafc       ??_C@_08GDMBKKIJ@TAILCALL?$AA@ 110b3afc     lopcodes.obj
 0002:0000ab08       ??_C@_04CAGKGBIO@CALL?$AA@ 110b3b08     lopcodes.obj
 0002:0000ab10       ??_C@_07GLDFODBB@TESTSET?$AA@ 110b3b10     lopcodes.obj
 0002:0000ab18       ??_C@_04OIKJMBFP@TEST?$AA@ 110b3b18     lopcodes.obj
 0002:0000ab20       ??_C@_02PEDAOJAJ@LE?$AA@   110b3b20     lopcodes.obj
 0002:0000ab24       ??_C@_02KHOJMKBJ@LT?$AA@   110b3b24     lopcodes.obj
 0002:0000ab28       ??_C@_02NFEPAFND@EQ?$AA@   110b3b28     lopcodes.obj
 0002:0000ab2c       ??_C@_03OIOLNLHN@JMP?$AA@  110b3b2c     lopcodes.obj
 0002:0000ab30       ??_C@_06CIJDJJIA@CONCAT?$AA@ 110b3b30     lopcodes.obj
 0002:0000ab38       ??_C@_03BHNCOKMG@LEN?$AA@  110b3b38     lopcodes.obj
 0002:0000ab3c       ??_C@_03GBFNEA@NOT?$AA@    110b3b3c     lopcodes.obj
 0002:0000ab40       ??_C@_03BNLLEOPB@UNM?$AA@  110b3b40     lopcodes.obj
 0002:0000ab44       ??_C@_03JLIKCOCP@POW?$AA@  110b3b44     lopcodes.obj
 0002:0000ab48       ??_C@_03FIBGOAPP@MOD?$AA@  110b3b48     lopcodes.obj
 0002:0000ab4c       ??_C@_03FJGHKDBE@DIV?$AA@  110b3b4c     lopcodes.obj
 0002:0000ab50       ??_C@_03IBHOEMFB@MUL?$AA@  110b3b50     lopcodes.obj
 0002:0000ab54       ??_C@_03KPDLEBHD@SUB?$AA@  110b3b54     lopcodes.obj
 0002:0000ab58       ??_C@_03BOJFLAKG@ADD?$AA@  110b3b58     lopcodes.obj
 0002:0000ab5c       ??_C@_04DFAHIJNB@SELF?$AA@ 110b3b5c     lopcodes.obj
 0002:0000ab64       ??_C@_08LPLGEMDO@NEWTABLE?$AA@ 110b3b64     lopcodes.obj
 0002:0000ab70       ??_C@_08NDNBPDIF@SETTABLE?$AA@ 110b3b70     lopcodes.obj
 0002:0000ab7c       ??_C@_08EDGMHGMA@SETUPVAL?$AA@ 110b3b7c     lopcodes.obj
 0002:0000ab88       ??_C@_09DECDCIIG@SETGLOBAL?$AA@ 110b3b88     lopcodes.obj
 0002:0000ab94       ??_C@_08CCPNOAPI@GETTABLE?$AA@ 110b3b94     lopcodes.obj
 0002:0000aba0       ??_C@_09BKGGAJBE@GETGLOBAL?$AA@ 110b3ba0     lopcodes.obj
 0002:0000abac       ??_C@_08LCEAGFLN@GETUPVAL?$AA@ 110b3bac     lopcodes.obj
 0002:0000abb8       ??_C@_07GHJHEMKM@LOADNIL?$AA@ 110b3bb8     lopcodes.obj
 0002:0000abc0       ??_C@_08GBBGHEAC@LOADBOOL?$AA@ 110b3bc0     lopcodes.obj
 0002:0000abcc       ??_C@_05KLLCNHFJ@LOADK?$AA@ 110b3bcc     lopcodes.obj
 0002:0000abd4       ??_C@_04LPPGDFDD@MOVE?$AA@ 110b3bd4     lopcodes.obj
 0002:0000abdc       ??_C@_07KOJJABMD@tmpname?$AA@ 110b3bdc     loslib.obj
 0002:0000abe4       ??_C@_09IOBOFJNA@setlocale?$AA@ 110b3be4     loslib.obj
 0002:0000abf0       ??_C@_06LMEAOBLB@rename?$AA@ 110b3bf0     loslib.obj
 0002:0000abf8       ??_C@_06LEMKAMD@remove?$AA@ 110b3bf8     loslib.obj
 0002:0000ac00       ??_C@_06EPDNLFGH@getenv?$AA@ 110b3c00     loslib.obj
 0002:0000ac08       ??_C@_04MKNBDEPB@exit?$AA@ 110b3c08     loslib.obj
 0002:0000ac10       ??_C@_07EMGJIMLB@execute?$AA@ 110b3c10     loslib.obj
 0002:0000ac18       ??_C@_08PDOPCMOG@difftime?$AA@ 110b3c18     loslib.obj
 0002:0000ac24       ??_C@_04JNIHBGGH@date?$AA@ 110b3c24     loslib.obj
 0002:0000ac2c       ??_C@_05DDECJJKE@clock?$AA@ 110b3c2c     loslib.obj
 0002:0000ac34       ??_C@_04CLCEDBPF@time?$AA@ 110b3c34     loslib.obj
 0002:0000ac3c       ??_C@_07MMLECJPG@numeric?$AA@ 110b3c3c     loslib.obj
 0002:0000ac44       ??_C@_08BIOBDOAM@monetary?$AA@ 110b3c44     loslib.obj
 0002:0000ac50       ??_C@_05JGEDHNAD@ctype?$AA@ 110b3c50     loslib.obj
 0002:0000ac58       ??_C@_07FCFLCBKH@collate?$AA@ 110b3c58     loslib.obj
 0002:0000ac60       ??_C@_03NFKEKGGK@all?$AA@  110b3c60     loslib.obj
 0002:0000ac64       ??_C@_0CF@CFMGMNIN@unable?5to?5generate?5a?5unique?5file@ 110b3c64     loslib.obj
 0002:0000ac8c       ??_C@_0CB@DJMEIEGF@field?5?8?$CFs?8?5missing?5in?5date?5table@ 110b3c8c     loslib.obj
 0002:0000acb0       ??_C@_02HODHFJCJ@?$CKt?$AA@ 110b3cb0     loslib.obj
 0002:0000acb4       ??_C@_03KHPNBODO@sec?$AA@  110b3cb4     loslib.obj
 0002:0000acb8       ??_C@_04LMOJGCPE@hour?$AA@ 110b3cb8     loslib.obj
 0002:0000acc0       ??_C@_03NNBHCDBP@day?$AA@  110b3cc0     loslib.obj
 0002:0000acc4       ??_C@_05MEBAADFH@month?$AA@ 110b3cc4     loslib.obj
 0002:0000accc       ??_C@_04JFPLDHAO@year?$AA@ 110b3ccc     loslib.obj
 0002:0000acd4       ??_C@_04HBIDDHMB@wday?$AA@ 110b3cd4     loslib.obj
 0002:0000acdc       ??_C@_04MOLDIJKA@yday?$AA@ 110b3cdc     loslib.obj
 0002:0000ace4       ??_C@_05HGBEJAHO@isdst?$AA@ 110b3ce4     loslib.obj
 0002:0000acec       ??_C@_0O@DDMAPLHE@?8?$CFs?8?5expected?$AA@ 110b3cec     lparser.obj
 0002:0000acfc       ??_C@_0CC@OKOPEFGK@main?5function?5has?5more?5than?5?$CFd?5?$CF@ 110b3cfc     lparser.obj
 0002:0000ad20       ??_C@_0CI@FLAOKACM@function?5at?5line?5?$CFd?5has?5more?5tha@ 110b3d20     lparser.obj
 0002:0000ad48       ??_C@_0CJ@IJEGBPEP@?8?$CFs?8?5expected?5?$CIto?5close?5?8?$CFs?8?5at?5@ 110b3d48     lparser.obj
 0002:0000ad74       ??_C@_0BJ@EGOMLGMD@too?5many?5local?5variables?$AA@ 110b3d74     lparser.obj
 0002:0000ad90       ??_C@_0BA@EIDMAHJI@local?5variables?$AA@ 110b3d90     lparser.obj
 0002:0000ada0       ??_C@_08JKPCMKJ@upvalues?$AA@ 110b3da0     lparser.obj
 0002:0000adac       ??_C@_0CB@OHOGAGIL@chunk?5has?5too?5many?5syntax?5levels@ 110b3dac     lparser.obj
 0002:0000add0       ??_C@_0BH@IAOKECIM@items?5in?5a?5constructor?$AA@ 110b3dd0     lparser.obj
 0002:0000ade8       ??_C@_03CAOIPBNL@arg?$AA@  110b3de8     lparser.obj
 0002:0000adec       ??_C@_0BJ@MHIGIDHO@?$DMname?$DO?5or?5?8?4?4?4?8?5expected?$AA@ 110b3dec     lparser.obj
 0002:0000ae08       ??_C@_04PJDNGLKJ@self?$AA@ 110b3e08     lparser.obj
 0002:0000ae10       ??_C@_0DB@LGGKFLCP@ambiguous?5syntax?5?$CIfunction?5call?5@ 110b3e10     lparser.obj
 0002:0000ae44       ??_C@_0BM@HEIHHEKF@function?5arguments?5expected?$AA@ 110b3e44     lparser.obj
 0002:0000ae60       ??_C@_0BC@KBCKKGAJ@unexpected?5symbol?$AA@ 110b3e60     lparser.obj
 0002:0000ae74       ??_C@_0CL@EJFFCAJP@cannot?5use?5?8?4?4?4?8?5outside?5a?5varar@ 110b3e74     lparser.obj
 0002:0000aea0       ??_C@_0N@MNJHOOI@syntax?5error?$AA@ 110b3ea0     lparser.obj
 0002:0000aeb0       ??_C@_0BI@MAKOOLPG@variables?5in?5assignment?$AA@ 110b3eb0     lparser.obj
 0002:0000aec8       ??_C@_0BB@DBFONGCK@no?5loop?5to?5break?$AA@ 110b3ec8     lparser.obj
 0002:0000aedc       ??_C@_0M@HHIHAJLG@?$CIfor?5index?$CJ?$AA@ 110b3edc     lparser.obj
 0002:0000aee8       ??_C@_0M@HGGGDCAE@?$CIfor?5limit?$CJ?$AA@ 110b3ee8     lparser.obj
 0002:0000aef4       ??_C@_0L@ELGHHMFI@?$CIfor?5step?$CJ?$AA@ 110b3ef4     lparser.obj
 0002:0000af00       ??_C@_0BA@IJIMMPHF@?$CIfor?5generator?$CJ?$AA@ 110b3f00     lparser.obj
 0002:0000af10       ??_C@_0M@CCNPGEGC@?$CIfor?5state?$CJ?$AA@ 110b3f10     lparser.obj
 0002:0000af1c       ??_C@_0O@PHJHAIC@?$CIfor?5control?$CJ?$AA@ 110b3f1c     lparser.obj
 0002:0000af2c       ??_C@_0BF@PACDFECJ@?8?$DN?8?5or?5?8in?8?5expected?$AA@ 110b3f2c     lparser.obj
 0002:0000af44       ??_C@_05NECKJAMC@upper?$AA@ 110b3f44     lstrlib.obj
 0002:0000af4c       ??_C@_03KCMAIMAP@sub?$AA@  110b3f4c     lstrlib.obj
 0002:0000af50       ??_C@_07KOIEOCCE@reverse?$AA@ 110b3f50     lstrlib.obj
 0002:0000af58       ??_C@_03HOKODIMJ@rep?$AA@  110b3f58     lstrlib.obj
 0002:0000af5c       ??_C@_05FNONLPDI@match?$AA@ 110b3f5c     lstrlib.obj
 0002:0000af64       ??_C@_05IPJEPLHL@lower?$AA@ 110b3f64     lstrlib.obj
 0002:0000af6c       ??_C@_03BKCJCHLK@len?$AA@  110b3f6c     lstrlib.obj
 0002:0000af70       ??_C@_04GOLEAPFD@gsub?$AA@ 110b3f70     lstrlib.obj
 0002:0000af78       ??_C@_06DPFCLDIO@gmatch?$AA@ 110b3f78     lstrlib.obj
 0002:0000af80       ??_C@_05EIEIBDFD@gfind?$AA@ 110b3f80     lstrlib.obj
 0002:0000af88       ??_C@_06DLEPGFEF@format?$AA@ 110b3f88     lstrlib.obj
 0002:0000af90       ??_C@_04CKFJHKAP@find?$AA@ 110b3f90     lstrlib.obj
 0002:0000af98       ??_C@_04GGLOKIEE@dump?$AA@ 110b3f98     lstrlib.obj
 0002:0000afa0       ??_C@_04ENMBGAPA@char?$AA@ 110b3fa0     lstrlib.obj
 0002:0000afa8       ??_C@_04IHGKJMLH@byte?$AA@ 110b3fa8     lstrlib.obj
 0002:0000afb0       ??_C@_0BG@DFAIEAEC@string?5slice?5too?5long?$AA@ 110b3fb0     lstrlib.obj
 0002:0000afc8       ??_C@_0O@EAJJMEEM@invalid?5value?$AA@ 110b3fc8     lstrlib.obj
 0002:0000afd8       ??_C@_0BO@BNLBHKJN@unable?5to?5dump?5given?5function?$AA@ 110b3fd8     lstrlib.obj
 0002:0000aff8       ??_C@_0BG@LEHNKOGD@invalid?5capture?5index?$AA@ 110b3ff8     lstrlib.obj
 0002:0000b010       ??_C@_0BI@ECNPHIBF@invalid?5pattern?5capture?$AA@ 110b4010     lstrlib.obj
 0002:0000b028       ??_C@_0CD@PLJBIEHA@malformed?5pattern?5?$CIends?5with?5?8?$CF?$CF@ 110b4028     lstrlib.obj
 0002:0000b04c       ??_C@_0CA@CFGACOGB@malformed?5pattern?5?$CImissing?5?8?$FN?8?$CJ?$AA@ 110b404c     lstrlib.obj
 0002:0000b06c       ??_C@_0BD@NGJIMPLI@unbalanced?5pattern?$AA@ 110b406c     lstrlib.obj
 0002:0000b080       ??_C@_0BC@IMEAEJPD@too?5many?5captures?$AA@ 110b4080     lstrlib.obj
 0002:0000b094       ??_C@_0CD@LOJJMDBH@missing?5?8?$FL?8?5after?5?8?$CF?$CFf?8?5in?5patte@ 110b4094     lstrlib.obj
 0002:0000b0b8       ??_C@_0BD@BFKNEALP@unfinished?5capture?$AA@ 110b40b8     lstrlib.obj
 0002:0000b0cc       ??_C@_0L@NLFJOONJ@?$FO$?$CK?$CL?$DP?4?$CI?$FL?$CF?9?$AA@ 110b40cc     lstrlib.obj
 0002:0000b0d8       ??_C@_0CO@MAGJPEI@?8string?4gfind?8?5was?5renamed?5to?5?8s@ 110b40d8     lstrlib.obj
 0002:0000b108       ??_C@_0CB@LPDIHGGA@invalid?5replacement?5value?5?$CIa?5?$CFs?$CJ@ 110b4108     lstrlib.obj
 0002:0000b12c       ??_C@_0BP@PPPOBACA@string?1function?1table?5expected?$AA@ 110b412c     lstrlib.obj
 0002:0000b14c       ??_C@_02HIBBOKEN@?2r?$AA@  110b414c     lstrlib.obj
 0002:0000b150       ??_C@_04MPDIABOK@?2000?$AA@ 110b4150     lstrlib.obj
 0002:0000b158       ??_C@_05GGBDHNF@?9?$CL?5?$CD0?$AA@ 110b4158     lstrlib.obj
 0002:0000b160       ??_C@_0CA@COOMGCAO@invalid?5format?5?$CIrepeated?5flags?$CJ?$AA@ 110b4160     lstrlib.obj
 0002:0000b180       ??_C@_0CN@KALFEKPN@invalid?5format?5?$CIwidth?5or?5precisi@ 110b4180     lstrlib.obj
 0002:0000b1b0       ??_C@_0CC@KIPBEOBI@invalid?5option?5?8?$CF?$CF?$CFc?8?5to?5?8format@ 110b41b0     lstrlib.obj
 0002:0000b1d4       ??_C@_0BG@FEBJBDLJ@invalid?5key?5to?5?8next?8?$AA@ 110b41d4     ltable.obj
 0002:0000b1ec       ??_C@_0P@KKABOKCO@table?5overflow?$AA@ 110b41ec     ltable.obj
 0002:0000b1fc       ??_C@_0BD@BDIKLFBP@table?5index?5is?5nil?$AA@ 110b41fc     ltable.obj
 0002:0000b210       ??_C@_0BD@BKBJANLJ@table?5index?5is?5NaN?$AA@ 110b4210     ltable.obj
 0002:0000b224       ??_C@_04PIMMHFGE@sort?$AA@ 110b4224     ltablib.obj
 0002:0000b22c       ??_C@_04CDNBBDGJ@setn?$AA@ 110b422c     ltablib.obj
 0002:0000b234       ??_C@_06OAOPNKHP@insert?$AA@ 110b4234     ltablib.obj
 0002:0000b23c       ??_C@_04HKHJFELJ@maxn?$AA@ 110b423c     ltablib.obj
 0002:0000b244       ??_C@_04LGLBCCCL@getn?$AA@ 110b4244     ltablib.obj
 0002:0000b24c       ??_C@_08GDLALCOF@foreachi?$AA@ 110b424c     ltablib.obj
 0002:0000b258       ??_C@_07ICLAOFOB@foreach?$AA@ 110b4258     ltablib.obj
 0002:0000b260       ??_C@_06CMLIEHFC@concat?$AA@ 110b4260     ltablib.obj
 0002:0000b268       ??_C@_0BD@OBDNDPKA@?8setn?8?5is?5obsolete?$AA@ 110b4268     ltablib.obj
 0002:0000b27c       ??_C@_0CG@LPGHMHCC@wrong?5number?5of?5arguments?5to?5?8in@ 110b427c     ltablib.obj
 0002:0000b2a4       ??_C@_0DF@OJJECDJJ@invalid?5value?5?$CI?$CFs?$CJ?5at?5index?5?$CFd?5i@ 110b42a4     ltablib.obj
 0002:0000b2dc       ??_C@_0CD@OFHMGIPD@invalid?5order?5function?5for?5sorti@ 110b42dc     ltablib.obj
 0002:0000b300       ??_C@_06JPFLIIOJ@__call?$AA@ 110b4300     ltm.obj
 0002:0000b308       ??_C@_08HGDAODEP@__concat?$AA@ 110b4308     ltm.obj
 0002:0000b314       ??_C@_04EJLHOCKK@__le?$AA@ 110b4314     ltm.obj
 0002:0000b31c       ??_C@_04BKGOMBLK@__lt?$AA@ 110b431c     ltm.obj
 0002:0000b324       ??_C@_05MNDELLDN@__len?$AA@ 110b4324     ltm.obj
 0002:0000b32c       ??_C@_05MHFNBPAK@__unm?$AA@ 110b432c     ltm.obj
 0002:0000b334       ??_C@_05EBGMHPNE@__pow?$AA@ 110b4334     ltm.obj
 0002:0000b33c       ??_C@_05ICPALBAE@__mod?$AA@ 110b433c     ltm.obj
 0002:0000b344       ??_C@_05IDIBPCOP@__div?$AA@ 110b4344     ltm.obj
 0002:0000b34c       ??_C@_05FLJIBNKK@__mul?$AA@ 110b434c     ltm.obj
 0002:0000b354       ??_C@_05HFNNBAII@__sub?$AA@ 110b4354     ltm.obj
 0002:0000b35c       ??_C@_05MEHDOBFN@__add?$AA@ 110b435c     ltm.obj
 0002:0000b364       ??_C@_04GIMIAOHA@__eq?$AA@ 110b4364     ltm.obj
 0002:0000b36c       ??_C@_0L@GADKNKH@__newindex?$AA@ 110b436c     ltm.obj
 0002:0000b378       ??_C@_05CCAJFIBN@upval?$AA@ 110b4378     ltm.obj
 0002:0000b380       ??_C@_05BENFLAID@proto?$AA@ 110b4380     ltm.obj
 0002:0000b388       ??_C@_06FJHNOCKE@thread?$AA@ 110b4388     ltm.obj
 0002:0000b390       ??_C@_06EBGNBFIA@number?$AA@ 110b4390     ltm.obj
 0002:0000b398       ??_C@_08NOEPOPLB@userdata?$AA@ 110b4398     ltm.obj
 0002:0000b3a4       ??_C@_07GOBOHMJA@boolean?$AA@ 110b43a4     ltm.obj
 0002:0000b3ac       ??_C@_0BM@EDNHGHJO@?$CFs?3?5?$CFs?5in?5precompiled?5chunk?$AA@ 110b43ac     lundump.obj
 0002:0000b3c8       ??_C@_0P@CLDJCNKP@unexpected?5end?$AA@ 110b43c8     lundump.obj
 0002:0000b3d8       ??_C@_0M@KLEMECJB@bad?5integer?$AA@ 110b43d8     lundump.obj
 0002:0000b3e4       ??_C@_0N@DOELNLHF@bad?5constant?$AA@ 110b43e4     lundump.obj
 0002:0000b3f4       ??_C@_0O@GNEOPCAJ@code?5too?5deep?$AA@ 110b43f4     lundump.obj
 0002:0000b404       ??_C@_08OFPEJJEA@bad?5code?$AA@ 110b4404     lundump.obj
 0002:0000b410       ??_C@_0L@PJHPAMCH@bad?5header?$AA@ 110b4410     lundump.obj
 0002:0000b41c       ??_C@_0O@CNJIDMJE@binary?5string?$AA@ 110b441c     lundump.obj
 0002:0000b42c       ??_C@_02HENDHKBC@?$DN?$DP?$AA@ 110b442c     lundump.obj
 0002:0000b430       ??_C@_05FKHKFDID@index?$AA@ 110b4430     lvm.obj
 0002:0000b438       ??_C@_0BB@JEECHIJH@loop?5in?5gettable?$AA@ 110b4438     lvm.obj
 0002:0000b44c       ??_C@_0BB@GFGOGLOK@loop?5in?5settable?$AA@ 110b444c     lvm.obj
 0002:0000b460       ??_C@_0BH@ONIKNOCM@string?5length?5overflow?$AA@ 110b4460     lvm.obj
 0002:0000b478       ??_C@_0O@MKOIIDGO@get?5length?5of?$AA@ 110b4478     lvm.obj
 0002:0000b488       ??_C@_0CF@JJFDEONC@?8for?8?5initial?5value?5must?5be?5a?5nu@ 110b4488     lvm.obj
 0002:0000b4b0       ??_C@_0BN@GHPMJMPH@?8for?8?5limit?5must?5be?5a?5number?$AA@ 110b44b0     lvm.obj
 0002:0000b4d0       ??_C@_0BM@EGCFKNIJ@?8for?8?5step?5must?5be?5a?5number?$AA@ 110b44d0     lvm.obj
 0002:0000b4ec       ??_C@_01MIFGBAGJ@?$CL?$AA@ 110b44ec     print.obj
 0002:0000b4f0       ??_C@_05MNCHLHCA@UTF16?$AA@ 110b44f0     sqlite3.obj
 0002:0000b4f8       ??_C@_06KNDPGIKI@UTF?916?$AA@ 110b44f8     sqlite3.obj
 0002:0000b500       ??_C@_07JDFIEPAG@UTF16be?$AA@ 110b4500     sqlite3.obj
 0002:0000b508       ??_C@_08HGGOPCBI@UTF?916be?$AA@ 110b4508     sqlite3.obj
 0002:0000b514       ??_C@_07JJMGGCAM@UTF16le?$AA@ 110b4514     sqlite3.obj
 0002:0000b51c       ??_C@_08HMPANPBC@UTF?916le?$AA@ 110b451c     sqlite3.obj
 0002:0000b528       ??_C@_04OOMJJNCF@UTF8?$AA@ 110b4528     sqlite3.obj
 0002:0000b530       ??_C@_05EGJIMALK@UTF?98?$AA@ 110b4530     sqlite3.obj
 0002:0000b538       ??_C@_0BB@KLHJNGLH@read_uncommitted?$AA@ 110b4538     sqlite3.obj
 0002:0000b54c       ??_C@_0O@FCIFIHH@omit_readlock?$AA@ 110b454c     sqlite3.obj
 0002:0000b55c       ??_C@_0BA@OHBCLCAL@writable_schema?$AA@ 110b455c     sqlite3.obj
 0002:0000b56c       ??_C@_0BJ@KLIMENGM@ignore_check_constraints?$AA@ 110b456c     sqlite3.obj
 0002:0000b588       ??_C@_09MLJLLBEB@fullfsync?$AA@ 110b4588     sqlite3.obj
 0002:0000b594       ??_C@_0BD@LEFOEGBK@legacy_file_format?$AA@ 110b4594     sqlite3.obj
 0002:0000b5a8       ??_C@_0BH@CMLDBHJP@empty_result_callbacks?$AA@ 110b45a8     sqlite3.obj
 0002:0000b5c0       ??_C@_0O@PEBBJPHD@count_changes?$AA@ 110b45c0     sqlite3.obj
 0002:0000b5d0       ??_C@_0BD@BFIEDLEP@short_column_names?$AA@ 110b45d0     sqlite3.obj
 0002:0000b5e4       ??_C@_0BC@CBBNFKC@full_column_names?$AA@ 110b45e4     sqlite3.obj
 0002:0000b5f8       ??_C@_0N@KKLIBDFO@group_concat?$AA@ 110b45f8     sqlite3.obj
 0002:0000b608       ??_C@_03CHOBFJAH@avg?$AA@  110b4608     sqlite3.obj
 0002:0000b60c       ??_C@_05KBOMEDGA@total?$AA@ 110b460c     sqlite3.obj
 0002:0000b614       ??_C@_03CFFIJAMA@sum?$AA@  110b4614     sqlite3.obj
 0002:0000b618       ??_C@_0P@BJKPICNH@load_extension?$AA@ 110b4618     sqlite3.obj
 0002:0000b628       ??_C@_08OAGHJJOG@zeroblob?$AA@ 110b4628     sqlite3.obj
 0002:0000b634       ??_C@_04GDOMMDLP@trim?$AA@ 110b4634     sqlite3.obj
 0002:0000b63c       ??_C@_05FCOGDJML@rtrim?$AA@ 110b463c     sqlite3.obj
 0002:0000b644       ??_C@_05GLDKFKCA@ltrim?$AA@ 110b4644     sqlite3.obj
 0002:0000b64c       ??_C@_07CLEHDIEJ@replace?$AA@ 110b464c     sqlite3.obj
 0002:0000b654       ??_C@_0O@MLEKHAGK@total_changes?$AA@ 110b4654     sqlite3.obj
 0002:0000b664       ??_C@_07HFLFHMNL@changes?$AA@ 110b4664     sqlite3.obj
 0002:0000b66c       ??_C@_0BC@EKKKCJJE@last_insert_rowid?$AA@ 110b466c     sqlite3.obj
 0002:0000b680       ??_C@_05JHEGFHLM@quote?$AA@ 110b4680     sqlite3.obj
 0002:0000b688       ??_C@_0P@IPDPEBN@sqlite_version?$AA@ 110b4688     sqlite3.obj
 0002:0000b698       ??_C@_06LLGGGFDC@nullif?$AA@ 110b4698     sqlite3.obj
 0002:0000b6a0       ??_C@_0L@IDMFPHDO@randomblob?$AA@ 110b46a0     sqlite3.obj
 0002:0000b6ac       ??_C@_06FAHGEKJN@ifnull?$AA@ 110b46ac     sqlite3.obj
 0002:0000b6b4       ??_C@_03IJNDAFDK@hex?$AA@  110b46b4     sqlite3.obj
 0002:0000b6b8       ??_C@_08FNGHHBID@coalesce?$AA@ 110b46b8     sqlite3.obj
 0002:0000b6c4       ??_C@_05MIMAKCN@round?$AA@ 110b46c4     sqlite3.obj
 0002:0000b6cc       ??_C@_06DAHFIGOC@substr?$AA@ 110b46cc     sqlite3.obj
 0002:0000b6d4       ??_C@_06IJDLPEM@length?$AA@ 110b46d4     sqlite3.obj
 0002:0000b6dc       ??_C@_06NDJPCPHC@typeof?$AA@ 110b46dc     sqlite3.obj
 0002:0000b6e4       ??_C@_0BG@DKJJOMDK@sqlite_rename_trigger?$AA@ 110b46e4     sqlite3.obj
 0002:0000b6fc       ??_C@_0BE@JHJAJICL@sqlite_rename_table?$AA@ 110b46fc     sqlite3.obj
 0002:0000b710       ??_C@_01HIHLOKLC@1?$AA@    110b4710     sqlite3.obj
 0002:0000b714       ??_C@_05NMJMPJJB@win32?$AA@ 110b4714     sqlite3.obj
 0002:0000b71c       ??_C@_06ICNNEOIM@ToReal?$AA@ 110b471c     sqlite3.obj
 0002:0000b724       ??_C@_05CNEGLJEO@ToInt?$AA@ 110b4724     sqlite3.obj
 0002:0000b72c       ??_C@_09IAEPJEPI@ToNumeric?$AA@ 110b472c     sqlite3.obj
 0002:0000b738       ??_C@_06LCIJGAA@ToBlob?$AA@ 110b4738     sqlite3.obj
 0002:0000b740       ??_C@_06JMHBLLIK@ToText?$AA@ 110b4740     sqlite3.obj
 0002:0000b748       ??_C@_0M@HFPJJKAF@NotUsed_137?$AA@ 110b4748     sqlite3.obj
 0002:0000b754       ??_C@_0M@GMOCKLEE@NotUsed_136?$AA@ 110b4754     sqlite3.obj
 0002:0000b760       ??_C@_0M@EHMPPIIH@NotUsed_135?$AA@ 110b4760     sqlite3.obj
 0002:0000b76c       ??_C@_0M@FONEMJMG@NotUsed_134?$AA@ 110b476c     sqlite3.obj
 0002:0000b778       ??_C@_0M@BBJFFPAB@NotUsed_133?$AA@ 110b4778     sqlite3.obj
 0002:0000b784       ??_C@_0M@IIOGOEA@NotUsed_132?$AA@ 110b4784     sqlite3.obj
 0002:0000b790       ??_C@_0M@CDKDDNID@NotUsed_131?$AA@ 110b4790     sqlite3.obj
 0002:0000b79c       ??_C@_0M@DKLIAMMC@NotUsed_130?$AA@ 110b479c     sqlite3.obj
 0002:0000b7a8       ??_C@_0M@OKLINNLM@NotUsed_129?$AA@ 110b47a8     sqlite3.obj
 0002:0000b7b4       ??_C@_0M@PDKDOMPN@NotUsed_128?$AA@ 110b47b4     sqlite3.obj
 0002:0000b7c0       ??_C@_0M@HEDLPADC@NotUsed_127?$AA@ 110b47c0     sqlite3.obj
 0002:0000b7cc       ??_C@_0M@GNCAMBHD@NotUsed_126?$AA@ 110b47cc     sqlite3.obj
 0002:0000b7d8       ??_C@_04PHKLBGME@Real?$AA@ 110b47d8     sqlite3.obj
 0002:0000b7e0       ??_C@_0M@FPBGKDPB@NotUsed_124?$AA@ 110b47e0     sqlite3.obj
 0002:0000b7ec       ??_C@_07HJJPPOKN@NullRow?$AA@ 110b47ec     sqlite3.obj
 0002:0000b7f4       ??_C@_05PMIMCOJP@IfPos?$AA@ 110b47f4     sqlite3.obj
 0002:0000b7fc       ??_C@_05JDGHEPJG@Found?$AA@ 110b47fc     sqlite3.obj
 0002:0000b804       ??_C@_07KDKHCOMM@VCreate?$AA@ 110b4804     sqlite3.obj
 0002:0000b80c       ??_C@_06KGOGOHGB@IfZero?$AA@ 110b480c     sqlite3.obj
 0002:0000b814       ??_C@_07NHABAPID@VUpdate?$AA@ 110b4814     sqlite3.obj
 0002:0000b81c       ??_C@_06CLFNNGGK@VBegin?$AA@ 110b481c     sqlite3.obj
 0002:0000b824       ??_C@_06KJNIJPEO@MoveGe?$AA@ 110b4824     sqlite3.obj
 0002:0000b82c       ??_C@_06MAOEIKCJ@Rewind?$AA@ 110b482c     sqlite3.obj
 0002:0000b834       ??_C@_04HOFOMOEI@Blob?$AA@ 110b4834     sqlite3.obj
 0002:0000b83c       ??_C@_04LCANPIEP@Move?$AA@ 110b483c     sqlite3.obj
 0002:0000b844       ??_C@_04KHKKIIL@Null?$AA@  110b4844     sqlite3.obj
 0002:0000b84c       ??_C@_0O@MHKNMBPC@OpenEphemeral?$AA@ 110b484c     sqlite3.obj
 0002:0000b85c       ??_C@_0L@PKPPHKBP@OpenPseudo?$AA@ 110b485c     sqlite3.obj
 0002:0000b868       ??_C@_07EMCFMDDO@Explain?$AA@ 110b4868     sqlite3.obj
 0002:0000b870       ??_C@_0N@FEAPPFEN@LoadAnalysis?$AA@ 110b4870     sqlite3.obj
 0002:0000b880       ??_C@_08PGPGCKGP@ForceInt?$AA@ 110b4880     sqlite3.obj
 0002:0000b88c       ??_C@_0L@LIFFPDNM@ReadCookie?$AA@ 110b488c     sqlite3.obj
 0002:0000b898       ??_C@_07BDCAJABG@Destroy?$AA@ 110b4898     sqlite3.obj
 0002:0000b8a0       ??_C@_06CPFCODOD@Insert?$AA@ 110b48a0     sqlite3.obj
 0002:0000b8a8       ??_C@_09ENCBCCAM@IdxInsert?$AA@ 110b48a8     sqlite3.obj
 0002:0000b8b4       ??_C@_04MDFHGMOB@Next?$AA@ 110b48b4     sqlite3.obj
 0002:0000b8bc       ??_C@_0L@NCJBPLPE@ContextPop?$AA@ 110b48bc     sqlite3.obj
 0002:0000b8c8       ??_C@_08JBEDGDCN@VDestroy?$AA@ 110b48c8     sqlite3.obj
 0002:0000b8d4       ??_C@_07OKDOHLDO@VFilter?$AA@ 110b48d4     sqlite3.obj
 0002:0000b8dc       ??_C@_0M@MEGKBOMN@Transaction?$AA@ 110b48dc     sqlite3.obj
 0002:0000b8e8       ??_C@_0O@GDDDBLCD@SetNumColumns?$AA@ 110b48e8     sqlite3.obj
 0002:0000b8f8       ??_C@_07NOMHFNIB@AggStep?$AA@ 110b48f8     sqlite3.obj
 0002:0000b900       ??_C@_0N@NKEHNBGM@VerifyCookie?$AA@ 110b4900     sqlite3.obj
 0002:0000b910       ??_C@_06PGFEFDLP@MoveLt?$AA@ 110b4910     sqlite3.obj
 0002:0000b918       ??_C@_05MDNHABIA@Clear?$AA@ 110b4918     sqlite3.obj
 0002:0000b920       ??_C@_08GMLBHKDC@FifoRead?$AA@ 110b4920     sqlite3.obj
 0002:0000b92c       ??_C@_09FDKNKOOK@TableLock?$AA@ 110b492c     sqlite3.obj
 0002:0000b938       ??_C@_04BNGNMAK@Goto?$AA@  110b4938     sqlite3.obj
 0002:0000b940       ??_C@_08FCKHNOBN@AggFinal?$AA@ 110b4940     sqlite3.obj
 0002:0000b94c       ??_C@_07KGFHIBD@String8?$AA@ 110b494c     sqlite3.obj
 0002:0000b954       ??_C@_06OBLNEDKN@BitNot?$AA@ 110b4954     sqlite3.obj
 0002:0000b95c       ??_C@_06JBKGCNBB@Delete?$AA@ 110b495c     sqlite3.obj
 0002:0000b964       ??_C@_09BKHKEBMD@ResultRow?$AA@ 110b4964     sqlite3.obj
 0002:0000b970       ??_C@_0L@PGPMFKDB@MakeRecord?$AA@ 110b4970     sqlite3.obj
 0002:0000b97c       ??_C@_06ODAFHOMO@Concat?$AA@ 110b497c     sqlite3.obj
 0002:0000b984       ??_C@_09DPOHBCHJ@Remainder?$AA@ 110b4984     sqlite3.obj
 0002:0000b990       ??_C@_06JKMEHOIB@Divide?$AA@ 110b4990     sqlite3.obj
 0002:0000b998       ??_C@_08EOBDLMOI@Multiply?$AA@ 110b4998     sqlite3.obj
 0002:0000b9a4       ??_C@_08DLEJPBEP@Subtract?$AA@ 110b49a4     sqlite3.obj
 0002:0000b9b0       ??_C@_03LDFMNCOE@Add?$AA@  110b49b0     sqlite3.obj
 0002:0000b9b4       ??_C@_0L@DHHFIOFJ@ShiftRight?$AA@ 110b49b4     sqlite3.obj
 0002:0000b9c0       ??_C@_09IIGOLNPP@ShiftLeft?$AA@ 110b49c0     sqlite3.obj
 0002:0000b9cc       ??_C@_05BKBNAGEF@BitOr?$AA@ 110b49cc     sqlite3.obj
 0002:0000b9d4       ??_C@_06PCNOCLJN@BitAnd?$AA@ 110b49d4     sqlite3.obj
 0002:0000b9dc       ??_C@_09ELPHDPAO@DropTable?$AA@ 110b49dc     sqlite3.obj
 0002:0000b9e8       ??_C@_02GNOBCCEK@Ge?$AA@   110b49e8     sqlite3.obj
 0002:0000b9ec       ??_C@_02DCGNOOLL@Lt?$AA@   110b49ec     sqlite3.obj
 0002:0000b9f0       ??_C@_02GBLEMNKL@Le?$AA@   110b49f0     sqlite3.obj
 0002:0000b9f4       ??_C@_02DODIABFK@Gt?$AA@   110b49f4     sqlite3.obj
 0002:0000b9f8       ??_C@_02EAMLCBHB@Eq?$AA@   110b49f8     sqlite3.obj
 0002:0000b9fc       ??_C@_02GCDABJMF@Ne?$AA@   110b49fc     sqlite3.obj
 0002:0000ba00       ??_C@_07HICACDPL@NotNull?$AA@ 110b4a00     sqlite3.obj
 0002:0000ba08       ??_C@_06NBBMPCN@IsNull?$AA@ 110b4a08     sqlite3.obj
 0002:0000ba10       ??_C@_05DALJIPE@IfNot?$AA@ 110b4a10     sqlite3.obj
 0002:0000ba18       ??_C@_06KFINHAKP@MoveLe?$AA@ 110b4a18     sqlite3.obj
 0002:0000ba20       ??_C@_06OBCEMCJB@Vacuum?$AA@ 110b4a20     sqlite3.obj
 0002:0000ba28       ??_C@_03LOMLFHDC@And?$AA@  110b4a28     sqlite3.obj
 0002:0000ba2c       ??_C@_02GGHBPHGE@Or?$AA@   110b4a2c     sqlite3.obj
 0002:0000ba30       ??_C@_09PDNFOMPO@IdxDelete?$AA@ 110b4a30     sqlite3.obj
 0002:0000ba3c       ??_C@_05FMIIHMAD@IdxGE?$AA@ 110b4a3c     sqlite3.obj
 0002:0000ba44       ??_C@_09KDDJLBNF@DropIndex?$AA@ 110b4a44     sqlite3.obj
 0002:0000ba50       ??_C@_0M@JKNINGPB@DropTrigger?$AA@ 110b4a50     sqlite3.obj
 0002:0000ba5c       ??_C@_0M@CKMEEPPD@ContextPush?$AA@ 110b4a5c     sqlite3.obj
 0002:0000ba68       ??_C@_09ILKOCOKG@FifoWrite?$AA@ 110b4a68     sqlite3.obj
 0002:0000ba74       ??_C@_0L@NDDNCBN@ResetCount?$AA@ 110b4a74     sqlite3.obj
 0002:0000ba80       ??_C@_08KLKOBEJ@IdxRowid?$AA@ 110b4a80     sqlite3.obj
 0002:0000ba8c       ??_C@_0L@POHPJECG@IncrVacuum?$AA@ 110b4a8c     sqlite3.obj
 0002:0000ba98       ??_C@_04DKKAEHDH@Last?$AA@ 110b4a98     sqlite3.obj
 0002:0000baa0       ??_C@_0M@BDPOJHGL@CreateTable?$AA@ 110b4aa0     sqlite3.obj
 0002:0000baac       ??_C@_07DOIHNMAE@VColumn?$AA@ 110b4aac     sqlite3.obj
 0002:0000bab4       ??_C@_04PHIBHIIF@Prev?$AA@ 110b4ab4     sqlite3.obj
 0002:0000babc       ??_C@_07EDADKEAH@Integer?$AA@ 110b4abc     sqlite3.obj
 0002:0000bac4       ??_C@_05DLHJCIPI@Gosub?$AA@ 110b4ac4     sqlite3.obj
 0002:0000bacc       ??_C@_09HMMGFEAA@NotExists?$AA@ 110b4acc     sqlite3.obj
 0002:0000bad8       ??_C@_06LJFJMLCE@MemMax?$AA@ 110b4ad8     sqlite3.obj
 0002:0000bae0       ??_C@_07OHPACBNN@RowData?$AA@ 110b4ae0     sqlite3.obj
 0002:0000bae8       ??_C@_09NLAGBMPK@Statement?$AA@ 110b4ae8     sqlite3.obj
 0002:0000baf4       ??_C@_06JHIJIKD@AddImm?$AA@ 110b4af4     sqlite3.obj
 0002:0000bafc       ??_C@_05DAELAPC@IdxLT?$AA@ 110b4afc     sqlite3.obj
 0002:0000bb04       ??_C@_05KEGGNBBF@Rowid?$AA@ 110b4b04     sqlite3.obj
 0002:0000bb0c       ??_C@_04NIFKAFLK@Halt?$AA@ 110b4b0c     sqlite3.obj
 0002:0000bb14       ??_C@_09LLJOBHN@MustBeInt?$AA@ 110b4b14     sqlite3.obj
 0002:0000bb20       ??_C@_05DPPJJBMK@Int64?$AA@ 110b4b20     sqlite3.obj
 0002:0000bb28       ??_C@_08MDBAGECB@NotFound?$AA@ 110b4b28     sqlite3.obj
 0002:0000bb34       ??_C@_08HBKIHNI@IsUnique?$AA@ 110b4b34     sqlite3.obj
 0002:0000bb40       ??_C@_0M@PLDABJLA@CreateIndex?$AA@ 110b4b40     sqlite3.obj
 0002:0000bb4c       ??_C@_05LGELBCGM@Close?$AA@ 110b4b4c     sqlite3.obj
 0002:0000bb54       ??_C@_05JABEJFFA@VOpen?$AA@ 110b4b54     sqlite3.obj
 0002:0000bb5c       ??_C@_0M@IPJMJJPI@ParseSchema?$AA@ 110b4b5c     sqlite3.obj
 0002:0000bb68       ??_C@_07BIPKCCHL@VRename?$AA@ 110b4b68     sqlite3.obj
 0002:0000bb70       ??_C@_0N@KGPEGHPK@RealAffinity?$AA@ 110b4b70     sqlite3.obj
 0002:0000bb80       ??_C@_06ENNEIMBA@String?$AA@ 110b4b80     sqlite3.obj
 0002:0000bb88       ??_C@_08DMMJCAML@Variable?$AA@ 110b4b88     sqlite3.obj
 0002:0000bb94       ??_C@_08FEDJPMPH@NewRowid?$AA@ 110b4b94     sqlite3.obj
 0002:0000bba0       ??_C@_06HCFIKKEA@Return?$AA@ 110b4ba0     sqlite3.obj
 0002:0000bba8       ??_C@_04NBOPPMHE@Noop?$AA@ 110b4ba8     sqlite3.obj
 0002:0000bbb0       ??_C@_05GPHDFMLA@IfNeg?$AA@ 110b4bb0     sqlite3.obj
 0002:0000bbb8       ??_C@_08PHKOHANG@Function?$AA@ 110b4bb8     sqlite3.obj
 0002:0000bbc4       ??_C@_05ILLBNNOP@Trace?$AA@ 110b4bc4     sqlite3.obj
 0002:0000bbcc       ??_C@_04OPMHGHMB@Copy?$AA@ 110b4bcc     sqlite3.obj
 0002:0000bbd4       ??_C@_04DJANFKGA@Sort?$AA@ 110b4bd4     sqlite3.obj
 0002:0000bbdc       ??_C@_03KNKIDPAC@Not?$AA@  110b4bdc     sqlite3.obj
 0002:0000bbe0       ??_C@_0M@KCIGPGBI@IntegrityCk?$AA@ 110b4be0     sqlite3.obj
 0002:0000bbec       ??_C@_0L@BPKAOEDK@AutoCommit?$AA@ 110b4bec     sqlite3.obj
 0002:0000bbf8       ??_C@_06GDNCIOGJ@Expire?$AA@ 110b4bf8     sqlite3.obj
 0002:0000bc00       ??_C@_08FJFCCPFB@OpenRead?$AA@ 110b4c00     sqlite3.obj
 0002:0000bc0c       ??_C@_07MCEFGNMJ@CollSeq?$AA@ 110b4c0c     sqlite3.obj
 0002:0000bc14       ??_C@_06MIMNHDEF@VRowid?$AA@ 110b4c14     sqlite3.obj
 0002:0000bc1c       ??_C@_02EMFCFMID@If?$AA@   110b4c1c     sqlite3.obj
 0002:0000bc20       ??_C@_09FPCAPNBB@OpenWrite?$AA@ 110b4c20     sqlite3.obj
 0002:0000bc2c       ??_C@_05BCDNELCG@SCopy?$AA@ 110b4c2c     sqlite3.obj
 0002:0000bc34       ??_C@_06JIHNENAH@RowKey?$AA@ 110b4c34     sqlite3.obj
 0002:0000bc3c       ??_C@_06PKABLMFO@MoveGt?$AA@ 110b4c3c     sqlite3.obj
 0002:0000bc44       ??_C@_08DOCONEG@Sequence?$AA@ 110b4c44     sqlite3.obj
 0002:0000bc50       ??_C@_09FEDANMPL@SetCookie?$AA@ 110b4c50     sqlite3.obj
 0002:0000bc5c       ??_C@_06FFIACGFC@Column?$AA@ 110b4c5c     sqlite3.obj
 0002:0000bc64       ??_C@_05GOGANBLF@VNext?$AA@ 110b4c64     sqlite3.obj
 0002:0000bc6c       ??_C@_0N@DJJJGBGD@current_date?$AA@ 110b4c6c     sqlite3.obj
 0002:0000bc7c       ??_C@_0BC@DDICBCEN@current_timestamp?$AA@ 110b4c7c     sqlite3.obj
 0002:0000bc90       ??_C@_0N@IPDKEGPB@current_time?$AA@ 110b4c90     sqlite3.obj
 0002:0000bca0       ??_C@_08EPGBJPHJ@strftime?$AA@ 110b4ca0     sqlite3.obj
 0002:0000bcac       ??_C@_08FGNPMIBK@datetime?$AA@ 110b4cac     sqlite3.obj
 0002:0000bcb8       ??_C@_09BPOICPEH@julianday?$AA@ 110b4cb8     sqlite3.obj
 0002:0000bcc4       ??_C@_03CGLHMDPP@now?$AA@  110b4cc4     sqlite3.obj
 0002:0000bcc8       ??_C@_09EKBOCLDN@localtime?$AA@ 110b4cc8     sqlite3.obj
 0002:0000bcd4       ??_C@_09KNIMKLBK@unixepoch?$AA@ 110b4cd4     sqlite3.obj
 0002:0000bce0       ??_C@_03JPHCIIKF@utc?$AA@  110b4ce0     sqlite3.obj
 0002:0000bce4       ??_C@_08IPAOEBNP@weekday?5?$AA@ 110b4ce4     sqlite3.obj
 0002:0000bcf0       ??_C@_09CABLEOFK@start?5of?5?$AA@ 110b4cf0     sqlite3.obj
 0002:0000bcfc       ??_C@_06JGJIJFNK@minute?$AA@ 110b4cfc     sqlite3.obj
 0002:0000bd04       ??_C@_06BJCFNGJP@second?$AA@ 110b4d04     sqlite3.obj
 0002:0000bd0c       ??_C@_0BO@NGNOHJIK@?$CF04d?9?$CF02d?9?$CF02d?5?$CF02d?3?$CF02d?3?$CF02d?$AA@ 110b4d0c     sqlite3.obj
 0002:0000bd2c       ??_C@_0P@PLMNPDMB@?$CF02d?3?$CF02d?3?$CF02d?$AA@ 110b4d2c     sqlite3.obj
 0002:0000bd3c       ??_C@_0P@MCDGMPHH@?$CF04d?9?$CF02d?9?$CF02d?$AA@ 110b4d3c     sqlite3.obj
 0002:0000bd4c       ??_C@_06IAGKDDNE@?$CF06?43f?$AA@ 110b4d4c     sqlite3.obj
 0002:0000bd54       ??_C@_04OHGLKFFN@?$CF03d?$AA@ 110b4d54     sqlite3.obj
 0002:0000bd5c       ??_C@_05CFGAKADK@?$CF?416g?$AA@ 110b4d5c     sqlite3.obj
 0002:0000bd64       ??_C@_04OCCELDNI@?$CF04d?$AA@ 110b4d64     sqlite3.obj
 0002:0000bd6c       ??_C@_03ICJPMMHB@NaN?$AA@  110b4d6c     sqlite3.obj
 0002:0000bd70       ??_C@_04JHHONOOL@?9Inf?$AA@ 110b4d70     sqlite3.obj
 0002:0000bd78       ??_C@_04BIDOCLEL@?$CLInf?$AA@ 110b4d78     sqlite3.obj
 0002:0000bd80       ??_C@_03EJEJBNFP@Inf?$AA@  110b4d80     sqlite3.obj
 0002:0000bd84       ??_C@_06LHGEHABH@?$CINULL?$CJ?$AA@ 110b4d84     sqlite3.obj
 0002:0000bd8c       ??_C@_0BD@FKIFACO@922337203685477580?$AA@ 110b4d8c     sqlite3.obj
 0002:0000bda0       ??_C@_0L@KBKJCPCN@?$CFs?2etilqs_?$AA@ 110b4da0     sqlite3.obj
 0002:0000bdac       ??_C@_01LOCGONAA@?$AA?$AA@ 110b4dac     sqlite3.obj
 0002:0000bdb0       ??_C@_08CADOGOJM@?3memory?3?$AA@ 110b4db0     sqlite3.obj
 0002:0000bdbc       ??_C@_08NFMECEIL@?9journal?$AA@ 110b4dbc     sqlite3.obj
 0002:0000bdc8       ??_C@_09KEIFNIBL@?9stmtjrnl?$AA@ 110b4dc8     sqlite3.obj
 0002:0000bdd4       ??_C@_0BH@LLKFEBHC@invalid?5page?5number?5?$CFd?$AA@ 110b4dd4     sqlite3.obj
 0002:0000bdec       ??_C@_0BJ@HHKCLCDH@2nd?5reference?5to?5page?5?$CFd?$AA@ 110b4dec     sqlite3.obj
 0002:0000be08       ??_C@_0BN@NJCBBLIO@Failed?5to?5read?5ptrmap?5key?$DN?$CFd?$AA@ 110b4e08     sqlite3.obj
 0002:0000be28       ??_C@_0DG@EAEHHDPC@Bad?5ptr?5map?5entry?5key?$DN?$CFd?5expecte@ 110b4e28     sqlite3.obj
 0002:0000be60       ??_C@_0DJ@PBFEOOMP@?$CFd?5of?5?$CFd?5pages?5missing?5from?5over@ 110b4e60     sqlite3.obj
 0002:0000be9c       ??_C@_0BG@GMIBDIEE@failed?5to?5get?5page?5?$CFd?$AA@ 110b4e9c     sqlite3.obj
 0002:0000beb4       ??_C@_0CH@LNHECGJJ@freelist?5leaf?5count?5too?5big?5on?5p@ 110b4eb4     sqlite3.obj
 0002:0000bedc       ??_C@_09OLGIMPDE@Page?5?$CFd?3?5?$AA@ 110b4edc     sqlite3.obj
 0002:0000bee8       ??_C@_0CG@ILLDAEJM@unable?5to?5get?5the?5page?4?5error?5co@ 110b4ee8     sqlite3.obj
 0002:0000bf10       ??_C@_0CN@PPGDAMCK@sqlite3BtreeInitPage?$CI?$CJ?5returns?5e@ 110b4f10     sqlite3.obj
 0002:0000bf40       ??_C@_0BK@DEBKKJM@On?5tree?5page?5?$CFd?5cell?5?$CFd?3?5?$AA@ 110b4f40     sqlite3.obj
 0002:0000bf5c       ??_C@_0BJ@FLOCKNJL@Child?5page?5depth?5differs?$AA@ 110b4f5c     sqlite3.obj
 0002:0000bf78       ??_C@_0BM@FMPLCKPB@On?5page?5?$CFd?5at?5right?5child?3?5?$AA@ 110b4f78     sqlite3.obj
 0002:0000bf94       ??_C@_0CK@JLHLDHFB@Corruption?5detected?5in?5cell?5?$CFd?5o@ 110b4f94     sqlite3.obj
 0002:0000bfc0       ??_C@_0CF@DKGAOHID@Multiple?5uses?5for?5byte?5?$CFd?5of?5pag@ 110b4fc0     sqlite3.obj
 0002:0000bfe8       ??_C@_0DG@NMEFLGAF@Fragmented?5space?5is?5?$CFd?5byte?5repo@ 110b4fe8     sqlite3.obj
 0002:0000c020       ??_C@_0CO@KJCLICBN@Unable?5to?5acquire?5a?5read?5lock?5on@ 110b5020     sqlite3.obj
 0002:0000c050       ??_C@_0BK@JIPGMNFI@Unable?5to?5malloc?5?$CFd?5bytes?$AA@ 110b5050     sqlite3.obj
 0002:0000c06c       ??_C@_0BA@EAICBBKE@Main?5freelist?3?5?$AA@ 110b506c     sqlite3.obj
 0002:0000c07c       ??_C@_0BF@CFAFGJN@List?5of?5tree?5roots?3?5?$AA@ 110b507c     sqlite3.obj
 0002:0000c094       ??_C@_0BG@NJBAMKDO@Page?5?$CFd?5is?5never?5used?$AA@ 110b5094     sqlite3.obj
 0002:0000c0ac       ??_C@_0CC@IBCKHFBM@Pointer?5map?5page?5?$CFd?5is?5reference@ 110b50ac     sqlite3.obj
 0002:0000c0d0       ??_C@_0DP@PJBOOLEO@Outstanding?5page?5count?5goes?5from@ 110b50d0     sqlite3.obj
 0002:0000c110       ??_C@_04BFAHMMK@?$CFlld?$AA@ 110b5110     sqlite3.obj
 0002:0000c118       ??_C@_06NJMDEJD@?$CF?$CB?415g?$AA@ 110b5118     sqlite3.obj
 0002:0000c120       ??_C@_0L@HDAMIFP@keyinfo?$CI?$CFd?$AA@ 110b5120     sqlite3.obj
 0002:0000c12c       ??_C@_0P@BMGKNHBK@collseq?$CI?$CF?420s?$CJ?$AA@ 110b512c     sqlite3.obj
 0002:0000c13c       ??_C@_06BPGFIOAL@?$CFs?$CI?$CFd?$CJ?$AA@ 110b513c     sqlite3.obj
 0002:0000c144       ??_C@_0L@IIBEKKAO@vtab?3?$CFp?3?$CFp?$AA@ 110b5144     sqlite3.obj
 0002:0000c150       ??_C@_04LABILCJL@?$CF?42x?$AA@ 110b5150     sqlite3.obj
 0002:0000c158       ??_C@_09PMECONDC@?$CFs?9mj?$CF08X?$AA@ 110b5158     sqlite3.obj
 0002:0000c164       ??_C@_0DD@BOPMNMAO@unable?5to?5use?5function?5?$CFs?5in?5the@ 110b5164     sqlite3.obj
 0002:0000c198       ??_C@_0CK@OGHLELOO@?5transaction?5?9?5SQL?5statements?5in@ 110b5198     sqlite3.obj
 0002:0000c1c4       ??_C@_08FBLICIPL@rollback?$AA@ 110b51c4     sqlite3.obj
 0002:0000c1d0       ??_C@_06IFNEBLAJ@commit?$AA@ 110b51d0     sqlite3.obj
 0002:0000c1d8       ??_C@_07FILNGEOC@cannot?5?$AA@ 110b51d8     sqlite3.obj
 0002:0000c1e0       ??_C@_0DA@CKKHGBEC@cannot?5start?5a?5transaction?5withi@ 110b51e0     sqlite3.obj
 0002:0000c210       ??_C@_0CL@DIEDEFLK@cannot?5rollback?5?9?5no?5transaction@ 110b5210     sqlite3.obj
 0002:0000c23c       ??_C@_0CJ@LALCBGBP@cannot?5commit?5?9?5no?5transaction?5i@ 110b523c     sqlite3.obj
 0002:0000c268       ??_C@_0BM@FKBOKANJ@database?5schema?5has?5changed?$AA@ 110b5268     sqlite3.obj
 0002:0000c284       ??_C@_0BD@OLGFAFA@sqlite_temp_master?$AA@ 110b5284     sqlite3.obj
 0002:0000c298       ??_C@_0O@JMEKHCEB@sqlite_master?$AA@ 110b5298     sqlite3.obj
 0002:0000c2a8       ??_C@_0DB@OFNJNGCG@SELECT?5name?0?5rootpage?0?5sql?5FROM?5@ 110b52a8     sqlite3.obj
 0002:0000c2dc       ??_C@_0BL@JCFDMLHP@database?5table?5is?5locked?3?5?$AA@ 110b52dc     sqlite3.obj
 0002:0000c2f8       ??_C@_0BA@FFEDMJJH@read?9only?5table?$AA@ 110b52f8     sqlite3.obj
 0002:0000c308       ??_C@_0BH@BEFJIDGM@string?5or?5blob?5too?5big?$AA@ 110b5308     sqlite3.obj
 0002:0000c320       ??_C@_0O@BNNCBLEN@out?5of?5memory?$AA@ 110b5320     sqlite3.obj
 0002:0000c330       ??_C@_0BF@IFOHJMAC@no?5such?5column?3?5?$CC?$CFs?$CC?$AA@ 110b5330     sqlite3.obj
 0002:0000c348       ??_C@_0CH@HDJFDCNH@cannot?5open?5indexed?5column?5for?5w@ 110b5348     sqlite3.obj
 0002:0000c370       ??_C@_04DGGKDJMA@real?$AA@ 110b5370     sqlite3.obj
 0002:0000c378       ??_C@_07LKHFMGFB@integer?$AA@ 110b5378     sqlite3.obj
 0002:0000c380       ??_C@_0BN@OFFACDFM@cannot?5open?5value?5of?5type?5?$CFs?$AA@ 110b5380     sqlite3.obj
 0002:0000c3a0       ??_C@_0BE@PGLAJEIK@no?5such?5rowid?3?5?$CFlld?$AA@ 110b53a0     sqlite3.obj
 0002:0000c3b4       ??_C@_0BI@CBJKLAIG@near?5?$CC?$CFT?$CC?3?5syntax?5error?$AA@ 110b53b4     sqlite3.obj
 0002:0000c3cc       ??_C@_0CL@MAPAMFMM@variable?5number?5must?5be?5between?5@ 110b53cc     sqlite3.obj
 0002:0000c3f8       ??_C@_0BH@KLMBLGJH@too?5many?5SQL?5variables?$AA@ 110b53f8     sqlite3.obj
 0002:0000c410       ??_C@_0BH@HJGFDJPB@too?5many?5columns?5in?5?$CFs?$AA@ 110b5410     sqlite3.obj
 0002:0000c428       ??_C@_07HKAAOBDA@_ROWID_?$AA@ 110b5428     sqlite3.obj
 0002:0000c430       ??_C@_05GIFMDDGN@ROWID?$AA@ 110b5430     sqlite3.obj
 0002:0000c438       ??_C@_03PGJCFEMG@OID?$AA@  110b5438     sqlite3.obj
 0002:0000c43c       ??_C@_03CLCAEGCJ@new?$AA@  110b543c     sqlite3.obj
 0002:0000c440       ??_C@_03PNKCFLFB@old?$AA@  110b5440     sqlite3.obj
 0002:0000c444       ??_C@_0BP@LIGNHLP@misuse?5of?5aliased?5aggregate?5?$CFs?$AA@ 110b5444     sqlite3.obj
 0002:0000c464       ??_C@_0P@OOEELNMH@no?5such?5column?$AA@ 110b5464     sqlite3.obj
 0002:0000c474       ??_C@_0BG@CPPEOILG@ambiguous?5column?5name?$AA@ 110b5474     sqlite3.obj
 0002:0000c48c       ??_C@_0N@GOMHGJCA@?$CFs?3?5?$CFs?4?$CFs?4?$CFs?$AA@ 110b548c     sqlite3.obj
 0002:0000c49c       ??_C@_09DEPFKOIN@?$CFs?3?5?$CFs?4?$CFs?$AA@ 110b549c     sqlite3.obj
 0002:0000c4a8       ??_C@_0CD@CLOCOINF@not?5authorized?5to?5use?5function?3?5@ 110b54a8     sqlite3.obj
 0002:0000c4cc       ??_C@_0CE@JOMBDPK@misuse?5of?5aggregate?5function?5?$CF?4?$CK@ 110b54cc     sqlite3.obj
 0002:0000c4f0       ??_C@_0BH@DEPAIHDK@no?5such?5function?3?5?$CF?4?$CKs?$AA@ 110b54f0     sqlite3.obj
 0002:0000c508       ??_C@_0CN@GBOJIJCC@wrong?5number?5of?5arguments?5to?5fun@ 110b5508     sqlite3.obj
 0002:0000c538       ??_C@_0CL@HPCDGFPK@subqueries?5prohibited?5in?5CHECK?5c@ 110b5538     sqlite3.obj
 0002:0000c564       ??_C@_0CL@HIKOHDBA@parameters?5prohibited?5in?5CHECK?5c@ 110b5564     sqlite3.obj
 0002:0000c590       ??_C@_0DA@HPOBBFJP@Expression?5tree?5is?5too?5large?5?$CIma@ 110b5590     sqlite3.obj
 0002:0000c5c0       ??_C@_0BI@KKBMAAI@misuse?5of?5aggregate?3?5?$CFT?$AA@ 110b55c0     sqlite3.obj
 0002:0000c5d8       ??_C@_0DC@JGGJAPOJ@RAISE?$CI?$CJ?5may?5only?5be?5used?5within?5@ 110b55d8     sqlite3.obj
 0002:0000c60c       ??_C@_08JLBDCDOJ@?$CF?4?$CKs?$CFQ?$CFs?$AA@ 110b560c     sqlite3.obj
 0002:0000c618       ??_C@_07IKCPJJF@name?$DN?$CFQ?$AA@ 110b5618     sqlite3.obj
 0002:0000c620       ??_C@_0O@JAFDLLMD@?$CFs?5OR?5name?$DN?$CFQ?$AA@ 110b5620     sqlite3.obj
 0002:0000c630       ??_C@_0M@FPJBBPLI@tbl_name?$DN?$CFQ?$AA@ 110b5630     sqlite3.obj
 0002:0000c63c       ??_C@_0DL@DAEIJKNC@there?5is?5already?5another?5table?5o@ 110b563c     sqlite3.obj
 0002:0000c678       ??_C@_07IOGLMIPM@sqlite_?$AA@ 110b5678     sqlite3.obj
 0002:0000c680       ??_C@_0BM@IAHFHDLE@table?5?$CFs?5may?5not?5be?5altered?$AA@ 110b5680     sqlite3.obj
 0002:0000c69c       ??_C@_0BL@FIDIAKLG@view?5?$CFs?5may?5not?5be?5altered?$AA@ 110b569c     sqlite3.obj
 0002:0000c6b8       ??_C@_0BHB@KHLCLKBH@UPDATE?5?$CFQ?4?$CFs?5SET?5sql?5?$DN?5CASE?5WHEN@ 110b56b8     sqlite3.obj
 0002:0000c82c       ??_C@_0BA@KDDGKFDH@sqlite_sequence?$AA@ 110b582c     sqlite3.obj
 0002:0000c83c       ??_C@_0DI@HNJIGNMM@UPDATE?5?$CFQ?4sqlite_sequence?5set?5na@ 110b583c     sqlite3.obj
 0002:0000c878       ??_C@_0FM@GJOILOPP@UPDATE?5sqlite_temp_master?5SET?5sq@ 110b5878     sqlite3.obj
 0002:0000c8d4       ??_C@_0CA@KEHKHMLG@Cannot?5add?5a?5PRIMARY?5KEY?5column?$AA@ 110b58d4     sqlite3.obj
 0002:0000c8f4       ??_C@_0BL@NAFLCLKF@Cannot?5add?5a?5UNIQUE?5column?$AA@ 110b58f4     sqlite3.obj
 0002:0000c910       ??_C@_0DF@JACFJFPO@Cannot?5add?5a?5NOT?5NULL?5column?5wit@ 110b5910     sqlite3.obj
 0002:0000c948       ??_C@_0CO@DPKGGDEF@Cannot?5add?5a?5column?5with?5non?9con@ 110b5948     sqlite3.obj
 0002:0000c978       ??_C@_0GL@MPFNILOA@UPDATE?5?$CFQ?4?$CFs?5SET?5sql?5?$DN?5substr?$CIsq@ 110b5978     sqlite3.obj
 0002:0000c9e4       ??_C@_0CC@HCCMFAJP@virtual?5tables?5may?5not?5be?5altere@ 110b59e4     sqlite3.obj
 0002:0000ca08       ??_C@_0BO@IKHDEECD@Cannot?5add?5a?5column?5to?5a?5view?$AA@ 110b5a08     sqlite3.obj
 0002:0000ca28       ??_C@_0N@EIGEIEIJ@sqlite_stat1?$AA@ 110b5a28     sqlite3.obj
 0002:0000ca38       ??_C@_0CL@CNIGKJFK@CREATE?5TABLE?5?$CFQ?4sqlite_stat1?$CItbl@ 110b5a38     sqlite3.obj
 0002:0000ca64       ??_C@_0CJ@MKNMEANI@DELETE?5FROM?5?$CFQ?4sqlite_stat1?5WHER@ 110b5a64     sqlite3.obj
 0002:0000ca90       ??_C@_03GINCELHE@aaa?$AA@  110b5a90     sqlite3.obj
 0002:0000ca94       ??_C@_0CG@NPAKAIJO@SELECT?5idx?0?5stat?5FROM?5?$CFQ?4sqlite_@ 110b5a94     sqlite3.obj
 0002:0000cabc       ??_C@_0BD@CLLJHPMJ@invalid?5name?3?5?$CC?$CFT?$CC?$AA@ 110b5abc     sqlite3.obj
 0002:0000cad0       ??_C@_0CF@FLFLBLIN@too?5many?5attached?5databases?5?9?5ma@ 110b5ad0     sqlite3.obj
 0002:0000caf8       ??_C@_0CK@JEFPBLHB@cannot?5ATTACH?5database?5within?5tr@ 110b5af8     sqlite3.obj
 0002:0000cb24       ??_C@_0BO@FOBANNIG@database?5?$CFs?5is?5already?5in?5use?$AA@ 110b5b24     sqlite3.obj
 0002:0000cb48       ??_C@_0EE@MLIDCBJA@attached?5databases?5must?5use?5the?5@ 110b5b48     sqlite3.obj
 0002:0000cb8c       ??_C@_0BM@JECJFHOP@unable?5to?5open?5database?3?5?$CFs?$AA@ 110b5b8c     sqlite3.obj
 0002:0000cba8       ??_C@_0BF@PJFCJDG@no?5such?5database?3?5?$CFs?$AA@ 110b5ba8     sqlite3.obj
 0002:0000cbc0       ??_C@_0BK@KGABJE@cannot?5detach?5database?5?$CFs?$AA@ 110b5bc0     sqlite3.obj
 0002:0000cbdc       ??_C@_0CK@NCGPBHIO@cannot?5DETACH?5database?5within?5tr@ 110b5bdc     sqlite3.obj
 0002:0000cc08       ??_C@_0BG@HKAEEBEM@database?5?$CFs?5is?5locked?$AA@ 110b5c08     sqlite3.obj
 0002:0000cc20       ??_C@_0O@PDAEIIFA@sqlite_detach?$AA@ 110b5c20     sqlite3.obj
 0002:0000cc30       ??_C@_0O@GJLGHGMJ@sqlite_attach?$AA@ 110b5c30     sqlite3.obj
 0002:0000cc40       ??_C@_0CO@IGOBCPDP@?$CFs?5?$CFT?5cannot?5reference?5objects?5i@ 110b5c40     sqlite3.obj
 0002:0000cc70       ??_C@_0GP@HDJMCODL@illegal?5return?5value?5?$CI?$CFd?$CJ?5from?5t@ 110b5c70     sqlite3.obj
 0002:0000cce0       ??_C@_0CB@NCPGIDCD@access?5to?5?$CFs?4?$CFs?4?$CFs?5is?5prohibited@ 110b5ce0     sqlite3.obj
 0002:0000cd04       ??_C@_0BO@CMCIGPCH@access?5to?5?$CFs?4?$CFs?5is?5prohibited?$AA@ 110b5d04     sqlite3.obj
 0002:0000cd24       ??_C@_0P@PEBGBLCC@not?5authorized?$AA@ 110b5d24     sqlite3.obj
 0002:0000cd34       ??_C@_0N@IAMBEAMM@no?5such?5view?$AA@ 110b5d34     sqlite3.obj
 0002:0000cd44       ??_C@_0O@HKMEEONL@no?5such?5table?$AA@ 110b5d44     sqlite3.obj
 0002:0000cd54       ??_C@_0BE@DADMKDCE@unknown?5database?5?$CFT?$AA@ 110b5d54     sqlite3.obj
 0002:0000cd68       ??_C@_0CK@DHAAGEMP@object?5name?5reserved?5for?5interna@ 110b5d68     sqlite3.obj
 0002:0000cd94       ??_C@_0CJ@GGBIBJLH@temporary?5table?5name?5must?5be?5unq@ 110b5d94     sqlite3.obj
 0002:0000cdc0       ??_C@_0BI@NMBJKJHP@table?5?$CFT?5already?5exists?$AA@ 110b5dc0     sqlite3.obj
 0002:0000cdd8       ??_C@_0CD@FJHICPML@there?5is?5already?5an?5index?5named?5@ 110b5dd8     sqlite3.obj
 0002:0000cdfc       ??_C@_0BH@KPDMNKOM@too?5many?5columns?5on?5?$CFs?$AA@ 110b5dfc     sqlite3.obj
 0002:0000ce14       ??_C@_0BK@CJJKBEHE@duplicate?5column?5name?3?5?$CFs?$AA@ 110b5e14     sqlite3.obj
 0002:0000ce30       ??_C@_0CN@MLPCOIJO@default?5value?5of?5column?5?$FL?$CFs?$FN?5is?5@ 110b5e30     sqlite3.obj
 0002:0000ce60       ??_C@_0CJ@LEOOFHMA@table?5?$CC?$CFs?$CC?5has?5more?5than?5one?5pri@ 110b5e60     sqlite3.obj
 0002:0000ce8c       ??_C@_07EHCIHKNF@INTEGER?$AA@ 110b5e8c     sqlite3.obj
 0002:0000ce94       ??_C@_0DI@IAIBDBA@AUTOINCREMENT?5is?5only?5allowed?5on@ 110b5e94     sqlite3.obj
 0002:0000cecc       ??_C@_0CB@NNGLIIOA@no?5such?5collation?5sequence?3?5?$CF?4?$CKs@ 110b5ecc     sqlite3.obj
 0002:0000cef0       ??_C@_01PKGAHCOL@?$CJ?$AA@ 110b5ef0     sqlite3.obj
 0002:0000cef4       ??_C@_03BMMPKCMF@?6?5?5?$AA@ 110b5ef4     sqlite3.obj
 0002:0000cef8       ??_C@_04PPJIEIMB@?0?6?5?5?$AA@ 110b5ef8     sqlite3.obj
 0002:0000cf00       ??_C@_02EJGPDMNA@?6?$CJ?$AA@ 110b5f00     sqlite3.obj
 0002:0000cf04       ??_C@_0BD@HKJEEOGH@CREATE?5TEMP?5TABLE?5?$AA@ 110b5f04     sqlite3.obj
 0002:0000cf18       ??_C@_0O@BLHKEBID@CREATE?5TABLE?5?$AA@ 110b5f18     sqlite3.obj
 0002:0000cf28       ??_C@_05HJCCDKBG@TABLE?$AA@ 110b5f28     sqlite3.obj
 0002:0000cf30       ??_C@_04CHADEDPO@view?$AA@ 110b5f30     sqlite3.obj
 0002:0000cf38       ??_C@_04OLDJKBIG@VIEW?$AA@ 110b5f38     sqlite3.obj
 0002:0000cf40       ??_C@_0P@BPBAOJCC@CREATE?5?$CFs?5?$CF?4?$CKs?$AA@ 110b5f40     sqlite3.obj
 0002:0000cf50       ??_C@_0FH@BLIGLCKI@UPDATE?5?$CFQ?4?$CFs?5SET?5type?$DN?8?$CFs?8?0?5name@ 110b5f50     sqlite3.obj
 0002:0000cfa8       ??_C@_0CK@BLJIJAMD@CREATE?5TABLE?5?$CFQ?4sqlite_sequence?$CI@ 110b5fa8     sqlite3.obj
 0002:0000cfd4       ??_C@_0O@LAHPKCHN@tbl_name?$DN?8?$CFq?8?$AA@ 110b5fd4     sqlite3.obj
 0002:0000cfe4       ??_C@_0CE@HIMMFEMD@parameters?5are?5not?5allowed?5in?5vi@ 110b5fe4     sqlite3.obj
 0002:0000d008       ??_C@_0BO@BLAOKNKN@view?5?$CFs?5is?5circularly?5defined?$AA@ 110b6008     sqlite3.obj
 0002:0000d028       ??_C@_0DI@GKCMDFKF@UPDATE?5?$CFQ?4?$CFs?5SET?5rootpage?$DN?$CFd?5WHE@ 110b6028     sqlite3.obj
 0002:0000d060       ??_C@_0BM@JEGMLIGC@table?5?$CFs?5may?5not?5be?5dropped?$AA@ 110b6060     sqlite3.obj
 0002:0000d07c       ??_C@_0CC@HNNEDPB@use?5DROP?5TABLE?5to?5delete?5table?5?$CF@ 110b607c     sqlite3.obj
 0002:0000d0a0       ??_C@_0CA@FJIHAAAA@use?5DROP?5VIEW?5to?5delete?5view?5?$CFs?$AA@ 110b60a0     sqlite3.obj
 0002:0000d0c0       ??_C@_0CN@DIEJHGCJ@DELETE?5FROM?5?$CFs?4sqlite_sequence?5W@ 110b60c0     sqlite3.obj
 0002:0000d0f0       ??_C@_0DI@FOLLFOLB@DELETE?5FROM?5?$CFQ?4?$CFs?5WHERE?5tbl_name@ 110b60f0     sqlite3.obj
 0002:0000d128       ??_C@_0DP@HFDIOLMB@foreign?5key?5on?5?$CFs?5should?5referen@ 110b6128     sqlite3.obj
 0002:0000d168       ??_C@_0FO@BDBBNOLJ@number?5of?5columns?5in?5foreign?5key@ 110b6168     sqlite3.obj
 0002:0000d1c8       ??_C@_0CO@ECJPGOGF@unknown?5column?5?$CC?$CFs?$CC?5in?5foreign?5k@ 110b61c8     sqlite3.obj
 0002:0000d1f8       ??_C@_0BP@NPACMCHA@indexed?5columns?5are?5not?5unique?$AA@ 110b61f8     sqlite3.obj
 0002:0000d218       ??_C@_0BM@KIGEJLNH@table?5?$CFs?5may?5not?5be?5indexed?$AA@ 110b6218     sqlite3.obj
 0002:0000d234       ??_C@_0BJ@CFGNJLOC@views?5may?5not?5be?5indexed?$AA@ 110b6234     sqlite3.obj
 0002:0000d250       ??_C@_0CC@FKDNLIPM@virtual?5tables?5may?5not?5be?5indexe@ 110b6250     sqlite3.obj
 0002:0000d274       ??_C@_0CC@CKJEJGLG@there?5is?5already?5a?5table?5named?5?$CF@ 110b6274     sqlite3.obj
 0002:0000d298       ??_C@_0BI@HPCDPJFN@index?5?$CFs?5already?5exists?$AA@ 110b6298     sqlite3.obj
 0002:0000d2b0       ??_C@_03HCMCBFLP@_?$CFd?$AA@ 110b62b0     sqlite3.obj
 0002:0000d2b4       ??_C@_0BC@FCCCAODM@sqlite_autoindex_?$AA@ 110b62b4     sqlite3.obj
 0002:0000d2c8       ??_C@_0CA@MKEFOFFD@table?5?$CFs?5has?5no?5column?5named?5?$CFs?$AA@ 110b62c8     sqlite3.obj
 0002:0000d2e8       ??_C@_0CK@BPKJMBLB@conflicting?5ON?5CONFLICT?5clauses?5@ 110b62e8     sqlite3.obj
 0002:0000d314       ??_C@_07OGDPOKCI@?5UNIQUE?$AA@ 110b6314     sqlite3.obj
 0002:0000d31c       ??_C@_0BE@NHCJMGDI@CREATE?$CFs?5INDEX?5?$CF?4?$CKs?$AA@ 110b631c     sqlite3.obj
 0002:0000d330       ??_C@_0DA@DLDDDEKN@INSERT?5INTO?5?$CFQ?4?$CFs?5VALUES?$CI?8index?8@ 110b6330     sqlite3.obj
 0002:0000d360       ??_C@_09NJDMOIOM@name?$DN?8?$CFq?8?$AA@ 110b6360     sqlite3.obj
 0002:0000d36c       ??_C@_0BC@JBPCAJCH@no?5such?5index?3?5?$CFS?$AA@ 110b636c     sqlite3.obj
 0002:0000d380       ??_C@_0EJ@MFMNFJHB@index?5associated?5with?5UNIQUE?5or?5@ 110b6380     sqlite3.obj
 0002:0000d3cc       ??_C@_0CA@IILCLBDE@DELETE?5FROM?5?$CFQ?4?$CFs?5WHERE?5name?$DN?$CFQ?$AA@ 110b63cc     sqlite3.obj
 0002:0000d3ec       ??_C@_05ILMMJGEC@BEGIN?$AA@ 110b63ec     sqlite3.obj
 0002:0000d3f4       ??_C@_06IBPPMFNL@COMMIT?$AA@ 110b63f4     sqlite3.obj
 0002:0000d3fc       ??_C@_08COBEBGNM@ROLLBACK?$AA@ 110b63fc     sqlite3.obj
 0002:0000d408       ??_C@_0EG@GIEOJFED@unable?5to?5open?5a?5temporary?5datab@ 110b6408     sqlite3.obj
 0002:0000d450       ??_C@_0CO@PMBDNHDC@unable?5to?5identify?5the?5object?5to@ 110b6450     sqlite3.obj
 0002:0000d480       ??_C@_0BP@CGLMEPGG@no?5such?5collation?5sequence?3?5?$CFs?$AA@ 110b6480     sqlite3.obj
 0002:0000d4a0       ??_C@_0BN@GLMOOAMK@table?5?$CFs?5may?5not?5be?5modified?$AA@ 110b64a0     sqlite3.obj
 0002:0000d4c0       ??_C@_0CG@CNPJIJGN@cannot?5modify?5?$CFs?5because?5it?5is?5a@ 110b64c0     sqlite3.obj
 0002:0000d4e8       ??_C@_0N@DAGIBCDP@rows?5deleted?$AA@ 110b64e8     sqlite3.obj
 0002:0000d4f8       ??_C@_04CIMGMMMG@text?$AA@ 110b64f8     sqlite3.obj
 0002:0000d500       ??_C@_04LPJPOBEM@blob?$AA@ 110b6500     sqlite3.obj
 0002:0000d508       ??_C@_0BB@KBEKGHFK@integer?5overflow?$AA@ 110b6508     sqlite3.obj
 0002:0000d51c       ??_C@_04HGGMHPIM@?$CF?4?$CKf?$AA@ 110b651c     sqlite3.obj
 0002:0000d524       ??_C@_0CB@LFIMBCA@LIKE?5or?5GLOB?5pattern?5too?5complex@ 110b6524     sqlite3.obj
 0002:0000d548       ??_C@_0CN@PAMOLCDH@ESCAPE?5expression?5must?5be?5a?5sing@ 110b6548     sqlite3.obj
 0002:0000d578       ??_C@_05JGHLFIHG@MATCH?$AA@ 110b6578     sqlite3.obj
 0002:0000d580       ??_C@_04HPDJJBAE@like?$AA@ 110b6580     sqlite3.obj
 0002:0000d588       ??_C@_04HHHPGODM@glob?$AA@ 110b6588     sqlite3.obj
 0002:0000d590       ??_C@_0DE@HLHNLKJ@table?5?$CFS?5has?5?$CFd?5columns?5but?5?$CFd?5v@ 110b6590     sqlite3.obj
 0002:0000d5c4       ??_C@_0BJ@IABIHKKK@?$CFd?5values?5for?5?$CFd?5columns?$AA@ 110b65c4     sqlite3.obj
 0002:0000d5e0       ??_C@_0CA@HKGLKLIP@table?5?$CFS?5has?5no?5column?5named?5?$CFs?$AA@ 110b65e0     sqlite3.obj
 0002:0000d600       ??_C@_0O@OMFDFDMH@rows?5inserted?$AA@ 110b6600     sqlite3.obj
 0002:0000d610       ??_C@_0BB@CJJGLMJD@?5may?5not?5be?5NULL?$AA@ 110b6610     sqlite3.obj
 0002:0000d624       ??_C@_0BL@MIGFAHKG@PRIMARY?5KEY?5must?5be?5unique?$AA@ 110b6624     sqlite3.obj
 0002:0000d640       ??_C@_08BLECJPKD@columns?5?$AA@ 110b6640     sqlite3.obj
 0002:0000d64c       ??_C@_07OJMCPGAK@column?5?$AA@ 110b664c     sqlite3.obj
 0002:0000d654       ??_C@_02KEGNLNML@?0?5?$AA@ 110b6654     sqlite3.obj
 0002:0000d658       ??_C@_0BA@IJKPAPH@?5are?5not?5unique?$AA@ 110b6658     sqlite3.obj
 0002:0000d668       ??_C@_0P@GKKFBNCL@?5is?5not?5unique?$AA@ 110b6668     sqlite3.obj
 0002:0000d678       ??_C@_0BH@NNAEMFED@sqlite3_extension_init?$AA@ 110b6678     sqlite3.obj
 0002:0000d690       ??_C@_0CD@FENJJFPL@unable?5to?5open?5shared?5library?5?$FL?$CF@ 110b6690     sqlite3.obj
 0002:0000d6b4       ??_C@_0CL@IHPFGADB@no?5entry?5point?5?$FL?$CFs?$FN?5in?5shared?5li@ 110b66b4     sqlite3.obj
 0002:0000d6e0       ??_C@_0CA@BPLHPOIJ@error?5during?5initialization?3?5?$CFs?$AA@ 110b66e0     sqlite3.obj
 0002:0000d700       ??_C@_0CH@EKKEGGML@automatic?5extension?5loading?5fail@ 110b6700     sqlite3.obj
 0002:0000d728       ??_C@_09JJPHINFN@exclusive?$AA@ 110b6728     sqlite3.obj
 0002:0000d734       ??_C@_0M@LPKHOAFP@incremental?$AA@ 110b6734     sqlite3.obj
 0002:0000d740       ??_C@_06HLKELJGF@memory?$AA@ 110b6740     sqlite3.obj
 0002:0000d748       ??_C@_0DO@MAKCDDCJ@temporary?5storage?5cannot?5be?5chan@ 110b6748     sqlite3.obj
 0002:0000d788       ??_C@_03GMLCELFL@?9?$CFT?$AA@ 110b6788     sqlite3.obj
 0002:0000d78c       ??_C@_0BD@EMJOENCP@default_cache_size?$AA@ 110b678c     sqlite3.obj
 0002:0000d7a0       ??_C@_0L@JIGNFOJJ@cache_size?$AA@ 110b67a0     sqlite3.obj
 0002:0000d7ac       ??_C@_09OGOMKHMG@page_size?$AA@ 110b67ac     sqlite3.obj
 0002:0000d7b8       ??_C@_0P@FMLMLOHD@max_page_count?$AA@ 110b67b8     sqlite3.obj
 0002:0000d7c8       ??_C@_0N@NOOMDJH@locking_mode?$AA@ 110b67c8     sqlite3.obj
 0002:0000d7d8       ??_C@_0M@ENMLGDH@auto_vacuum?$AA@ 110b67d8     sqlite3.obj
 0002:0000d7e4       ??_C@_0BD@IEMDKFHA@incremental_vacuum?$AA@ 110b67e4     sqlite3.obj
 0002:0000d7f8       ??_C@_0L@JEPCDDIC@temp_store?$AA@ 110b67f8     sqlite3.obj
 0002:0000d804       ??_C@_0BF@OPALIJKE@temp_store_directory?$AA@ 110b6804     sqlite3.obj
 0002:0000d81c       ??_C@_0BJ@INLPNACB@not?5a?5writable?5directory?$AA@ 110b681c     sqlite3.obj
 0002:0000d838       ??_C@_0M@GKGFOGDE@synchronous?$AA@ 110b6838     sqlite3.obj
 0002:0000d844       ??_C@_0DF@GMDBDCKL@Safety?5level?5may?5not?5be?5changed?5@ 110b6844     sqlite3.obj
 0002:0000d87c       ??_C@_0L@NEMFJAGM@table_info?$AA@ 110b687c     sqlite3.obj
 0002:0000d888       ??_C@_03LBLPCGAC@cid?$AA@  110b6888     sqlite3.obj
 0002:0000d88c       ??_C@_07EAJHGOKJ@notnull?$AA@ 110b688c     sqlite3.obj
 0002:0000d894       ??_C@_0L@KNDFGGNJ@dflt_value?$AA@ 110b6894     sqlite3.obj
 0002:0000d8a0       ??_C@_02NCEGPMNB@pk?$AA@   110b68a0     sqlite3.obj
 0002:0000d8a4       ??_C@_0L@CKPANNIC@index_info?$AA@ 110b68a4     sqlite3.obj
 0002:0000d8b0       ??_C@_05OBPGIPLF@seqno?$AA@ 110b68b0     sqlite3.obj
 0002:0000d8b8       ??_C@_0L@MMBMMAEK@index_list?$AA@ 110b68b8     sqlite3.obj
 0002:0000d8c4       ??_C@_03NPAJGOON@seq?$AA@  110b68c4     sqlite3.obj
 0002:0000d8c8       ??_C@_06ODCMFGLL@unique?$AA@ 110b68c8     sqlite3.obj
 0002:0000d8d0       ??_C@_0O@EBMNDACF@database_list?$AA@ 110b68d0     sqlite3.obj
 0002:0000d8e0       ??_C@_0P@KOJNIGCH@collation_list?$AA@ 110b68e0     sqlite3.obj
 0002:0000d8f0       ??_C@_0BB@KJMCGNAI@foreign_key_list?$AA@ 110b68f0     sqlite3.obj
 0002:0000d904       ??_C@_02EGCJHIOB@id?$AA@   110b6904     sqlite3.obj
 0002:0000d908       ??_C@_04HNEBHLOP@from?$AA@ 110b6908     sqlite3.obj
 0002:0000d910       ??_C@_02LBCDJBAJ@to?$AA@   110b6910     sqlite3.obj
 0002:0000d914       ??_C@_0BE@LKBHCIHN@case_sensitive_like?$AA@ 110b6914     sqlite3.obj
 0002:0000d928       ??_C@_0BA@EDNFHOBJ@integrity_check?$AA@ 110b6928     sqlite3.obj
 0002:0000d938       ??_C@_0M@EDPCDMIO@quick_check?$AA@ 110b6938     sqlite3.obj
 0002:0000d944       ??_C@_0BI@FOLPKNAK@?$CK?$CK?$CK?5in?5database?5?$CFs?5?$CK?$CK?$CK?6?$AA@ 110b6944     sqlite3.obj
 0002:0000d95c       ??_C@_06DHEAJPAE@rowid?5?$AA@ 110b695c     sqlite3.obj
 0002:0000d964       ??_C@_0BF@JGBLFHJL@?5missing?5from?5index?5?$AA@ 110b6964     sqlite3.obj
 0002:0000d97c       ??_C@_0BN@JKHLHJNK@wrong?5?$CD?5of?5entries?5in?5index?5?$AA@ 110b697c     sqlite3.obj
 0002:0000d99c       ??_C@_02MFDMBIJM@ok?$AA@   110b699c     sqlite3.obj
 0002:0000d9a0       ??_C@_08MLPGAEIK@encoding?$AA@ 110b69a0     sqlite3.obj
 0002:0000d9ac       ??_C@_0BJ@GJBMJNNI@unsupported?5encoding?3?5?$CFs?$AA@ 110b69ac     sqlite3.obj
 0002:0000d9c8       ??_C@_0P@JGMMHBPP@schema_version?$AA@ 110b69c8     sqlite3.obj
 0002:0000d9d8       ??_C@_0N@MPKCHLKL@user_version?$AA@ 110b69d8     sqlite3.obj
 0002:0000d9e8       ??_C@_0P@GDKICNML@freelist_count?$AA@ 110b69e8     sqlite3.obj
 0002:0000d9f8       ??_C@_03NLJIHOMM@?5?9?5?$AA@ 110b69f8     sqlite3.obj
 0002:0000d9fc       ??_C@_0BK@KDGONMLG@malformed?5database?5schema?$AA@ 110b69fc     sqlite3.obj
 0002:0000da18       ??_C@_06FJHKNKMG@BINARY?$AA@ 110b6a18     sqlite3.obj
 0002:0000da20       ??_C@_0BI@FFDCNLCF@unsupported?5file?5format?$AA@ 110b6a20     sqlite3.obj
 0002:0000da38       ??_C@_0CI@FDECACCL@SELECT?5name?0?5rootpage?0?5sql?5FROM?5@ 110b6a38     sqlite3.obj
 0002:0000da60       ??_C@_0BO@EBFEALBC@database?5schema?5is?5locked?3?5?$CFs?$AA@ 110b6a60     sqlite3.obj
 0002:0000da80       ??_C@_05NDNMCCJH@order?$AA@ 110b6a80     sqlite3.obj
 0002:0000da88       ??_C@_06EENFNEPD@detail?$AA@ 110b6a88     sqlite3.obj
 0002:0000da90       ??_C@_04HLBMEOMD@addr?$AA@ 110b6a90     sqlite3.obj
 0002:0000da98       ??_C@_06POMMAHJK@opcode?$AA@ 110b6a98     sqlite3.obj
 0002:0000daa0       ??_C@_02JCBCEJAP@p1?$AA@   110b6aa0     sqlite3.obj
 0002:0000daa4       ??_C@_02LJDPBKMM@p2?$AA@   110b6aa4     sqlite3.obj
 0002:0000daa8       ??_C@_02KACECLIN@p3?$AA@   110b6aa8     sqlite3.obj
 0002:0000daac       ??_C@_02OPGFLNEK@p4?$AA@   110b6aac     sqlite3.obj
 0002:0000dab0       ??_C@_02PGHOIMAL@p5?$AA@   110b6ab0     sqlite3.obj
 0002:0000dab4       ??_C@_07GJGNEJFD@comment?$AA@ 110b6ab4     sqlite3.obj
 0002:0000dabc       ??_C@_0CN@CENKDKHG@unknown?5or?5unsupported?5join?5type@ 110b6abc     sqlite3.obj
 0002:0000daec       ??_C@_0DH@LJEHIDDA@RIGHT?5and?5FULL?5OUTER?5JOINs?5are?5n@ 110b6aec     sqlite3.obj
 0002:0000db24       ??_C@_04ODDMBDHP@?$CC?$CFw?$CC?$AA@ 110b6b24     sqlite3.obj
 0002:0000db2c       ??_C@_0DC@NBGJANJH@a?5NATURAL?5join?5may?5not?5have?5an?5O@ 110b6b2c     sqlite3.obj
 0002:0000db60       ??_C@_0DH@DHMOHNCE@cannot?5have?5both?5ON?5and?5USING?5cl@ 110b6b60     sqlite3.obj
 0002:0000db98       ??_C@_0EA@LFCKDDII@cannot?5join?5using?5column?5?$CFs?5?9?5co@ 110b6b98     sqlite3.obj
 0002:0000dbd8       ??_C@_0EI@FMCKEHHB@only?5a?5single?5result?5allowed?5for@ 110b6bd8     sqlite3.obj
 0002:0000dc20       ??_C@_04OEPMCOLO@TEXT?$AA@ 110b6c20     sqlite3.obj
 0002:0000dc28       ??_C@_05KDMKNECD@rowid?$AA@ 110b6c28     sqlite3.obj
 0002:0000dc30       ??_C@_08OHGGEHKA@column?$CFd?$AA@ 110b6c30     sqlite3.obj
 0002:0000dc3c       ??_C@_09CDPONBKL@UNION?5ALL?$AA@ 110b6c3c     sqlite3.obj
 0002:0000dc48       ??_C@_09JBOBNLLF@INTERSECT?$AA@ 110b6c48     sqlite3.obj
 0002:0000dc54       ??_C@_06JFIPMMLD@EXCEPT?$AA@ 110b6c54     sqlite3.obj
 0002:0000dc5c       ??_C@_05GJNJOPB@UNION?$AA@ 110b6c5c     sqlite3.obj
 0002:0000dc64       ??_C@_02OAOPDKLG@?$CFT?$AA@ 110b6c64     sqlite3.obj
 0002:0000dc68       ??_C@_05KLPAANK@?$CFz?3?$CFd?$AA@ 110b6c68     sqlite3.obj
 0002:0000dc70       ??_C@_0BE@EGABPGJI@sqlite_subquery_?$CFp_?$AA@ 110b6c70     sqlite3.obj
 0002:0000dc84       ??_C@_05NNFHCGPF@?$CFs?4?$CFs?$AA@ 110b6c84     sqlite3.obj
 0002:0000dc8c       ??_C@_0BC@OFCALFBN@no?5such?5table?3?5?$CFs?$AA@ 110b6c8c     sqlite3.obj
 0002:0000dca0       ??_C@_0BE@EGLAAHPP@no?5tables?5specified?$AA@ 110b6ca0     sqlite3.obj
 0002:0000dcb4       ??_C@_0BP@JFMLENOH@too?5many?5columns?5in?5result?5set?$AA@ 110b6cb4     sqlite3.obj
 0002:0000dcd4       ??_C@_05BIEKMFNJ@ORDER?$AA@ 110b6cd4     sqlite3.obj
 0002:0000dcdc       ??_C@_05NAIABEH@GROUP?$AA@ 110b6cdc     sqlite3.obj
 0002:0000dce4       ??_C@_0BP@OLNMGBH@too?5many?5terms?5in?5?$CFs?5BY?5clause?$AA@ 110b6ce4     sqlite3.obj
 0002:0000dd04       ??_C@_0DI@IJOLPLNO@?$CFr?5?$CFs?5BY?5term?5out?5of?5range?5?9?5sho@ 110b6d04     sqlite3.obj
 0002:0000dd3c       ??_C@_0CC@GEJJPDIE@too?5many?5terms?5in?5ORDER?5BY?5claus@ 110b6d3c     sqlite3.obj
 0002:0000dd60       ??_C@_0DL@PHMENBPN@?$CFr?5ORDER?5BY?5term?5out?5of?5range?5?9?5@ 110b6d60     sqlite3.obj
 0002:0000dd9c       ??_C@_0DN@KHANHMIL@?$CFr?5ORDER?5BY?5term?5does?5not?5match?5@ 110b6d9c     sqlite3.obj
 0002:0000dddc       ??_C@_0DA@GPNKNMMI@ORDER?5BY?5clause?5should?5come?5afte@ 110b6ddc     sqlite3.obj
 0002:0000de0c       ??_C@_0CN@DDIHOHHL@LIMIT?5clause?5should?5come?5after?5?$CF@ 110b6e0c     sqlite3.obj
 0002:0000de40       ??_C@_0FC@CMDCIIHA@SELECTs?5to?5the?5left?5and?5right?5of@ 110b6e40     sqlite3.obj
 0002:0000de94       ??_C@_0CM@CFGBPLAG@a?5GROUP?5BY?5clause?5is?5required?5be@ 110b6e94     sqlite3.obj
 0002:0000dec0       ??_C@_0DL@LDIIFJFH@aggregate?5functions?5are?5not?5allo@ 110b6ec0     sqlite3.obj
 0002:0000defc       ??_C@_0DI@BMJPLCG@DISTINCT?5in?5aggregate?5must?5be?5fo@ 110b6efc     sqlite3.obj
 0002:0000df34       ??_C@_0CC@DHLFNDIF@too?5many?5terms?5in?5compound?5SELEC@ 110b6f34     sqlite3.obj
 0002:0000df58       ??_C@_0EB@PHGCKHIG@sqlite3_get_table?$CI?$CJ?5called?5with?5@ 110b6f58     sqlite3.obj
 0002:0000df9c       ??_C@_0CO@CGGBEMGD@temporary?5trigger?5may?5not?5have?5q@ 110b6f9c     sqlite3.obj
 0002:0000dfcc       ??_C@_07DIDNFGDE@trigger?$AA@ 110b6fcc     sqlite3.obj
 0002:0000dfd4       ??_C@_0CJ@KLDCMPKB@cannot?5create?5triggers?5on?5virtua@ 110b6fd4     sqlite3.obj
 0002:0000e000       ??_C@_0BK@IACDKJFA@trigger?5?$CFT?5already?5exists?$AA@ 110b7000     sqlite3.obj
 0002:0000e01c       ??_C@_0CG@JAGCNIHD@cannot?5create?5trigger?5on?5system?5@ 110b701c     sqlite3.obj
 0002:0000e044       ??_C@_06BIGAHLBC@BEFORE?$AA@ 110b7044     sqlite3.obj
 0002:0000e04c       ??_C@_05OHDJMCHE@AFTER?$AA@ 110b704c     sqlite3.obj
 0002:0000e054       ??_C@_0CF@CNPIEMED@cannot?5create?5?$CFs?5trigger?5on?5view@ 110b7054     sqlite3.obj
 0002:0000e07c       ??_C@_0CO@GJNALGCE@cannot?5create?5INSTEAD?5OF?5trigger@ 110b707c     sqlite3.obj
 0002:0000e0b0       ??_C@_0EA@IJNEMIHP@INSERT?5INTO?5?$CFQ?4?$CFs?5VALUES?$CI?8trigge@ 110b70b0     sqlite3.obj
 0002:0000e0f0       ??_C@_0BN@JFPIJHCG@type?$DN?8trigger?8?5AND?5name?$DN?8?$CFq?8?$AA@ 110b70f0     sqlite3.obj
 0002:0000e110       ??_C@_0BE@ELCABEID@no?5such?5trigger?3?5?$CFS?$AA@ 110b7110     sqlite3.obj
 0002:0000e124       ??_C@_0O@JKBKLFDA@?9?9?5TRIGGER?5?$CFs?$AA@ 110b7124     sqlite3.obj
 0002:0000e134       ??_C@_0BD@IEIMFPKF@no?5such?5column?3?5?$CFs?$AA@ 110b7134     sqlite3.obj
 0002:0000e148       ??_C@_0N@KMEMLEEO@rows?5updated?$AA@ 110b7148     sqlite3.obj
 0002:0000e158       ??_C@_07OLKPBLEA@_rowid_?$AA@ 110b7158     sqlite3.obj
 0002:0000e160       ??_C@_0CI@CPMJIPOI@cannot?5VACUUM?5from?5within?5a?5tran@ 110b7160     sqlite3.obj
 0002:0000e188       ??_C@_0BI@OOHLJPLG@ATTACH?5?8?8?5AS?5vacuum_db?$DL?$AA@ 110b7188     sqlite3.obj
 0002:0000e1a0       ??_C@_0CB@NBNOHMDI@PRAGMA?5vacuum_db?4synchronous?$DNOFF@ 110b71a0     sqlite3.obj
 0002:0000e1c4       ??_C@_0BB@JEGCAHMF@BEGIN?5EXCLUSIVE?$DL?$AA@ 110b71c4     sqlite3.obj
 0002:0000e1d8       ??_C@_0II@FEBAKHNN@SELECT?5?8CREATE?5TABLE?5vacuum_db?4?8@ 110b71d8     sqlite3.obj
 0002:0000e260       ??_C@_0GI@FEDHFMIE@SELECT?5?8CREATE?5INDEX?5vacuum_db?4?8@ 110b7260     sqlite3.obj
 0002:0000e2c8       ??_C@_0HG@GKDDPPFI@SELECT?5?8CREATE?5UNIQUE?5INDEX?5vacu@ 110b72c8     sqlite3.obj
 0002:0000e340       ??_C@_0KO@HAGDHKLJ@SELECT?5?8INSERT?5INTO?5vacuum_db?4?8?5@ 110b7340     sqlite3.obj
 0002:0000e3f0       ??_C@_0HB@CJENIKHO@SELECT?5?8DELETE?5FROM?5vacuum_db?4?8?5@ 110b73f0     sqlite3.obj
 0002:0000e468       ??_C@_0JG@FGPGEBNJ@SELECT?5?8INSERT?5INTO?5vacuum_db?4?8?5@ 110b7468     sqlite3.obj
 0002:0000e500       ??_C@_0LD@KNCLPPMC@INSERT?5INTO?5vacuum_db?4sqlite_mas@ 110b7500     sqlite3.obj
 0002:0000e5b4       ??_C@_0CP@FJGAICJB@Cannot?5use?5virtual?5tables?5in?5sha@ 110b75b4     sqlite3.obj
 0002:0000e5e4       ??_C@_0BI@PDMEEOA@CREATE?5VIRTUAL?5TABLE?5?$CFT?$AA@ 110b75e4     sqlite3.obj
 0002:0000e600       ??_C@_0FI@IFIJAFLJ@UPDATE?5?$CFQ?4?$CFs?5SET?5type?$DN?8table?8?0?5n@ 110b7600     sqlite3.obj
 0002:0000e658       ??_C@_0BO@DEKEKMPI@vtable?5constructor?5failed?3?5?$CFs?$AA@ 110b7658     sqlite3.obj
 0002:0000e678       ??_C@_0CO@NAIIFAKI@vtable?5constructor?5did?5not?5decla@ 110b7678     sqlite3.obj
 0002:0000e6a8       ??_C@_06JIKFICKK@hidden?$AA@ 110b76a8     sqlite3.obj
 0002:0000e6b0       ??_C@_07JJJNOAOL@?5hidden?$AA@ 110b76b0     sqlite3.obj
 0002:0000e6b8       ??_C@_0BD@KBJCCNMM@no?5such?5module?3?5?$CFs?$AA@ 110b76b8     sqlite3.obj
 0002:0000e6cc       ??_C@_0BM@BLDEAGOK@at?5most?5?$CFd?5tables?5in?5a?5join?$AA@ 110b76cc     sqlite3.obj
 0002:0000e6e8       ??_C@_08HCMEEBCG@TABLE?5?$CFs?$AA@ 110b76e8     sqlite3.obj
 0002:0000e6f4       ??_C@_08CKMPFKL@?$CFz?5AS?5?$CFs?$AA@ 110b76f4     sqlite3.obj
 0002:0000e700       ??_C@_0BB@BIEKKNLE@?$CFz?5WITH?5INDEX?5?$CFs?$AA@ 110b7700     sqlite3.obj
 0002:0000e714       ??_C@_0BF@ILEGLOOO@?$CFz?5USING?5PRIMARY?5KEY?$AA@ 110b7714     sqlite3.obj
 0002:0000e72c       ??_C@_0BN@GIJPKDIL@?$CFz?5VIRTUAL?5TABLE?5INDEX?5?$CFd?3?$CFs?$AA@ 110b772c     sqlite3.obj
 0002:0000e74c       ??_C@_0M@FEBHOCCB@?$CFz?5ORDER?5BY?$AA@ 110b774c     sqlite3.obj
 0002:0000e758       ??_C@_0BG@FMAEELCM@parser?5stack?5overflow?$AA@ 110b7758     sqlite3.obj
 0002:0000e770       ??_C@_08FAFAADKO@set?5list?$AA@ 110b7770     sqlite3.obj
 0002:0000e77c       ??_C@_0CC@BHLMPGNH@too?5many?5arguments?5on?5function?5?$CF@ 110b777c     sqlite3.obj
 0002:0000e7a0       ??_C@_09NCAJIFEE@interrupt?$AA@ 110b77a0     sqlite3.obj
 0002:0000e7ac       ??_C@_0BJ@EMNEDDKJ@unrecognized?5token?3?5?$CC?$CFT?$CC?$AA@ 110b77ac     sqlite3.obj
 0002:0000e7c8       ??_C@_04FGEHGIFJ@temp?$AA@ 110b77c8     sqlite3.obj
 0002:0000e7d0       ??_C@_09CAHPDAG@temporary?$AA@ 110b77d0     sqlite3.obj
 0002:0000e7dc       ??_C@_07LFFDKBGI@explain?$AA@ 110b77dc     sqlite3.obj
 0002:0000e7e4       ??_C@_0CO@MAICLPMM@Unable?5to?5close?5due?5to?5unfinalis@ 110b77e4     sqlite3.obj
 0002:0000e814       ??_C@_0N@FKKFHCIB@not?5an?5error?$AA@ 110b7814     sqlite3.obj
 0002:0000e824       ??_C@_0CE@BCMAPMOL@SQL?5logic?5error?5or?5missing?5datab@ 110b7824     sqlite3.obj
 0002:0000e848       ??_C@_0BJ@OFHFLJKH@access?5permission?5denied?$AA@ 110b7848     sqlite3.obj
 0002:0000e864       ??_C@_0BP@BFMDEDKN@callback?5requested?5query?5abort?$AA@ 110b7864     sqlite3.obj
 0002:0000e884       ??_C@_0BD@DAAAMHOI@database?5is?5locked?$AA@ 110b7884     sqlite3.obj
 0002:0000e898       ??_C@_0BJ@DNPONIEG@database?5table?5is?5locked?$AA@ 110b7898     sqlite3.obj
 0002:0000e8b4       ??_C@_0CF@JBLJEMGC@attempt?5to?5write?5a?5readonly?5data@ 110b78b4     sqlite3.obj
 0002:0000e8dc       ??_C@_0M@EGEKIIMP@interrupted?$AA@ 110b78dc     sqlite3.obj
 0002:0000e8e8       ??_C@_0P@FOPPKBJH@disk?5I?1O?5error?$AA@ 110b78e8     sqlite3.obj
 0002:0000e8f8       ??_C@_0CB@ONDDCPGK@database?5disk?5image?5is?5malformed@ 110b78f8     sqlite3.obj
 0002:0000e91c       ??_C@_0BJ@GDNBBAEL@database?5or?5disk?5is?5full?$AA@ 110b791c     sqlite3.obj
 0002:0000e938       ??_C@_0BN@JLONMGIA@unable?5to?5open?5database?5file?$AA@ 110b7938     sqlite3.obj
 0002:0000e958       ??_C@_0BH@OCNELEJF@table?5contains?5no?5data?$AA@ 110b7958     sqlite3.obj
 0002:0000e970       ??_C@_0CD@CFCKODOJ@String?5or?5BLOB?5exceeded?5size?5lim@ 110b7970     sqlite3.obj
 0002:0000e994       ??_C@_0BC@IFKPGMGK@constraint?5failed?$AA@ 110b7994     sqlite3.obj
 0002:0000e9a8       ??_C@_0BC@FILINGOB@datatype?5mismatch?$AA@ 110b79a8     sqlite3.obj
 0002:0000e9bc       ??_C@_0CH@GCDGLLPA@library?5routine?5called?5out?5of?5se@ 110b79bc     sqlite3.obj
 0002:0000e9e4       ??_C@_0CA@GPEHDHDC@kernel?5lacks?5large?5file?5support?$AA@ 110b79e4     sqlite3.obj
 0002:0000ea04       ??_C@_0BF@LMCDAPDN@authorization?5denied?$AA@ 110b7a04     sqlite3.obj
 0002:0000ea1c       ??_C@_0CA@DBBJFBEG@auxiliary?5database?5format?5error?$AA@ 110b7a1c     sqlite3.obj
 0002:0000ea3c       ??_C@_0CC@OHMKLHEA@bind?5or?5column?5index?5out?5of?5rang@ 110b7a3c     sqlite3.obj
 0002:0000ea60       ??_C@_0CH@JKOMOHHH@file?5is?5encrypted?5or?5is?5not?5a?5da@ 110b7a60     sqlite3.obj
 0002:0000ea88       ??_C@_0O@BFJCFAAK@unknown?5error?$AA@ 110b7a88     sqlite3.obj
 0002:0000ea98       ??_C@_0P@OGLLBPDH@bad?5parameters?$AA@ 110b7a98     sqlite3.obj
 0002:0000eaa8       ??_C@_0DP@FEHMPAL@Unable?5to?5delete?1modify?5user?9fun@ 110b7aa8     sqlite3.obj
 0002:0000eae8       ??_C@_0BB@ICOLFIAA@unknown?5encoding?$AA@ 110b7ae8     sqlite3.obj
 0002:0000eb00       ??_C@_0EE@JLKKONPB@Unable?5to?5delete?1modify?5collatio@ 110b7b00     sqlite3.obj
 0002:0000eb44       ??_C@_0BA@JNKNNOBA@no?5such?5vfs?3?5?$CFs?$AA@ 110b7b44     sqlite3.obj
 0002:0000eb54       ??_C@_05JJHANOIF@RTRIM?$AA@ 110b7b54     sqlite3.obj
 0002:0000eb5c       ??_C@_06FHKGKAHE@NOCASE?$AA@ 110b7b5c     sqlite3.obj
 0002:0000eb64       ??_C@_0BL@NLBFJAPJ@PRAGMA?5encoding?5?$DN?5?8UTF?916?8?$AA@ 110b7b64     sqlite3.obj
 0002:0000eb80       __real@4024000000000000    110b7b80      CIL library: CIL module
 0002:0000eb88       __real@3ff0000000000000    110b7b88      CIL library: CIL module
 0002:0000eb90       __real@4141978ac0000000    110b7b90      CIL library: CIL module
 0002:0000eb98       __real@3d745c7fe3bc40b0    110b7b98      CIL library: CIL module
 0002:0000eba0       __real@41f0000000000000    110b7ba0      CIL library: CIL module
 0002:0000eba8       __real@40c3880000000000    110b7ba8      CIL library: CIL module
 0002:0000ebb0       __real@4341c37937e08000    110b7bb0      CIL library: CIL module
 0002:0000ebb8       __real@4d384f03e93ff9f5    110b7bb8      CIL library: CIL module
 0002:0000ebc0       __real@0000000000000000    110b7bc0      CIL library: CIL module
 0002:0000ebc8       __real@403e99a027525461    110b7bc8      CIL library: CIL module
 0002:0000ebd0       __real@3fa0bb627b5c1c3f    110b7bd0      CIL library: CIL module
 0002:0000ebd8       __real@4076d40000000000    110b7bd8      CIL library: CIL module
 0002:0000ebe0       __real@3f666db072f2284d    110b7be0      CIL library: CIL module
 0002:0000ebe8       __real@405e866666666666    110b7be8      CIL library: CIL module
 0002:0000ebf0       __real@3efcb5835e647c31    110b7bf0      CIL library: CIL module
 0002:0000ebf8       __real@413c7dd040000000    110b7bf8      CIL library: CIL module
 0002:0000ec00       __real@3fe0000000000000    110b7c00      CIL library: CIL module
 0002:0000ec08       __real@3ee845c8a0ce5129    110b7c08      CIL library: CIL module
 0002:0000ec10       __real@40ac200000000000    110b7c10      CIL library: CIL module
 0002:0000ec18       __real@404e000000000000    110b7c18      CIL library: CIL module
 0002:0000ec20       __real@4097d20000000000    110b7c20      CIL library: CIL module
 0002:0000ec28       __real@c03e99a027525461    110b7c28      CIL library: CIL module
 0002:0000ec30       __real@3f50624dd2f1a9fc    110b7c30      CIL library: CIL module
 0002:0000ec38       __real@4194997000000000    110b7c38      CIL library: CIL module
 0002:0000ec40       __real@bf800000            110b7c40      CIL library: CIL module
 0002:0000ec44       __real@40000000            110b7c44      CIL library: CIL module
 0002:0000ec48       __real@41a00000            110b7c48      CIL library: CIL module
 0002:0000ec4c       __real@447a0000            110b7c4c      CIL library: CIL module
 0002:0000ec50       __real@459c4000            110b7c50      CIL library: CIL module
 0002:0000ec58       __real@4048000000000000    110b7c58      CIL library: CIL module
 0002:0000ec60       __real@3949f623d5a8a733    110b7c60      CIL library: CIL module
 0002:0000ec68       __real@3e45798ee2308c3a    110b7c68      CIL library: CIL module
 0002:0000ec70       __real@4197d78400000000    110b7c70      CIL library: CIL module
 0002:0000ec78       __real@4693b8b5b5056e17    110b7c78      CIL library: CIL module
 0002:0000ec80       __real@3fb999999999999a    110b7c80      CIL library: CIL module
 0002:0000ec88       __real@40f5180000000000    110b7c88      CIL library: CIL module
 0002:0000ec90       __real@41429ec5c0000000    110b7c90      CIL library: CIL module
 0002:0000ec98       __real@403e000000000000    110b7c98      CIL library: CIL module
 0002:0000eca0       __real@3f46c16c16c16c17    110b7ca0      CIL library: CIL module
 0002:0000eca8       __real@3fa5555555555555    110b7ca8      CIL library: CIL module
 0002:0000ecb0       __real@3ff8000000000000    110b7cb0      CIL library: CIL module
 0002:0000ecb8       __real@401c000000000000    110b7cb8      CIL library: CIL module
 0002:0000ecc0       __real@546d42aea2879f2e    110b7cc0      CIL library: CIL module
 0002:0000ecc8       __real@404dffdf3b645a1d    110b7cc8      CIL library: CIL module
 0002:0000ecd0       __real@bff0000000000000    110b7cd0      CIL library: CIL module
 0002:0000ecd8       __real@4039000000000000    110b7cd8      CIL library: CIL module
 0002:0000ece0       __real@3fd5555555555555    110b7ce0      CIL library: CIL module
 0002:0000ece8       __real@4069000000000000    110b7ce8      CIL library: CIL module
 0002:0000ecf0       __real@547d42aea2879f2e    110b7cf0      CIL library: CIL module
 0002:0000ecf8       __real@400921fb54442d18    110b7cf8      CIL library: CIL module
 0002:0000ed00       __real@3f00002000400080    110b7d00      CIL library: CIL module
 0002:0000ed08       __real@3f91df46a2529d39    110b7d08      CIL library: CIL module
 0002:0000ed10       __real@404ca5dc1a63c1f8    110b7d10      CIL library: CIL module
 0002:0000ed18       __real@3f50000000000000    110b7d18      CIL library: CIL module
 0002:0000ed20       __real@42d3a52453c00000    110b7d20      CIL library: CIL module
 0002:000126c8       __DEFAULT_CW_in_mem        110bb6c8     LIBCMT:_common_.obj
 0002:000126ca       __pi_by_2_to_61            110bb6ca     LIBCMT:_common_.obj
 0002:00015740       __load_config_used         110be740     LIBCMT:loadcfg.obj
 0002:000157d4       ??_R4exception@std@@6B@    110be7d4     LIBCMT:stdexcpt.obj
 0002:000157e8       ??_R4type_info@@6B@        110be7e8     LIBCMT:typinfo.obj
 0002:000157fc       ??_R3type_info@@8          110be7fc     LIBCMT:typinfo.obj
 0002:0001580c       ??_R2type_info@@8          110be80c     LIBCMT:typinfo.obj
 0002:00015814       ??_R1A@?0A@EA@type_info@@8 110be814     LIBCMT:typinfo.obj
 0002:00015830       ??_R4out_of_range@std@@6B@ 110be830     libcpmt:string.obj
 0002:00015844       ??_R3out_of_range@std@@8   110be844     libcpmt:string.obj
 0002:00015854       ??_R2out_of_range@std@@8   110be854     libcpmt:string.obj
 0002:00015864       ??_R1A@?0A@EA@out_of_range@std@@8 110be864     libcpmt:string.obj
 0002:00015880       ??_R4bad_exception@std@@6B@ 110be880     LIBCMT:frame.obj
 0002:00015894       ??_R3bad_exception@std@@8  110be894     LIBCMT:frame.obj
 0002:000158a4       ??_R2bad_exception@std@@8  110be8a4     LIBCMT:frame.obj
 0002:000158b0       ??_R1A@?0A@EA@bad_exception@std@@8 110be8b0     LIBCMT:frame.obj
 0002:000158cc       ??_R4bad_alloc@std@@6B@    110be8cc     engine_gm.obj
 0002:000158e0       ??_R3bad_alloc@std@@8      110be8e0     engine_gm.obj
 0002:000158f0       ??_R2bad_alloc@std@@8      110be8f0     engine_gm.obj
 0002:000158fc       ??_R1A@?0A@EA@exception@std@@8 110be8fc     engine_gm.obj
 0002:00015918       ??_R3exception@std@@8      110be918     engine_gm.obj
 0002:00015928       ??_R2exception@std@@8      110be928     engine_gm.obj
 0002:00015930       ??_R1A@?0A@EA@bad_alloc@std@@8 110be930     engine_gm.obj
 0002:0001594c       ??_R4length_error@std@@6B@ 110be94c     gmcommandclass.obj
 0002:00015960       ??_R3length_error@std@@8   110be960     gmcommandclass.obj
 0002:00015970       ??_R2length_error@std@@8   110be970     gmcommandclass.obj
 0002:00015980       ??_R1A@?0A@EA@length_error@std@@8 110be980     gmcommandclass.obj
 0002:0001599c       ??_R4logic_error@std@@6B@  110be99c     gmcommandclass.obj
 0002:000159b0       ??_R3logic_error@std@@8    110be9b0     gmcommandclass.obj
 0002:000159c0       ??_R2logic_error@std@@8    110be9c0     gmcommandclass.obj
 0002:000159cc       ??_R1A@?0A@EA@logic_error@std@@8 110be9cc     gmcommandclass.obj
 0002:000159e8       ??_R4?$VectorClass@PAE@@6B@ 110be9e8     engine_bhs.obj
 0002:000159fc       ??_R3?$VectorClass@PAE@@8  110be9fc     engine_bhs.obj
 0002:00015a0c       ??_R2?$VectorClass@PAE@@8  110bea0c     engine_bhs.obj
 0002:00015a14       ??_R1A@?0A@EA@?$VectorClass@PAE@@8 110bea14     engine_bhs.obj
 0002:00015a30       ??_R4_Vector4MathFunctionsSSE@@6B@ 110bea30     engine_math.obj
 0002:00015a44       ??_R3_Vector4MathFunctionsSSE@@8 110bea44     engine_math.obj
 0002:00015a54       ??_R2_Vector4MathFunctionsSSE@@8 110bea54     engine_math.obj
 0002:00015a60       ??_R1A@?0A@EA@_Vector4MathFunctionsSSE@@8 110bea60     engine_math.obj
 0002:00015a7c       ??_R4_Vector4MathFunctions@@6B@ 110bea7c     engine_math.obj
 0002:00015a90       ??_R3_Vector4MathFunctions@@8 110bea90     engine_math.obj
 0002:00015aa0       ??_R2_Vector4MathFunctions@@8 110beaa0     engine_math.obj
 0002:00015aa8       ??_R1A@?0A@EA@_Vector4MathFunctions@@8 110beaa8     engine_math.obj
 0002:00015ac4       ??_R4_Vector3MathFunctions@@6B@ 110beac4     engine_math.obj
 0002:00015ad8       ??_R3_Vector3MathFunctions@@8 110bead8     engine_math.obj
 0002:00015ae8       ??_R2_Vector3MathFunctions@@8 110beae8     engine_math.obj
 0002:00015af0       ??_R1A@?0A@EA@_Vector3MathFunctions@@8 110beaf0     engine_math.obj
 0002:00015b0c       ??_R4ScriptFactory@@6B@    110beb0c     scriptfactory.obj
 0002:00015b20       ??_R3ScriptFactory@@8      110beb20     scriptfactory.obj
 0002:00015b30       ??_R2ScriptFactory@@8      110beb30     scriptfactory.obj
 0002:00015b38       ??_R1A@?0A@EA@ScriptFactory@@8 110beb38     scriptfactory.obj
 0002:00015b54       ??_R4ScriptImpClass@@6B@   110beb54     scripts.obj
 0002:00015b68       ??_R3ScriptImpClass@@8     110beb68     scripts.obj
 0002:00015b78       ??_R2ScriptImpClass@@8     110beb78     scripts.obj
 0002:00015b88       ??_R1A@?0A@EA@ScriptImpClass@@8 110beb88     scripts.obj
 0002:00015ba4       ??_R4GameObjObserverClass@@6B@ 110beba4     scripts.obj
 0002:00015bb8       ??_R3ScriptClass@@8        110bebb8     scripts.obj
 0002:00015bc8       ??_R2ScriptClass@@8        110bebc8     scripts.obj
 0002:00015bd4       ??_R1A@?0A@EA@GameObjObserverClass@@8 110bebd4     scripts.obj
 0002:00015bf0       ??_R3GameObjObserverClass@@8 110bebf0     scripts.obj
 0002:00015c00       ??_R2GameObjObserverClass@@8 110bec00     scripts.obj
 0002:00015c08       ??_R1A@?0A@EA@ScriptClass@@8 110bec08     scripts.obj
 0002:00015c24       ??_R4?$ScriptRegistrant@VLuaScript@LuaScriptManager@@@@6B@ 110bec24     LuaManager.obj
 0002:00015c38       ??_R3?$ScriptRegistrant@VLuaScript@LuaScriptManager@@@@8 110bec38     LuaManager.obj
 0002:00015c48       ??_R2?$ScriptRegistrant@VLuaScript@LuaScriptManager@@@@8 110bec48     LuaManager.obj
 0002:00015c54       ??_R1A@?0A@EA@?$ScriptRegistrant@VLuaScript@LuaScriptManager@@@@8 110bec54     LuaManager.obj
 0002:00015c70       ??_R4LuaScript@LuaScriptManager@@6B@ 110bec70     LuaManager.obj
 0002:00015c84       ??_R3LuaScript@LuaScriptManager@@8 110bec84     LuaManager.obj
 0002:00015c94       ??_R2LuaScript@LuaScriptManager@@8 110bec94     LuaManager.obj
 0002:00015ca8       ??_R1A@?0A@EA@LuaScript@LuaScriptManager@@8 110beca8     LuaManager.obj
 0002:00015cd0       ___safe_se_handler_table   110becd0     <linker-defined>
 0002:00015d00       ___rtc_iaa                 110bed00     LIBCMT:_initsect_.obj
 0002:00015d04       ___rtc_izz                 110bed04     LIBCMT:_initsect_.obj
 0002:00015d08       ___rtc_taa                 110bed08     LIBCMT:_initsect_.obj
 0002:00015d0c       ___rtc_tzz                 110bed0c     LIBCMT:_initsect_.obj
 0002:000165e8       __TI3?AVout_of_range@std@@ 110bf5e8     libcpmt:string.obj
 0002:000165f8       __CTA3?AVout_of_range@std@@ 110bf5f8     libcpmt:string.obj
 0002:00016608       __CT??_R0?AVout_of_range@std@@@8??0out_of_range@std@@QAE@ABV01@@Z40 110bf608     libcpmt:string.obj
 0002:0001672c       __TI2?AVbad_exception@std@@ 110bf72c     LIBCMT:frame.obj
 0002:0001673c       __CTA2?AVbad_exception@std@@ 110bf73c     LIBCMT:frame.obj
 0002:00016748       __CT??_R0?AVbad_exception@std@@@8??0bad_exception@std@@QAE@ABV01@@Z12 110bf748     LIBCMT:frame.obj
 0002:00016764       __CT??_R0?AVexception@std@@@8??0exception@std@@QAE@ABV01@@Z12 110bf764     engine_gm.obj
 0002:00016780       __CT??_R0?AVbad_alloc@std@@@8??0bad_alloc@std@@QAE@ABV01@@Z12 110bf780     engine_gm.obj
 0002:0001679c       __CTA2?AVbad_alloc@std@@   110bf79c     engine_gm.obj
 0002:000167a8       __TI2?AVbad_alloc@std@@    110bf7a8     engine_gm.obj
 0002:000167b8       __CT??_R0?AVlogic_error@std@@@8??0logic_error@std@@QAE@ABV01@@Z40 110bf7b8     gmcommandclass.obj
 0002:000167d4       __CT??_R0?AVlength_error@std@@@8??0length_error@std@@QAE@ABV01@@Z40 110bf7d4     gmcommandclass.obj
 0002:000167f0       __CTA3?AVlength_error@std@@ 110bf7f0     gmcommandclass.obj
 0002:00016800       __TI3?AVlength_error@std@@ 110bf800     gmcommandclass.obj
 0002:0001694c       __IMPORT_DESCRIPTOR_WS2_32 110bf94c     ws2_32:WS2_32.dll
 0002:00016960       __IMPORT_DESCRIPTOR_USER32 110bf960     user32:USER32.dll
 0002:00016974       __IMPORT_DESCRIPTOR_WININET 110bf974     Wininet:WININET.dll
 0002:00016988       __IMPORT_DESCRIPTOR_KERNEL32 110bf988     kernel32:KERNEL32.dll
 0002:0001699c       __NULL_IMPORT_DESCRIPTOR   110bf99c     ws2_32:WS2_32.dll
 0003:00000008       ??_R0?AVtype_info@@@8      110c1008     LIBCMT:typinfo.obj
 0003:00000030       ___lconv_static_decimal    110c1030     LIBCMT:lconv.obj
 0003:00000034       ___lconv_c                 110c1034     LIBCMT:lconv.obj
 0003:00000064       ___lconv                   110c1064     LIBCMT:lconv.obj
 0003:00000070       __iob                      110c1070     LIBCMT:_file.obj
 0003:00000460       __aexit_rtn                110c1460     LIBCMT:crt0dat.obj
 0003:00000470       __HUGE                     110c1470     LIBCMT:_huge_.obj
 0003:00000480       ___lc_time_c               110c1480     LIBCMT:strftime.obj
 0003:00000538       ___lc_time_curr            110c1538     LIBCMT:strftime.obj
 0003:00000540       ___nullstring              110c1540     LIBCMT:output.obj
 0003:00000544       ___wnullstring             110c1544     LIBCMT:output.obj
 0003:00000560       __timezone                 110c1560     LIBCMT:timeset.obj
 0003:00000564       __daylight                 110c1564     LIBCMT:timeset.obj
 0003:00000568       __dstbias                  110c1568     LIBCMT:timeset.obj
 0003:000005f0       __tzname                   110c15f0     LIBCMT:timeset.obj
 0003:00000600       ___initialmbcinfo          110c1600     LIBCMT:mbctype.obj
 0003:00000820       __mbctype                  110c1820     LIBCMT:mbctype.obj
 0003:00000928       __mbcasemap                110c1928     LIBCMT:mbctype.obj
 0003:00000a28       ___ptmbcinfo               110c1a28     LIBCMT:mbctype.obj
 0003:00000b20       ___globallocalestatus      110c1b20     LIBCMT:glstatus.obj
 0003:00000b28       ___clocalestr              110c1b28     LIBCMT:nlsdata2.obj
 0003:00000b30       ___initiallocinfo          110c1b30     LIBCMT:nlsdata2.obj
 0003:00000c08       ___ptlocinfo               110c1c08     LIBCMT:nlsdata2.obj
 0003:00000c0c       ___lc_clike                110c1c0c     LIBCMT:nlsdata2.obj
 0003:00000c10       ___initiallocalestructinfo 110c1c10     LIBCMT:nlsdata2.obj
 0003:00000c18       ___flsindex                110c1c18     LIBCMT:tidtable.obj
 0003:00000c1c       ___getvalueindex           110c1c1c     LIBCMT:tidtable.obj
 0003:00000c20       ___security_cookie         110c1c20     LIBCMT:gs_cookie.obj
 0003:00000c24       ___security_cookie_complement 110c1c24     LIBCMT:gs_cookie.obj
 0003:00000c30       ___badioinfo               110c1c30     LIBCMT:ioinit.obj
 0003:00000c70       __amblksiz                 110c1c70     LIBCMT:heapinit.obj
 0003:00000d98       ___abort_behavior          110c1d98     LIBCMT:abort.obj
 0003:00000e58       __fltused                  110c1e58     LIBCMT:_fpinit_.obj
 0003:00000e5c       __ldused                   110c1e5c     LIBCMT:_fpinit_.obj
 0003:00000e60       __sys_errlist              110c1e60     LIBCMT:syserr.obj
 0003:00000f10       __sys_nerr                 110c1f10     LIBCMT:syserr.obj
 0003:00000f18       __lookuptrailbytes         110c1f18     LIBCMT:read.obj
 0003:00001018       __NLG_Destination          110c2018     LIBCMT:exsup.obj
 0003:00001028       __cfltcvt_tab              110c2028     LIBCMT:cmiscdat.obj
 0003:00001050       __First_FPE_Indx           110c2050     LIBCMT:winxfltr.obj
 0003:00001054       __Num_FPE                  110c2054     LIBCMT:winxfltr.obj
 0003:00001058       __XcptActTabSize           110c2058     LIBCMT:winxfltr.obj
 0003:0000105c       __XcptActTabCount          110c205c     LIBCMT:winxfltr.obj
 0003:00001060       __tmpoff                   110c2060     LIBCMT:rmtmp.obj
 0003:00001064       __tempoff                  110c2064     LIBCMT:rmtmp.obj
 0003:00001070       __d_inf                    110c2070     LIBCMT:_util_.obj
 0003:00001078       __d_ind                    110c2078     LIBCMT:_util_.obj
 0003:00001080       __d_max                    110c2080     LIBCMT:_util_.obj
 0003:00001088       __d_min                    110c2088     LIBCMT:_util_.obj
 0003:00001090       __d_mzero                  110c2090     LIBCMT:_util_.obj
 0003:0000119c       __lpdays                   110c219c     LIBCMT:days.obj
 0003:000011d0       __days                     110c21d0     LIBCMT:days.obj
 0003:00001220       __pctype                   110c2220     LIBCMT:ctype.obj
 0003:00001224       __pwctype                  110c2224     LIBCMT:ctype.obj
 0003:00001228       ___mb_cur_max              110c2228     LIBCMT:nlsdata1.obj
 0003:0000122c       ___decimal_point           110c222c     LIBCMT:nlsdata1.obj
 0003:00001230       ___decimal_point_length    110c2230     LIBCMT:nlsdata1.obj
 0003:00001278       __pow10pos                 110c2278     LIBCMT:_constpow_.obj
 0003:000013d8       __pow10neg                 110c23d8     LIBCMT:_constpow_.obj
 0003:00001534       __matherr_flag             110c2534     LIBCMT:_matherr_.obj
 0003:00001538       __p_overlay                110c2538     LIBCMT:dospawn.obj
 0003:0000153c       __coninpfh                 110c253c     LIBCMT:initcon.obj
 0003:00001540       __confh                    110c2540     LIBCMT:initcon.obj
 0003:00001554       ??_R0?AVout_of_range@std@@@8 110c2554     libcpmt:string.obj
 0003:00001578       ?_Sync@ios_base@std@@0_NA  110c2578     libcpmt:ios.obj
 0003:00001598       ?_PJP_CPP_Copyright@@3PADA 110c2598     libcpmt:iosptrs.obj
 0003:000015f8       ??_R0?AVbad_exception@std@@@8 110c25f8     LIBCMT:frame.obj
 0003:00001750       ?crc_table@@3PAKA          110c2750     engine_io.obj
 0003:00001b54       ?Exe@@3HA                  110c2b54     engine_common.obj
 0003:00001bac       ?days@@3PAHA               110c2bac     date.obj
 0003:00001be0       ??_R0?AVexception@std@@@8  110c2be0     engine_gm.obj
 0003:00001bfc       ??_R0?AVbad_alloc@std@@@8  110c2bfc     engine_gm.obj
 0003:00001c18       ??_R0?AVlogic_error@std@@@8 110c2c18     gmcommandclass.obj
 0003:00001c38       ??_R0?AVlength_error@std@@@8 110c2c38     gmcommandclass.obj
 0003:00001c58       ??_R0?AV?$VectorClass@PAE@@@8 110c2c58     engine_bhs.obj
 0003:00001c78       ??_R0?AV_Vector4MathFunctionsSSE@@@8 110c2c78     engine_math.obj
 0003:00001ca0       ??_R0?AV_Vector4MathFunctions@@@8 110c2ca0     engine_math.obj
 0003:00001cc4       ??_R0?AV_Vector3MathFunctions@@@8 110c2cc4     engine_math.obj
 0003:00001ce8       ??_R0?AVScriptFactory@@@8  110c2ce8     scriptfactory.obj
 0003:00001d04       ??_R0?AVScriptImpClass@@@8 110c2d04     scripts.obj
 0003:00001d24       ??_R0?AVGameObjObserverClass@@@8 110c2d24     scripts.obj
 0003:00001d48       ??_R0?AVScriptClass@@@8    110c2d48     scripts.obj
 0003:00001d64       ??_R0?AV?$ScriptRegistrant@VLuaScript@LuaScriptManager@@@@@8 110c2d64     LuaManager.obj
 0003:00001da4       ??_R0?AVLuaScript@LuaScriptManager@@@8 110c2da4     LuaManager.obj
 0003:00001dd0       __half                     110c2dd0     LIBCMT:_pow_.obj
 0003:00001de0       __OP_FMODjmptab            110c2de0     LIBCMT:_87fmod_.obj
 0003:00001e50       __infinity                 110c2e50     LIBCMT:_87tran_.obj
 0003:00001e5a       __minfinity                110c2e5a     LIBCMT:_87tran_.obj
 0003:00001e64       __logemax                  110c2e64     LIBCMT:_87tran_.obj
 0003:00001e8a       __OP_EXPjmptab             110c2e8a     LIBCMT:_87tran_.obj
 0003:00001eb0       __indefinite               110c2eb0     LIBCMT:_87disp_.obj
 0003:00001eba       __piby2                    110c2eba     LIBCMT:_87disp_.obj
 0003:0000205a       __OP_SINHjmptab            110c305a     LIBCMT:_87trigh_.obj
 0003:0000207a       __OP_COSHjmptab            110c307a     LIBCMT:_87trigh_.obj
 0003:0000209a       __OP_TANHjmptab            110c309a     LIBCMT:_87trigh_.obj
 0003:000020d0       ___pInvalidArgHandler      110c30d0     LIBCMT:invarg.obj
 0003:000020d4       ___lconv_static_null       110c30d4     LIBCMT:lconv.obj
 0003:000020e8       __cflush                   110c30e8     LIBCMT:_file.obj
 0003:000020ec       __umaskval                 110c30ec     LIBCMT:crt0dat.obj
 0003:000020f0       ___argc                    110c30f0     LIBCMT:crt0dat.obj
 0003:000020f4       ___argv                    110c30f4     LIBCMT:crt0dat.obj
 0003:000020f8       ___wargv                   110c30f8     LIBCMT:crt0dat.obj
 0003:000020fc       __environ                  110c30fc     LIBCMT:crt0dat.obj
 0003:00002100       ___initenv                 110c3100     LIBCMT:crt0dat.obj
 0003:00002104       __wenviron                 110c3104     LIBCMT:crt0dat.obj
 0003:00002108       ___winitenv                110c3108     LIBCMT:crt0dat.obj
 0003:0000210c       __pgmptr                   110c310c     LIBCMT:crt0dat.obj
 0003:00002110       __wpgmptr                  110c3110     LIBCMT:crt0dat.obj
 0003:00002114       __exitflag                 110c3114     LIBCMT:crt0dat.obj
 0003:00002118       __C_Termination_Done       110c3118     LIBCMT:crt0dat.obj
 0003:0000211c       __C_Exit_Done              110c311c     LIBCMT:crt0dat.obj
 0003:00002158       ___idtabsiz                110c3158     LIBCMT:popen.obj
 0003:0000215c       ___idpairs                 110c315c     LIBCMT:popen.obj
 0003:00002160       ___locale_changed          110c3160     LIBCMT:setlocal.obj
 0003:00002168       __aenvptr                  110c3168     LIBCMT:dllcrt0.obj
 0003:0000216c       __wenvptr                  110c316c     LIBCMT:dllcrt0.obj
 0003:00002170       ___error_mode              110c3170     LIBCMT:dllcrt0.obj
 0003:00002174       ___app_type                110c3174     LIBCMT:dllcrt0.obj
 0003:00002234       ___mbulinfo                110c3234     LIBCMT:mbctype.obj
 0003:00002240       ___mbcodepage              110c3240     LIBCMT:mbctype.obj
 0003:00002244       ___ismbcodepage            110c3244     LIBCMT:mbctype.obj
 0003:00002248       ___mblcid                  110c3248     LIBCMT:mbctype.obj
 0003:0000224c       ___lc_handle               110c324c     LIBCMT:nlsdata2.obj
 0003:00002264       ___lc_codepage             110c3264     LIBCMT:nlsdata2.obj
 0003:00002268       ___lc_collate_cp           110c3268     LIBCMT:nlsdata2.obj
 0003:0000226c       _gpFlsAlloc                110c326c     LIBCMT:tidtable.obj
 0003:00002270       _gpFlsGetValue             110c3270     LIBCMT:tidtable.obj
 0003:00002274       _gpFlsSetValue             110c3274     LIBCMT:tidtable.obj
 0003:00002278       _gpFlsFree                 110c3278     LIBCMT:tidtable.obj
 0003:00002284       ?_pnhHeap@@3P6AHI@ZA       110c3284     LIBCMT:handler.obj
 0003:00002288       __crtheap                  110c3288     LIBCMT:heapinit.obj
 0003:000023e0       ___sbh_pHeaderDefer        110c33e0     LIBCMT:sbheap.obj
 0003:000023e8       __stdbuf                   110c33e8     LIBCMT:_sftbuf.obj
 0003:000023f0       __maxwait                  110c33f0     LIBCMT:crtheap.obj
 0003:00002714       ___pPurecall               110c3714     LIBCMT:inithelp.obj
 0003:00002718       ___fastflag                110c3718     LIBCMT:_fpinit_.obj
 0003:0000271c       __adjust_fdiv              110c371c     LIBCMT:_fpinit_.obj
 0003:00002720       __newmode                  110c3720     LIBCMT:_newmode.obj
 0003:00002724       ?__pInconsistency@@3P6AXXZA 110c3724     LIBCMT:hooks.obj
 0003:00002744       __old_pfxlen               110c3744     LIBCMT:rmtmp.obj
 0003:00002748       __commode                  110c3748     LIBCMT:ncommode.obj
 0003:00002ba0       ?pArgList@UnDecorator@@0PAVReplicator@@A 110c3ba0     LIBCMT:undname.obj
 0003:00002ba4       ?pZNameList@UnDecorator@@0PAVReplicator@@A 110c3ba4     LIBCMT:undname.obj
 0003:00002ba8       ?pTemplateArgList@UnDecorator@@0PAVReplicator@@A 110c3ba8     LIBCMT:undname.obj
 0003:00002bac       ?gName@UnDecorator@@0PBDB  110c3bac     LIBCMT:undname.obj
 0003:00002bb0       ?name@UnDecorator@@0PBDB   110c3bb0     LIBCMT:undname.obj
 0003:00002bb4       ?outputString@UnDecorator@@0PADA 110c3bb4     LIBCMT:undname.obj
 0003:00002bb8       ?maxStringLength@UnDecorator@@0HA 110c3bb8     LIBCMT:undname.obj
 0003:00002bbc       ?disableFlags@UnDecorator@@0KA 110c3bbc     LIBCMT:undname.obj
 0003:00002bc0       ?m_pGetParameter@UnDecorator@@0P6APADJ@ZA 110c3bc0     LIBCMT:undname.obj
 0003:00002bc4       ?fExplicitTemplateParams@UnDecorator@@0_NA 110c3bc4     LIBCMT:undname.obj
 0003:00002bc5       ?fGetTemplateArgumentList@UnDecorator@@0_NA 110c3bc5     LIBCMT:undname.obj
 0003:00002be0       __outputformat             110c3be0     LIBCMT:outputformat.obj
 0003:00002be4       __fmode                    110c3be4     LIBCMT:txtmode.obj
 0003:00002be8       ?_Fpz@std@@3_JA            110c3be8     libcpmt:ios.obj
 0003:00002bf0       ?_Index@ios_base@std@@0HA  110c3bf0     libcpmt:ios.obj
 0003:00002c30       ?_Clocptr@_Locimp@locale@std@@0PAV123@A 110c3c30     libcpmt:locale0.obj
 0003:00002c34       ?_Id_cnt@id@locale@std@@0HA 110c3c34     libcpmt:locale0.obj
 0003:00002c38       ?id@?$ctype@D@std@@2V0locale@2@A 110c3c38     libcpmt:locale0.obj
 0003:00002c3c       ?id@?$codecvt@GDH@std@@2V0locale@2@A 110c3c3c     libcpmt:locale0.obj
 0003:00002c40       ?id@?$ctype@_W@std@@2V0locale@2@A 110c3c40     libcpmt:locale0.obj
 0003:00002c44       ?id@?$codecvt@_WDH@std@@2V0locale@2@A 110c3c44     libcpmt:locale0.obj
 0003:00002c4c       ?id@?$ctype@G@std@@2V0locale@2@A 110c3c4c     libcpmt:locale0.obj
 0003:00002db0       ?_Ptr_cin@std@@3PAV?$basic_istream@DU?$char_traits@D@std@@@1@A 110c3db0     libcpmt:iosptrs.obj
 0003:00002db4       ?_Ptr_cout@std@@3PAV?$basic_ostream@DU?$char_traits@D@std@@@1@A 110c3db4     libcpmt:iosptrs.obj
 0003:00002db8       ?_Ptr_cerr@std@@3PAV?$basic_ostream@DU?$char_traits@D@std@@@1@A 110c3db8     libcpmt:iosptrs.obj
 0003:00002dbc       ?_Ptr_clog@std@@3PAV?$basic_ostream@DU?$char_traits@D@std@@@1@A 110c3dbc     libcpmt:iosptrs.obj
 0003:00002dc0       ?_Ptr_wcin@std@@3PAV?$basic_istream@_WU?$char_traits@_W@std@@@1@A 110c3dc0     libcpmt:iosptrs.obj
 0003:00002dc4       ?_Ptr_wcout@std@@3PAV?$basic_ostream@_WU?$char_traits@_W@std@@@1@A 110c3dc4     libcpmt:iosptrs.obj
 0003:00002dc8       ?_Ptr_wcerr@std@@3PAV?$basic_ostream@_WU?$char_traits@_W@std@@@1@A 110c3dc8     libcpmt:iosptrs.obj
 0003:00002dcc       ?_Ptr_wclog@std@@3PAV?$basic_ostream@_WU?$char_traits@_W@std@@@1@A 110c3dcc     libcpmt:iosptrs.obj
 0003:00002e00       ?out_string@date@@1PADA    110c3e00     date.obj
 0003:00002e1c       ?last_date@date@@1PADA     110c3e1c     date.obj
 0003:00002e38       ?Get_Next_Definition@@3P6APAVDefinitionClass@@PAV1@KD@ZA 110c3e38     engine_gm.obj
 0003:00002e3c       ?Get_First_Definition@@3P6APAVDefinitionClass@@KD@ZA 110c3e3c     engine_gm.obj
 0003:00002e40       ?ObjectsFile@@3PADA        110c3e40     engine_gm.obj
 0003:00002e44       ?bhs@@3PAUHINSTANCE__@@A   110c3e44     dllmain.obj
 0003:00002e48       ?Commands@@3PAUScriptCommands@@A 110c3e48     dllmain.obj
 0003:00002e4c       ?Fade_Background_Music_Player@@3P6AXPAEPBDHH@ZA 110c3e4c     engine_bhs.obj
 0003:00002e50       ?AddPowerupPurchaseHook@@3P6AHP6AHPAVBaseControllerClass@@PAEIIPBD@Z2@ZA 110c3e50     engine_bhs.obj
 0003:00002e54       ?Set_Shader_Number@@3P6AXPAEIM@ZA 110c3e54     engine_bhs.obj
 0003:00002e58       ?Send_Message@@3P6AXIIIPBD@ZA 110c3e58     engine_bhs.obj
 0003:00002e5c       ?AddVehiclePurchaseHook@@3P6AHP6AHPAVBaseControllerClass@@PAEIIPBD@Z2@ZA 110c3e5c     engine_bhs.obj
 0003:00002e60       ?Change_Radar_Map@@3P6AXMMMPBD@ZA 110c3e60     engine_bhs.obj
 0003:00002e64       ?Display_GDI_Player_Terminal_Player@@3P6AXPAE@ZA 110c3e64     engine_bhs.obj
 0003:00002e68       ?Stop_Background_Music_Player@@3P6AXPAE@ZA 110c3e68     engine_bhs.obj
 0003:00002e6c       ?Display_NOD_Sidebar@@3P6AXPAE@ZA 110c3e6c     engine_bhs.obj
 0003:00002e70       ?Display_GDI_Sidebar@@3P6AXPAE@ZA 110c3e70     engine_bhs.obj
 0003:00002e74       ?Set_HUD_Texture@@3P6AXPAEPBD@ZA 110c3e74     engine_bhs.obj
 0003:00002e78       ?Set_Fog_Color@@3P6AXIII@ZA 110c3e78     engine_bhs.obj
 0003:00002e7c       ?AddDataHook@@3P6AXP6AXHIPAI@Z@ZA 110c3e7c     engine_bhs.obj
 0003:00002e80       ?RemovePowerupPurchaseHook@@3P6AXH@ZA 110c3e80     engine_bhs.obj
 0003:00002e84       ?AddHostHook@@3P6AXP6AXHW4TextMessageEnum@@PBD@Z@ZA 110c3e84     engine_bhs.obj
 0003:00002e88       ?Set_Fog_Density@@3P6AXM@ZA 110c3e88     engine_bhs.obj
 0003:00002e8c       ?AddCharacterPurchaseHook@@3P6AHP6AHPAVBaseControllerClass@@PAEIIPBD@Z2@ZA 110c3e8c     engine_bhs.obj
 0003:00002e90       ?Display_Text_Player@@3P6AXPAEH@ZA 110c3e90     engine_bhs.obj
 0003:00002e94       ?Set_Display_Color_Player@@3P6AXPAEEEE@ZA 110c3e94     engine_bhs.obj
 0003:00002e98       ?AddGameOverHook@@3P6AXP6AXXZ@ZA 110c3e98     engine_bhs.obj
 0003:00002e9c       ?Set_Screen_Fade_Color_Player@@3P6AXPAEMMMM@ZA 110c3e9c     engine_bhs.obj
 0003:00002ea0       ?Set_Fog_Enable_Player@@3P6AXPAE_N@ZA 110c3ea0     engine_bhs.obj
 0003:00002ea4       ?Create_3D_WAV_Sound_At_Bone_Player@@3P6AHPAEPBD01@ZA 110c3ea4     engine_bhs.obj
 0003:00002ea8       ?Set_Info_Texture@@3P6AXPAEPBD@ZA 110c3ea8     engine_bhs.obj
 0003:00002eac       ?AddVersionHook@@3P6AXP6AXHM@Z@ZA 110c3eac     engine_bhs.obj
 0003:00002eb0       ?Set_Fog_Mode@@3P6AXI@ZA   110c3eb0     engine_bhs.obj
 0003:00002eb4       ?GetExplosionObj@@3P6APAEXZA 110c3eb4     engine_bhs.obj
 0003:00002eb8       ?Set_Vehicle_Limit@@3P6AXI@ZA 110c3eb8     engine_bhs.obj
 0003:00002ebc       ?AddCharacterPurchaseMonHook@@3P6AHP6AXPAVBaseControllerClass@@PAEIIIPBD@Z2@ZA 110c3ebc     engine_bhs.obj
 0003:00002ec0       ?RemovePowerupPurchaseMonHook@@3P6AXH@ZA 110c3ec0     engine_bhs.obj
 0003:00002ec4       ?Set_Currently_Building@@3P6AX_NH@ZA 110c3ec4     engine_bhs.obj
 0003:00002ec8       ?Send_Message_Player@@3P6AXPAEIIIPBD@ZA 110c3ec8     engine_bhs.obj
 0003:00002ecc       ?Change_Time_Limit@@3P6AXH@ZA 110c3ecc     engine_bhs.obj
 0003:00002ed0       ?RemoveCharacterPurchaseHook@@3P6AXH@ZA 110c3ed0     engine_bhs.obj
 0003:00002ed4       ?Display_NOD_Player_Terminal_Player@@3P6AXPAE@ZA 110c3ed4     engine_bhs.obj
 0003:00002ed8       ?Enable_HUD_Player@@3P6AXPAE_N@ZA 110c3ed8     engine_bhs.obj
 0003:00002edc       ?Set_Fog_Color_Player@@3P6AXPAEIII@ZA 110c3edc     engine_bhs.obj
 0003:00002ee0       ?Clear_Info_Texture@@3P6AXPAE@ZA 110c3ee0     engine_bhs.obj
 0003:00002ee4       ?Set_Fog_Range_Player@@3P6AXPAEMMM@ZA 110c3ee4     engine_bhs.obj
 0003:00002ee8       ?Force_Camera_Look_Player@@3P6AXPAEABUVector3@@@ZA 110c3ee8     engine_bhs.obj
 0003:00002eec       ?Set_Wireframe_Mode@@3P6AXH@ZA 110c3eec     engine_bhs.obj
 0003:00002ef0       ?RemoveKeyHook@@3P6AXH@ZA  110c3ef0     engine_bhs.obj
 0003:00002ef4       ?AddChatHook@@3P6AXP6AXHW4TextMessageEnum@@PB_W@Z@ZA 110c3ef4     engine_bhs.obj
 0003:00002ef8       ?Create_Sound_Player@@3P6AHPAEPBDABUVector3@@0@ZA 110c3ef8     engine_bhs.obj
 0003:00002efc       ?RemoveVehiclePurchaseMonHook@@3P6AXH@ZA 110c3efc     engine_bhs.obj
 0003:00002f00       ?Load_New_HUD_INI@@3P6AXPAEPBD@ZA 110c3f00     engine_bhs.obj
 0003:00002f04       ?Create_3D_Sound_At_Bone_Player@@3P6AHPAEPBD01@ZA 110c3f04     engine_bhs.obj
 0003:00002f08       ?Set_Screen_Fade_Opacity_Player@@3P6AXPAEMM@ZA 110c3f08     engine_bhs.obj
 0003:00002f0c       ?AddConsoleOutputHook@@3P6AXP6AXPBD@Z@ZA 110c3f0c     engine_bhs.obj
 0003:00002f10       ?RemoveObjectCreateHook@@3P6AXH@ZA 110c3f10     engine_bhs.obj
 0003:00002f14       ?Set_Background_Music_Player@@3P6AXPAEPBD@ZA 110c3f14     engine_bhs.obj
 0003:00002f18       ?Set_Reticle_Texture2@@3P6AXPAEPBD@ZA 110c3f18     engine_bhs.obj
 0003:00002f1c       ?Display_Int_Player@@3P6AXPAEHPBD@ZA 110c3f1c     engine_bhs.obj
 0003:00002f20       ?AddKeyHook@@3P6AHPAUKeyHookStruct@@@ZA 110c3f20     engine_bhs.obj
 0003:00002f24       ?Set_Fog_Mode_Player@@3P6AXPAEI@ZA 110c3f24     engine_bhs.obj
 0003:00002f28       ?RemoveCharacterPurchaseMonHook@@3P6AXH@ZA 110c3f28     engine_bhs.obj
 0003:00002f2c       ?RemoveVehiclePurchaseHook@@3P6AXH@ZA 110c3f2c     engine_bhs.obj
 0003:00002f30       ?Set_Obj_Radar_Blip_Shape_Player@@3P6AXPAE0H@ZA 110c3f30     engine_bhs.obj
 0003:00002f34       ?AddVehiclePurchaseMonHook@@3P6AHP6AXPAVBaseControllerClass@@PAEIIIPBD@Z2@ZA 110c3f34     engine_bhs.obj
 0003:00002f38       ?Set_Fog_Density_Player@@3P6AXPAEM@ZA 110c3f38     engine_bhs.obj
 0003:00002f3c       ?Get_Vehicle_Limit@@3P6AKXZA 110c3f3c     engine_bhs.obj
 0003:00002f40       ?Set_Obj_Radar_Blip_Color_Player@@3P6AXPAE0H@ZA 110c3f40     engine_bhs.obj
 0003:00002f44       ?AddCRCHook@@3P6AXP6AXIH@Z@ZA 110c3f44     engine_bhs.obj
 0003:00002f48       ?Display_Float_Player@@3P6AXPAEMPBD@ZA 110c3f48     engine_bhs.obj
 0003:00002f4c       ?Create_2D_WAV_Sound_Player@@3P6AHPAEPBD@ZA 110c3f4c     engine_bhs.obj
 0003:00002f50       ?GetCurrentMusicTrack@@3P6APBDXZA 110c3f50     engine_bhs.obj
 0003:00002f54       ?AddPlayerLeaveHook@@3P6AXP6AXH@Z@ZA 110c3f54     engine_bhs.obj
 0003:00002f58       ?AddLoadLevelHook@@3P6AXP6AXXZ@ZA 110c3f58     engine_bhs.obj
 0003:00002f5c       ?Set_Scope@@3P6AXPAEH@ZA   110c3f5c     engine_bhs.obj
 0003:00002f60       ?AddPlayerJoinHook@@3P6AXP6AXHPBD@Z@ZA 110c3f60     engine_bhs.obj
 0003:00002f64       ?Remove_Weapon@@3P6AXPAEPBD@ZA 110c3f64     engine_bhs.obj
 0003:00002f68       ?Display_Security_Dialog@@3P6AXPAE@ZA 110c3f68     engine_bhs.obj
 0003:00002f6c       ?AddObjectCreateHook@@3P6AHPAUObjectCreateHookStruct@@@ZA 110c3f6c     engine_bhs.obj
 0003:00002f70       ?AddPowerupPurchaseMonHook@@3P6AHP6AXPAVBaseControllerClass@@PAEIIIPBD@Z2@ZA 110c3f70     engine_bhs.obj
 0003:00002f74       ?Create_2D_Sound_Player@@3P6AHPAEPBD@ZA 110c3f74     engine_bhs.obj
 0003:00002f78       ?Is_Currently_Building@@3P6A_NH@ZA 110c3f78     engine_bhs.obj
 0003:00002f7c       ?Enable_Stealth_Player@@3P6AXPAE0_N@ZA 110c3f7c     engine_bhs.obj
 0003:00002f80       ?Set_Reticle_Texture1@@3P6AXPAEPBD@ZA 110c3f80     engine_bhs.obj
 0003:00002f84       ?Change_Time_Remaining@@3P6AXM@ZA 110c3f84     engine_bhs.obj
 0003:00002f88       ?Update_PT_Data@@3P6AXXZA  110c3f88     engine_bhs.obj
 0003:00002f8c       ?Enable_Radar_Player@@3P6AXPAE_N@ZA 110c3f8c     engine_bhs.obj
 0003:00002f90       ?Get_Build_Time_Multiplier@@3P6AMH@ZA 110c3f90     engine_bhs.obj
 0003:00002f94       ?Output_To_Console@@3PAXA  110c3f94     engine_common.obj
 0003:00002f98       ?RenDelete@@3P6AXPAX@ZA    110c3f98     engine_common.obj
 0003:00002f9c       ?RenVecDelete@@3P6AXPAX@ZA 110c3f9c     engine_common.obj
 0003:00002fa0       ?Parse_Console_Input@@3P6AXPBD@ZA 110c3fa0     engine_common.obj
 0003:00002fa4       ?Has3DNow@@3PA_NA          110c3fa4     engine_common.obj
 0003:00002fa8       ?HasSSE@@3PA_NA            110c3fa8     engine_common.obj
 0003:00002fac       ?FindNamedDef@@3P6APAVDefinitionClass@@PBD_N@ZA 110c3fac     engine_def.obj
 0003:00002fb0       ?Set_Safe_Data_Float_Ref@@3P6A_NPAXAAM@ZA 110c3fb0     engine_def.obj
 0003:00002fb4       ?Get_Safe_Data_Uint@@3PAXA 110c3fb4     engine_def.obj
 0003:00002fb8       ?Set_Safe_Data_Uint_Ref@@3P6A_NPAXAAI@ZA 110c3fb8     engine_def.obj
 0003:00002fbc       ?Set_Safe_Data_Int_Ref@@3P6A_NPAXAAH@ZA 110c3fbc     engine_def.obj
 0003:00002fc0       ?Get_Safe_Data_Float@@3PAXA 110c3fc0     engine_def.obj
 0003:00002fc4       ?Find_Def@@3P6APAVDefinitionClass@@K_N@ZA 110c3fc4     engine_def.obj
 0003:00002fc8       ?Get_Safe_Data_Int@@3PAXA  110c3fc8     engine_def.obj
 0003:00002fcc       ?Get_Armor_Type@@3P6AIPBD@ZA 110c3fcc     engine_dmg.obj
 0003:00002fd0       ?Get_Armor_Name@@3P6APBDI@ZA 110c3fd0     engine_dmg.obj
 0003:00002fd4       ?EnableRadar@@3PAXA        110c3fd4     engine_game.obj
 0003:00002fd8       ?FindBuilding@@3PAXA       110c3fd8     engine_game.obj
 0003:00002fdc       ?IsListed@@3PA_NA          110c3fdc     engine_game.obj
 0003:00002fe0       ?Skirmish_Game@@3PAXA      110c3fe0     engine_game.obj
 0003:00002fe4       ?DestroyBase@@3PAXA        110c3fe4     engine_game.obj
 0003:00002fe8       ?GDIHouseColor@@3PAMA      110c3fe8     engine_game.obj
 0003:00002fec       ?Single_Player_Game@@3PAXA 110c3fec     engine_game.obj
 0003:00002ff0       ?SetBeaconDestroyedBase@@3PAXA 110c3ff0     engine_game.obj
 0003:00002ff4       ?PrivateMessageColor@@3PAMA 110c3ff4     engine_game.obj
 0003:00002ff8       ?Game@@3PAXA               110c3ff8     engine_game.obj
 0003:00002ffc       ?NodHouseColor@@3PAMA      110c3ffc     engine_game.obj
 0003:00003000       ?IsMapVTOL@@3PA_NA         110c4000     engine_game.obj
 0003:00003004       ?GetHarvester@@3PAXA       110c4004     engine_game.obj
 0003:00003008       ?GameMode@@3PAIA           110c4008     engine_game.obj
 0003:0000300c       ?PowerBase@@3PAXA          110c400c     engine_game.obj
 0003:00003010       ?Game_Mode_Find@@3P6APAXPBD@ZA 110c4010     engine_game.obj
 0003:00003014       ?SetCanGenerateSoldiers@@3PAXA 110c4014     engine_game.obj
 0003:00003018       ?Cnc_Game@@3PAXA           110c4018     engine_game.obj
 0003:0000301c       ?GameType@@3PAHA           110c401c     engine_game.obj
 0003:00003020       ?PublicMessageColor@@3PAMA 110c4020     engine_game.obj
 0003:00003024       ?FindBase@@3PAXA           110c4024     engine_game.obj
 0003:00003028       ?Collect_Building_Components@@3P6AXXZA 110c4028     engine_game.obj
 0003:0000302c       ?SetCanGenerateVehicles@@3PAXA 110c402c     engine_game.obj
 0003:00003030       ?IniClassGetInt@@3PAXA     110c4030     engine_io.obj
 0003:00003034       ?TheFileFactory@@3PAPAVFileFactoryClass@@A 110c4034     engine_io.obj
 0003:00003038       ?ReleaseINI@@3PAXA         110c4038     engine_io.obj
 0003:0000303c       ?GetINI@@3PAXA             110c403c     engine_io.obj
 0003:00003040       ?IniClassGetString@@3PAXA  110c4040     engine_io.obj
 0003:00003044       ?IniClassGetFloat@@3PAXA   110c4044     engine_io.obj
 0003:00003048       ?IniClassGetBool@@3PAXA    110c4048     engine_io.obj
 0003:0000304c       ?Vector4Math@@3PAV_Vector4MathFunctions@@A 110c404c     engine_math.obj
 0003:00003050       ?Vector3Math@@3PAV_Vector3MathFunctions@@A 110c4050     engine_math.obj
 0003:00003054       ?Bandwidth_Out@@3P6AHPAUsockaddr_in@@@ZA 110c4054     engine_net.obj
 0003:00003058       ?Get_Address@@3P6APAUsockaddr_in@@XZA 110c4058     engine_net.obj
 0003:0000305c       ?ServerConnection@@3PAPADA 110c405c     engine_net.obj
 0003:00003060       ?PacketManager@@3PAXA      110c4060     engine_net.obj
 0003:00003064       ?Get_Remote_Host@@3P6APADH@ZA 110c4064     engine_net.obj
 0003:00003068       ?ServerKillConnection@@3PAXA 110c4068     engine_net.obj
 0003:0000306c       ?SetMaxHealth@@3PAXA       110c406c     engine_obj.obj
 0003:00003070       ?BaseGameObjList@@3PAV?$SList@E@@A 110c4070     engine_obj.obj
 0003:00003074       ?SmartGameObjList@@3PAV?$SList@E@@A 110c4074     engine_obj.obj
 0003:00003078       ?BuildingGameObjList@@3PAV?$SList@E@@A 110c4078     engine_obj.obj
 0003:0000307c       ?MarkOwnerDirty@@3PAXA     110c407c     engine_obj.obj
 0003:00003080       ?Powerup_Grant@@3PAXA      110c4080     engine_obj.obj
 0003:00003084       ?Get_Obj_Color@@3PAXA      110c4084     engine_obj.obj
 0003:00003088       ?StartObservers@@3PAXA     110c4088     engine_obj.obj
 0003:0000308c       ?SetMaxShieldStrength@@3PAXA 110c408c     engine_obj.obj
 0003:00003090       ?CheckTransitions@@3PAXA   110c4090     engine_obj2.obj
 0003:00003094       ?Request_Vehicle@@3P6A_NHMPAE@ZA 110c4094     engine_obj2.obj
 0003:00003098       ?FindClosestZone@@3PAXA    110c4098     engine_obj2.obj
 0003:0000309c       ?GetVehicleCount@@3P6AIXZA 110c409c     engine_obj2.obj
 0003:000030a0       ?Is_Available_For_Purchase@@3P6A_NXZA 110c40a0     engine_obj2.obj
 0003:000030a4       ?SpawnCharNod@@3PADA       110c40a4     engine_obj2.obj
 0003:000030a8       ?Create_Library_Object@@3P6APAEPBD@ZA 110c40a8     engine_obj2.obj
 0003:000030ac       ?SoldierReInit@@3P6AXPAVDefinitionClass@@@ZA 110c40ac     engine_obj2.obj
 0003:000030b0       ?overlap@@3PAXA            110c40b0     engine_obj2.obj
 0003:000030b4       ?ToggleFly@@3P6AXXZA       110c40b4     engine_obj2.obj
 0003:000030b8       ?SpawnCharGDI@@3PADA       110c40b8     engine_obj2.obj
 0003:000030bc       ?Grant_Supplies@@3PAXA     110c40bc     engine_obj2.obj
 0003:000030c0       ?InsideMe@@3PAXA           110c40c0     engine_obj2.obj
 0003:000030c4       ?Physical_Set_Transform@@3PAXA 110c40c4     engine_phys.obj
 0003:000030c8       ?Physical_Get_Transform@@3PAXA 110c40c8     engine_phys.obj
 0003:000030cc       ?TallyTeamSize@@3P6AHH@ZA  110c40cc     engine_player.obj
 0003:000030d0       ?FindPlayer@@3P6APAVcPlayer@@H@ZA 110c40d0     engine_player.obj
 0003:000030d4       ?SetRung@@3PAXA            110c40d4     engine_player.obj
 0003:000030d8       ?SetPlayerType@@3PAXA      110c40d8     engine_player.obj
 0003:000030dc       ?Get_Color_For_Team@@3P6AXPAUVector3@@H@ZA 110c40dc     engine_player.obj
 0003:000030e0       ?PlayerList@@3PAV?$SList@PAVcPlayer@@@@A 110c40e0     engine_player.obj
 0003:000030e4       ?Find_Team@@3P6APADH@ZA    110c40e4     engine_player.obj
 0003:000030e8       ?GetPlayerCount@@3PAXA     110c40e8     engine_player.obj
 0003:000030ec       ?GetColor@@3PAXA           110c40ec     engine_player.obj
 0003:000030f0       ?SetLadderPoints@@3PAXA    110c40f0     engine_player.obj
 0003:000030f4       ?DefinitionArray@@3PAPAVPurchaseSettingsDefClass@@A 110c40f4     engine_pt.obj
 0003:000030f8       ?Find_Team_Purchase_Definition@@3PAXA 110c40f8     engine_pt.obj
 0003:000030fc       ?Find_Purchase_Definition@@3PAXA 110c40fc     engine_pt.obj
 0003:00003100       ?m_TempMutex@WideStringClass@@2PAVCriticalSectionClass@@A 110c4100     engine_string.obj
 0003:00003104       ?m_FreeTempPtr@WideStringClass@@2PAPA_WA 110c4104     engine_string.obj
 0003:00003108       ?m_Mutex@StringClass@@2PAVCriticalSectionClass@@A 110c4108     engine_string.obj
 0003:0000310c       ?m_TempStrings@StringClass@@2PADA 110c410c     engine_string.obj
 0003:00003110       ?m_NullChar@WideStringClass@@2PA_WA 110c4110     engine_string.obj
 0003:00003114       ?m_NullChar@StringClass@@2PADA 110c4114     engine_string.obj
 0003:00003118       ?m_ResTempPtr@WideStringClass@@2PAPA_WA 110c4118     engine_string.obj
 0003:0000311c       ?m_EmptyString@WideStringClass@@2PAPA_WA 110c411c     engine_string.obj
 0003:00003120       ?m_EmptyString@StringClass@@2PAPADA 110c4120     engine_string.obj
 0003:00003124       ?ReservedMask@StringClass@@2PAIA 110c4124     engine_string.obj
 0003:00003128       ?m_UsedTempStringCount@WideStringClass@@2PAHA 110c4128     engine_string.obj
 0003:0000312c       ?Get_VehicleName@@3P6APA_WXZA 110c412c     engine_tdb.obj
 0003:00003130       ?Get_TDB_Object@@3P6APAVTDBObjClass@@K@ZA 110c4130     engine_tdb.obj
 0003:00003134       ?CriticalLock@@3PAXA       110c4134     engine_threading.obj
 0003:00003138       ?Mine_Limit@@3PADA         110c4138     engine_weap.obj
 0003:0000313c       ?GetBeaconOwner@@3PAXA     110c413c     engine_weap.obj
 0003:00003140       ?C4Defuse@@3PAXA           110c4140     engine_weap.obj
 0003:00003144       ?mScriptFactories@ScriptRegistrar@@0PAVScriptFactory@@A 110c4144     scriptregistrar.obj
 0003:00003148       ?RequestDestroyScript@ScriptImpClass@@0P6AXPAVScriptClass@@@ZA 110c4148     scripts.obj
 0003:0000314c       ?Upload_Error@LuaSocketManager@@0HA 110c414c     LuaManager.obj
 0003:00003150       ?Scripts@LuaScriptManager@@2PAPAUScript@1@A 110c4150     LuaManager.obj
 0003:00003550       ?Lua@LuaManager@@0PAPAUlua_State@@A 110c4550     LuaManager.obj
 0003:00003950       ?Sockets@LuaSocketManager@@0PAPAVTCPSocket@@A 110c4950     LuaManager.obj
 0003:00003a50       ?Upload_State@LuaSocketManager@@0HA 110c4a50     LuaManager.obj
 0003:00003c4c       ?List@ChatCommandList@@2PAV?$vector@PAUChatCommandInfo@@V?$allocator@PAUChatCommandInfo@@@std@@@std@@A 110c4c4c     gmcommandclass.obj
 0003:00003c50       ?Settings@@3PAUSettingsStruct@@A 110c4c50     gmmain.obj
 0003:00003c54       ?Data@@3PAUDataStruct@@A   110c4c54     gmmain.obj
 0003:00003c58       ?RequestSerial@@3P6AXHAAVStringClass@@@ZA 110c4c58     Hooks.obj
 0003:00003c5c       ?AddSerialHook@@3P6AXP6AXHPBD@Z@ZA 110c4c5c     Hooks.obj
 0003:00003c60       ?AddLoadingEHook@@3P6AXP6AXH_N@Z@ZA 110c4c60     Hooks.obj
 0003:00003c64       ?AddDamageHook@@3P6AXP6A_NHHHMI@Z@ZA 110c4c64     Hooks.obj
 0003:00003c68       ?AddChatEHook@@3P6AXP6A_NHHAAVWideStringClass@@H@Z@ZA 110c4c68     Hooks.obj
 0003:00003c6c       ?AddPingHook@@3P6AXP6AXHH@Z@ZA 110c4c6c     Hooks.obj
 0003:00003c70       ?AddSuicideHook@@3P6AXP6A_NH@Z@ZA 110c4c70     Hooks.obj
 0003:00003c74       ?AddRadioHook@@3P6AXP6A_NHHHHH@Z@ZA 110c4c74     Hooks.obj
 0003:00003c78       ?AddThinkHook@@3P6AXP6AXXZ@ZA 110c4c78     Hooks.obj
 0003:00003c7c       ?RenNew@@3P6APAXK@ZA       110c4c7c     engine_common.obj
 0003:00003c80       ?RenVecNew@@3P6APAXK@ZA    110c4c80     engine_common.obj
 0003:00003c84       ?noparams@@3PADA           110c4c84     scripts.obj
 0003:00003c88       ?Reload_Flag@LuaManager@@2_NA 110c4c88     LuaManager.obj
 0003:00003cb4       _sqlite3_temp_directory    110c4cb4     sqlite3.obj
 0003:00003cb8       ?id@?$num_put@DV?$ostreambuf_iterator@DU?$char_traits@D@std@@@std@@@std@@2V0locale@2@A 110c4cb8     gmfunc.obj
 0003:00003cbc       ?id@?$numpunct@D@std@@2V0locale@2@A 110c4cbc     gmfunc.obj
 0003:00003cc0       ?id@?$codecvt@DDH@std@@2V0locale@2@A 110c4cc0     gmfunc.obj
 0003:00003cc4       ___use_sse2_mathfcns       110c4cc4     <common>
 0003:00003cc8       ___sse2_available          110c4cc8     <common>
 0003:00003ccc       __pmatherr                 110c4ccc     <common>
 0003:00003cd0       ___sbh_cntHeaderList       110c4cd0     <common>
 0003:00003cd4       ___sbh_pHeaderList         110c4cd4     <common>
 0003:00003cd8       ___sbh_threshold           110c4cd8     <common>
 0003:00003cdc       ___sbh_pHeaderScan         110c4cdc     <common>
 0003:00003ce0       ___sbh_sizeHeaderList      110c4ce0     <common>
 0003:00003ce4       ___sbh_indGroupDefer       110c4ce4     <common>
 0003:00003ce8       ___active_heap             110c4ce8     <common>
 0003:00003cec       __nhandle                  110c4cec     <common>
 0003:00003d00       ___pioinfo                 110c4d00     <common>
 0003:00003e00       __debugger_hook_dummy      110c4e00     <common>
 0003:00003e04       __acmdln                   110c4e04     <common>
 0003:00003e08       ___env_initialized         110c4e08     <common>
 0003:00003e0c       ___onexitend               110c4e0c     <common>
 0003:00003e10       ___onexitbegin             110c4e10     <common>
 0003:00003e14       ___mbctype_initialized     110c4e14     <common>
 0003:00003e18       ___dyn_tls_init_callback   110c4e18     <common>
 0003:00003e1c       ___piob                    110c4e1c     <common>
 0003:00003e20       __bufin                    110c4e20     <common>
 0003:00004e20       __nstream                  110c5e20     <common>

 entry point at        0001:0008ecb9

 Static symbols

 0001:00000490       __catch$?_Copy@?$basic_string@DU?$char_traits@D@std@@V?$allocator@D@2@@std@@IAEXII@Z$0 11001490 f i  CIL library: CIL module
 0001:0000051e       __catch$?_Copy@?$basic_string@DU?$char_traits@D@std@@V?$allocator@D@2@@std@@IAEXII@Z$1 1100151e f i  CIL library: CIL module
 0001:0001fc50       _index2adr                 11020c50 f    CIL library: CIL module
 0001:00020670       _f_call                    11021670 f    CIL library: CIL module
 0001:00021640       _emptybuffer               11022640 f    CIL library: CIL module
 0001:000216b0       _adjuststack               110226b0 f    CIL library: CIL module
 0001:00021970       _getF                      11022970 f    CIL library: CIL module
 0001:000219d0       _errfile                   110229d0 f    CIL library: CIL module
 0001:00021cb0       _getS                      11022cb0 f    CIL library: CIL module
 0001:00021cd0       _l_alloc                   11022cd0 f    CIL library: CIL module
 0001:00021d00       _panic                     11022d00 f    CIL library: CIL module
 0001:00021d60       _luaB_print                11022d60 f    CIL library: CIL module
 0001:00021f00       _luaB_tonumber             11022f00 f    CIL library: CIL module
 0001:00022090       _luaB_error                11023090 f    CIL library: CIL module
 0001:00022180       _luaB_getmetatable         11023180 f    CIL library: CIL module
 0001:00022270       _luaB_setmetatable         11023270 f    CIL library: CIL module
 0001:000223b0       _getfunc                   110233b0 f    CIL library: CIL module
 0001:000224a0       _luaB_getfenv              110234a0 f    CIL library: CIL module
 0001:000224f0       _luaB_setfenv              110234f0 f    CIL library: CIL module
 0001:00022680       _luaB_rawequal             11023680 f    CIL library: CIL module
 0001:00022730       _luaB_rawget               11023730 f    CIL library: CIL module
 0001:00022820       _luaB_rawset               11023820 f    CIL library: CIL module
 0001:00022910       _luaB_gcinfo               11023910 f    CIL library: CIL module
 0001:00022950       _luaB_collectgarbage       11023950 f    CIL library: CIL module
 0001:00022a40       _luaB_type                 11023a40 f    CIL library: CIL module
 0001:00022ab0       _luaB_next                 11023ab0 f    CIL library: CIL module
 0001:00022b90       _luaB_pairs                11023b90 f    CIL library: CIL module
 0001:00022c60       _ipairsaux                 11023c60 f    CIL library: CIL module
 0001:00022d50       _luaB_ipairs               11023d50 f    CIL library: CIL module
 0001:00022e20       _load_aux                  11023e20 f    CIL library: CIL module
 0001:00022e80       _luaB_loadstring           11023e80 f    CIL library: CIL module
 0001:00022f30       _luaB_loadfile             11023f30 f    CIL library: CIL module
 0001:00022f80       _generic_reader            11023f80 f    CIL library: CIL module
 0001:00023090       _luaB_load                 11024090 f    CIL library: CIL module
 0001:000231a0       _luaB_dofile               110241a0 f    CIL library: CIL module
 0001:00023220       _luaB_assert               11024220 f    CIL library: CIL module
 0001:000232c0       _luaB_unpack               110242c0 f    CIL library: CIL module
 0001:00023440       _luaB_select               11024440 f    CIL library: CIL module
 0001:00023540       _luaB_pcall                11024540 f    CIL library: CIL module
 0001:00023630       _luaB_xpcall               11024630 f    CIL library: CIL module
 0001:00023770       _luaB_tostring             11024770 f    CIL library: CIL module
 0001:00023910       _luaB_newproxy             11024910 f    CIL library: CIL module
 0001:00023b20       _luaB_costatus             11024b20 f    CIL library: CIL module
 0001:00023bd0       _auxresume                 11024bd0 f    CIL library: CIL module
 0001:00023d00       _luaB_coresume             11024d00 f    CIL library: CIL module
 0001:00023da0       _luaB_auxwrap              11024da0 f    CIL library: CIL module
 0001:00023e50       _luaB_cocreate             11024e50 f    CIL library: CIL module
 0001:00023f20       _luaB_cowrap               11024f20 f    CIL library: CIL module
 0001:00023f50       _luaB_yield                11024f50 f    CIL library: CIL module
 0001:00023f90       _luaB_corunning            11024f90 f    CIL library: CIL module
 0001:00023fd0       _auxopen                   11024fd0 f    CIL library: CIL module
 0001:00024050       _base_open                 11025050 f    CIL library: CIL module
 0001:00024370       _condjump                  11025370 f    CIL library: CIL module
 0001:000243d0       _fixjump                   110253d0 f    CIL library: CIL module
 0001:00024420       _need_value                11025420 f    CIL library: CIL module
 0001:00024480       _patchtestreg              11025480 f    CIL library: CIL module
 0001:00024500       _removevalues              11025500 f    CIL library: CIL module
 0001:00024590       _patchlistaux              11025590 f    CIL library: CIL module
 0001:00024700       _freeexp                   11025700 f    CIL library: CIL module
 0001:00024720       _addk                      11025720 f    CIL library: CIL module
 0001:00024880       _nilK                      11025880 f    CIL library: CIL module
 0001:00024a60       _discharge2reg             11025a60 f    CIL library: CIL module
 0001:00024bc0       _discharge2anyreg          11025bc0 f    CIL library: CIL module
 0001:00024c10       _exp2reg                   11025c10 f    CIL library: CIL module
 0001:00025140       _invertjump                11026140 f    CIL library: CIL module
 0001:00025190       _jumponcond                11026190 f    CIL library: CIL module
 0001:00025330       _luaK_goiffalse            11026330 f    CIL library: CIL module
 0001:000253c0       _codenot                   110263c0 f    CIL library: CIL module
 0001:00025490       _constfolding              11026490 f    CIL library: CIL module
 0001:00025580       _codearith                 11026580 f    CIL library: CIL module
 0001:00025680       _codecomp                  11026680 f    CIL library: CIL module
 0001:00025a60       _luaK_code                 11026a60 f    CIL library: CIL module
 0001:00025bc0       _db_getregistry            11026bc0 f    CIL library: CIL module
 0001:00025bf0       _db_getmetatable           11026bf0 f    CIL library: CIL module
 0001:00025c80       _db_setmetatable           11026c80 f    CIL library: CIL module
 0001:00025d10       _db_getfenv                11026d10 f    CIL library: CIL module
 0001:00025d30       _db_setfenv                11026d30 f    CIL library: CIL module
 0001:00025df0       _settabss                  11026df0 f    CIL library: CIL module
 0001:00025e60       _setfield                  11026e60 f    CIL library: CIL module
 0001:00025e60       _settabsi                  11026e60 f    CIL library: CIL module
 0001:00025ed0       _treatstackoption          11026ed0 f    CIL library: CIL module
 0001:00025fa0       _db_getinfo                11026fa0 f    CIL library: CIL module
 0001:00026300       _db_getlocal               11027300 f    CIL library: CIL module
 0001:00026430       _db_setlocal               11027430 f    CIL library: CIL module
 0001:00026580       _auxupvalue                11027580 f    CIL library: CIL module
 0001:00026650       _db_getupvalue             11027650 f    CIL library: CIL module
 0001:00026660       _db_setupvalue             11027660 f    CIL library: CIL module
 0001:000266a0       _hookf                     110276a0 f    CIL library: CIL module
 0001:00026780       _gethooktable              11027780 f    CIL library: CIL module
 0001:00026850       _db_sethook                11027850 f    CIL library: CIL module
 0001:00026a40       _db_gethook                11027a40 f    CIL library: CIL module
 0001:00026b90       _db_debug                  11027b90 f    CIL library: CIL module
 0001:00026e00       _db_errorfb                11027e00 f    CIL library: CIL module
 0001:00027210       _currentline               11028210 f    CIL library: CIL module
 0001:000272d0       _findlocal                 110282d0 f    CIL library: CIL module
 0001:00027350       _funcinfo                  11028350 f    CIL library: CIL module
 0001:000273c0       _collectvalidlines         110283c0 f    CIL library: CIL module
 0001:000274b0       _auxgetinfo                110284b0 f    CIL library: CIL module
 0001:000276c0       _precheck                  110286c0 f    CIL library: CIL module
 0001:00027750       _checkArgMode              11028750 f    CIL library: CIL module
 0001:000277a0       _symbexec                  110287a0 f    CIL library: CIL module
 0001:00027c50       _kname                     11028c50 f    CIL library: CIL module
 0001:00027c80       _getobjname                11028c80 f    CIL library: CIL module
 0001:00027e00       _getfuncname               11028e00 f    CIL library: CIL module
 0001:00027fc0       _addinfo                   11028fc0 f    CIL library: CIL module
 0001:00028180       _resetstack                11029180 f    CIL library: CIL module
 0001:000282b0       _correctstack              110292b0 f    CIL library: CIL module
 0001:00028440       _growCI                    11029440 f    CIL library: CIL module
 0001:00028560       _adjust_varargs            11029560 f    CIL library: CIL module
 0001:00028790       _tryfuncTM                 11029790 f    CIL library: CIL module
 0001:00028a30       _callrethooks              11029a30 f    CIL library: CIL module
 0001:00028ba0       _resume                    11029ba0 f    CIL library: CIL module
 0001:00028c20       _resume_error              11029c20 f    CIL library: CIL module
 0001:00028e30       _f_parser                  11029e30 f    CIL library: CIL module
 0001:00029010       _DumpString                1102a010 f    CIL library: CIL module
 0001:00029090       _DumpConstants             1102a090 f    CIL library: CIL module
 0001:000291d0       _DumpDebug                 1102a1d0 f    CIL library: CIL module
 0001:00029320       _DumpFunction              1102a320 f    CIL library: CIL module
 0001:00029940       _reallymarkobject          1102a940 f    CIL library: CIL module
 0001:00029ad0       _traversetable             1102aad0 f    CIL library: CIL module
 0001:00029c80       _traverseproto             1102ac80 f    CIL library: CIL module
 0001:00029d50       _traverseclosure           1102ad50 f    CIL library: CIL module
 0001:00029df0       _traversestack             1102adf0 f    CIL library: CIL module
 0001:00029f40       _propagatemark             1102af40 f    CIL library: CIL module
 0001:0002a040       _cleartable                1102b040 f    CIL library: CIL module
 0001:0002a140       _freeobj                   1102b140 f    CIL library: CIL module
 0001:0002a1e0       _sweeplist                 1102b1e0 f    CIL library: CIL module
 0001:0002a270       _checkSizes                1102b270 f    CIL library: CIL module
 0001:0002a300       _GCTM                      1102b300 f    CIL library: CIL module
 0001:0002a400       _markmt                    1102b400 f    CIL library: CIL module
 0001:0002a440       _markroot                  1102b440 f    CIL library: CIL module
 0001:0002a4b0       _remarkupvals              1102b4b0 f    CIL library: CIL module
 0001:0002a4f0       _atomic                    1102b4f0 f    CIL library: CIL module
 0001:0002a5f0       _singlestep                1102b5f0 f    CIL library: CIL module
 0001:0002a960       _fileerror                 1102b960 f    CIL library: CIL module
 0001:0002a9f0       _io_type                   1102b9f0 f    CIL library: CIL module
 0001:0002ab50       _newfile                   1102bb50 f    CIL library: CIL module
 0001:0002ac50       _io_noclose                1102bc50 f    CIL library: CIL module
 0001:0002aca0       _io_pclose                 1102bca0 f    CIL library: CIL module
 0001:0002ad40       _io_fclose                 1102bd40 f    CIL library: CIL module
 0001:0002ade0       _aux_close                 1102bde0 f    CIL library: CIL module
 0001:0002ae60       _io_close                  1102be60 f    CIL library: CIL module
 0001:0002aee0       _io_gc                     1102bee0 f    CIL library: CIL module
 0001:0002af10       _io_tostring               1102bf10 f    CIL library: CIL module
 0001:0002af80       _io_open                   1102bf80 f    CIL library: CIL module
 0001:0002b050       _io_popen                  1102c050 f    CIL library: CIL module
 0001:0002b120       _io_tmpfile                1102c120 f    CIL library: CIL module
 0001:0002b190       _getiofile                 1102c190 f    CIL library: CIL module
 0001:0002b210       _g_iofile                  1102c210 f    CIL library: CIL module
 0001:0002b350       _io_input                  1102c350 f    CIL library: CIL module
 0001:0002b370       _io_output                 1102c370 f    CIL library: CIL module
 0001:0002b390       _f_lines                   1102c390 f    CIL library: CIL module
 0001:0002b410       _io_lines                  1102c410 f    CIL library: CIL module
 0001:0002b500       _read_number               1102c500 f    CIL library: CIL module
 0001:0002b540       _test_eof                  1102c540 f    CIL library: CIL module
 0001:0002b5a0       _read_line                 1102c5a0 f    CIL library: CIL module
 0001:0002b6e0       _read_chars                1102c6e0 f    CIL library: CIL module
 0001:0002b800       _g_read                    1102c800 f    CIL library: CIL module
 0001:0002ba20       _io_read                   1102ca20 f    CIL library: CIL module
 0001:0002ba40       _f_read                    1102ca40 f    CIL library: CIL module
 0001:0002ba80       _io_readline               1102ca80 f    CIL library: CIL module
 0001:0002bba0       _g_write                   1102cba0 f    CIL library: CIL module
 0001:0002bde0       _io_write                  1102cde0 f    CIL library: CIL module
 0001:0002be00       _f_write                   1102ce00 f    CIL library: CIL module
 0001:0002be40       _f_seek                    1102ce40 f    CIL library: CIL module
 0001:0002bf40       _f_setvbuf                 1102cf40 f    CIL library: CIL module
 0001:0002c030       _io_flush                  1102d030 f    CIL library: CIL module
 0001:0002c0c0       _f_flush                   1102d0c0 f    CIL library: CIL module
 0001:0002c170       _createmeta                1102d170 f    CIL library: CIL module
 0001:0002c1f0       _createstdfile             1102d1f0 f    CIL library: CIL module
 0001:0002c2b0       _newfenv                   1102d2b0 f    CIL library: CIL module
 0001:0002c4a0       _save                      1102d4a0 f    CIL library: CIL module
 0001:0002c5b0       _txtToken                  1102d5b0 f    CIL library: CIL module
 0001:0002c6e0       _inclinenumber             1102d6e0 f    CIL library: CIL module
 0001:0002c870       _check_next                1102d870 f    CIL library: CIL module
 0001:0002c900       _trydecpoint               1102d900 f    CIL library: CIL module
 0001:0002c990       _read_numeral              1102d990 f    CIL library: CIL module
 0001:0002cb20       _skip_sep                  1102db20 f    CIL library: CIL module
 0001:0002cc10       _read_long_string          1102dc10 f    CIL library: CIL module
 0001:0002cf20       _read_string               1102df20 f    CIL library: CIL module
 0001:0002d3b0       _llex                      1102e3b0 f    CIL library: CIL module
 0001:0002dc90       _math_abs                  1102ec90 f    CIL library: CIL module
 0001:0002dcd0       _math_sin                  1102ecd0 f    CIL library: CIL module
 0001:0002dd10       _math_sinh                 1102ed10 f    CIL library: CIL module
 0001:0002dd50       _math_cos                  1102ed50 f    CIL library: CIL module
 0001:0002dd90       _math_cosh                 1102ed90 f    CIL library: CIL module
 0001:0002ddd0       _math_tan                  1102edd0 f    CIL library: CIL module
 0001:0002de10       _math_tanh                 1102ee10 f    CIL library: CIL module
 0001:0002de50       _math_asin                 1102ee50 f    CIL library: CIL module
 0001:0002de90       _math_acos                 1102ee90 f    CIL library: CIL module
 0001:0002ded0       _math_atan                 1102eed0 f    CIL library: CIL module
 0001:0002df10       _math_atan2                1102ef10 f    CIL library: CIL module
 0001:0002df60       _math_ceil                 1102ef60 f    CIL library: CIL module
 0001:0002dfa0       _math_floor                1102efa0 f    CIL library: CIL module
 0001:0002dfe0       _math_fmod                 1102efe0 f    CIL library: CIL module
 0001:0002e030       _math_modf                 1102f030 f    CIL library: CIL module
 0001:0002e090       _math_sqrt                 1102f090 f    CIL library: CIL module
 0001:0002e0d0       _math_pow                  1102f0d0 f    CIL library: CIL module
 0001:0002e120       _math_log                  1102f120 f    CIL library: CIL module
 0001:0002e160       _math_log10                1102f160 f    CIL library: CIL module
 0001:0002e1a0       _math_exp                  1102f1a0 f    CIL library: CIL module
 0001:0002e1f0       _math_deg                  1102f1f0 f    CIL library: CIL module
 0001:0002e230       _math_rad                  1102f230 f    CIL library: CIL module
 0001:0002e270       _math_frexp                1102f270 f    CIL library: CIL module
 0001:0002e2d0       _math_ldexp                1102f2d0 f    CIL library: CIL module
 0001:0002e320       _math_min                  1102f320 f    CIL library: CIL module
 0001:0002e3a0       _math_max                  1102f3a0 f    CIL library: CIL module
 0001:0002e420       _math_random               1102f420 f    CIL library: CIL module
 0001:0002e570       _math_randomseed           1102f570 f    CIL library: CIL module
 0001:0002e7e0       _setprogdir                1102f7e0 f    CIL library: CIL module
 0001:0002e890       _pusherror                 1102f890 f    CIL library: CIL module
 0001:0002e8f0       _ll_register               1102f8f0 f    CIL library: CIL module
 0001:0002ea10       _gctm                      1102fa10 f    CIL library: CIL module
 0001:0002ea40       _ll_loadfunc               1102fa40 f    CIL library: CIL module
 0001:0002eab0       _ll_loadlib                1102fab0 f    CIL library: CIL module
 0001:0002eb20       _pushnexttemplate          1102fb20 f    CIL library: CIL module
 0001:0002eba0       _findfile                  1102fba0 f    CIL library: CIL module
 0001:0002ee30       _loaderror                 1102fe30 f    CIL library: CIL module
 0001:0002eed0       _loader_Lua                1102fed0 f    CIL library: CIL module
 0001:0002ef20       _mkfuncname                1102ff20 f    CIL library: CIL module
 0001:0002ef90       _loader_C                  1102ff90 f    CIL library: CIL module
 0001:0002eff0       _loader_Croot              1102fff0 f    CIL library: CIL module
 0001:0002f0f0       _loader_preload            110300f0 f    CIL library: CIL module
 0001:0002f1f0       _ll_require                110301f0 f    CIL library: CIL module
 0001:0002f770       _setfenv                   11030770 f    CIL library: CIL module
 0001:0002f7f0       _dooptions                 110307f0 f    CIL library: CIL module
 0001:0002f860       _modinit                   11030860 f    CIL library: CIL module
 0001:0002f9a0       _ll_module                 110309a0 f    CIL library: CIL module
 0001:0002fb60       _ll_seeall                 11030b60 f    CIL library: CIL module
 0001:0002fcc0       _setpath                   11030cc0 f    CIL library: CIL module
 0001:000302b0       _pushstr                   110312b0 f    CIL library: CIL module
 0001:00030730       _os_pushresult             11031730 f    CIL library: CIL module
 0001:000307b0       _os_execute                110317b0 f    CIL library: CIL module
 0001:00030810       _os_remove                 11031810 f    CIL library: CIL module
 0001:00030840       _os_rename                 11031840 f    CIL library: CIL module
 0001:00030880       _os_tmpname                11031880 f    CIL library: CIL module
 0001:000308d0       _os_getenv                 110318d0 f    CIL library: CIL module
 0001:00030900       _os_clock                  11031900 f    CIL library: CIL module
 0001:00030930       _getboolfield              11031930 f    CIL library: CIL module
 0001:000309d0       _getfield                  110319d0 f    CIL library: CIL module
 0001:00030a80       _os_date                   11031a80 f    CIL library: CIL module
 0001:00030d40       _os_time                   11031d40 f    CIL library: CIL module
 0001:00030ee0       _os_difftime               11031ee0 f    CIL library: CIL module
 0001:00030f60       _os_setlocale              11031f60 f    CIL library: CIL module
 0001:00030fc0       _os_exit                   11031fc0 f    CIL library: CIL module
 0001:00031010       _anchor_token              11032010 f    CIL library: CIL module
 0001:00031070       _error_expected            11032070 f    CIL library: CIL module
 0001:000310d0       _errorlimit                110320d0 f    CIL library: CIL module
 0001:00031110       _testnext                  11032110 f    CIL library: CIL module
 0001:00031160       _checknext                 11032160 f    CIL library: CIL module
 0001:000311c0       _check_match               110321c0 f    CIL library: CIL module
 0001:00031260       _str_checkname             11032260 f    CIL library: CIL module
 0001:000312e0       _codestring                110322e0 f    CIL library: CIL module
 0001:00031320       _registerlocalvar          11032320 f    CIL library: CIL module
 0001:000313e0       _adjustlocalvars           110323e0 f    CIL library: CIL module
 0001:00031420       _removevars                11032420 f    CIL library: CIL module
 0001:00031460       _indexupvalue              11032460 f    CIL library: CIL module
 0001:00031580       _singlevaraux              11032580 f    CIL library: CIL module
 0001:00031660       _singlevar                 11032660 f    CIL library: CIL module
 0001:000316b0       _adjust_assign             110326b0 f    CIL library: CIL module
 0001:00031750       _leaveblock                11032750 f    CIL library: CIL module
 0001:000317b0       _pushclosure               110327b0 f    CIL library: CIL module
 0001:000318c0       _open_func                 110328c0 f    CIL library: CIL module
 0001:000319a0       _close_func                110329a0 f    CIL library: CIL module
 0001:00031db0       _field                     11032db0 f    CIL library: CIL module
 0001:00031e90       _yindex                    11032e90 f    CIL library: CIL module
 0001:00031f90       _recfield                  11032f90 f    CIL library: CIL module
 0001:00032090       _lastlistfield             11033090 f    CIL library: CIL module
 0001:00032100       _constructor               11033100 f    CIL library: CIL module
 0001:000323f0       _parlist                   110333f0 f    CIL library: CIL module
 0001:000325e0       _body                      110335e0 f    CIL library: CIL module
 0001:000327b0       _explist1                  110337b0 f    CIL library: CIL module
 0001:000328a0       _funcargs                  110338a0 f    CIL library: CIL module
 0001:000329e0       _prefixexp                 110339e0 f    CIL library: CIL module
 0001:00032a80       _primaryexp                11033a80 f    CIL library: CIL module
 0001:00032d50       _simpleexp                 11033d50 f    CIL library: CIL module
 0001:00032f30       _getbinopr                 11033f30 f    CIL library: CIL module
 0001:000330e0       _subexpr                   110340e0 f    CIL library: CIL module
 0001:00033260       _block                     11034260 f    CIL library: CIL module
 0001:000332b0       _check_conflict            110342b0 f    CIL library: CIL module
 0001:00033340       _assignment                11034340 f    CIL library: CIL module
 0001:00033480       _breakstat                 11034480 f    CIL library: CIL module
 0001:00033520       _whilestat                 11034520 f    CIL library: CIL module
 0001:00033710       _repeatstat                11034710 f    CIL library: CIL module
 0001:000338f0       _forbody                   110348f0 f    CIL library: CIL module
 0001:00033b70       _fornum                    11034b70 f    CIL library: CIL module
 0001:00033ed0       _forlist                   11034ed0 f    CIL library: CIL module
 0001:00034230       _forstat                   11035230 f    CIL library: CIL module
 0001:00034310       _test_then_block           11035310 f    CIL library: CIL module
 0001:00034430       _ifstat                    11035430 f    CIL library: CIL module
 0001:00034720       _localfunc                 11035720 f    CIL library: CIL module
 0001:00034820       _localstat                 11035820 f    CIL library: CIL module
 0001:000349b0       _funcname                  110359b0 f    CIL library: CIL module
 0001:00034a40       _funcstat                  11035a40 f    CIL library: CIL module
 0001:00034ad0       _exprstat                  11035ad0 f    CIL library: CIL module
 0001:00034b30       _retstat                   11035b30 f    CIL library: CIL module
 0001:00034c60       _statement                 11035c60 f    CIL library: CIL module
 0001:00034da0       _chunk                     11035da0 f    CIL library: CIL module
 0001:00034e80       _stack_init                11035e80 f    CIL library: CIL module
 0001:00034f50       _f_luaopen                 11035f50 f    CIL library: CIL module
 0001:00034fd0       _close_state               11035fd0 f    CIL library: CIL module
 0001:00035300       _callallgcTM               11036300 f    CIL library: CIL module
 0001:00035450       _newlstr                   11036450 f    CIL library: CIL module
 0001:00035680       _str_len                   11036680 f    CIL library: CIL module
 0001:000356b0       _str_sub                   110366b0 f    CIL library: CIL module
 0001:000357d0       _str_reverse               110367d0 f    CIL library: CIL module
 0001:000358d0       _str_lower                 110368d0 f    CIL library: CIL module
 0001:00035a80       _str_upper                 11036a80 f    CIL library: CIL module
 0001:00035c30       _str_rep                   11036c30 f    CIL library: CIL module
 0001:00035cc0       _str_byte                  11036cc0 f    CIL library: CIL module
 0001:00035e90       _str_char                  11036e90 f    CIL library: CIL module
 0001:00036070       _writer                    11037070 f    CIL library: CIL module
 0001:00036090       _str_dump                  11037090 f    CIL library: CIL module
 0001:000361a0       _classend                  110371a0 f    CIL library: CIL module
 0001:00036220       _match_class               11037220 f    CIL library: CIL module
 0001:00036330       _matchbracketclass         11037330 f    CIL library: CIL module
 0001:000363d0       _matchbalance              110373d0 f    CIL library: CIL module
 0001:00036440       _max_expand                11037440 f    CIL library: CIL module
 0001:000364e0       _min_expand                110374e0 f    CIL library: CIL module
 0001:00036570       _start_capture             11037570 f    CIL library: CIL module
 0001:000365c0       _end_capture               110375c0 f    CIL library: CIL module
 0001:00036620       _match_capture             11037620 f    CIL library: CIL module
 0001:000366b0       _match                     110376b0 f    CIL library: CIL module
 0001:000369b0       _lmemfind                  110379b0 f    CIL library: CIL module
 0001:00036a70       _push_onecapture           11037a70 f    CIL library: CIL module
 0001:00036b40       _push_captures             11037b40 f    CIL library: CIL module
 0001:00036bb0       _str_find_aux              11037bb0 f    CIL library: CIL module
 0001:00036dd0       _str_find                  11037dd0 f    CIL library: CIL module
 0001:00036df0       _str_match                 11037df0 f    CIL library: CIL module
 0001:00036e10       _gmatch_aux                11037e10 f    CIL library: CIL module
 0001:00036fa0       _gmatch                    11037fa0 f    CIL library: CIL module
 0001:00037020       _gfind_nodef               11038020 f    CIL library: CIL module
 0001:00037040       _add_s                     11038040 f    CIL library: CIL module
 0001:00037140       _add_value                 11038140 f    CIL library: CIL module
 0001:000372c0       _str_gsub                  110382c0 f    CIL library: CIL module
 0001:00037510       _addquoted                 11038510 f    CIL library: CIL module
 0001:00037700       _scanformat                11038700 f    CIL library: CIL module
 0001:000377e0       _str_format                110387e0 f    CIL library: CIL module
 0001:00037b70       _createmetatable           11038b70 f    CIL library: CIL module
 0001:00037d20       _hashnum                   11038d20 f    CIL library: CIL module
 0001:00037d60       _mainposition              11038d60 f    CIL library: CIL module
 0001:00037df0       _findindex                 11038df0 f    CIL library: CIL module
 0001:00037fa0       _computesizes              11038fa0 f    CIL library: CIL module
 0001:00038000       _countint                  11039000 f    CIL library: CIL module
 0001:00038080       _numusearray               11039080 f    CIL library: CIL module
 0001:00038100       _numusehash                11039100 f    CIL library: CIL module
 0001:00038160       _setarrayvector            11039160 f    CIL library: CIL module
 0001:000381d0       _setnodevector             110391d0 f    CIL library: CIL module
 0001:000382b0       _resize                    110392b0 f    CIL library: CIL module
 0001:000384d0       _rehash                    110394d0 f    CIL library: CIL module
 0001:00038680       _newkey                    11039680 f    CIL library: CIL module
 0001:000389f0       _unbound_search            110399f0 f    CIL library: CIL module
 0001:00038b10       _foreachi                  11039b10 f    CIL library: CIL module
 0001:00038cb0       _foreach                   11039cb0 f    CIL library: CIL module
 0001:00038e40       _maxn                      11039e40 f    CIL library: CIL module
 0001:00038f70       _getn                      11039f70 f    CIL library: CIL module
 0001:00039000       _setn                      1103a000 f    CIL library: CIL module
 0001:000390a0       _tinsert                   1103a0a0 f    CIL library: CIL module
 0001:000391d0       _tremove                   1103a1d0 f    CIL library: CIL module
 0001:00039340       _addfield                  1103a340 f    CIL library: CIL module
 0001:000393e0       _tconcat                   1103a3e0 f    CIL library: CIL module
 0001:00039630       _sort_comp                 1103a630 f    CIL library: CIL module
 0001:00039730       _auxsort                   1103a730 f    CIL library: CIL module
 0001:00039ba0       _sort                      1103aba0 f    CIL library: CIL module
 0001:00039df0       _error                     1103adf0 f    CIL library: CIL module
 0001:00039e10       _LoadString                1103ae10 f    CIL library: CIL module
 0001:00039e90       _LoadCode                  1103ae90 f    CIL library: CIL module
 0001:00039f70       _LoadConstants             1103af70 f    CIL library: CIL module
 0001:0003a240       _LoadDebug                 1103b240 f    CIL library: CIL module
 0001:0003a560       _LoadFunction              1103b560 f    CIL library: CIL module
 0001:0003a760       _LoadHeader                1103b760 f    CIL library: CIL module
 0001:0003a920       _traceexec                 1103b920 f    CIL library: CIL module
 0001:0003a9b0       _callTMres                 1103b9b0 f    CIL library: CIL module
 0001:0003aa70       _callTM                    1103ba70 f    CIL library: CIL module
 0001:0003ae40       _call_binTM                1103be40 f    CIL library: CIL module
 0001:0003af10       _get_compTM                1103bf10 f    CIL library: CIL module
 0001:0003af80       _call_orderTM              1103bf80 f    CIL library: CIL module
 0001:0003b070       _l_strcmp                  1103c070 f    CIL library: CIL module
 0001:0003b190       _lessequal                 1103c190 f    CIL library: CIL module
 0001:0003b580       _Arith                     1103c580 f    CIL library: CIL module
 0001:0003cad0       _getDigits                 1103dad0 f    CIL library: CIL module
 0001:0003cb90       _parseTimezone             1103db90 f    CIL library: CIL module
 0001:0003cc70       _parseHhMmSs               1103dc70 f    CIL library: CIL module
 0001:0003cdb0       _computeJD                 1103ddb0 f    CIL library: CIL module
 0001:0003cec0       _parseYyyyMmDd             1103dec0 f    CIL library: CIL module
 0001:0003cfa0       _parseDateOrTime           1103dfa0 f    CIL library: CIL module
 0001:0003d040       _computeYMD                1103e040 f    CIL library: CIL module
 0001:0003d150       _computeHMS                1103e150 f    CIL library: CIL module
 0001:0003d210       _localtimeOffset           1103e210 f    CIL library: CIL module
 0001:0003d350       _parseModifier             1103e350 f    CIL library: CIL module
 0001:0003db80       _isDate                    1103eb80 f    CIL library: CIL module
 0001:0003dc00       _juliandayFunc             1103ec00 f    CIL library: CIL module
 0001:0003dc50       _datetimeFunc              1103ec50 f    CIL library: CIL module
 0001:0003dd10       _timeFunc                  1103ed10 f    CIL library: CIL module
 0001:0003ddb0       _dateFunc                  1103edb0 f    CIL library: CIL module
 0001:0003de50       _strftimeFunc              1103ee50 f    CIL library: CIL module
 0001:0003e3d0       _ctimeFunc                 1103f3d0 f    CIL library: CIL module
 0001:0003e3f0       _cdateFunc                 1103f3f0 f    CIL library: CIL module
 0001:0003e410       _ctimestampFunc            1103f410 f    CIL library: CIL module
 0001:0003e430       _sqlite3RegisterDateTimeFunctions 1103f430 f    CIL library: CIL module
 0001:0003e480       _sqlite3OsClose            1103f480 f    CIL library: CIL module
 0001:0003e4a0       _sqlite3OsRead             1103f4a0 f    CIL library: CIL module
 0001:0003e4d0       _sqlite3OsWrite            1103f4d0 f    CIL library: CIL module
 0001:0003e4f0       _sqlite3OsSectorSize       1103f4f0 f    CIL library: CIL module
 0001:0003e510       _sqlite3OsOpenMalloc       1103f510 f    CIL library: CIL module
 0001:0003e570       _sqlite3OsCloseFree        1103f570 f    CIL library: CIL module
 0001:0003e650       _vfsUnlink                 1103f650 f    CIL library: CIL module
 0001:0003e8a0       _sqlite3MemsysAlarm        1103f8a0 f    CIL library: CIL module
 0001:0003eda0       _sqlite3MallocZero         1103fda0 f    CIL library: CIL module
 0001:0003edc0       _sqlite3DbMallocZero       1103fdc0 f    CIL library: CIL module
 0001:0003ee00       _sqlite3DbMallocRaw        1103fe00 f    CIL library: CIL module
 0001:0003ee30       _sqlite3DbReallocOrFree    1103fe30 f    CIL library: CIL module
 0001:0003ee60       _sqlite3DbStrDup           1103fe60 f    CIL library: CIL module
 0001:0003eeb0       _sqlite3DbStrNDup          1103feb0 f    CIL library: CIL module
 0001:0003ef00       _sqlite3SetString          1103ff00 f    CIL library: CIL module
 0001:0003ef90       _sqlite3ApiExit            1103ff90 f    CIL library: CIL module
 0001:0003efd0       _vxprintf                  1103ffd0 f    CIL library: CIL module
 0001:0003fd80       _sqlite3StrAccumAppend     11040d80 f    CIL library: CIL module
 0001:0003fe50       _sqlite3StrAccumFinish     11040e50 f    CIL library: CIL module
 0001:0003fea0       _sqlite3StrAccumReset      11040ea0 f    CIL library: CIL module
 0001:0003fec0       _sqlite3VMPrintf           11040ec0 f    CIL library: CIL module
 0001:0003ff70       _sqlite3MPrintf            11040f70 f    CIL library: CIL module
 0001:000400b0       _randomByte                110410b0 f    CIL library: CIL module
 0001:000401b0       _sqlite3Randomness         110411b0 f    CIL library: CIL module
 0001:00040210       _sqlite3Utf8Read           11041210 f    CIL library: CIL module
 0001:00040270       _sqlite3VdbeMemTranslate   11041270 f    CIL library: CIL module
 0001:00040670       _sqlite3VdbeMemHandleBom   11041670 f    CIL library: CIL module
 0001:00040710       _sqlite3Utf8CharLen        11041710 f    CIL library: CIL module
 0001:00040760       _sqlite3Utf16to8           11041760 f    CIL library: CIL module
 0001:000407f0       _sqlite3Utf16ByteLen       110417f0 f    CIL library: CIL module
 0001:00040870       _sqlite3Error              11041870 f    CIL library: CIL module
 0001:00040900       _sqlite3ErrorMsg           11041900 f    CIL library: CIL module
 0001:00040940       _sqlite3Dequote            11041940 f    CIL library: CIL module
 0001:00040a10       _sqlite3StrICmp            11041a10 f    CIL library: CIL module
 0001:00040a60       _sqlite3StrNICmp           11041a60 f    CIL library: CIL module
 0001:00040ac0       _sqlite3IsNumber           11041ac0 f    CIL library: CIL module
 0001:00040be0       _sqlite3AtoF               11041be0 f    CIL library: CIL module
 0001:00040e20       _compare2pow63             11041e20 f    CIL library: CIL module
 0001:00040e90       _sqlite3Atoi64             11041e90 f    CIL library: CIL module
 0001:00040f80       _sqlite3FitsIn64Bits       11041f80 f    CIL library: CIL module
 0001:00041000       _sqlite3GetInt32           11042000 f    CIL library: CIL module
 0001:000410c0       _sqlite3PutVarint          110420c0 f    CIL library: CIL module
 0001:000411a0       _sqlite3GetVarint          110421a0 f    CIL library: CIL module
 0001:000412b0       _sqlite3GetVarint32        110422b0 f    CIL library: CIL module
 0001:00041310       _sqlite3VarintLen          11042310 f    CIL library: CIL module
 0001:00041340       _sqlite3Get4byte           11042340 f    CIL library: CIL module
 0001:00041360       _sqlite3HexToBlob          11042360 f    CIL library: CIL module
 0001:00041400       _sqlite3HashClear          11042400 f    CIL library: CIL module
 0001:00041500       _strHash                   11042500 f    CIL library: CIL module
 0001:00041550       _strCompare                11042550 f    CIL library: CIL module
 0001:00041580       _binHash                   11042580 f    CIL library: CIL module
 0001:000415b0       _binCompare                110425b0 f    CIL library: CIL module
 0001:00041640       _insertElement             11042640 f    CIL library: CIL module
 0001:00041690       _rehash                    11042690 f    CIL library: CIL module
 0001:00041790       _findElementGivenHash      11042790 f    CIL library: CIL module
 0001:000417f0       _removeElementGivenHash    110427f0 f    CIL library: CIL module
 0001:00041860       _sqlite3HashFind           11042860 f    CIL library: CIL module
 0001:000418b0       _sqlite3HashInsert         110428b0 f    CIL library: CIL module
 0001:000419f0       _utf8ToUnicode             110429f0 f    CIL library: CIL module
 0001:00041a50       _unicodeToUtf8             11042a50 f    CIL library: CIL module
 0001:00041ab0       _mbcsToUnicode             11042ab0 f    CIL library: CIL module
 0001:00041b20       _unicodeToMbcs             11042b20 f    CIL library: CIL module
 0001:00041b90       _winClose                  11042b90 f    CIL library: CIL module
 0001:00041be0       _winRead                   11042be0 f    CIL library: CIL module
 0001:00041c80       _winWrite                  11042c80 f    CIL library: CIL module
 0001:00041d30       _winTruncate               11042d30 f    CIL library: CIL module
 0001:00041d70       _winSync                   11042d70 f    CIL library: CIL module
 0001:00041d90       _winFileSize               11042d90 f    CIL library: CIL module
 0001:00041dd0       _getReadLock               11042dd0 f    CIL library: CIL module
 0001:00041e90       _unlockReadLock            11042e90 f    CIL library: CIL module
 0001:00041f10       _winLock                   11042f10 f    CIL library: CIL module
 0001:00042050       _winCheckReservedLock      11043050 f    CIL library: CIL module
 0001:000420a0       _winUnlock                 110430a0 f    CIL library: CIL module
 0001:00042140       _winFileControl            11043140 f    CIL library: CIL module
 0001:00042160       _winSectorSize             11043160 f    CIL library: CIL module
 0001:00042170       _winDeviceCharacteristics  11043170 f    CIL library: CIL module
 0001:00042180       _convertUtf8Filename       11043180 f    CIL library: CIL module
 0001:00042200       _winOpen                   11043200 f    CIL library: CIL module
 0001:00042380       _winDelete                 11043380 f    CIL library: CIL module
 0001:00042490       _winAccess                 11043490 f    CIL library: CIL module
 0001:00042550       _winGetTempname            11043550 f    CIL library: CIL module
 0001:000427c0       _winFullPathname           110437c0 f    CIL library: CIL module
 0001:00042900       _winDlOpen                 11043900 f    CIL library: CIL module
 0001:00042980       _winDlError                11043980 f    CIL library: CIL module
 0001:000429e0       _winRandomness             110439e0 f    CIL library: CIL module
 0001:00042a80       _winSleep                  11043a80 f    CIL library: CIL module
 0001:00042b10       _listRemove                11043b10 f    CIL library: CIL module
 0001:00042b70       _pageInStatement           11043b70 f    CIL library: CIL module
 0001:00042bc0       _pager_resize_hash_table   11043bc0 f    CIL library: CIL module
 0001:00042c60       _read32bits                11043c60 f    CIL library: CIL module
 0001:00042cc0       _write32bits               11043cc0 f    CIL library: CIL module
 0001:00042d00       _pager_error               11043d00 f    CIL library: CIL module
 0001:00042d40       _readMasterJournal         11043d40 f    CIL library: CIL module
 0001:00042e80       _seekJournalHdr            11043e80 f    CIL library: CIL module
 0001:00042ee0       _writeJournalHdr           11043ee0 f    CIL library: CIL module
 0001:000430c0       _readJournalHdr            110440c0 f    CIL library: CIL module
 0001:00043210       _writeMasterJournal        11044210 f    CIL library: CIL module
 0001:00043390       _page_add_to_stmt_list     11044390 f    CIL library: CIL module
 0001:000433d0       _pager_lookup              110443d0 f    CIL library: CIL module
 0001:00043400       _pager_reset               11044400 f    CIL library: CIL module
 0001:00043500       _pager_unlock              11044500 f    CIL library: CIL module
 0001:000435d0       _pager_end_transaction     110445d0 f    CIL library: CIL module
 0001:00043720       _pager_cksum               11044720 f    CIL library: CIL module
 0001:00043790       _pager_playback_one_page   11044790 f    CIL library: CIL module
 0001:00043970       _pager_delmaster           11044970 f    CIL library: CIL module
 0001:00043bb0       _pager_truncate            11044bb0 f    CIL library: CIL module
 0001:00043c20       _setSectorSize             11044c20 f    CIL library: CIL module
 0001:00043c60       _pager_playback            11044c60 f    CIL library: CIL module
 0001:00043ec0       _pager_stmt_playback       11044ec0 f    CIL library: CIL module
 0001:000440c0       _sqlite3PagerOpen          110450c0 f    CIL library: CIL module
 0001:000444c0       _sqlite3PagerSetPagesize   110454c0 f    CIL library: CIL module
 0001:00044550       _sqlite3PagerReadFileheader 11045550 f    CIL library: CIL module
 0001:000445a0       _sqlite3PagerPagecount     110455a0 f    CIL library: CIL module
 0001:00044670       _unlinkHashChain           11045670 f    CIL library: CIL module
 0001:000446e0       _pager_truncate_cache      110456e0 f    CIL library: CIL module
 0001:00044800       _pager_wait_on_lock        11045800 f    CIL library: CIL module
 0001:00044880       _sqlite3PagerTruncate      11045880 f    CIL library: CIL module
 0001:000448e0       _sqlite3PagerClose         110458e0 f    CIL library: CIL module
 0001:000449a0       __page_ref                 110459a0 f    CIL library: CIL module
 0001:000449d0       _sqlite3PagerRef           110459d0 f    CIL library: CIL module
 0001:00044a10       _syncJournal               11045a10 f    CIL library: CIL module
 0001:00044af0       _merge_pagelist            11045af0 f    CIL library: CIL module
 0001:00044b60       _sort_pagelist             11045b60 f    CIL library: CIL module
 0001:00044bf0       _pager_write_pagelist      11045bf0 f    CIL library: CIL module
 0001:00044d00       _hasHotJournal             11045d00 f    CIL library: CIL module
 0001:00044d60       _pager_recycle             11045d60 f    CIL library: CIL module
 0001:00044e30       _readDbPage                11045e30 f    CIL library: CIL module
 0001:00044ec0       _pagerSharedLock           11045ec0 f    CIL library: CIL module
 0001:000450e0       _pagerAllocatePage         110460e0 f    CIL library: CIL module
 0001:000451d0       _pager_get_content         110461d0 f    CIL library: CIL module
 0001:00045200       _pagerAcquire              11046200 f    CIL library: CIL module
 0001:00045420       _sqlite3PagerLookup        11046420 f    CIL library: CIL module
 0001:00045480       _sqlite3PagerUnref         11046480 f    CIL library: CIL module
 0001:00045530       _pager_open_journal        11046530 f    CIL library: CIL module
 0001:00045650       _sqlite3PagerBegin         11046650 f    CIL library: CIL module
 0001:00045720       _makeDirty                 11046720 f    CIL library: CIL module
 0001:00045750       _makeClean                 11046750 f    CIL library: CIL module
 0001:00045790       _pager_write               11046790 f    CIL library: CIL module
 0001:00045ab0       _sqlite3PagerWrite         11046ab0 f    CIL library: CIL module
 0001:00045c60       _sqlite3PagerOverwrite     11046c60 f    CIL library: CIL module
 0001:00045cc0       _sqlite3PagerDontWrite     11046cc0 f    CIL library: CIL module
 0001:00045cf0       _sqlite3PagerDontRollback  11046cf0 f    CIL library: CIL module
 0001:00045d50       _pager_incr_changecounter  11046d50 f    CIL library: CIL module
 0001:00045e00       _sqlite3PagerCommitPhaseOne 11046e00 f    CIL library: CIL module
 0001:00045f90       _sqlite3PagerCommitPhaseTwo 11046f90 f    CIL library: CIL module
 0001:00046100       _sqlite3PagerRollback      11047100 f    CIL library: CIL module
 0001:00046300       _pagerStmtBegin            11047300 f    CIL library: CIL module
 0001:000463f0       _sqlite3PagerStmtCommit    110473f0 f    CIL library: CIL module
 0001:000464d0       _sqlite3PagerStmtRollback  110474d0 f    CIL library: CIL module
 0001:00046570       _sqlite3PagerMovepage      11047570 f    CIL library: CIL module
 0001:00046760       _sqlite3BtreeEnter         11047760 f    CIL library: CIL module
 0001:00046800       _sqlite3BtreeLeave         11047800 f    CIL library: CIL module
 0001:00046830       _sqlite3BtreeEnterAll      11047830 f    CIL library: CIL module
 0001:00046910       _sqlite3BtreeLeaveAll      11047910 f    CIL library: CIL module
 0001:00046960       _sqlite3BtreeMutexArrayInsert 11047960 f    CIL library: CIL module
 0001:000469c0       _sqlite3BtreeMutexArrayEnter 110479c0 f    CIL library: CIL module
 0001:00046a30       _sqlite3BtreeMutexArrayLeave 11047a30 f    CIL library: CIL module
 0001:00046a90       _queryTableLock            11047a90 f    CIL library: CIL module
 0001:00046af0       _lockTable                 11047af0 f    CIL library: CIL module
 0001:00046b80       _unlockAllTables           11047b80 f    CIL library: CIL module
 0001:00046c20       _invalidateAllOverflowCache 11047c20 f    CIL library: CIL module
 0001:00046ca0       _saveCursorPosition        11047ca0 f    CIL library: CIL module
 0001:00046d70       _saveAllCursors            11047d70 f    CIL library: CIL module
 0001:00046db0       _sqlite3BtreeRestoreOrClearCursorPosition 11047db0 f    CIL library: CIL module
 0001:00046e20       _ptrmapPageno              11047e20 f    CIL library: CIL module
 0001:00046e60       _ptrmapPut                 11047e60 f    CIL library: CIL module
 0001:00046f60       _ptrmapGet                 11047f60 f    CIL library: CIL module
 0001:00047060       _findOverflowCell          11048060 f    CIL library: CIL module
 0001:000470b0       _sqlite3BtreeParseCellPtr  110480b0 f    CIL library: CIL module
 0001:000471f0       _cellSizePtr               110481f0 f    CIL library: CIL module
 0001:00047210       _ptrmapPutOvflPtr          11048210 f    CIL library: CIL module
 0001:000472a0       _defragmentPage            110482a0 f    CIL library: CIL module
 0001:000473b0       _allocateSpace             110483b0 f    CIL library: CIL module
 0001:00047520       _freeSpace                 11048520 f    CIL library: CIL module
 0001:000476d0       _decodeFlags               110486d0 f    CIL library: CIL module
 0001:00047750       _sqlite3BtreeInitPage      11048750 f    CIL library: CIL module
 0001:000478c0       _zeroPage                  110488c0 f    CIL library: CIL module
 0001:00047950       _sqlite3BtreeGetPage       11048950 f    CIL library: CIL module
 0001:000479a0       _getAndInitPage            110489a0 f    CIL library: CIL module
 0001:00047a10       _pageDestructor            11048a10 f    CIL library: CIL module
 0001:00047a40       _pageReinit                11048a40 f    CIL library: CIL module
 0001:00047a70       _sqlite3BtreeInvokeBusyHandler 11048a70 f    CIL library: CIL module
 0001:00047ab0       _sqlite3BtreeOpen          11048ab0 f    CIL library: CIL module
 0001:00047f30       _removeFromSharingList     11048f30 f    CIL library: CIL module
 0001:00047fc0       _sqlite3BtreeClose         11048fc0 f    CIL library: CIL module
 0001:00048090       _sqlite3BtreeSetCacheSize  11049090 f    CIL library: CIL module
 0001:000480e0       _sqlite3BtreeSetSafetyLevel 110490e0 f    CIL library: CIL module
 0001:00048160       _sqlite3BtreeSyncDisabled  11049160 f    CIL library: CIL module
 0001:000481a0       _sqlite3BtreeSetPageSize   110491a0 f    CIL library: CIL module
 0001:00048270       _sqlite3BtreeMaxPageCount  11049270 f    CIL library: CIL module
 0001:000482c0       _sqlite3BtreeSetAutoVacuum 110492c0 f    CIL library: CIL module
 0001:00048320       _sqlite3BtreeGetAutoVacuum 11049320 f    CIL library: CIL module
 0001:00048370       _lockBtree                 11049370 f    CIL library: CIL module
 0001:00048530       _unlockBtreeIfUnused       11049530 f    CIL library: CIL module
 0001:00048570       _newDatabase               11049570 f    CIL library: CIL module
 0001:00048660       _sqlite3BtreeBeginTrans    11049660 f    CIL library: CIL module
 0001:00048800       _setChildPtrmaps           11049800 f    CIL library: CIL module
 0001:00048900       _modifyPagePointer         11049900 f    CIL library: CIL module
 0001:00048ae0       _relocatePage              11049ae0 f    CIL library: CIL module
 0001:00048c00       _incrVacuumStep            11049c00 f    CIL library: CIL module
 0001:00048e20       _sqlite3BtreeIncrVacuum    11049e20 f    CIL library: CIL module
 0001:00048e80       _autoVacuumCommit          11049e80 f    CIL library: CIL module
 0001:00049020       _sqlite3BtreeCommitPhaseOne 1104a020 f    CIL library: CIL module
 0001:000490d0       _sqlite3BtreeCommitPhaseTwo 1104a0d0 f    CIL library: CIL module
 0001:00049190       _sqlite3BtreeCommit        1104a190 f    CIL library: CIL module
 0001:000491e0       _sqlite3BtreeTripAllCursors 1104a1e0 f    CIL library: CIL module
 0001:000492a0       _sqlite3BtreeRollback      1104a2a0 f    CIL library: CIL module
 0001:000493d0       _sqlite3BtreeBeginStmt     1104a3d0 f    CIL library: CIL module
 0001:00049440       _sqlite3BtreeCommitStmt    1104a440 f    CIL library: CIL module
 0001:000494a0       _sqlite3BtreeRollbackStmt  1104a4a0 f    CIL library: CIL module
 0001:00049500       _dfltCompare               1104a500 f    CIL library: CIL module
 0001:00049590       _btreeCursor               1104a590 f    CIL library: CIL module
 0001:00049710       _sqlite3BtreeCursor        1104a710 f    CIL library: CIL module
 0001:00049770       _sqlite3BtreeCloseCursor   1104a770 f    CIL library: CIL module
 0001:00049830       _sqlite3BtreeGetTempCursor 1104a830 f    CIL library: CIL module
 0001:00049870       _getCellInfo               1104a870 f    CIL library: CIL module
 0001:000498b0       _sqlite3BtreeKeySize       1104a8b0 f    CIL library: CIL module
 0001:00049900       _sqlite3BtreeDataSize      1104a900 f    CIL library: CIL module
 0001:00049950       _getOverflowPage           1104a950 f    CIL library: CIL module
 0001:00049af0       _copyPayload               1104aaf0 f    CIL library: CIL module
 0001:00049b20       _accessPayload             1104ab20 f    CIL library: CIL module
 0001:00049e30       _sqlite3BtreeKey           1104ae30 f    CIL library: CIL module
 0001:00049e70       _sqlite3BtreeData          1104ae70 f    CIL library: CIL module
 0001:00049eb0       _sqlite3BtreeKeyFetch      1104aeb0 f    CIL library: CIL module
 0001:00049f20       _sqlite3BtreeDataFetch     1104af20 f    CIL library: CIL module
 0001:00049fa0       _moveToChild               1104afa0 f    CIL library: CIL module
 0001:0004a000       _sqlite3BtreeMoveToParent  1104b000 f    CIL library: CIL module
 0001:0004a070       _moveToRoot                1104b070 f    CIL library: CIL module
 0001:0004a160       _moveToLeftmost            1104b160 f    CIL library: CIL module
 0001:0004a270       _moveToRightmost           1104b270 f    CIL library: CIL module
 0001:0004a380       _sqlite3BtreeLast          1104b380 f    CIL library: CIL module
 0001:0004a3b0       _sqlite3BtreeMoveto        1104b3b0 f    CIL library: CIL module
 0001:0004a7e0       _btreeNext                 1104b7e0 f    CIL library: CIL module
 0001:0004a920       _btreePrevious             1104b920 f    CIL library: CIL module
 0001:0004aa60       _allocateBtreePage         1104ba60 f    CIL library: CIL module
 0001:0004b0b0       _freePage                  1104c0b0 f    CIL library: CIL module
 0001:0004b320       _clearCell                 1104c320 f    CIL library: CIL module
 0001:0004b420       _fillInCell                1104c420 f    CIL library: CIL module
 0001:0004b6e0       _reparentPage              1104c6e0 f    CIL library: CIL module
 0001:0004b770       _reparentChildPages        1104c770 f    CIL library: CIL module
 0001:0004b830       _dropCell                  1104c830 f    CIL library: CIL module
 0001:0004b8b0       _insertCell                1104c8b0 f    CIL library: CIL module
 0001:0004baa0       _assemblePage              1104caa0 f    CIL library: CIL module
 0001:0004bbb0       _balance_quick             1104cbb0 f    CIL library: CIL module
 0001:0004bdb0       _balance_nonroot           1104cdb0 f    CIL library: CIL module
 0001:0004ca40       _balance_shallower         1104da40 f    CIL library: CIL module
 0001:0004cc80       _balance_deeper            1104dc80 f    CIL library: CIL module
 0001:0004ce00       _balance                   1104de00 f    CIL library: CIL module
 0001:0004ce90       _checkReadLocks            1104de90 f    CIL library: CIL module
 0001:0004cf10       _sqlite3BtreeInsert        1104df10 f    CIL library: CIL module
 0001:0004d100       _sqlite3BtreeDelete        1104e100 f    CIL library: CIL module
 0001:0004d3d0       _btreeCreateTable          1104e3d0 f    CIL library: CIL module
 0001:0004d640       _sqlite3BtreeCreateTable   1104e640 f    CIL library: CIL module
 0001:0004d690       _clearDatabasePage         1104e690 f    CIL library: CIL module
 0001:0004d7f0       _sqlite3BtreeClearTable    1104e7f0 f    CIL library: CIL module
 0001:0004d880       _btreeDropTable            1104e880 f    CIL library: CIL module
 0001:0004dab0       _sqlite3BtreeDropTable     1104eab0 f    CIL library: CIL module
 0001:0004db00       _sqlite3BtreeGetMeta       1104eb00 f    CIL library: CIL module
 0001:0004dc00       _sqlite3BtreeUpdateMeta    1104ec00 f    CIL library: CIL module
 0001:0004dca0       _sqlite3BtreeFlags         1104eca0 f    CIL library: CIL module
 0001:0004dcd0       _checkAppendMsg            1104ecd0 f    CIL library: CIL module
 0001:0004dd60       _checkRef                  1104ed60 f    CIL library: CIL module
 0001:0004ddc0       _checkPtrmap               1104edc0 f    CIL library: CIL module
 0001:0004de40       _checkList                 1104ee40 f    CIL library: CIL module
 0001:0004e030       _checkTreePage             1104f030 f    CIL library: CIL module
 0001:0004e5c0       _sqlite3BtreeIntegrityCheck 1104f5c0 f    CIL library: CIL module
 0001:0004ea20       _btreeCopyFile             1104fa20 f    CIL library: CIL module
 0001:0004ec20       _sqlite3BtreeCopyFile      1104fc20 f    CIL library: CIL module
 0001:0004ec90       _sqlite3BtreeSchema        1104fc90 f    CIL library: CIL module
 0001:0004ed00       _sqlite3BtreeSchemaLocked  1104fd00 f    CIL library: CIL module
 0001:0004ed80       _sqlite3BtreeLockTable     1104fd80 f    CIL library: CIL module
 0001:0004edf0       _sqlite3BtreePutData       1104fdf0 f    CIL library: CIL module
 0001:0004ee70       _sqlite3VdbeFifoPush       1104fe70 f    CIL library: CIL module
 0001:0004ef10       _sqlite3VdbeFifoPop        1104ff10 f    CIL library: CIL module
 0001:0004ef60       _sqlite3VdbeFifoClear      1104ff60 f    CIL library: CIL module
 0001:0004efe0       _sqlite3VdbeChangeEncoding 1104ffe0 f    CIL library: CIL module
 0001:0004f000       _sqlite3VdbeMemDynamicify  11050000 f    CIL library: CIL module
 0001:0004f090       _sqlite3VdbeMemExpandBlob  11050090 f    CIL library: CIL module
 0001:0004f140       _sqlite3VdbeMemMakeWriteable 11050140 f    CIL library: CIL module
 0001:0004f1e0       _sqlite3VdbeMemNulTerminate 110501e0 f    CIL library: CIL module
 0001:0004f2a0       _sqlite3VdbeMemStringify   110502a0 f    CIL library: CIL module
 0001:0004f320       _sqlite3VdbeMemFinalize    11050320 f    CIL library: CIL module
 0001:0004f3b0       _sqlite3VdbeMemRelease     110503b0 f    CIL library: CIL module
 0001:0004f410       _doubleToInt64             11050410 f    CIL library: CIL module
 0001:0004f470       _sqlite3VdbeIntValue       11050470 f    CIL library: CIL module
 0001:0004f500       _sqlite3VdbeRealValue      11050500 f    CIL library: CIL module
 0001:0004f580       _sqlite3VdbeIntegerAffinity 11050580 f    CIL library: CIL module
 0001:0004f5b0       _sqlite3VdbeMemIntegerify  110505b0 f    CIL library: CIL module
 0001:0004f5e0       _sqlite3VdbeMemRealify     110505e0 f    CIL library: CIL module
 0001:0004f610       _sqlite3VdbeMemNumerify    11050610 f    CIL library: CIL module
 0001:0004f690       _sqlite3VdbeMemSetNull     11050690 f    CIL library: CIL module
 0001:0004f6b0       _sqlite3VdbeMemSetDouble   110506b0 f    CIL library: CIL module
 0001:0004f710       _sqlite3VdbeMemTooBig      11050710 f    CIL library: CIL module
 0001:0004f740       _sqlite3VdbeMemShallowCopy 11050740 f    CIL library: CIL module
 0001:0004f780       _sqlite3VdbeMemCopy        11050780 f    CIL library: CIL module
 0001:0004f7e0       _sqlite3VdbeMemMove        110507e0 f    CIL library: CIL module
 0001:0004f830       _sqlite3VdbeMemSetStr      11050830 f    CIL library: CIL module
 0001:0004f950       _sqlite3MemCompare         11050950 f    CIL library: CIL module
 0001:0004fb90       _sqlite3VdbeMemFromBtree   11050b90 f    CIL library: CIL module
 0001:0004fcc0       _sqlite3ValueText          11050cc0 f    CIL library: CIL module
 0001:0004fd60       _sqlite3ValueNew           11050d60 f    CIL library: CIL module
 0001:0004fdb0       _sqlite3ValueFromExpr      11050db0 f    CIL library: CIL module
 0001:0004ffb0       _sqlite3ValueFree          11050fb0 f    CIL library: CIL module
 0001:0004ffe0       _sqlite3VdbeCreate         11050fe0 f    CIL library: CIL module
 0001:00050050       _sqlite3VdbeSetSql         11051050 f    CIL library: CIL module
 0001:000500b0       _sqlite3VdbeSwap           110510b0 f    CIL library: CIL module
 0001:00050140       _resizeOpArray             11051140 f    CIL library: CIL module
 0001:000501a0       _sqlite3VdbeAddOp3         110511a0 f    CIL library: CIL module
 0001:00050210       _sqlite3VdbeAddOp2         11051210 f    CIL library: CIL module
 0001:00050230       _sqlite3VdbeAddOp4         11051230 f    CIL library: CIL module
 0001:00050260       _sqlite3VdbeMakeLabel      11051260 f    CIL library: CIL module
 0001:000502d0       _sqlite3VdbeResolveLabel   110512d0 f    CIL library: CIL module
 0001:000502f0       _resolveP2Values           110512f0 f    CIL library: CIL module
 0001:00050470       _sqlite3VdbeAddOpList      11051470 f    CIL library: CIL module
 0001:00050530       _sqlite3VdbeChangeP1       11051530 f    CIL library: CIL module
 0001:00050550       _sqlite3VdbeChangeP2       11051550 f    CIL library: CIL module
 0001:00050570       _sqlite3VdbeChangeP3       11051570 f    CIL library: CIL module
 0001:00050590       _sqlite3VdbeChangeP5       11051590 f    CIL library: CIL module
 0001:000505b0       _sqlite3VdbeJumpHere       110515b0 f    CIL library: CIL module
 0001:000505d0       _freeP4                    110515d0 f    CIL library: CIL module
 0001:00050660       _sqlite3VdbeChangeToNoop   11051660 f    CIL library: CIL module
 0001:000506b0       _sqlite3VdbeChangeP4       110516b0 f    CIL library: CIL module
 0001:000507c0       _displayP4                 110517c0 f    CIL library: CIL module
 0001:00050a10       _sqlite3VdbeUsesBtree      11051a10 f    CIL library: CIL module
 0001:00050a50       _releaseMemArray           11051a50 f    CIL library: CIL module
 0001:00050b30       _sqlite3VdbeList           11051b30 f    CIL library: CIL module
 0001:00050d20       _sqlite3VdbeMakeReady      11051d20 f    CIL library: CIL module
 0001:00050ec0       _sqlite3VdbeFreeCursor     11051ec0 f    CIL library: CIL module
 0001:00050f30       _closeAllCursorsExceptActiveVtabs 11051f30 f    CIL library: CIL module
 0001:00050f80       _Cleanup                   11051f80 f    CIL library: CIL module
 0001:000510a0       _sqlite3VdbeSetNumCols     110520a0 f    CIL library: CIL module
 0001:00051140       _sqlite3VdbeSetColName     11052140 f    CIL library: CIL module
 0001:00051210       _vdbeCommit                11052210 f    CIL library: CIL module
 0001:000517c0       _invalidateCursorsOnModifiedBtrees 110527c0 f    CIL library: CIL module
 0001:00051800       _sqlite3VdbeHalt           11052800 f    CIL library: CIL module
 0001:00051ac0       _sqlite3VdbeReset          11052ac0 f    CIL library: CIL module
 0001:00051ba0       _sqlite3VdbeFinalize       11052ba0 f    CIL library: CIL module
 0001:00051be0       _sqlite3VdbeDeleteAuxData  11052be0 f    CIL library: CIL module
 0001:00051c30       _sqlite3VdbeDelete         11052c30 f    CIL library: CIL module
 0001:00051e90       _sqlite3VdbeCursorMoveto   11052e90 f    CIL library: CIL module
 0001:00051f10       _sqlite3VdbeSerialType     11052f10 f    CIL library: CIL module
 0001:00051ff0       _sqlite3VdbeSerialTypeLen  11052ff0 f    CIL library: CIL module
 0001:00052010       _sqlite3VdbeSerialPut      11053010 f    CIL library: CIL module
 0001:000520c0       _sqlite3VdbeSerialGet      110530c0 f    CIL library: CIL module
 0001:000522c0       _sqlite3VdbeRecordCompare  110532c0 f    CIL library: CIL module
 0001:00052730       _sqlite3VdbeIdxRowidLen    11053730 f    CIL library: CIL module
 0001:00052770       _sqlite3VdbeIdxRowid       11053770 f    CIL library: CIL module
 0001:00052850       _sqlite3VdbeIdxKeyCompare  11053850 f    CIL library: CIL module
 0001:00052930       _sqlite3ExpirePreparedStatements 11053930 f    CIL library: CIL module
 0001:00052e80       _sqlite3Step               11053e80 f    CIL library: CIL module
 0001:00053190       _sqlite3InvalidFunction    11054190 f    CIL library: CIL module
 0001:00053400       _columnMem                 11054400 f    CIL library: CIL module
 0001:00053970       _columnName                11054970 f    CIL library: CIL module
 0001:00053a70       _vdbeUnbind                11054a70 f    CIL library: CIL module
 0001:00053af0       _bindText                  11054af0 f    CIL library: CIL module
 0001:00053e90       _createVarMap              11054e90 f    CIL library: CIL module
 0001:00054070       __storeTypeInfo            11055070 f    CIL library: CIL module
 0001:000540a0       _allocateCursor            110550a0 f    CIL library: CIL module
 0001:00054100       _applyNumericAffinity      11055100 f    CIL library: CIL module
 0001:000541c0       _applyAffinity             110551c0 f    CIL library: CIL module
 0001:00054290       _sqlite3VdbeExec           11055290 f    CIL library: CIL module
 0001:00058620       _blobReadWrite             11059620 f    CIL library: CIL module
 0001:00058780       _sqlite3ExprAffinity       11059780 f    CIL library: CIL module
 0001:000587b0       _sqlite3ExprSetColl        110597b0 f    CIL library: CIL module
 0001:00058800       _sqlite3ExprCollSeq        11059800 f    CIL library: CIL module
 0001:00058870       _sqlite3CompareAffinity    11059870 f    CIL library: CIL module
 0001:000588d0       _comparisonAffinity        110598d0 f    CIL library: CIL module
 0001:00058940       _sqlite3IndexAffinityOk    11059940 f    CIL library: CIL module
 0001:00058980       _sqlite3BinaryCompareCollSeq 11059980 f    CIL library: CIL module
 0001:000589c0       _codeCompare               110599c0 f    CIL library: CIL module
 0001:00058b00       _sqlite3Expr               11059b00 f    CIL library: CIL module
 0001:00058c00       _sqlite3RegisterExpr       11059c00 f    CIL library: CIL module
 0001:00058cd0       _sqlite3ExprSpan           11059cd0 f    CIL library: CIL module
 0001:00058d10       _sqlite3ExprFunction       11059d10 f    CIL library: CIL module
 0001:00058da0       _sqlite3ExprAssignVarNumber 11059da0 f    CIL library: CIL module
 0001:00058fa0       _sqlite3ExprDelete         11059fa0 f    CIL library: CIL module
 0001:00059010       _sqlite3DequoteExpr        1105a010 f    CIL library: CIL module
 0001:00059040       _sqlite3ExprDup            1105a040 f    CIL library: CIL module
 0001:00059100       _sqlite3TokenCopy          1105a100 f    CIL library: CIL module
 0001:00059190       _sqlite3ExprListDup        1105a190 f    CIL library: CIL module
 0001:000592b0       _sqlite3SrcListDup         1105a2b0 f    CIL library: CIL module
 0001:000594a0       _sqlite3IdListDup          1105a4a0 f    CIL library: CIL module
 0001:00059570       _sqlite3SelectDup          1105a570 f    CIL library: CIL module
 0001:00059670       _sqlite3ExprListAppend     1105a670 f    CIL library: CIL module
 0001:00059740       _sqlite3ExprListCheckLength 1105a740 f    CIL library: CIL module
 0001:00059760       _heightOfSelect            1105a760 f    CIL library: CIL module
 0001:00059850       _sqlite3ExprSetHeight      1105a850 f    CIL library: CIL module
 0001:000598d0       _sqlite3SelectExprHeight   1105a8d0 f    CIL library: CIL module
 0001:000598f0       _sqlite3ExprListDelete     1105a8f0 f    CIL library: CIL module
 0001:00059a30       _walkExprTree              1105aa30 f    CIL library: CIL module
 0001:00059ab0       _walkExprList              1105aab0 f    CIL library: CIL module
 0001:00059b00       _walkSelectExpr            1105ab00 f    CIL library: CIL module
 0001:00059b60       _exprNodeIsConstant        1105ab60 f    CIL library: CIL module
 0001:00059c50       _sqlite3ExprIsConstant     1105ac50 f    CIL library: CIL module
 0001:00059c70       _sqlite3ExprIsInteger      1105ac70 f    CIL library: CIL module
 0001:00059ce0       _sqlite3IsRowid            1105ace0 f    CIL library: CIL module
 0001:00059d20       _lookupName                1105ad20 f    CIL library: CIL module
 0001:0005a5d0       _nameResolverStep          1105b5d0 f    CIL library: CIL module
 0001:0005a920       _sqlite3ExprResolveNames   1105b920 f    CIL library: CIL module
 0001:0005a9d0       _sqlite3FindInIndex        1105b9d0 f    CIL library: CIL module
 0001:0005ad00       _sqlite3CodeSubselect      1105bd00 f    CIL library: CIL module
 0001:0005b090       _dup8bytes                 1105c090 f    CIL library: CIL module
 0001:0005b0d0       _codeReal                  1105c0d0 f    CIL library: CIL module
 0001:0005b1b0       _codeInteger               1105c1b0 f    CIL library: CIL module
 0001:0005b2e0       _sqlite3ExprCodeGetColumn  1105c2e0 f    CIL library: CIL module
 0001:0005b380       _sqlite3ExprCodeTarget     1105c380 f    CIL library: CIL module
 0001:0005c0b0       _sqlite3ExprCodeTemp       1105d0b0 f    CIL library: CIL module
 0001:0005c110       _sqlite3ExprCode           1105d110 f    CIL library: CIL module
 0001:0005c150       _sqlite3ExprCodeAndCache   1105d150 f    CIL library: CIL module
 0001:0005c1c0       _sqlite3ExprCodeExprList   1105d1c0 f    CIL library: CIL module
 0001:0005c210       _sqlite3ExprIfTrue         1105d210 f    CIL library: CIL module
 0001:0005c500       _sqlite3ExprIfFalse        1105d500 f    CIL library: CIL module
 0001:0005c7c0       _sqlite3ExprCompare        1105d7c0 f    CIL library: CIL module
 0001:0005c8e0       _analyzeAggregate          1105d8e0 f    CIL library: CIL module
 0001:0005cba0       _sqlite3ExprAnalyzeAggList 1105dba0 f    CIL library: CIL module
 0001:0005cbe0       _sqlite3GetTempReg         1105dbe0 f    CIL library: CIL module
 0001:0005cc00       _sqlite3ReleaseTempReg     1105dc00 f    CIL library: CIL module
 0001:0005cc20       _sqlite3GetTempRange       1105dc20 f    CIL library: CIL module
 0001:0005cc50       _renameTableFunc           1105dc50 f    CIL library: CIL module
 0001:0005cd10       _renameTriggerFunc         1105dd10 f    CIL library: CIL module
 0001:0005ce10       _whereTempTriggers         1105de10 f    CIL library: CIL module
 0001:0005ce90       _reloadTableSchema         1105de90 f    CIL library: CIL module
 0001:0005d300       _sqlite3AlterRenameTable   1105e300 f    CIL library: CIL module
 0001:0005d5b0       _sqlite3AlterFinishAddColumn 1105e5b0 f    CIL library: CIL module
 0001:0005d7e0       _sqlite3AlterBeginAddColumn 1105e7e0 f    CIL library: CIL module
 0001:0005d9c0       _openStatTable             1105e9c0 f    CIL library: CIL module
 0001:0005dac0       _analyzeOneTable           1105eac0 f    CIL library: CIL module
 0001:0005efd0       _analyzeDatabase           1105ffd0 f    CIL library: CIL module
 0001:0005f130       _analyzeTable              11060130 f    CIL library: CIL module
 0001:0005f1c0       _sqlite3Analyze            110601c0 f    CIL library: CIL module
 0001:0005f320       _analysisLoader            11060320 f    CIL library: CIL module
 0001:0005f3a0       _sqlite3AnalysisLoad       110603a0 f    CIL library: CIL module
 0001:0005f4d0       _resolveAttachExpr         110604d0 f    CIL library: CIL module
 0001:0005f540       _attachFunc                11060540 f    CIL library: CIL module
 0001:0005f8f0       _detachFunc                110608f0 f    CIL library: CIL module
 0001:0005fb10       _codeAttach                11060b10 f    CIL library: CIL module
 0001:0005fd20       _sqlite3FixInit            11060d20 f    CIL library: CIL module
 0001:0005fd50       _sqlite3FixSrcList         11060d50 f    CIL library: CIL module
 0001:0005fe60       _sqlite3FixSelect          11060e60 f    CIL library: CIL module
 0001:0005fef0       _sqlite3FixExpr            11060ef0 f    CIL library: CIL module
 0001:0005ff70       _sqlite3FixTriggerStep     11060f70 f    CIL library: CIL module
 0001:00060050       _sqliteAuthBadReturnCode   11061050 f    CIL library: CIL module
 0001:00060070       _sqlite3AuthRead           11061070 f    CIL library: CIL module
 0001:00060220       _sqlite3AuthCheck          11061220 f    CIL library: CIL module
 0001:000602b0       _sqlite3AuthContextPush    110612b0 f    CIL library: CIL module
 0001:000602d0       _sqlite3TableLock          110612d0 f    CIL library: CIL module
 0001:00060410       _codeTableLocks            11061410 f    CIL library: CIL module
 0001:000605a0       _sqlite3FinishCoding       110615a0 f    CIL library: CIL module
 0001:00060820       _sqlite3NestedParse        11061820 f    CIL library: CIL module
 0001:000608c0       _sqlite3FindTable          110618c0 f    CIL library: CIL module
 0001:000609c0       _sqlite3LocateTable        110619c0 f    CIL library: CIL module
 0001:00060a50       _sqlite3FindIndex          11061a50 f    CIL library: CIL module
 0001:00060b60       _sqliteDeleteIndex         11061b60 f    CIL library: CIL module
 0001:00060be0       _sqlite3UnlinkAndDeleteIndex 11061be0 f    CIL library: CIL module
 0001:00060d20       _sqlite3ResetInternalSchema 11061d20 f    CIL library: CIL module
 0001:00060f50       _sqliteResetColumnNames    11061f50 f    CIL library: CIL module
 0001:00061110       _sqlite3DeleteTable        11062110 f    CIL library: CIL module
 0001:00061520       _sqlite3UnlinkAndDeleteTable 11062520 f    CIL library: CIL module
 0001:00061670       _sqlite3NameFromToken      11062670 f    CIL library: CIL module
 0001:000616e0       _sqlite3OpenMasterTable    110626e0 f    CIL library: CIL module
 0001:00061770       _sqlite3FindDb             11062770 f    CIL library: CIL module
 0001:00061830       _sqlite3TwoPartName        11062830 f    CIL library: CIL module
 0001:00061880       _sqlite3CheckObjectName    11062880 f    CIL library: CIL module
 0001:000618d0       _sqlite3StartTable         110628d0 f    CIL library: CIL module
 0001:00061d70       _sqlite3AddColumn          11062d70 f    CIL library: CIL module
 0001:00061eb0       _sqlite3AffinityType       11062eb0 f    CIL library: CIL module
 0001:00061f70       _sqlite3AddColumnType      11062f70 f    CIL library: CIL module
 0001:00061fc0       _sqlite3AddDefaultValue    11062fc0 f    CIL library: CIL module
 0001:00062060       _sqlite3AddPrimaryKey      11063060 f    CIL library: CIL module
 0001:000621f0       _sqlite3AddCheckConstraint 110631f0 f    CIL library: CIL module
 0001:00062260       _sqlite3AddCollateType     11063260 f    CIL library: CIL module
 0001:000622e0       _sqlite3LocateCollSeq      110632e0 f    CIL library: CIL module
 0001:00062370       _sqlite3ChangeCookie       11063370 f    CIL library: CIL module
 0001:000623e0       _identPut                  110633e0 f    CIL library: CIL module
 0001:000624a0       _createTableStmt           110634a0 f    CIL library: CIL module
 0001:000626b0       _sqlite3EndTable           110636b0 f    CIL library: CIL module
 0001:00062b30       _sqlite3CreateView         11063b30 f    CIL library: CIL module
 0001:00063020       _sqlite3ViewGetColumnNames 11064020 f    CIL library: CIL module
 0001:00063160       _sqliteViewResetAll        11064160 f    CIL library: CIL module
 0001:000631b0       _sqlite3RootPageMoved      110641b0 f    CIL library: CIL module
 0001:00063200       _destroyRootPage           11064200 f    CIL library: CIL module
 0001:00063280       _destroyTable              11064280 f    CIL library: CIL module
 0001:00063310       _sqlite3DropTable          11064310 f    CIL library: CIL module
 0001:00063650       _sqlite3CreateForeignKey   11064650 f    CIL library: CIL module
 0001:00063950       _sqlite3DeferForeignKey    11064950 f    CIL library: CIL module
 0001:00063970       _sqlite3RefillIndex        11064970 f    CIL library: CIL module
 0001:00063d50       _sqlite3CreateIndex        11064d50 f    CIL library: CIL module
 0001:000646a0       _sqlite3MinimumFileFormat  110656a0 f    CIL library: CIL module
 0001:000647d0       _sqlite3DefaultRowEst      110657d0 f    CIL library: CIL module
 0001:00064820       _sqlite3DropIndex          11065820 f    CIL library: CIL module
 0001:00064a00       _sqlite3ArrayAllocate      11065a00 f    CIL library: CIL module
 0001:00064a80       _sqlite3IdListAppend       11065a80 f    CIL library: CIL module
 0001:00064b20       _sqlite3IdListDelete       11065b20 f    CIL library: CIL module
 0001:00064c40       _sqlite3IdListIndex        11065c40 f    CIL library: CIL module
 0001:00064cb0       _sqlite3SrcListAppend      11065cb0 f    CIL library: CIL module
 0001:00064db0       _sqlite3SrcListAssignCursors 11065db0 f    CIL library: CIL module
 0001:00064e10       _sqlite3SrcListDelete      11065e10 f    CIL library: CIL module
 0001:00064fd0       _sqlite3SrcListAppendFromTerm 11065fd0 f    CIL library: CIL module
 0001:00065080       _sqlite3SrcListShiftJoinType 11066080 f    CIL library: CIL module
 0001:000650c0       _sqlite3BeginTransaction   110660c0 f    CIL library: CIL module
 0001:000651a0       _sqlite3CommitTransaction  110661a0 f    CIL library: CIL module
 0001:00065230       _sqlite3RollbackTransaction 11066230 f    CIL library: CIL module
 0001:000652c0       _sqlite3OpenTempDatabase   110662c0 f    CIL library: CIL module
 0001:00065370       _sqlite3CodeVerifySchema   11066370 f    CIL library: CIL module
 0001:00065430       _sqlite3BeginWriteOperation 11066430 f    CIL library: CIL module
 0001:000654b0       _collationMatch            110664b0 f    CIL library: CIL module
 0001:00065500       _reindexTable              11066500 f    CIL library: CIL module
 0001:00065580       _reindexDatabases          11066580 f    CIL library: CIL module
 0001:000655e0       _sqlite3Reindex            110665e0 f    CIL library: CIL module
 0001:00065760       _sqlite3IndexKeyinfo       11066760 f    CIL library: CIL module
 0001:00065860       _callCollNeeded            11066860 f    CIL library: CIL module
 0001:00065970       _synthCollSeq              11066970 f    CIL library: CIL module
 0001:00065a80       _sqlite3GetCollSeq         11066a80 f    CIL library: CIL module
 0001:00065b30       _findCollSeqEntry          11066b30 f    CIL library: CIL module
 0001:00065c50       _sqlite3FindCollSeq        11066c50 f    CIL library: CIL module
 0001:00065c80       _sqlite3FindFunction       11066c80 f    CIL library: CIL module
 0001:00065e50       _sqlite3SchemaFree         11066e50 f    CIL library: CIL module
 0001:000660e0       _sqlite3SchemaGet          110670e0 f    CIL library: CIL module
 0001:00066180       _sqlite3SrcListLookup      11067180 f    CIL library: CIL module
 0001:00066250       _sqlite3IsReadOnly         11067250 f    CIL library: CIL module
 0001:000662c0       _sqlite3OpenTable          110672c0 f    CIL library: CIL module
 0001:00066320       _sqlite3DeleteFrom         11067320 f    CIL library: CIL module
 0001:00066b00       _sqlite3GenerateRowDelete  11067b00 f    CIL library: CIL module
 0001:00066bd0       _sqlite3GenerateRowIndexDelete 11067bd0 f    CIL library: CIL module
 0001:00066d30       _sqlite3GenerateIndexKey   11067d30 f    CIL library: CIL module
 0001:00067000       _minmaxFunc                11068000 f    CIL library: CIL module
 0001:000670e0       _typeofFunc                110680e0 f    CIL library: CIL module
 0001:000671a0       _lengthFunc                110681a0 f    CIL library: CIL module
 0001:000672a0       _absFunc                   110682a0 f    CIL library: CIL module
 0001:000673b0       _substrFunc                110683b0 f    CIL library: CIL module
 0001:00067610       _roundFunc                 11068610 f    CIL library: CIL module
 0001:000676b0       _contextMalloc             110686b0 f    CIL library: CIL module
 0001:00067700       _upperFunc                 11068700 f    CIL library: CIL module
 0001:000677c0       _lowerFunc                 110687c0 f    CIL library: CIL module
 0001:00067880       _ifnullFunc                11068880 f    CIL library: CIL module
 0001:00067950       _randomFunc                11068950 f    CIL library: CIL module
 0001:000679f0       _randomBlob                110689f0 f    CIL library: CIL module
 0001:00067a90       _last_insert_rowid         11068a90 f    CIL library: CIL module
 0001:00067ad0       _changes                   11068ad0 f    CIL library: CIL module
 0001:00067b10       _total_changes             11068b10 f    CIL library: CIL module
 0001:00067b50       _patternCompare            11068b50 f    CIL library: CIL module
 0001:00067f10       _likeFunc                  11068f10 f    CIL library: CIL module
 0001:00068080       _nullifFunc                11069080 f    CIL library: CIL module
 0001:000680c0       _versionFunc               110690c0 f    CIL library: CIL module
 0001:00068100       _quoteFunc                 11069100 f    CIL library: CIL module
 0001:00068340       _hexFunc                   11069340 f    CIL library: CIL module
 0001:00068460       _zeroblobFunc              11069460 f    CIL library: CIL module
 0001:00068510       _replaceFunc               11069510 f    CIL library: CIL module
 0001:00068790       _trimFunc                  11069790 f    CIL library: CIL module
 0001:00068b90       _loadExt                   11069b90 f    CIL library: CIL module
 0001:00068ca0       _sumStep                   11069ca0 f    CIL library: CIL module
 0001:00068dd0       _sumFinalize               11069dd0 f    CIL library: CIL module
 0001:00068e80       _avgFinalize               11069e80 f    CIL library: CIL module
 0001:00068ee0       _totalFinalize             11069ee0 f    CIL library: CIL module
 0001:00068f30       _countStep                 11069f30 f    CIL library: CIL module
 0001:00068fb0       _countFinalize             11069fb0 f    CIL library: CIL module
 0001:00069010       _minmaxStep                1106a010 f    CIL library: CIL module
 0001:00069080       _minMaxFinalize            1106a080 f    CIL library: CIL module
 0001:000690d0       _groupConcatStep           1106a0d0 f    CIL library: CIL module
 0001:000691a0       _groupConcatFinalize       1106a1a0 f    CIL library: CIL module
 0001:00069240       _sqlite3RegisterBuiltinFunctions 1106a240 f    CIL library: CIL module
 0001:000695c0       _sqlite3RegisterLikeFunctions 1106a5c0 f    CIL library: CIL module
 0001:00069670       _sqlite3IsLikeFunction     1106a670 f    CIL library: CIL module
 0001:000696e0       _sqlite3IndexAffinityStr   1106a6e0 f    CIL library: CIL module
 0001:00069810       _sqlite3TableAffinityStr   1106a810 f    CIL library: CIL module
 0001:00069900       _readsTable                1106a900 f    CIL library: CIL module
 0001:00069990       _autoIncBegin              1106a990 f    CIL library: CIL module
 0001:00069b80       _autoIncStep               1106ab80 f    CIL library: CIL module
 0001:00069ba0       _autoIncEnd                1106aba0 f    CIL library: CIL module
 0001:00069cb0       _sqlite3Insert             1106acb0 f    CIL library: CIL module
 0001:0006ae30       _sqlite3GenerateConstraintChecks 1106be30 f    CIL library: CIL module
 0001:0006beb0       _sqlite3CompleteInsertion  1106ceb0 f    CIL library: CIL module
 0001:0006c290       _sqlite3OpenTableAndIndices 1106d290 f    CIL library: CIL module
 0001:0006c480       _xferCompatibleIndex       1106d480 f    CIL library: CIL module
 0001:0006c4e0       _xferOptimization          1106d4e0 f    CIL library: CIL module
 0001:0006cef0       _sqlite3LoadExtension      1106def0 f    CIL library: CIL module
 0001:0006d100       _sqlite3CloseExtensions    1106e100 f    CIL library: CIL module
 0001:0006d180       _sqlite3AutoLoadExtensions 1106e180 f    CIL library: CIL module
 0001:0006d250       _getSafetyLevel            1106e250 f    CIL library: CIL module
 0001:0006d2d0       _getLockingMode            1106e2d0 f    CIL library: CIL module
 0001:0006d300       _getAutoVacuum             1106e300 f    CIL library: CIL module
 0001:0006d360       _invalidateTempStorage     1106e360 f    CIL library: CIL module
 0001:0006d3b0       _changeTempStorage         1106e3b0 f    CIL library: CIL module
 0001:0006d420       _returnSingleInt           1106e420 f    CIL library: CIL module
 0001:0006d4f0       _flagPragma                1106e4f0 f    CIL library: CIL module
 0001:0006d670       _sqlite3Pragma             1106e670 f    CIL library: CIL module
 0001:0006f6d0       _corruptSchema             110706d0 f    CIL library: CIL module
 0001:0006f710       _sqlite3InitCallback       11070710 f    CIL library: CIL module
 0001:0006f890       _sqlite3InitOne            11070890 f    CIL library: CIL module
 0001:0006fce0       _sqlite3Init               11070ce0 f    CIL library: CIL module
 0001:0006fdb0       _sqlite3ReadSchema         11070db0 f    CIL library: CIL module
 0001:0006fde0       _schemaIsValid             11070de0 f    CIL library: CIL module
 0001:0006fee0       _sqlite3SchemaToIndex      11070ee0 f    CIL library: CIL module
 0001:0006ff10       _sqlite3Prepare            11070f10 f    CIL library: CIL module
 0001:000703e0       _sqlite3LockAndPrepare     110713e0 f    CIL library: CIL module
 0001:00070460       _sqlite3Reprepare          11071460 f    CIL library: CIL module
 0001:00070550       _sqlite3Prepare16          11071550 f    CIL library: CIL module
 0001:000706a0       _clearSelect               110716a0 f    CIL library: CIL module
 0001:00070710       _sqlite3SelectNew          11071710 f    CIL library: CIL module
 0001:00070870       _sqlite3SelectDelete       11071870 f    CIL library: CIL module
 0001:00070890       _sqlite3JoinType           11071890 f    CIL library: CIL module
 0001:000709c0       _columnIndex               110719c0 f    CIL library: CIL module
 0001:00070a30       _addWhereTerm              11071a30 f    CIL library: CIL module
 0001:00070bc0       _setJoinExpr               11071bc0 f    CIL library: CIL module
 0001:00070bf0       _sqliteProcessJoin         11071bf0 f    CIL library: CIL module
 0001:00070e00       _pushOntoSorter            11071e00 f    CIL library: CIL module
 0001:00070fd0       _codeOffset                11071fd0 f    CIL library: CIL module
 0001:00071040       _codeDistinct              11072040 f    CIL library: CIL module
 0001:000710b0       _checkForMultiColumnSelectError 110720b0 f    CIL library: CIL module
 0001:000710e0       _selectInnerLoop           110720e0 f    CIL library: CIL module
 0001:00071660       _keyInfoFromExprList       11072660 f    CIL library: CIL module
 0001:00071720       _generateSortTail          11072720 f    CIL library: CIL module
 0001:00071b40       _columnType                11072b40 f    CIL library: CIL module
 0001:00071d30       _generateColumnTypes       11072d30 f    CIL library: CIL module
 0001:00071fa0       _generateColumnNames       11072fa0 f    CIL library: CIL module
 0001:000722b0       _selectOpName              110732b0 f    CIL library: CIL module
 0001:000722e0       _sqlite3ResultSetOfSelect  110732e0 f    CIL library: CIL module
 0001:00072600       _prepSelectStmt            11073600 f    CIL library: CIL module
 0001:00072ce0       _matchOrderByTermToExprList 11073ce0 f    CIL library: CIL module
 0001:00072e80       _processOrderGroupBy       11073e80 f    CIL library: CIL module
 0001:00072ff0       _processCompoundOrderBy    11073ff0 f    CIL library: CIL module
 0001:00073370       _sqlite3GetVdbe            11074370 f    CIL library: CIL module
 0001:000733e0       _computeLimitRegisters     110743e0 f    CIL library: CIL module
 0001:00073520       _createSortingIndex        11074520 f    CIL library: CIL module
 0001:00073550       _multiSelectCollSeq        11074550 f    CIL library: CIL module
 0001:00073590       _multiSelect               11074590 f    CIL library: CIL module
 0001:00073e70       _substExpr                 11074e70 f    CIL library: CIL module
 0001:00073fa0       _substExprList             11074fa0 f    CIL library: CIL module
 0001:00073fe0       _substSelect               11074fe0 f    CIL library: CIL module
 0001:00074130       _flattenSubquery           11075130 f    CIL library: CIL module
 0001:000745c0       _minMaxQuery               110755c0 f    CIL library: CIL module
 0001:00074630       _sqlite3SelectResolve      11075630 f    CIL library: CIL module
 0001:00074820       _resetAccumulator          11075820 f    CIL library: CIL module
 0001:00074af0       _finalizeAggFunctions      11075af0 f    CIL library: CIL module
 0001:00074c70       _updateAccumulator         11075c70 f    CIL library: CIL module
 0001:00075410       _sqlite3SelectMask         11076410 f    CIL library: CIL module
 0001:000754a0       _sqlite3Select             110764a0 f    CIL library: CIL module
 0001:00076730       _sqlite3_get_table_cb      11077730 f    CIL library: CIL module
 0001:00076af0       _sqlite3DeleteTriggerStep  11077af0 f    CIL library: CIL module
 0001:00076df0       _sqlite3BeginTrigger       11077df0 f    CIL library: CIL module
 0001:000771e0       _sqlite3FinishTrigger      110781e0 f    CIL library: CIL module
 0001:00077480       _sqlitePersistTriggerStep  11078480 f    CIL library: CIL module
 0001:00077560       _sqlite3TriggerSelectStep  11078560 f    CIL library: CIL module
 0001:000775e0       _sqlite3TriggerInsertStep  110785e0 f    CIL library: CIL module
 0001:000776a0       _sqlite3TriggerUpdateStep  110786a0 f    CIL library: CIL module
 0001:00077730       _sqlite3TriggerDeleteStep  11078730 f    CIL library: CIL module
 0001:000777b0       _sqlite3DeleteTrigger      110787b0 f    CIL library: CIL module
 0001:00077800       _sqlite3DropTrigger        11078800 f    CIL library: CIL module
 0001:00077980       _tableOfTrigger            11078980 f    CIL library: CIL module
 0001:000779e0       _sqlite3DropTriggerPtr     110789e0 f    CIL library: CIL module
 0001:00077c80       _sqlite3UnlinkAndDeleteTrigger 11078c80 f    CIL library: CIL module
 0001:00077d60       _checkColumnOverLap        11078d60 f    CIL library: CIL module
 0001:00077dc0       _sqlite3TriggersExist      11078dc0 f    CIL library: CIL module
 0001:00077e40       _targetSrcList             11078e40 f    CIL library: CIL module
 0001:00077ee0       _codeTriggerProgram        11078ee0 f    CIL library: CIL module
 0001:000782a0       _sqlite3CodeRowTrigger     110792a0 f    CIL library: CIL module
 0001:000785c0       _sqlite3ColumnDefault      110795c0 f    CIL library: CIL module
 0001:00078650       _sqlite3Update             11079650 f    CIL library: CIL module
 0001:0007a710       _updateVirtualTable        1107b710 f    CIL library: CIL module
 0001:0007b480       _execSql                   1107c480 f    CIL library: CIL module
 0001:0007b510       _execExecSql               1107c510 f    CIL library: CIL module
 0001:0007b6a0       _sqlite3Vacuum             1107c6a0 f    CIL library: CIL module
 0001:0007b700       _sqlite3RunVacuum          1107c700 f    CIL library: CIL module
 0001:0007b980       _createModule              1107c980 f    CIL library: CIL module
 0001:0007bac0       _sqlite3VtabUnlock         1107cac0 f    CIL library: CIL module
 0001:0007baf0       _sqlite3VtabClear          1107caf0 f    CIL library: CIL module
 0001:0007bc00       _addModuleArgument         1107cc00 f    CIL library: CIL module
 0001:0007bd90       _sqlite3VtabBeginParse     1107cd90 f    CIL library: CIL module
 0001:0007bea0       _sqlite3VtabFinishParse    1107cea0 f    CIL library: CIL module
 0001:0007c120       _sqlite3VtabArgInit        1107d120 f    CIL library: CIL module
 0001:0007c170       _sqlite3VtabArgExtend      1107d170 f    CIL library: CIL module
 0001:0007c1c0       _vtabCallConstructor       1107d1c0 f    CIL library: CIL module
 0001:0007c430       _sqlite3VtabCallConnect    1107d430 f    CIL library: CIL module
 0001:0007c4d0       _addToVTrans               1107d4d0 f    CIL library: CIL module
 0001:0007c550       _sqlite3VtabCallCreate     1107d550 f    CIL library: CIL module
 0001:0007c730       _sqlite3VtabCallDestroy    1107d730 f    CIL library: CIL module
 0001:0007c780       _callFinaliser             1107d780 f    CIL library: CIL module
 0001:0007c860       _sqlite3VtabSync           1107d860 f    CIL library: CIL module
 0001:0007c8b0       _sqlite3VtabBegin          1107d8b0 f    CIL library: CIL module
 0001:0007c920       _sqlite3VtabOverloadFunction 1107d920 f    CIL library: CIL module
 0001:0007ca30       _whereClauseClear          1107da30 f    CIL library: CIL module
 0001:0007cac0       _whereClauseInsert         1107dac0 f    CIL library: CIL module
 0001:0007cb60       _whereSplit                1107db60 f    CIL library: CIL module
 0001:0007cbb0       _getMask                   1107dbb0 f    CIL library: CIL module
 0001:0007cbe0       _exprTableUsage            1107dbe0 f    CIL library: CIL module
 0001:0007ccb0       _exprListTableUsage        1107dcb0 f    CIL library: CIL module
 0001:0007cd10       _exprSelectTableUsage      1107dd10 f    CIL library: CIL module
 0001:0007ce80       _exprCommute               1107de80 f    CIL library: CIL module
 0001:0007cf10       _operatorMask              1107df10 f    CIL library: CIL module
 0001:0007cf40       _findTerm                  1107df40 f    CIL library: CIL module
 0001:0007d060       _isLikeOrGlob              1107e060 f    CIL library: CIL module
 0001:0007d170       _orTermIsOptCandidate      1107e170 f    CIL library: CIL module
 0001:0007d1e0       _exprAnalyze               1107e1e0 f    CIL library: CIL module
 0001:0007de40       _referencesOtherTables     1107ee40 f    CIL library: CIL module
 0001:0007dee0       _isSortingIndex            1107eee0 f    CIL library: CIL module
 0001:0007e060       _sortableByRowid           1107f060 f    CIL library: CIL module
 0001:0007e0a0       _estLog                    1107f0a0 f    CIL library: CIL module
 0001:0007e0e0       _bestVirtualIndex          1107f0e0 f    CIL library: CIL module
 0001:0007e3e0       _bestIndex                 1107f3e0 f    CIL library: CIL module
 0001:0007e9b0       _disableTerm               1107f9b0 f    CIL library: CIL module
 0001:0007ea00       _codeEqualityTerm          1107fa00 f    CIL library: CIL module
 0001:0007eb80       _codeAllEqualityTerms      1107fb80 f    CIL library: CIL module
 0001:0007ecb0       _whereInfoFree             1107fcb0 f    CIL library: CIL module
 0001:0007ed90       _sqlite3WhereBegin         1107fd90 f    CIL library: CIL module
 0001:000819f0       _sqlite3WhereEnd           110829f0 f    CIL library: CIL module
 0001:00082250       _yy_destructor             11083250 f    CIL library: CIL module
 0001:00082340       _sqlite3ParserFree         11083340 f    CIL library: CIL module
 0001:00082380       _yy_find_shift_action      11083380 f    CIL library: CIL module
 0001:00082400       _yyStackOverflow           11083400 f    CIL library: CIL module
 0001:00082450       _yy_reduce                 11083450 f    CIL library: CIL module
 0001:00084380       _yy_accept                 11085380 f    CIL library: CIL module
 0001:00084380       _yy_parse_failed           11085380 f    CIL library: CIL module
 0001:000843c0       _sqlite3Parser             110853c0 f    CIL library: CIL module
 0001:000844e0       _keywordCode               110854e0 f    CIL library: CIL module
 0001:00084580       _getToken                  11085580 f    CIL library: CIL module
 0001:00084be0       _sqlite3RunParser          11085be0 f    CIL library: CIL module
 0001:00085380       _binCollFunc               11086380 f    CIL library: CIL module
 0001:00085460       _nocaseCollatingFunc       11086460 f    CIL library: CIL module
 0001:000859c0       _sqlite3RollbackAll        110869c0 f    CIL library: CIL module
 0001:00085a70       _sqlite3ErrStr             11086a70 f    CIL library: CIL module
 0001:00085be0       _sqliteDefaultBusyCallback 11086be0 f    CIL library: CIL module
 0001:00085de0       _sqlite3CreateFunc         11086de0 f    CIL library: CIL module
 0001:00086270       _sqlite3BtreeFactory       11087270 f    CIL library: CIL module
 0001:00086540       _createCollation           11087540 f    CIL library: CIL module
 0001:000866e0       _openDatabase              110876e0 f    CIL library: CIL module
 0001:00086e30       _softHeapLimitEnforcer     11087e30 f    CIL library: CIL module
 0001:00087e2d       _flsall                    11088e2d f   LIBCMT:fflush.obj
 0001:00088a33       ?_mbrtowc_s_l@@YAHPAHPA_WPBDI0PAUlocaleinfo_struct@@@Z 11089a33 f   LIBCMT:mbrtowc.obj
 0001:0008a0cb       ?strtoxl@@YAKPAUlocaleinfo_struct@@PBDPAPBDHH@Z 1108b0cb f   LIBCMT:strtol.obj
 0001:0008a5fb       __initterm                 1108b5fb f   LIBCMT:crt0dat.obj
 0001:0008a6c1       _doexit                    1108b6c1 f   LIBCMT:crt0dat.obj
 0001:0008a9a0       _init_namebuf              1108b9a0 f   LIBCMT:tmpfile.obj
 0001:0008aa67       _genfname                  1108ba67 f   LIBCMT:tmpfile.obj
 0001:0008aeb9       _idtab                     1108beb9 f   LIBCMT:popen.obj
 0001:0008c1b8       __make__time64_t           1108d1b8 f   LIBCMT:mktime64.obj
 0001:0008c7e9       ?_store_str@@YAXPADPAPADPAI@Z 1108d7e9 f   LIBCMT:strftime.obj
 0001:0008c809       ?_store_num@@YAXHHPAPADPAII@Z 1108d809 f   LIBCMT:strftime.obj
 0001:0008c884       ?_expandtime@@YAHPAUlocaleinfo_struct@@DPBUtm@@PAPADPAIPAU__lc_time_data@@I@Z 1108d884 f   LIBCMT:strftime.obj
 0001:0008cc6c       ?_store_winword@@YAHPAUlocaleinfo_struct@@HPBUtm@@PAPADPAIPAU__lc_time_data@@@Z 1108dc6c f   LIBCMT:strftime.obj
 0001:0008d501       __copytlocinfo_nolock      1108e501 f   LIBCMT:setlocal.obj
 0001:0008d527       __updatetlocinfoEx_nolock  1108e527 f   LIBCMT:setlocal.obj
 0001:0008d5db       _sync_legacy_variables_lk  1108e5db f   LIBCMT:setlocal.obj
 0001:0008d8c6       __setlocale_get_all        1108e8c6 f   LIBCMT:setlocal.obj
 0001:0008dc74       __setlocale_set_cat        1108ec74 f   LIBCMT:setlocal.obj
 0001:0008df76       __setlocale_nolock         1108ef76 f   LIBCMT:setlocal.obj
 0001:0008ebc3       ___DllMainCRTStartup       1108fbc3 f   LIBCMT:dllcrt0.obj
 0001:0008ee40       _write_char                1108fe40 f   LIBCMT:output.obj
 0001:0008ee73       _write_multi_char          1108fe73 f   LIBCMT:output.obj
 0001:0008ee99       _write_string              1108fe99 f   LIBCMT:output.obj
 0001:0008fab1       __tzset_nolock             11090ab1 f   LIBCMT:tzset.obj
 0001:0008fdf7       _cvtdate                   11090df7 f   LIBCMT:tzset.obj
 0001:0008ffee       __isindst_nolock           11090fee f   LIBCMT:tzset.obj
 0001:000909a5       ?CPtoLCID@@YAHH@Z          110919a5 f   LIBCMT:mbctype.obj
 0001:000909d4       ?setSBCS@@YAXPAUthreadmbcinfostruct@@@Z 110919d4 f   LIBCMT:mbctype.obj
 0001:00090a38       ?setSBUpLow@@YAXPAUthreadmbcinfostruct@@@Z 11091a38 f   LIBCMT:mbctype.obj
 0001:00090c6f       ?getSystemCP@@YAHH@Z       11091c6f f   LIBCMT:mbctype.obj
 0001:000917b8       __onexit_nolock            110927b8 f   LIBCMT:onexit.obj
 0001:00093697       ?__crtLCMapStringA_stat@@YAHPAUlocaleinfo_struct@@KKPBDHPADHHH@Z 11094697 f   LIBCMT:a_map.obj
 0001:00094504       __unwind_handler4          11095504 f   LIBCMT:exsup4.obj
 0001:00094a71       ___check_float_string      11095a71 f   LIBCMT:input.obj
 0001:00094ac8       __hextodec                 11095ac8 f   LIBCMT:input.obj
 0001:00094ae8       __inc                      11095ae8 f   LIBCMT:input.obj
 0001:00094afe       __un_inc                   11095afe f   LIBCMT:input.obj
 0001:00094b11       __whiteout                 11095b11 f   LIBCMT:input.obj
 0001:00096b94       __unwind_handler           11097b94 f   LIBCMT:exsup.obj
 0001:000970f1       _siglookup                 110980f1 f   LIBCMT:winsig.obj
 0001:000973d7       _xtoa_s@20                 110983d7 f   LIBCMT:xtoas.obj
 0001:00097758       __tsopen_nolock            11098758 f   LIBCMT:open.obj
 0001:00099930       _comexecmd                 1109a930 f   LIBCMT:spawnve.obj
 0001:00099bfc       __get_lc_time              1109abfc f   LIBCMT:inittime.obj
 0001:0009ab50       _TranslateName             1109bb50 f   LIBCMT:getqloc.obj
 0001:0009abb2       _ProcessCodePage           1109bbb2 f   LIBCMT:getqloc.obj
 0001:0009ac56       _TestDefaultCountry        1109bc56 f   LIBCMT:getqloc.obj
 0001:0009ac7a       _LcidFromHexString         1109bc7a f   LIBCMT:getqloc.obj
 0001:0009acae       _GetPrimaryLen             1109bcae f   LIBCMT:getqloc.obj
 0001:0009acc9       _CountryEnumProc@4         1109bcc9 f   LIBCMT:getqloc.obj
 0001:0009ad61       _TestDefaultLanguage       1109bd61 f   LIBCMT:getqloc.obj
 0001:0009add5       _LangCountryEnumProc@4     1109bdd5 f   LIBCMT:getqloc.obj
 0001:0009afa7       _LanguageEnumProc@4        1109bfa7 f   LIBCMT:getqloc.obj
 0001:0009b068       _GetLcidFromLangCountry    1109c068 f   LIBCMT:getqloc.obj
 0001:0009b0cf       _GetLcidFromLanguage       1109c0cf f   LIBCMT:getqloc.obj
 0001:0009c97c       ?__crtGetStringTypeA_stat@@YAHPAUlocaleinfo_struct@@KPBDHPAGHHH@Z 1109d97c f   LIBCMT:a_str.obj
 0001:0009cb78       ?strncnt@@YAHPBDH@Z        1109db78 f   LIBCMT:a_cmp.obj
 0001:0009cb96       ?__crtCompareStringA_stat@@YAHPAUlocaleinfo_struct@@KKPBDH1HH@Z 1109db96 f   LIBCMT:a_cmp.obj
 0001:0009cf48       _fastcopy_I                1109df48 f   LIBCMT:p4_memcpy.obj
 0001:0009d190       _parse_cmdline             1109e190 f   LIBCMT:stdargv.obj
 0001:0009d9d5       _fastzero_I                1109e9d5 f   LIBCMT:p4_memset.obj
 0001:0009ebb7       ?__crtGetLocaleInfoA_stat@@YAHPAUlocaleinfo_struct@@KKPADHH@Z 1109fbb7 f   LIBCMT:a_loc.obj
 0001:0009f928       __shift                    110a0928 f   LIBCMT:cvt.obj
 0001:0009f96d       __cftoe2_l                 110a096d f   LIBCMT:cvt.obj
 0001:0009ff3f       __cftof2_l                 110a0f3f f   LIBCMT:cvt.obj
 0001:000a07ad       _has_osfxsr_set            110a17ad f   LIBCMT:cpu_disp.obj
 0001:000a097a       _findenv                   110a197a f   LIBCMT:setenv.obj
 0001:000a09cc       _copy_environ              110a19cc f   LIBCMT:setenv.obj
 0001:000a147c       ?x_ismbbtype_l@@YAHPAUlocaleinfo_struct@@IHH@Z 110a247c f   LIBCMT:ismbbyte.obj
 0001:000a2565       __hw_cw                    110a3565 f   LIBCMT:_ieee87_.obj
 0001:000a25f3       ___hw_cw_sse2              110a35f3 f   LIBCMT:_ieee87_.obj
 0001:000a2b17       __ReleaseCPLocHash         110a3b17 f   libcpmt:xmbtowc.obj
 0001:000a2b57       __InitCPLocHash            110a3b57 f   libcpmt:xmbtowc.obj
 0001:000a2c99       ?CatchGuardHandler@@YA?AW4_EXCEPTION_DISPOSITION@@PAUEHExceptionRecord@@PAUCatchGuardRN@@PAX2@Z 110a3c99 f   LIBCMT:_trnsctrl_.obj
 0001:000a2da3       ?TranslatorGuardHandler@@YA?AW4_EXCEPTION_DISPOSITION@@PAUEHExceptionRecord@@PAUTranslatorGuardRN@@PAX2@Z 110a3da3 f   LIBCMT:_trnsctrl_.obj
 0001:000a31fe       ?ExFilterRethrow@@YAHPAU_EXCEPTION_POINTERS@@@Z 110a41fe f   LIBCMT:frame.obj
 0001:000a32c1       ?IsInExceptionSpec@@YAEPAUEHExceptionRecord@@PBU_s_ESTypeList@@@Z 110a42c1 f   LIBCMT:frame.obj
 0001:000a333c       ?CallUnexpected@@YAXPBU_s_ESTypeList@@@Z 110a433c f   LIBCMT:frame.obj
 0001:000a336d       __catch$?CallUnexpected@@YAXPBU_s_ESTypeList@@@Z$0 110a436d f   LIBCMT:frame.obj
 0001:000a3385       ?CallCatchBlock@@YAPAXPAUEHExceptionRecord@@PAUEHRegistrationNode@@PAU_CONTEXT@@PBU_s_FuncInfo@@PAXHK@Z 110a4385 f   LIBCMT:frame.obj
 0001:000a3732       ?CatchIt@@YAXPAUEHExceptionRecord@@PAUEHRegistrationNode@@PAU_CONTEXT@@PAXPBU_s_FuncInfo@@PBU_s_HandlerType@@PBU_s_CatchableType@@PBU_s_TryBlockMapEntry@@H1E@Z 110a4732 f   LIBCMT:frame.obj
 0001:000a37a0       ?FindHandlerForForeignException@@YAXPAUEHExceptionRecord@@PAUEHRegistrationNode@@PAU_CONTEXT@@PAXPBU_s_FuncInfo@@HH1@Z 110a47a0 f   LIBCMT:frame.obj
 0001:000a3894       ?FindHandler@@YAXPAUEHExceptionRecord@@PAUEHRegistrationNode@@PAU_CONTEXT@@PAXPBU_s_FuncInfo@@EH1@Z 110a4894 f   LIBCMT:frame.obj
 0001:000a76f0       __unwindfunclet$?_Xran@_String_base@std@@SAXXZ$0 110a86f0 f   libcpmt:string.obj
 0001:000a76f0       __unwindfunclet$?_Xlen@_String_base@std@@SAXXZ$0 110a86f0 f   libcpmt:string.obj
 0001:000a76f8       __ehhandler$?_Xran@_String_base@std@@SAXXZ 110a86f8 f   libcpmt:string.obj
 0001:000a76f8       __ehhandler$?_Xlen@_String_base@std@@SAXXZ 110a86f8 f   libcpmt:string.obj
 0001:000a7713       __ehhandler$?CallUnexpected@@YAXPBU_s_ESTypeList@@@Z 110a8713 f   LIBCMT:frame.obj
 0001:000a7730       __unwindfunclet$?Force_Occupants_Exit_Team@@YAXPAEH@Z$0 110a8730 f    CIL library: CIL module
 0001:000a7738       __ehhandler$?Force_Occupants_Exit_Team@@YAXPAEH@Z 110a8738 f    CIL library: CIL module
 0001:000a7750       __ehhandler$?_Copy@?$basic_string@DU?$char_traits@D@std@@V?$allocator@D@2@@std@@IAEXII@Z 110a8750 f    CIL library: CIL module
 0001:000a7760       __unwindfunclet$??0logic_error@std@@QAE@ABV01@@Z$0 110a8760 f    CIL library: CIL module
 0001:000a7760       __unwindfunclet$??0logic_error@std@@QAE@ABV?$basic_string@DU?$char_traits@D@std@@V?$allocator@D@2@@1@@Z$0 110a8760 f    CIL library: CIL module
 0001:000a7768       __ehhandler$??0logic_error@std@@QAE@ABV?$basic_string@DU?$char_traits@D@std@@V?$allocator@D@2@@1@@Z 110a8768 f    CIL library: CIL module
 0001:000a7768       __ehhandler$??0logic_error@std@@QAE@ABV01@@Z 110a8768 f    CIL library: CIL module
 0001:000a7780       __unwindfunclet$?RegisterTable@Lua_sqlite_wrapper@@CAHPAUlua_State@@@Z$0 110a8780 f    CIL library: CIL module
 0001:000a778b       __ehhandler$?RegisterTable@Lua_sqlite_wrapper@@CAHPAUlua_State@@@Z 110a878b f    CIL library: CIL module
 0001:000a77a0       __unwindfunclet$?Lua_RequestSerial@@YAHPAUlua_State@@@Z$0 110a87a0 f    CIL library: CIL module
 0001:000a77a8       __ehhandler$?Lua_RequestSerial@@YAHPAUlua_State@@@Z 110a87a8 f    CIL library: CIL module
 0001:000a77b2       ??__Eclassic_locale@std@@YAXXZ 110a87b2 f   libcpmt:locale0.obj
 0001:000a77be       ??__Einitlocks@std@@YAXXZ  110a87be f   libcpmt:xlock.obj
 0001:000a77d4       ??__Einitlocks@std@@YAXXZ  110a87d4 f   libcpmt:iosptrs.obj
 0001:000a77ea       ??__Einit_atexit@@YAXXZ    110a87ea f   libcpmt:iosptrs.obj
 0001:000a77f6       ??__Fnomem@?5???2@YAPAXI@Z@YAXXZ 110a87f6 f   LIBCMT:new.obj
 0001:000a780a       ??__Fclassic_locale@std@@YAXXZ 110a880a f   libcpmt:locale0.obj
 0001:000a7814       ??__Finitlocks@std@@YAXXZ  110a8814 f   libcpmt:xlock.obj
 0001:000a781e       ??__Finitlocks@std@@YAXXZ  110a881e f   libcpmt:iosptrs.obj
 0001:000a7828       ??__Finit_atexit@@YAXXZ    110a8828 f   libcpmt:iosptrs.obj
